 jpackage

 Timestamp is c0a4633f (reproducible build file hash)

 Preferred load address is 0000000180000000

 Start         Length     Name                   Class
 0001:00000000 00000020H .text$di                CODE
 0001:00000020 00011090H .text$mn                CODE
 0001:000110b0 00000036H .text$mn$00             CODE
 0001:000110e6 00001322H .text$x                 CODE
 0001:00012408 00000067H .text$yd                CODE
 0002:00000000 00000798H .idata$5                DATA
 0002:00000798 00000038H .00cfg                  DATA
 0002:000007d0 00000008H .CRT$XCA                DATA
 0002:000007d8 00000008H .CRT$XCL                DATA
 0002:000007e0 00000008H .CRT$XCU                DATA
 0002:000007e8 00000008H .CRT$XCZ                DATA
 0002:000007f0 00000008H .CRT$XIA                DATA
 0002:000007f8 00000008H .CRT$XIZ                DATA
 0002:00000800 00000008H .CRT$XPA                DATA
 0002:00000808 00000008H .CRT$XPZ                DATA
 0002:00000810 00000008H .CRT$XTA                DATA
 0002:00000818 00000008H .CRT$XTZ                DATA
 0002:00000820 00000000H .gehcont$y              DATA
 0002:00000820 00000000H .gfids$y                DATA
 0002:00000820 00001be0H .rdata                  DATA
 0002:00002400 00000000H .rdata$CastGuardVftablesA DATA
 0002:00002400 00000000H .rdata$CastGuardVftablesC DATA
 0002:00002400 000016a4H .rdata$r                DATA
 0002:00003aa4 00000118H .rdata$voltmd           DATA
 0002:00003bbc 0000035cH .rdata$zzzdbg           DATA
 0002:00003f18 00000008H .rtc$IAA                DATA
 0002:00003f20 00000008H .rtc$IZZ                DATA
 0002:00003f28 00000008H .rtc$TAA                DATA
 0002:00003f30 00000008H .rtc$TZZ                DATA
 0002:00003f38 00002380H .xdata                  DATA
 0002:000062b8 000004b8H .xdata$x                DATA
 0002:00006770 00000320H .edata                  DATA
 0002:00006a90 000000f0H .idata$2                DATA
 0002:00006b80 00000018H .idata$3                DATA
 0002:00006b98 00000798H .idata$4                DATA
 0002:00007330 000028eeH .idata$6                DATA
 0003:00000000 000002c8H .data                   DATA
 0003:000002c8 00000298H .data$r                 DATA
 0003:00000560 00000730H .data$rs                DATA
 0003:00000c90 00000668H .bss                    DATA
 0004:00000000 00001320H .pdata                  DATA
 0005:00000000 00000060H .rsrc$01                DATA
 0005:00000060 00000320H .rsrc$02                DATA

  Address         Publics by Value              Rva+Base               Lib:Object

 0000:00000000       __AbsoluteZero             0000000000000000     <absolute>
 0000:00000000       ___safe_se_handler_count   0000000000000000     <absolute>
 0000:00000000       ___safe_se_handler_table   0000000000000000     <absolute>
 0000:00000000       __arm64x_extra_rfe_table   0000000000000000     <absolute>
 0000:00000000       __arm64x_extra_rfe_table_size 0000000000000000     <absolute>
 0000:00000000       __arm64x_native_entrypoint 0000000000000000     <absolute>
 0000:00000000       __arm64x_redirection_metadata 0000000000000000     <absolute>
 0000:00000000       __arm64x_redirection_metadata_count 0000000000000000     <absolute>
 0000:00000000       __dynamic_value_reloc_table 0000000000000000     <absolute>
 0000:00000000       __enclave_config           0000000000000000     <absolute>
 0000:00000000       __guard_check_icall_a64n_fptr 0000000000000000     <absolute>
 0000:00000000       __guard_eh_cont_count      0000000000000000     <absolute>
 0000:00000000       __guard_eh_cont_table      0000000000000000     <absolute>
 0000:00000000       __guard_fids_count         0000000000000000     <absolute>
 0000:00000000       __guard_fids_table         0000000000000000     <absolute>
 0000:00000000       __guard_iat_count          0000000000000000     <absolute>
 0000:00000000       __guard_iat_table          0000000000000000     <absolute>
 0000:00000000       __guard_longjmp_count      0000000000000000     <absolute>
 0000:00000000       __guard_longjmp_table      0000000000000000     <absolute>
 0000:00000000       __hybrid_auxiliary_delayload_iat 0000000000000000     <absolute>
 0000:00000000       __hybrid_auxiliary_delayload_iat_copy 0000000000000000     <absolute>
 0000:00000000       __hybrid_auxiliary_iat     0000000000000000     <absolute>
 0000:00000000       __hybrid_auxiliary_iat_copy 0000000000000000     <absolute>
 0000:00000000       __hybrid_code_map          0000000000000000     <absolute>
 0000:00000000       __hybrid_code_map_count    0000000000000000     <absolute>
 0000:00000000       __hybrid_image_info_bitfield 0000000000000000     <absolute>
 0000:00000000       __x64_code_ranges_to_entry_points 0000000000000000     <absolute>
 0000:00000000       __x64_code_ranges_to_entry_points_count 0000000000000000     <absolute>
 0000:00000100       __guard_flags              0000000000000100     <absolute>
 0000:00000000       __ImageBase                0000000180000000     <linker-defined>
 0001:00000020       ??$?6GU?$char_traits@G@std@@@std@@YAAEAV?$basic_ostream@GU?$char_traits@G@std@@@0@AEAV10@PEBD@Z 0000000180001020 f i ErrorHandling.obj
 0001:00000294       ??$?6GU?$char_traits@G@std@@@std@@YAAEAV?$basic_ostream@GU?$char_traits@G@std@@@0@AEAV10@PEBG@Z 0000000180001294 f i ErrorHandling.obj
 0001:00000484       ??$?6U?$char_traits@D@std@@@std@@YAAEAV?$basic_ostream@DU?$char_traits@D@std@@@0@AEAV10@PEBD@Z 0000000180001484 f i ErrorHandling.obj
 0001:0000065c       ??$_Allocate_manually_vector_aligned@U_Default_allocate_traits@std@@@std@@YAPEAX_K@Z 000000018000165c f i ErrorHandling.obj
 0001:00000698       ??$_Construct@$00PEBD@?$basic_string@DU?$char_traits@D@std@@V?$allocator@D@2@@std@@AEAAXQEBD_K@Z 0000000180001698 f i ErrorHandling.obj
 0001:00000778       ??$_Construct@$00PEAG@?$basic_string@GU?$char_traits@G@std@@V?$allocator@G@2@@std@@AEAAXQEAG_K@Z 0000000180001778 f i Guid.obj
 0001:00000778       ??$_Construct@$00PEBG@?$basic_string@GU?$char_traits@G@std@@V?$allocator@G@2@@std@@AEAAXQEBG_K@Z 0000000180001778 f i ErrorHandling.obj
 0001:0000087c       ??$_Construct@$01PEBD@?$basic_string@DU?$char_traits@D@std@@V?$allocator@D@2@@std@@AEAAXQEBD_K@Z 000000018000187c f i ErrorHandling.obj
 0001:00000944       ??$_Insert_string@DU?$char_traits@D@std@@_K@std@@YAAEAV?$basic_ostream@DU?$char_traits@D@std@@@0@AEAV10@QEBD_K@Z 0000000180001944 f i ErrorHandling.obj
 0001:00000b18       ??$_Insert_string@GU?$char_traits@G@std@@_K@std@@YAAEAV?$basic_ostream@GU?$char_traits@G@std@@@0@AEAV10@QEBG_K@Z 0000000180001b18 f i ErrorHandling.obj
 0001:00000d04       ??$_Reallocate_for@V<lambda_1>@?1??assign@?$basic_string@DU?$char_traits@D@std@@V?$allocator@D@2@@std@@QEAAAEAV34@QEBD_K@Z@PEBD@?$basic_string@DU?$char_traits@D@std@@V?$allocator@D@2@@std@@AEAAAEAV01@_KV<lambda_1>@?1??assign@01@QEAAAEAV01@QEBD0@Z@PEBD@Z 0000000180001d04 f i ErrorHandling.obj
 0001:00000e10       ??$_Reallocate_for@V<lambda_1>@?1??assign@?$basic_string@GU?$char_traits@G@std@@V?$allocator@G@2@@std@@QEAAAEAV34@QEBG_K@Z@PEBG@?$basic_string@GU?$char_traits@G@std@@V?$allocator@G@2@@std@@AEAAAEAV01@_KV<lambda_1>@?1??assign@01@QEAAAEAV01@QEBG0@Z@PEBG@Z 0000000180001e10 f i ErrorHandling.obj
 0001:00000f50       ??$_Traits_find_last_of@U?$char_traits@D@std@@$00@std@@YA_KQEBD_K101@Z 0000000180001f50 f i ErrorHandling.obj
 0001:00001004       ??$use_facet@V?$ctype@G@std@@@std@@YAAEBV?$ctype@G@0@AEBVlocale@0@@Z 0000000180002004 f i ErrorHandling.obj
 0001:000010e4       ??0?$basic_ostringstream@DU?$char_traits@D@std@@V?$allocator@D@2@@std@@QEAA@XZ 00000001800020e4 f i ErrorHandling.obj
 0001:0000118c       ??0?$basic_ostringstream@GU?$char_traits@G@std@@V?$allocator@G@2@@std@@QEAA@XZ 000000018000218c f i ErrorHandling.obj
 0001:00001234       ??0bad_alloc@std@@QEAA@AEBV01@@Z 0000000180002234 f i ErrorHandling.obj
 0001:00001270       ??0bad_array_new_length@std@@QEAA@AEBV01@@Z 0000000180002270 f i ErrorHandling.obj
 0001:000012ac       ??0bad_array_new_length@std@@QEAA@XZ 00000001800022ac f i ErrorHandling.obj
 0001:000012cc       ??0bad_cast@std@@QEAA@AEBV01@@Z 00000001800022cc f i ErrorHandling.obj
 0001:00001308       ??0bad_cast@std@@QEAA@XZ   0000000180002308 f i ErrorHandling.obj
 0001:00001328       ??0exception@std@@QEAA@AEBV01@@Z 0000000180002328 f i ErrorHandling.obj
 0001:0000135c       ??0sentry@?$basic_ostream@DU?$char_traits@D@std@@@std@@QEAA@AEAV12@@Z 000000018000235c f i ErrorHandling.obj
 0001:00001400       ??0sentry@?$basic_ostream@GU?$char_traits@G@std@@@std@@QEAA@AEAV12@@Z 0000000180002400 f i ErrorHandling.obj
 0001:000014a4       ??1?$basic_ostringstream@DU?$char_traits@D@std@@V?$allocator@D@2@@std@@UEAA@XZ 00000001800024a4 f i ErrorHandling.obj
 0001:0000151c       ??1?$basic_ostringstream@GU?$char_traits@G@std@@V?$allocator@G@2@@std@@UEAA@XZ 000000018000251c f i ErrorHandling.obj
 0001:00001594       ??1?$basic_string@DU?$char_traits@D@std@@V?$allocator@D@2@@std@@QEAA@XZ 0000000180002594 f i ErrorHandling.obj
 0001:000015f0       ??1?$basic_string@GU?$char_traits@G@std@@V?$allocator@G@2@@std@@QEAA@XZ 00000001800025f0 f i ErrorHandling.obj
 0001:000015f8       ??1?$unique_ptr@V_Facet_base@std@@U?$default_delete@V_Facet_base@std@@@2@@std@@QEAA@XZ 00000001800025f8 f i ErrorHandling.obj
 0001:00001614       ??1_Sentry_base@?$basic_ostream@DU?$char_traits@D@std@@@std@@QEAA@XZ 0000000180002614 f i ErrorHandling.obj
 0001:00001640       ??1_Sentry_base@?$basic_ostream@GU?$char_traits@G@std@@@std@@QEAA@XZ 0000000180002640 f i ErrorHandling.obj
 0001:0000166c       ??1any@tstrings@@QEAA@XZ   000000018000266c f i ErrorHandling.obj
 0001:0000166c       ??_D?$basic_ostringstream@GU?$char_traits@G@std@@V?$allocator@G@2@@std@@QEAAXXZ 000000018000266c f i ErrorHandling.obj
 0001:00001690       ??1Error@msi@@UEAA@XZ      0000000180002690 f i MsiCA.obj
 0001:00001690       ??1NoMoreItemsError@msi@@UEAA@XZ 0000000180002690 f i MsiDb.obj
 0001:00001690       ??1SysError@@UEAA@XZ       0000000180002690 f i Executor.obj
 0001:00001690       ??1bad_alloc@std@@UEAA@XZ  0000000180002690 f i MSVCRT:throw_bad_alloc.obj
 0001:00001690       ??1bad_array_new_length@std@@UEAA@XZ 0000000180002690 f i ErrorHandling.obj
 0001:00001690       ??1bad_cast@std@@UEAA@XZ   0000000180002690 f i ErrorHandling.obj
 0001:00001690       ??1invalid_argument@std@@UEAA@XZ 0000000180002690 f i tstrings.obj
 0001:00001690       ??1runtime_error@std@@UEAA@XZ 0000000180002690 f i Guid.obj
 0001:000016a4       ??1locale@std@@QEAA@XZ     00000001800026a4 f i ErrorHandling.obj
 0001:000016d0       ??1sentry@?$basic_ostream@DU?$char_traits@D@std@@@std@@QEAA@XZ 00000001800026d0 f i ErrorHandling.obj
 0001:00001714       ??1sentry@?$basic_ostream@GU?$char_traits@G@std@@@std@@QEAA@XZ 0000000180002714 f i ErrorHandling.obj
 0001:00001758       ??6@YAAEAV?$basic_ostream@DU?$char_traits@D@std@@@std@@AEAV01@AEBVany@tstrings@@@Z 0000000180002758 f i ErrorHandling.obj
 0001:00001810       ??_D?$basic_ostringstream@DU?$char_traits@D@std@@V?$allocator@D@2@@std@@QEAAXXZ 0000000180002810 f i ErrorHandling.obj
 0001:00001834       ??_E?$basic_ostringstream@DU?$char_traits@D@std@@V?$allocator@D@2@@std@@$4PPPPPPPM@A@EAAPEAXI@Z 0000000180002834 f i ErrorHandling.obj
 0001:00001840       ??_E?$basic_ostringstream@GU?$char_traits@G@std@@V?$allocator@G@2@@std@@$4PPPPPPPM@A@EAAPEAXI@Z 0000000180002840 f i ErrorHandling.obj
 0001:0000184c       ??_E?$basic_ostringstream@DU?$char_traits@D@std@@V?$allocator@D@2@@std@@UEAAPEAXI@Z 000000018000284c f i ErrorHandling.obj
 0001:0000184c       ??_G?$basic_ostringstream@DU?$char_traits@D@std@@V?$allocator@D@2@@std@@UEAAPEAXI@Z 000000018000284c f i ErrorHandling.obj
 0001:0000189c       ??_E?$basic_ostringstream@GU?$char_traits@G@std@@V?$allocator@G@2@@std@@UEAAPEAXI@Z 000000018000289c f i ErrorHandling.obj
 0001:0000189c       ??_G?$basic_ostringstream@GU?$char_traits@G@std@@V?$allocator@G@2@@std@@UEAAPEAXI@Z 000000018000289c f i ErrorHandling.obj
 0001:000018ec       ??_E?$basic_stringbuf@DU?$char_traits@D@std@@V?$allocator@D@2@@std@@UEAAPEAXI@Z 00000001800028ec f i ErrorHandling.obj
 0001:000018ec       ??_G?$basic_stringbuf@DU?$char_traits@D@std@@V?$allocator@D@2@@std@@UEAAPEAXI@Z 00000001800028ec f i ErrorHandling.obj
 0001:00001934       ??_E?$basic_stringbuf@GU?$char_traits@G@std@@V?$allocator@G@2@@std@@UEAAPEAXI@Z 0000000180002934 f i ErrorHandling.obj
 0001:00001934       ??_G?$basic_stringbuf@GU?$char_traits@G@std@@V?$allocator@G@2@@std@@UEAAPEAXI@Z 0000000180002934 f i ErrorHandling.obj
 0001:0000197c       ??_ESysError@@UEAAPEAXI@Z  000000018000297c f i Executor.obj
 0001:0000197c       ??_Ebad_alloc@std@@UEAAPEAXI@Z 000000018000297c f i ErrorHandling.obj
 0001:0000197c       ??_Ebad_array_new_length@std@@UEAAPEAXI@Z 000000018000297c f i ErrorHandling.obj
 0001:0000197c       ??_Ebad_cast@std@@UEAAPEAXI@Z 000000018000297c f i ErrorHandling.obj
 0001:0000197c       ??_Eexception@std@@UEAAPEAXI@Z 000000018000297c f i ErrorHandling.obj
 0001:0000197c       ??_Einvalid_argument@std@@UEAAPEAXI@Z 000000018000297c f i tstrings.obj
 0001:0000197c       ??_Elogic_error@std@@UEAAPEAXI@Z 000000018000297c f i tstrings.obj
 0001:0000197c       ??_Eruntime_error@std@@UEAAPEAXI@Z 000000018000297c f i Executor.obj
 0001:0000197c       ??_GSysError@@UEAAPEAXI@Z  000000018000297c f i Executor.obj
 0001:0000197c       ??_Gbad_alloc@std@@UEAAPEAXI@Z 000000018000297c f i ErrorHandling.obj
 0001:0000197c       ??_Gbad_array_new_length@std@@UEAAPEAXI@Z 000000018000297c f i ErrorHandling.obj
 0001:0000197c       ??_Gbad_cast@std@@UEAAPEAXI@Z 000000018000297c f i ErrorHandling.obj
 0001:0000197c       ??_Gexception@std@@UEAAPEAXI@Z 000000018000297c f i ErrorHandling.obj
 0001:0000197c       ??_Ginvalid_argument@std@@UEAAPEAXI@Z 000000018000297c f i tstrings.obj
 0001:0000197c       ??_Glogic_error@std@@UEAAPEAXI@Z 000000018000297c f i tstrings.obj
 0001:0000197c       ??_Gruntime_error@std@@UEAAPEAXI@Z 000000018000297c f i Executor.obj
 0001:000019c0       ?_Get_buffer_view@?$basic_stringbuf@DU?$char_traits@D@std@@V?$allocator@D@2@@std@@QEBA?AU_Buffer_view@12@XZ 00000001800029c0 f i ErrorHandling.obj
 0001:00001a78       ?_Get_buffer_view@?$basic_stringbuf@GU?$char_traits@G@std@@V?$allocator@G@2@@std@@QEBA?AU_Buffer_view@12@XZ 0000000180002a78 f i ErrorHandling.obj
 0001:00001b38       ?_Throw_bad_array_new_length@std@@YAXXZ 0000000180002b38 f i ErrorHandling.obj
 0001:00001b38       ?__scrt_throw_std_bad_array_new_length@@YAXXZ 0000000180002b38 f i MSVCRT:throw_bad_alloc.obj
 0001:00001b58       ?_Throw_bad_cast@std@@YAXXZ 0000000180002b58 f i ErrorHandling.obj
 0001:00001b78       ?_Tidy@?$basic_stringbuf@DU?$char_traits@D@std@@V?$allocator@D@2@@std@@IEAAXXZ 0000000180002b78 f i ErrorHandling.obj
 0001:00001c34       ?_Tidy@?$basic_stringbuf@GU?$char_traits@G@std@@V?$allocator@G@2@@std@@IEAAXXZ 0000000180002c34 f i ErrorHandling.obj
 0001:00001cf4       ?_Tidy_deallocate@?$basic_string@GU?$char_traits@G@std@@V?$allocator@G@2@@std@@AEAAXXZ 0000000180002cf4 f i ErrorHandling.obj
 0001:00001d58       ?_Xlen_string@std@@YAXXZ   0000000180002d58 f i ErrorHandling.obj
 0001:00001d6c       ?_Xran@?$_String_val@U?$_Simple_types@D@std@@@std@@SAXXZ 0000000180002d6c f i ErrorHandling.obj
 0001:00001d6c       ?_Xran@?$_String_val@U?$_Simple_types@G@std@@@std@@SAXXZ 0000000180002d6c f i FileUtils.obj
 0001:00001f70       ?joinErrorMessages@@YA?AV?$basic_string@DU?$char_traits@D@std@@V?$allocator@D@2@@std@@AEBV12@0@Z 0000000180002f70 f   ErrorHandling.obj
 0001:00002324       ?makeMessage@@YA?AV?$basic_string@DU?$char_traits@D@std@@V?$allocator@D@2@@std@@AEBVruntime_error@2@AEBUSourceCodePos@@@Z 0000000180003324 f   ErrorHandling.obj
 0001:00002478       ?overflow@?$basic_stringbuf@DU?$char_traits@D@std@@V?$allocator@D@2@@std@@MEAAHH@Z 0000000180003478 f i ErrorHandling.obj
 0001:00002614       ?overflow@?$basic_stringbuf@GU?$char_traits@G@std@@V?$allocator@G@2@@std@@MEAAGG@Z 0000000180003614 f i ErrorHandling.obj
 0001:000027f0       ?pbackfail@?$basic_stringbuf@DU?$char_traits@D@std@@V?$allocator@D@2@@std@@MEAAHH@Z 00000001800037f0 f i ErrorHandling.obj
 0001:0000287c       ?pbackfail@?$basic_stringbuf@GU?$char_traits@G@std@@V?$allocator@G@2@@std@@MEAAGG@Z 000000018000387c f i ErrorHandling.obj
 0001:00002b34       ?reportError@@YAXAEBUSourceCodePos@@AEBVruntime_error@std@@@Z 0000000180003b34 f   ErrorHandling.obj
 0001:00002c10       ?reportUnknownError@@YAXAEBUSourceCodePos@@@Z 0000000180003c10 f   ErrorHandling.obj
 0001:00002cc4       ?seekoff@?$basic_stringbuf@DU?$char_traits@D@std@@V?$allocator@D@2@@std@@MEAA?AV?$fpos@U_Mbstatet@@@2@_JHH@Z 0000000180003cc4 f i ErrorHandling.obj
 0001:00002e6c       ?seekoff@?$basic_stringbuf@GU?$char_traits@G@std@@V?$allocator@G@2@@std@@MEAA?AV?$fpos@U_Mbstatet@@@2@_JHH@Z 0000000180003e6c f i ErrorHandling.obj
 0001:00003018       ?seekpos@?$basic_stringbuf@DU?$char_traits@D@std@@V?$allocator@D@2@@std@@MEAA?AV?$fpos@U_Mbstatet@@@2@V32@H@Z 0000000180004018 f i ErrorHandling.obj
 0001:0000315c       ?seekpos@?$basic_stringbuf@GU?$char_traits@G@std@@V?$allocator@G@2@@std@@MEAA?AV?$fpos@U_Mbstatet@@@2@V32@H@Z 000000018000415c f i ErrorHandling.obj
 0001:000032a0       ?str@?$basic_stringbuf@DU?$char_traits@D@std@@V?$allocator@D@2@@std@@QEBA?AV?$basic_string@DU?$char_traits@D@std@@V?$allocator@D@2@@2@XZ 00000001800042a0 f i ErrorHandling.obj
 0001:00003344       ?str@?$basic_stringbuf@GU?$char_traits@G@std@@V?$allocator@G@2@@std@@QEBA?AV?$basic_string@GU?$char_traits@G@std@@V?$allocator@G@2@@2@XZ 0000000180004344 f i ErrorHandling.obj
 0001:000033ec       ?underflow@?$basic_stringbuf@DU?$char_traits@D@std@@V?$allocator@D@2@@std@@MEAAHXZ 00000001800043ec f i ErrorHandling.obj
 0001:00003490       ?underflow@?$basic_stringbuf@GU?$char_traits@G@std@@V?$allocator@G@2@@std@@MEAAGXZ 0000000180004490 f i ErrorHandling.obj
 0001:00003538       ?what@exception@std@@UEBAPEBDXZ 0000000180004538 f i ErrorHandling.obj
 0001:0000354c       ??$?6PEBD@any@tstrings@@QEAAAEAV01@PEBD@Z 000000018000454c f i Executor.obj
 0001:00003564       ??$_Construct@$01PEBG@?$basic_string@GU?$char_traits@G@std@@V?$allocator@G@2@@std@@AEAAXQEBG_K@Z 0000000180004564 f i Executor.obj
 0001:00003648       ??$_Copy_memmove@PEAEPEAE@std@@YAPEAEPEAE00@Z 0000000180004648 f i ResourceEditor.obj
 0001:00003648       ??$_Copy_memmove@PEAGPEAG@std@@YAPEAGPEAG00@Z 0000000180004648 f i Executor.obj
 0001:00003678       ??$_Destroy_range@V?$allocator@V?$basic_string@GU?$char_traits@G@std@@V?$allocator@G@2@@std@@@std@@@std@@YAXPEAV?$basic_string@GU?$char_traits@G@std@@V?$allocator@G@2@@0@QEAV10@AEAV?$allocator@V?$basic_string@GU?$char_traits@G@std@@V?$allocator@G@2@@std@@@0@@Z 0000000180004678 f i Executor.obj
 0001:000036ac       ??$_Uninitialized_move@PEAV?$basic_string@GU?$char_traits@G@std@@V?$allocator@G@2@@std@@V?$allocator@V?$basic_string@GU?$char_traits@G@std@@V?$allocator@G@2@@std@@@2@@std@@YAPEAV?$basic_string@GU?$char_traits@G@std@@V?$allocator@G@2@@0@QEAV10@0PEAV10@AEAV?$allocator@V?$basic_string@GU?$char_traits@G@std@@V?$allocator@G@2@@std@@@0@@Z 00000001800046ac f i Executor.obj
 0001:0000373c       ??$makeException@VSysError@@@@YA?AV?$JpError@VSysError@@@@AEBVSysError@@AEBUSourceCodePos@@@Z 000000018000473c f i Executor.obj
 0001:00003754       ??0?$JpError@VSysError@@@@QEAA@AEBV0@@Z 0000000180004754 f i Executor.obj
 0001:000037e4       ??0?$JpError@VSysError@@@@QEAA@AEBVSysError@@AEBUSourceCodePos@@@Z 00000001800047e4 f i Executor.obj
 0001:00003864       ??0?$basic_string@GU?$char_traits@G@std@@V?$allocator@G@2@@std@@QEAA@U_String_constructor_concat_tag@1@AEBV01@QEBG_K23@Z 0000000180004864 f i Executor.obj
 0001:00003978       ??0JpErrorBase@@QEAA@AEBV0@@Z 0000000180004978 f i Executor.obj
 0001:00003988       ??0SourceCodePos@@QEAA@PEBD0H@Z 0000000180004988 f i Executor.obj
 0001:00003998       ??0SysError@@QEAA@AEBV0@@Z 0000000180004998 f i Executor.obj
 0001:000039d4       ??0any@tstrings@@QEAA@PEBD@Z 00000001800049d4 f i Executor.obj
 0001:00003acc       ??0any@tstrings@@QEAA@XZ   0000000180004acc f i Executor.obj
 0001:00003ae8       ??0runtime_error@std@@QEAA@AEBV01@@Z 0000000180004ae8 f i Executor.obj
 0001:00003b24       ??1?$JpError@VSysError@@@@UEAA@XZ 0000000180004b24 f i Executor.obj
 0001:00003bac       ??1?$_Tidy_guard@V?$vector@GV?$allocator@G@std@@@std@@@std@@QEAA@XZ 0000000180004bac f i Executor.obj
 0001:00003c10       ??1?$vector@GV?$allocator@G@std@@@std@@QEAA@XZ 0000000180004c10 f i Executor.obj
 0001:00003c70       ??1?$vector@V?$basic_string@GU?$char_traits@G@std@@V?$allocator@G@2@@std@@V?$allocator@V?$basic_string@GU?$char_traits@G@std@@V?$allocator@G@2@@std@@@2@@std@@QEAA@XZ 0000000180004c70 f i Executor.obj
 0001:00003c78       ??_E?$JpError@VSysError@@@@W7EAAPEAXI@Z 0000000180004c78 f i Executor.obj
 0001:00003c84       ??_E?$JpError@VSysError@@@@UEAAPEAXI@Z 0000000180004c84 f i Executor.obj
 0001:00003c84       ??_G?$JpError@VSysError@@@@UEAAPEAXI@Z 0000000180004c84 f i Executor.obj
 0001:00003cb8       ?_Change_array@?$vector@GV?$allocator@G@std@@@std@@AEAAXQEAG_K1@Z 0000000180004cb8 f i Executor.obj
 0001:00003d44       ?_Change_array@?$vector@V?$basic_string@GU?$char_traits@G@std@@V?$allocator@G@2@@std@@V?$allocator@V?$basic_string@GU?$char_traits@G@std@@V?$allocator@G@2@@std@@@2@@std@@AEAAXQEAV?$basic_string@GU?$char_traits@G@std@@V?$allocator@G@2@@2@_K1@Z 0000000180004d44 f i Executor.obj
 0001:00003df4       ?_Tidy@?$vector@V?$basic_string@GU?$char_traits@G@std@@V?$allocator@G@2@@std@@V?$allocator@V?$basic_string@GU?$char_traits@G@std@@V?$allocator@G@2@@std@@@2@@std@@AEAAXXZ 0000000180004df4 f i Executor.obj
 0001:00003e80       ?_Xlength@?$vector@EV?$allocator@E@std@@@std@@CAXXZ 0000000180004e80 f i ResourceEditor.obj
 0001:00003e80       ?_Xlength@?$vector@GV?$allocator@G@std@@@std@@CAXXZ 0000000180004e80 f i Executor.obj
 0001:00003e80       ?_Xlength@?$vector@V?$basic_string@GU?$char_traits@G@std@@V?$allocator@G@2@@std@@V?$allocator@V?$basic_string@GU?$char_traits@G@std@@V?$allocator@G@2@@std@@@2@@std@@CAXXZ 0000000180004e80 f i Executor.obj
 0001:00003e94       ?deallocate@?$allocator@G@std@@QEAAXQEAG_K@Z 0000000180004e94 f i Executor.obj
 0001:00003ed4       ?deallocate@?$allocator@V?$basic_string@GU?$char_traits@G@std@@V?$allocator@G@2@@std@@@std@@QEAAXQEAV?$basic_string@GU?$char_traits@G@std@@V?$allocator@G@2@@2@_K@Z 0000000180004ed4 f i Executor.obj
 0001:00003f18       ?log@Logger@@QEBAXW4LogLevel@1@PEBGH1AEBVany@tstrings@@@Z 0000000180004f18 f i Executor.obj
 0001:00003fa0       ?rawMessage@?$JpError@VError@msi@@@@UEBAPEBDXZ 0000000180004fa0 f i MsiCA.obj
 0001:00003fa0       ?rawMessage@?$JpError@VNoMoreItemsError@msi@@@@UEBAPEBDXZ 0000000180004fa0 f i MsiDb.obj
 0001:00003fa0       ?rawMessage@?$JpError@VSysError@@@@UEBAPEBDXZ 0000000180004fa0 f i Executor.obj
 0001:00003fa0       ?rawMessage@?$JpError@Vruntime_error@std@@@@UEBAPEBDXZ 0000000180004fa0 f i Guid.obj
 0001:00003fb4       ?what@?$JpError@VSysError@@@@UEBAPEBDXZ 0000000180004fb4 f i Executor.obj
 0001:00003fb4       ?what@?$JpError@Vruntime_error@std@@@@UEBAPEBDXZ 0000000180004fb4 f i Guid.obj
 0001:00003fc4       wmemchr                    0000000180004fc4 f i Executor.obj
 0001:000040dc       ??$_Reallocate_grow_by@V<lambda_1>@?1??append@?$basic_string@GU?$char_traits@G@std@@V?$allocator@G@2@@std@@QEAAAEAV34@QEBG_K@Z@PEBG_K@?$basic_string@GU?$char_traits@G@std@@V?$allocator@G@2@@std@@AEAAAEAV01@_KV<lambda_1>@?1??append@01@QEAAAEAV01@QEBG0@Z@PEBG_K@Z 00000001800050dc f i FileUtils.obj
 0001:00004264       ??$_Reallocate_grow_by@V<lambda_1>@?1??append@?$basic_string@GU?$char_traits@G@std@@V?$allocator@G@2@@std@@QEAAAEAV34@_KG@Z@_KG@?$basic_string@GU?$char_traits@G@std@@V?$allocator@G@2@@std@@AEAAAEAV01@_KV<lambda_1>@?1??append@01@QEAAAEAV01@0G@Z@_KG@Z 0000000180005264 f i FileUtils.obj
 0001:000043e8       ??$_Traits_find_last_of@U?$char_traits@G@std@@$00@std@@YA_KQEBG_K101@Z 00000001800053e8 f i FileUtils.obj
 0001:00004500       ?append@?$basic_string@GU?$char_traits@G@std@@V?$allocator@G@2@@std@@QEAAAEAV12@QEBG_K@Z 0000000180005500 f i FileUtils.obj
 0001:0000457c       ?append@?$basic_string@GU?$char_traits@G@std@@V?$allocator@G@2@@std@@QEAAAEAV12@_KG@Z 000000018000557c f i FileUtils.obj
 0001:000045f4       ?basename@FileUtils@@YA?AV?$basic_string@GU?$char_traits@G@std@@V?$allocator@G@2@@std@@AEBV23@@Z 00000001800055f4 f   FileUtils.obj
 0001:000046c8       ?combinePath@FileUtils@@YA?AV?$basic_string@GU?$char_traits@G@std@@V?$allocator@G@2@@std@@AEBV23@0@Z 00000001800056c8 f   FileUtils.obj
 0001:000049c0       ?removeTrailingSlash@FileUtils@@YA?AV?$basic_string@GU?$char_traits@G@std@@V?$allocator@G@2@@std@@AEBV23@@Z 00000001800059c0 f   FileUtils.obj
 0001:00004a74       ??$?HGU?$char_traits@G@std@@V?$allocator@G@1@@std@@YA?AV?$basic_string@GU?$char_traits@G@std@@V?$allocator@G@2@@0@$$QEAV10@QEBG@Z 0000000180005a74 f i Guid.obj
 0001:00004af4       ??$?HGU?$char_traits@G@std@@V?$allocator@G@1@@std@@YA?AV?$basic_string@GU?$char_traits@G@std@@V?$allocator@G@2@@0@QEBGAEBV10@@Z 0000000180005af4 f i Guid.obj
 0001:00004b78       ??$?MGU?$char_traits@G@std@@V?$allocator@G@1@@std@@YA_NAEBV?$basic_string@GU?$char_traits@G@std@@V?$allocator@G@2@@0@0@Z 0000000180005b78 f i Guid.obj
 0001:00004be0       ??$_Reallocate_grow_by@V<lambda_1>@?1??insert@?$basic_string@GU?$char_traits@G@std@@V?$allocator@G@2@@std@@QEAAAEAV34@_K0G@Z@_K_KG@?$basic_string@GU?$char_traits@G@std@@V?$allocator@G@2@@std@@AEAAAEAV01@_KV<lambda_1>@?1??insert@01@QEAAAEAV01@00G@Z@_K2G@Z 0000000180005be0 f i Guid.obj
 0001:00004d44       ??0?$JpError@Vruntime_error@std@@@@QEAA@AEBV0@@Z 0000000180005d44 f i Guid.obj
 0001:00004dd4       ??0?$JpError@Vruntime_error@std@@@@QEAA@AEBVruntime_error@std@@AEBUSourceCodePos@@@Z 0000000180005dd4 f i Guid.obj
 0001:00004e54       ??0Guid@@QEAA@AEBV?$basic_string@GU?$char_traits@G@std@@V?$allocator@G@2@@std@@@Z 0000000180005e54 f   Guid.obj
 0001:000050a4       ??1?$JpError@Vruntime_error@std@@@@UEAA@XZ 00000001800060a4 f i Guid.obj
 0001:0000512c       ??4?$basic_string@GU?$char_traits@G@std@@V?$allocator@G@2@@std@@QEAAAEAV01@AEBV01@@Z 000000018000612c f i Guid.obj
 0001:000051a4       ??6any@tstrings@@QEAAAEAV01@AEBV?$basic_string@GU?$char_traits@G@std@@V?$allocator@G@2@@std@@@Z 00000001800061a4 f i Guid.obj
 0001:000051d0       ??R<lambda_1>@?1??insert@?$basic_string@GU?$char_traits@G@std@@V?$allocator@G@2@@std@@QEAAAEAV23@_K0G@Z@QEBA@QEAGQEBG000G@Z 00000001800061d0 f i Guid.obj
 0001:00005258       ??_E?$JpError@Vruntime_error@std@@@@W7EAAPEAXI@Z 0000000180006258 f i Guid.obj
 0001:00005264       ??_E?$JpError@Vruntime_error@std@@@@UEAAPEAXI@Z 0000000180006264 f i Guid.obj
 0001:00005264       ??_G?$JpError@Vruntime_error@std@@@@UEAAPEAXI@Z 0000000180006264 f i Guid.obj
 0001:00005378       ?insert@?$basic_string@GU?$char_traits@G@std@@V?$allocator@G@2@@std@@QEAAAEAV12@_K0G@Z 0000000180006378 f i Guid.obj
 0001:00005424       ?makeException@@YA?AV?$JpError@Vruntime_error@std@@@@AEBV?$basic_string@DU?$char_traits@D@std@@V?$allocator@D@2@@std@@AEBUSourceCodePos@@@Z 0000000180006424 f i Guid.obj
 0001:000054b0       ?makeException@@YA?AV?$JpError@Vruntime_error@std@@@@AEBVany@tstrings@@AEBUSourceCodePos@@@Z 00000001800064b0 f i Guid.obj
 0001:00005574       ?makeException@@YA?AV?$JpError@Vruntime_error@std@@@@PEBDAEBUSourceCodePos@@@Z 0000000180006574 f i Guid.obj
 0001:0000562c       ?toString@Guid@@QEBA?AV?$basic_string@GU?$char_traits@G@std@@V?$allocator@G@2@@std@@H@Z 000000018000662c f   Guid.obj
 0001:00005b54       wmemcmp                    0000000180006b54 f i Guid.obj
 0001:00005c80       ?ChangeIcon@@YA_NPEAXAEBV?$basic_string@GU?$char_traits@G@std@@V?$allocator@G@2@@std@@@Z 0000000180006c80 f   IconSwap.obj
 0001:00005f64       ?PrintError@@YAXXZ         0000000180006f64 f   IconSwap.obj
 0001:00005fc4       __local_stdio_printf_options 0000000180006fc4 f i IconSwap.obj
 0001:00005fcc       printf                     0000000180006fcc f i IconSwap.obj
 0001:00006020       ??$_Emplace_reallocate@V?$basic_string@GU?$char_traits@G@std@@V?$allocator@G@2@@std@@@?$vector@V?$basic_string@GU?$char_traits@G@std@@V?$allocator@G@2@@std@@V?$allocator@V?$basic_string@GU?$char_traits@G@std@@V?$allocator@G@2@@std@@@2@@std@@AEAAPEAV?$basic_string@GU?$char_traits@G@std@@V?$allocator@G@2@@1@QEAV21@$$QEAV21@@Z 0000000180007020 f i JniUtils.obj
 0001:000061e8       ??1?$unique_ptr@UJniObjWithEnv@jni@@ULocalRefDeleter@12@@std@@QEAA@XZ 00000001800071e8 f i JniUtils.obj
 0001:00006224       ?toJString@jni@@YAPEAV_jstring@@PEAUJNIEnv_@@AEBV?$basic_string@GU?$char_traits@G@std@@V?$allocator@G@2@@std@@@Z 0000000180007224 f   JniUtils.obj
 0001:000062bc       ?toUnicodeString@jni@@YA?AV?$basic_string@GU?$char_traits@G@std@@V?$allocator@G@2@@std@@PEAUJNIEnv_@@PEAV_jstring@@@Z 00000001800072bc f   JniUtils.obj
 0001:000063bc       ?toUnicodeStringArray@jni@@YA?AV?$vector@V?$basic_string@GU?$char_traits@G@std@@V?$allocator@G@2@@std@@V?$allocator@V?$basic_string@GU?$char_traits@G@std@@V?$allocator@G@2@@std@@@2@@std@@PEAUJNIEnv_@@PEAV_jobjectArray@@@Z 00000001800073bc f   JniUtils.obj
 0001:00006518       ??$endl@DU?$char_traits@D@std@@@std@@YAAEAV?$basic_ostream@DU?$char_traits@D@std@@@0@AEAV10@@Z 0000000180007518 f i Log.obj
 0001:00006550       ??0LogEvent@@QEAA@XZ       0000000180007550 f   Log.obj
 0001:00006828       ??1LogEvent@@QEAA@XZ       0000000180007828 f i Log.obj
 0001:00006860       ??6?$basic_ostream@GU?$char_traits@G@std@@@std@@QEAAAEAV01@G@Z 0000000180007860 f i Log.obj
 0001:00006a48       ??_ELogAppender@@UEAAPEAXI@Z 0000000180007a48 f i Log.obj
 0001:00006a48       ??_GLogAppender@@UEAAPEAXI@Z 0000000180007a48 f i Log.obj
 0001:00006a74       ??_EStreamLogAppender@@UEAAPEAXI@Z 0000000180007a74 f i Log.obj
 0001:00006a74       ??_GStreamLogAppender@@UEAAPEAXI@Z 0000000180007a74 f i Log.obj
 0001:00006aa0       ?append@StreamLogAppender@@UEAAXAEBULogEvent@@@Z 0000000180007aa0 f   Log.obj
 0001:00006d40       ?assign@?$basic_string@GU?$char_traits@G@std@@V?$allocator@G@2@@std@@QEAAAEAV12@QEBG@Z 0000000180007d40 f i Log.obj
 0001:00006dc4       ?defaultLogger@Logger@@SAAEAV1@XZ 0000000180007dc4 f   Log.obj
 0001:00006e38       ?isLoggable@Logger@@QEBA_NW4LogLevel@1@@Z 0000000180007e38 f   Log.obj
 0001:00006e40       ?log@Logger@@QEBAXW4LogLevel@1@PEBGH1AEBV?$basic_string@GU?$char_traits@G@std@@V?$allocator@G@2@@std@@@Z 0000000180007e40 f   Log.obj
 0001:00007064       ??$?0AEBUpiecewise_construct_t@std@@V?$tuple@AEBV?$basic_string@GU?$char_traits@G@std@@V?$allocator@G@2@@std@@@1@V?$tuple@$$V@1@@?$_Tree_temp_node@V?$allocator@U?$_Tree_node@U?$pair@$$CBV?$basic_string@GU?$char_traits@G@std@@V?$allocator@G@2@@std@@V12@@std@@PEAX@std@@@std@@@std@@QEAA@AEAV?$allocator@U?$_Tree_node@U?$pair@$$CBV?$basic_string@GU?$char_traits@G@std@@V?$allocator@G@2@@std@@V12@@std@@PEAX@std@@@1@PEAU?$_Tree_node@U?$pair@$$CBV?$basic_string@GU?$char_traits@G@std@@V?$allocator@G@2@@std@@V12@@std@@PEAX@1@AEBUpiecewise_construct_t@1@$$QEAV?$tuple@AEBV?$basic_string@GU?$char_traits@G@std@@V?$allocator@G@2@@std@@@1@$$QEAV?$tuple@$$V@1@@Z 0000000180008064 f i MsiCA.obj
 0001:00007128       ??$_Erase_tree@V?$allocator@U?$_Tree_node@U?$pair@$$CBV?$basic_string@GU?$char_traits@G@std@@V?$allocator@G@2@@std@@V12@@std@@PEAX@std@@@std@@@?$_Tree_val@U?$_Tree_simple_types@U?$pair@$$CBV?$basic_string@GU?$char_traits@G@std@@V?$allocator@G@2@@std@@V12@@std@@@std@@@std@@QEAAXAEAV?$allocator@U?$_Tree_node@U?$pair@$$CBV?$basic_string@GU?$char_traits@G@std@@V?$allocator@G@2@@std@@V12@@std@@PEAX@std@@@1@PEAU?$_Tree_node@U?$pair@$$CBV?$basic_string@GU?$char_traits@G@std@@V?$allocator@G@2@@std@@V12@@std@@PEAX@1@@Z 0000000180008128 f i MsiCA.obj
 0001:000071a8       ??$_Find_lower_bound@V?$basic_string@GU?$char_traits@G@std@@V?$allocator@G@2@@std@@@?$_Tree@V?$_Tmap_traits@V?$basic_string@GU?$char_traits@G@std@@V?$allocator@G@2@@std@@V12@U?$less@V?$basic_string@GU?$char_traits@G@std@@V?$allocator@G@2@@std@@@2@V?$allocator@U?$pair@$$CBV?$basic_string@GU?$char_traits@G@std@@V?$allocator@G@2@@std@@V12@@std@@@2@$0A@@std@@@std@@IEBA?AU?$_Tree_find_result@PEAU?$_Tree_node@U?$pair@$$CBV?$basic_string@GU?$char_traits@G@std@@V?$allocator@G@2@@std@@V12@@std@@PEAX@std@@@1@AEBV?$basic_string@GU?$char_traits@G@std@@V?$allocator@G@2@@1@@Z 00000001800081a8 f i MsiCA.obj
 0001:00007214       ??$_Try_emplace@AEBV?$basic_string@GU?$char_traits@G@std@@V?$allocator@G@2@@std@@$$V@?$map@V?$basic_string@GU?$char_traits@G@std@@V?$allocator@G@2@@std@@V12@U?$less@V?$basic_string@GU?$char_traits@G@std@@V?$allocator@G@2@@std@@@2@V?$allocator@U?$pair@$$CBV?$basic_string@GU?$char_traits@G@std@@V?$allocator@G@2@@std@@V12@@std@@@2@@std@@AEAA?AU?$pair@PEAU?$_Tree_node@U?$pair@$$CBV?$basic_string@GU?$char_traits@G@std@@V?$allocator@G@2@@std@@V12@@std@@PEAX@std@@_N@1@AEBV?$basic_string@GU?$char_traits@G@std@@V?$allocator@G@2@@1@@Z 0000000180008214 f i MsiCA.obj
 0001:00007324       ??$makeException@VError@msi@@@@YA?AV?$JpError@VError@msi@@@@AEBVError@msi@@AEBUSourceCodePos@@@Z 0000000180008324 f i MsiCA.obj
 0001:0000733c       ??0?$JpError@VError@msi@@@@QEAA@AEBV0@@Z 000000018000833c f i MsiCA.obj
 0001:000073dc       ??0?$JpError@VError@msi@@@@QEAA@AEBVError@msi@@AEBUSourceCodePos@@@Z 00000001800083dc f i MsiCA.obj
 0001:0000746c       ??0?$basic_string@DU?$char_traits@D@std@@V?$allocator@D@2@@std@@QEAA@QEBD@Z 000000018000846c f i MsiCA.obj
 0001:000074b0       ??0Error@msi@@QEAA@AEBV01@@Z 00000001800084b0 f i MsiCA.obj
 0001:000074fc       ??1?$JpError@VError@msi@@@@UEAA@XZ 00000001800084fc f i MsiCA.obj
 0001:00007584       ??1?$_Alloc_construct_ptr@V?$allocator@U?$_Tree_node@U?$pair@$$CBV?$basic_string@GU?$char_traits@G@std@@V?$allocator@G@2@@std@@V12@@std@@PEAX@std@@@std@@@std@@QEAA@XZ 0000000180008584 f i MsiCA.obj
 0001:00007584       ??1?$_Tree_temp_node_alloc@V?$allocator@U?$_Tree_node@U?$pair@$$CBV?$basic_string@GU?$char_traits@G@std@@V?$allocator@G@2@@std@@V12@@std@@PEAX@std@@@std@@@std@@QEAA@XZ 0000000180008584 f i MsiCA.obj
 0001:000075a0       ??1DatabaseRecord@msi@@QEAA@XZ 00000001800085a0 f i MsiCA.obj
 0001:000075b8       ??_E?$JpError@VError@msi@@@@W7EAAPEAXI@Z 00000001800085b8 f i MsiCA.obj
 0001:000075c4       ??_E?$JpError@VError@msi@@@@UEAAPEAXI@Z 00000001800085c4 f i MsiCA.obj
 0001:000075c4       ??_G?$JpError@VError@msi@@@@UEAAPEAXI@Z 00000001800085c4 f i MsiCA.obj
 0001:000075f8       ??_EError@msi@@UEAAPEAXI@Z 00000001800085f8 f i MsiCA.obj
 0001:000075f8       ??_ENoMoreItemsError@msi@@UEAAPEAXI@Z 00000001800085f8 f i MsiDb.obj
 0001:000075f8       ??_GError@msi@@UEAAPEAXI@Z 00000001800085f8 f i MsiCA.obj
 0001:000075f8       ??_GNoMoreItemsError@msi@@UEAAPEAXI@Z 00000001800085f8 f i MsiDb.obj
 0001:0000763c       ?_Insert_node@?$_Tree_val@U?$_Tree_simple_types@U?$pair@$$CBV?$basic_string@GU?$char_traits@G@std@@V?$allocator@G@2@@std@@V12@@std@@@std@@@std@@QEAAPEAU?$_Tree_node@U?$pair@$$CBV?$basic_string@GU?$char_traits@G@std@@V?$allocator@G@2@@std@@V12@@std@@PEAX@2@U?$_Tree_id@PEAU?$_Tree_node@U?$pair@$$CBV?$basic_string@GU?$char_traits@G@std@@V?$allocator@G@2@@std@@V12@@std@@PEAX@std@@@2@QEAU32@@Z 000000018000863c f i MsiCA.obj
 0001:00007868       ?_Throw_tree_length_error@std@@YAXXZ 0000000180008868 f i MsiCA.obj
 0001:0000787c       ?what@?$JpError@VError@msi@@@@UEBAPEBDXZ 000000018000887c f i MsiCA.obj
 0001:0000787c       ?what@?$JpError@VNoMoreItemsError@msi@@@@UEBAPEBDXZ 000000018000887c f i MsiDb.obj
 0001:0000788c       ??$?6I@any@tstrings@@QEAAAEAV01@I@Z 000000018000888c f i MsiDb.obj
 0001:000078a4       ??$_Reallocate_grow_by@V<lambda_1>@?1??push_back@?$basic_string@DU?$char_traits@D@std@@V?$allocator@D@2@@std@@QEAAXD@Z@D@?$basic_string@DU?$char_traits@D@std@@V?$allocator@D@2@@std@@AEAAAEAV01@_KV<lambda_1>@?1??push_back@01@QEAAXD@Z@D@Z 00000001800088a4 f i MsiDb.obj
 0001:000079e4       ??$makeException@VNoMoreItemsError@msi@@@@YA?AV?$JpError@VNoMoreItemsError@msi@@@@AEBVNoMoreItemsError@msi@@AEBUSourceCodePos@@@Z 00000001800089e4 f i MsiDb.obj
 0001:000079fc       ??$use_facet@V?$codecvt@DDU_Mbstatet@@@std@@@std@@YAAEBV?$codecvt@DDU_Mbstatet@@@0@AEBVlocale@0@@Z 00000001800089fc f i MsiDb.obj
 0001:00007adc       ??0?$JpError@VNoMoreItemsError@msi@@@@QEAA@AEBV0@@Z 0000000180008adc f i MsiDb.obj
 0001:00007b7c       ??0?$JpError@VNoMoreItemsError@msi@@@@QEAA@AEBVNoMoreItemsError@msi@@AEBUSourceCodePos@@@Z 0000000180008b7c f i MsiDb.obj
 0001:00007c0c       ??0Database@msi@@QEAA@AEBV?$basic_string@GU?$char_traits@G@std@@V?$allocator@G@2@@std@@@Z 0000000180008c0c f   MsiDb.obj
 0001:00007c60       ??0DatabaseView@msi@@QEAA@AEBVDatabase@1@AEBV?$basic_string@GU?$char_traits@G@std@@V?$allocator@G@2@@std@@AEBVDatabaseRecord@1@@Z 0000000180008c60 f   MsiDb.obj
 0001:00007e38       ??0NoMoreItemsError@msi@@QEAA@AEBV01@@Z 0000000180008e38 f i MsiDb.obj
 0001:00007e90       ??0NoMoreItemsError@msi@@QEAA@AEBVany@tstrings@@@Z 0000000180008e90 f i MsiDb.obj
 0001:00007eb8       ??1?$JpError@VNoMoreItemsError@msi@@@@UEAA@XZ 0000000180008eb8 f i MsiDb.obj
 0001:00007f40       ??1?$basic_filebuf@DU?$char_traits@D@std@@@std@@UEAA@XZ 0000000180008f40 f i MsiDb.obj
 0001:00007fa4       ??1DatabaseView@msi@@QEAA@XZ 0000000180008fa4 f i MsiDb.obj
 0001:00007fc8       ??_E?$JpError@VNoMoreItemsError@msi@@@@W7EAAPEAXI@Z 0000000180008fc8 f i MsiDb.obj
 0001:00007fd4       ??_E?$JpError@VNoMoreItemsError@msi@@@@UEAAPEAXI@Z 0000000180008fd4 f i MsiDb.obj
 0001:00007fd4       ??_G?$JpError@VNoMoreItemsError@msi@@@@UEAAPEAXI@Z 0000000180008fd4 f i MsiDb.obj
 0001:00008008       ??_E?$basic_filebuf@DU?$char_traits@D@std@@@std@@UEAAPEAXI@Z 0000000180009008 f i MsiDb.obj
 0001:00008008       ??_G?$basic_filebuf@DU?$char_traits@D@std@@@std@@UEAAPEAXI@Z 0000000180009008 f i MsiDb.obj
 0001:0000803c       ?_Endwrite@?$basic_filebuf@DU?$char_traits@D@std@@@std@@IEAA_NXZ 000000018000903c f i MsiDb.obj
 0001:00008104       ?_Init@?$basic_filebuf@DU?$char_traits@D@std@@@std@@IEAAXPEAU_iobuf@@W4_Initfl@12@@Z 0000000180009104 f i MsiDb.obj
 0001:000081a0       ?_Lock@?$basic_filebuf@DU?$char_traits@D@std@@@std@@UEAAXXZ 00000001800091a0 f i MsiDb.obj
 0001:000081bc       ?_Unlock@?$basic_filebuf@DU?$char_traits@D@std@@@std@@UEAAXXZ 00000001800091bc f i MsiDb.obj
 0001:000081d8       ?close@?$basic_filebuf@DU?$char_traits@D@std@@@std@@QEAAPEAV12@XZ 00000001800091d8 f i MsiDb.obj
 0001:00008284       ?fetch@DatabaseRecord@msi@@QEAAAEAV12@AEAVDatabaseView@2@@Z 0000000180009284 f   MsiDb.obj
 0001:000082c8       ?fetch@DatabaseView@msi@@QEAA?AVDatabaseRecord@2@XZ 00000001800092c8 f   MsiDb.obj
 0001:000083b8       ?getFieldCount@DatabaseRecord@msi@@QEBAIXZ 00000001800093b8 f   MsiDb.obj
 0001:00008468       ?getProperty@Database@msi@@QEBA?AV?$basic_string@GU?$char_traits@G@std@@V?$allocator@G@2@@std@@AEBV34@@Z 0000000180009468 f   MsiDb.obj
 0001:00008664       ?imbue@?$basic_filebuf@DU?$char_traits@D@std@@@std@@MEAAXAEBVlocale@2@@Z 0000000180009664 f i MsiDb.obj
 0001:000087a0       ?overflow@?$basic_filebuf@DU?$char_traits@D@std@@@std@@MEAAHH@Z 00000001800097a0 f i MsiDb.obj
 0001:00008920       ?pbackfail@?$basic_filebuf@DU?$char_traits@D@std@@@std@@MEAAHH@Z 0000000180009920 f i MsiDb.obj
 0001:00008a2c       ?seekoff@?$basic_filebuf@DU?$char_traits@D@std@@@std@@MEAA?AV?$fpos@U_Mbstatet@@@2@_JHH@Z 0000000180009a2c f i MsiDb.obj
 0001:00008b18       ?seekpos@?$basic_filebuf@DU?$char_traits@D@std@@@std@@MEAA?AV?$fpos@U_Mbstatet@@@2@V32@H@Z 0000000180009b18 f i MsiDb.obj
 0001:00008bd0       ?setbuf@?$basic_filebuf@DU?$char_traits@D@std@@@std@@MEAAPEAV?$basic_streambuf@DU?$char_traits@D@std@@@2@PEAD_J@Z 0000000180009bd0 f i MsiDb.obj
 0001:00008c28       ?sync@?$basic_filebuf@DU?$char_traits@D@std@@@std@@MEAAHXZ 0000000180009c28 f i MsiDb.obj
 0001:00008c74       ?tryFetch@DatabaseView@msi@@QEAA?AVDatabaseRecord@2@XZ 0000000180009c74 f   MsiDb.obj
 0001:00008d84       ?uflow@?$basic_filebuf@DU?$char_traits@D@std@@@std@@MEAAHXZ 0000000180009d84 f i MsiDb.obj
 0001:00009020       ?underflow@?$basic_filebuf@DU?$char_traits@D@std@@@std@@MEAAHXZ 000000018000a020 f i MsiDb.obj
 0001:0000908c       ?xsgetn@?$basic_filebuf@DU?$char_traits@D@std@@@std@@MEAA_JPEAD_J@Z 000000018000a08c f i MsiDb.obj
 0001:000091bc       ?xsputn@?$basic_filebuf@DU?$char_traits@D@std@@@std@@MEAA_JPEBD_J@Z 000000018000a1bc f i MsiDb.obj
 0001:0000926c       ??$?6K@any@tstrings@@QEAAAEAV01@K@Z 000000018000a26c f i MsiUtils.obj
 0001:00009284       ??$_Construct_n@$$V@?$vector@GV?$allocator@G@std@@@std@@AEAAX_K@Z 000000018000a284 f i MsiUtils.obj
 0001:00009320       ??$_Resize@U_Value_init_tag@std@@@?$vector@GV?$allocator@G@std@@@std@@AEAAX_KAEBU_Value_init_tag@1@@Z 000000018000a320 f i MsiUtils.obj
 0001:00009394       ??$_Resize_reallocate@U_Value_init_tag@std@@@?$vector@GV?$allocator@G@std@@@std@@AEAAX_KAEBU_Value_init_tag@1@@Z 000000018000a394 f i MsiUtils.obj
 0001:00009694       ??0Error@msi@@QEAA@AEBV?$basic_string@DU?$char_traits@D@std@@V?$allocator@D@2@@std@@I@Z 000000018000a694 f   MsiUtils.obj
 0001:0000976c       ??0Error@msi@@QEAA@AEBVany@tstrings@@I@Z 000000018000a76c f   MsiUtils.obj
 0001:000098b8       ??1?$unique_ptr@PEAUHINSTANCE__@@ULibraryReleaser@Dll@@@std@@QEAA@XZ 000000018000a8b8 f i MsiUtils.obj
 0001:000098d0       ??1StringResource@@QEAA@XZ 000000018000a8d0 f i MsiUtils.obj
 0001:000098f0       ?closeMSIHANDLE@msi@@YAXK@Z 000000018000a8f0 f   MsiUtils.obj
 0001:000099e0       ?getString@DatabaseRecord@msi@@QEBA?AV?$basic_string@GU?$char_traits@G@std@@V?$allocator@G@2@@std@@I@Z 000000018000a9e0 f   MsiUtils.obj
 0001:00009f3c       ??0PlatformLogEvent@@QEAA@XZ 000000018000af3c f   PlatformLogEvent.obj
 0001:00009f5c       ?appendFormatted@LogEvent@@CAXAEBUPlatformLogEvent@@AEAV?$basic_string@GU?$char_traits@G@std@@V?$allocator@G@2@@std@@@Z 000000018000af5c f   PlatformLogEvent.obj
 0001:0000a030       ?init@LogEvent@@CAXAEAUPlatformLogEvent@@@Z 000000018000b030 f   PlatformLogEvent.obj
 0001:0000a064       ?initializeLogging@Logger@@CAXXZ 000000018000b064 f   PlatformLogEvent.obj
 0001:0000a128       ?initializingLogging@Logger@@CAXXZ 000000018000b128 f   PlatformLogEvent.obj
 0001:0000a190       ??$?6PEAX@any@tstrings@@QEAAAEAV01@PEAX@Z 000000018000b190 f i ResourceEditor.obj
 0001:0000a1a8       ??$_Append_uncounted_range@V?$istreambuf_iterator@DU?$char_traits@D@std@@@std@@V12@@?$vector@EV?$allocator@E@std@@@std@@AEAAXV?$istreambuf_iterator@DU?$char_traits@D@std@@@1@V21@@Z 000000018000b1a8 f i ResourceEditor.obj
 0001:0000a2cc       ??$_Emplace_reallocate@D@?$vector@EV?$allocator@E@std@@@std@@AEAAPEAEQEAE$$QEAD@Z 000000018000b2cc f i ResourceEditor.obj
 0001:0000a3d8       ??$_Resize@U_Value_init_tag@std@@@?$vector@EV?$allocator@E@std@@@std@@AEAAX_KAEBU_Value_init_tag@1@@Z 000000018000b3d8 f i ResourceEditor.obj
 0001:0000a448       ??$_Resize_reallocate@U_Value_init_tag@std@@@?$vector@EV?$allocator@E@std@@@std@@AEAAX_KAEBU_Value_init_tag@1@@Z 000000018000b448 f i ResourceEditor.obj
 0001:0000a534       ??0?$basic_ifstream@DU?$char_traits@D@std@@@std@@QEAA@PEBGHH@Z 000000018000b534 f i ResourceEditor.obj
 0001:0000a644       ??0FileLock@ResourceEditor@@QEAA@AEBV?$basic_string@GU?$char_traits@G@std@@V?$allocator@G@2@@std@@@Z 000000018000b644 f   ResourceEditor.obj
 0001:0000a768       ??0FileLock@ResourceEditor@@QEAA@PEAX@Z 000000018000b768 f   ResourceEditor.obj
 0001:0000a77c       ??0ResourceEditor@@QEAA@XZ 000000018000b77c f   ResourceEditor.obj
 0001:0000a7d4       ??1?$_Tidy_guard@V?$vector@EV?$allocator@E@std@@@std@@@std@@QEAA@XZ 000000018000b7d4 f i ResourceEditor.obj
 0001:0000a834       ??1?$vector@EV?$allocator@E@std@@@std@@QEAA@XZ 000000018000b834 f i ResourceEditor.obj
 0001:0000a890       ??1FileLock@ResourceEditor@@QEAA@XZ 000000018000b890 f   ResourceEditor.obj
 0001:0000a9a4       ??_D?$basic_ifstream@DU?$char_traits@D@std@@@std@@QEAAXXZ 000000018000b9a4 f i ResourceEditor.obj
 0001:0000aa08       ??_E?$basic_ifstream@DU?$char_traits@D@std@@@std@@$4PPPPPPPM@A@EAAPEAXI@Z 000000018000ba08 f i ResourceEditor.obj
 0001:0000aa14       ??_E?$basic_ifstream@DU?$char_traits@D@std@@@std@@UEAAPEAXI@Z 000000018000ba14 f i ResourceEditor.obj
 0001:0000aa14       ??_G?$basic_ifstream@DU?$char_traits@D@std@@@std@@UEAAPEAXI@Z 000000018000ba14 f i ResourceEditor.obj
 0001:0000aa50       ?_Change_array@?$vector@EV?$allocator@E@std@@@std@@AEAAXQEAE_K1@Z 000000018000ba50 f i ResourceEditor.obj
 0001:0000aad4       ?apply@ResourceEditor@@QEAAAEAV1@AEBVFileLock@1@AEAV?$basic_istream@DU?$char_traits@D@std@@@std@@_J@Z 000000018000bad4 f   ResourceEditor.obj
 0001:0000acd8       ?apply@ResourceEditor@@QEAAAEAV1@AEBVFileLock@1@AEBV?$basic_string@GU?$char_traits@G@std@@V?$allocator@G@2@@std@@@Z 000000018000bcd8 f   ResourceEditor.obj
 0001:0000ad90       ?deallocate@?$allocator@E@std@@QEAAXQEAE_K@Z 000000018000bd90 f i ResourceEditor.obj
 0001:0000add0       ?id@ResourceEditor@@QEAAAEAV1@PEBG@Z 000000018000bdd0 f   ResourceEditor.obj
 0001:0000aee8       ?open@?$basic_filebuf@DU?$char_traits@D@std@@@std@@QEAAPEAV12@PEBGHH@Z 000000018000bee8 f i ResourceEditor.obj
 0001:0000afa0       ?type@ResourceEditor@@QEAAAEAV1@PEBG@Z 000000018000bfa0 f   ResourceEditor.obj
 0001:0000b0c8       ??0Resource@@QEAA@IPEBGPEAUHINSTANCE__@@@Z 000000018000c0c8 f   Resources.obj
 0001:0000b110       ??0any@tstrings@@QEAA@AEBV?$basic_string@DU?$char_traits@D@std@@V?$allocator@D@2@@std@@@Z 000000018000c110 f i Resources.obj
 0001:0000b198       ?findResource@Resource@@AEBAPEAUHRSRC__@@XZ 000000018000c198 f   Resources.obj
 0001:0000b1bc       ?getErrMsg@Resource@@AEBA?AV?$basic_string@DU?$char_traits@D@std@@V?$allocator@D@2@@std@@AEBV23@@Z 000000018000c1bc f   Resources.obj
 0001:0000b2f8       ?getPtr@Resource@@AEBAPEAXAEAK@Z 000000018000c2f8 f   Resources.obj
 0001:0000b508       ?init@Resource@@AEAAXPEBG0PEAUHINSTANCE__@@@Z 000000018000c508 f   Resources.obj
 0001:0000b6d0       ?string@StringResource@@QEBA?AV?$basic_string@GU?$char_traits@G@std@@V?$allocator@G@2@@std@@XZ 000000018000c6d0 f   Resources.obj
 0001:0000b840       ??$_Traits_rfind@U?$char_traits@G@std@@@std@@YA_KQEBG_K101@Z 000000018000c840 f i VersionInfo.obj
 0001:0000b8cc       ??0?$basic_stringstream@DU?$char_traits@D@std@@V?$allocator@D@2@@std@@QEAA@H@Z 000000018000c8cc f i VersionInfo.obj
 0001:0000b9a4       ??0?$basic_stringstream@GU?$char_traits@G@std@@V?$allocator@G@2@@std@@QEAA@XZ 000000018000c9a4 f i VersionInfo.obj
 0001:0000bb58       ??0VersionInfo@@QEAA@XZ    000000018000cb58 f   VersionInfo.obj
 0001:0000bb94       ??1?$basic_stringstream@DU?$char_traits@D@std@@V?$allocator@D@2@@std@@UEAA@XZ 000000018000cb94 f i VersionInfo.obj
 0001:0000bc0c       ??1?$basic_stringstream@GU?$char_traits@G@std@@V?$allocator@G@2@@std@@UEAA@XZ 000000018000cc0c f i VersionInfo.obj
 0001:0000bc84       ??1ResourceEditor@@QEAA@XZ 000000018000cc84 f i VersionInfo.obj
 0001:0000bdb8       ??_D?$basic_stringstream@DU?$char_traits@D@std@@V?$allocator@D@2@@std@@QEAAXXZ 000000018000cdb8 f i VersionInfo.obj
 0001:0000bddc       ??_D?$basic_stringstream@GU?$char_traits@G@std@@V?$allocator@G@2@@std@@QEAAXXZ 000000018000cddc f i VersionInfo.obj
 0001:0000be00       ??_E?$basic_stringstream@DU?$char_traits@D@std@@V?$allocator@D@2@@std@@$4PPPPPPPM@A@EAAPEAXI@Z 000000018000ce00 f i VersionInfo.obj
 0001:0000be0c       ??_E?$basic_stringstream@GU?$char_traits@G@std@@V?$allocator@G@2@@std@@$4PPPPPPPM@A@EAAPEAXI@Z 000000018000ce0c f i VersionInfo.obj
 0001:0000be18       ??_E?$basic_stringstream@DU?$char_traits@D@std@@V?$allocator@D@2@@std@@UEAAPEAXI@Z 000000018000ce18 f i VersionInfo.obj
 0001:0000be18       ??_G?$basic_stringstream@DU?$char_traits@D@std@@V?$allocator@D@2@@std@@UEAAPEAXI@Z 000000018000ce18 f i VersionInfo.obj
 0001:0000be68       ??_E?$basic_stringstream@GU?$char_traits@G@std@@V?$allocator@G@2@@std@@UEAAPEAXI@Z 000000018000ce68 f i VersionInfo.obj
 0001:0000be68       ??_G?$basic_stringstream@GU?$char_traits@G@std@@V?$allocator@G@2@@std@@UEAAPEAXI@Z 000000018000ce68 f i VersionInfo.obj
 0001:0000bf90       ?apply@VersionInfo@@QEBAAEBV1@AEBVFileLock@ResourceEditor@@@Z 000000018000cf90 f   VersionInfo.obj
 0001:0000c1a0       ?createFIXEDFILEINFO@VersionInfo@@AEBA?AUtagVS_FIXEDFILEINFO@@XZ 000000018000d1a0 f   VersionInfo.obj
 0001:0000c424       ?fillBuffer@VersionInfo@@AEBAXAEAV?$basic_ostream@DU?$char_traits@D@std@@@std@@@Z 000000018000d424 f   VersionInfo.obj
 0001:0000ca8c       ?hex@std@@YAAEAVios_base@1@AEAV21@@Z 000000018000da8c f i VersionInfo.obj
 0001:0000cab0       ?setProperty@VersionInfo@@QEAAAEAV1@AEBV?$basic_string@GU?$char_traits@G@std@@V?$allocator@G@2@@std@@0@Z 000000018000dab0 f   VersionInfo.obj
 0001:0000cb4c       ?uppercase@std@@YAAEAVios_base@1@AEAV21@@Z 000000018000db4c f i VersionInfo.obj
 0001:0000cc00       __local_stdio_scanf_options 000000018000dc00 f i VersionInfo.obj
 0001:0000cc08       swscanf_s                  000000018000dc08 f i VersionInfo.obj
 0001:0000cc58       ?freeLibrary@Dll@@SAXPEAUHINSTANCE__@@@Z 000000018000dc58 f   WinDll.obj
 0001:0000cc6c       ??0SysError@@QEAA@AEBVany@tstrings@@PEBXKPEBD@Z 000000018000dc6c f   WinErrorHandling.obj
 0001:0000cdc8       ?getSysErrorMessage@SysError@@SA?AV?$basic_string@GU?$char_traits@G@std@@V?$allocator@G@2@@std@@KPEAUHINSTANCE__@@@Z 000000018000ddc8 f   WinErrorHandling.obj
 0001:0000d2b8       ?toShortPath@FileUtils@@YA?AV?$basic_string@GU?$char_traits@G@std@@V?$allocator@G@2@@std@@AEBV23@@Z 000000018000e2b8 f   WinFileUtils.obj
 0001:0000d540       ??$?HDU?$char_traits@D@std@@V?$allocator@D@1@@std@@YA?AV?$basic_string@DU?$char_traits@D@std@@V?$allocator@D@2@@0@AEBV10@QEBD@Z 000000018000e540 f i WinSysInfo.obj
 0001:0000d5c4       ??$?HDU?$char_traits@D@std@@V?$allocator@D@1@@std@@YA?AV?$basic_string@DU?$char_traits@D@std@@V?$allocator@D@2@@0@QEBDAEBV10@@Z 000000018000e5c4 f i WinSysInfo.obj
 0001:0000d8d0       ??0?$basic_string@DU?$char_traits@D@std@@V?$allocator@D@2@@std@@QEAA@U_String_constructor_concat_tag@1@AEBV01@QEBD_K23@Z 000000018000e8d0 f i WinSysInfo.obj
 0001:0000d9c4       ?getCurrentModuleHandle@SysInfo@@YAPEAUHINSTANCE__@@XZ 000000018000e9c4 f   WinSysInfo.obj
 0001:0000dabc       ?getCurrentModulePath@SysInfo@@YA?AV?$basic_string@GU?$char_traits@G@std@@V?$allocator@G@2@@std@@XZ 000000018000eabc f   WinSysInfo.obj
 0001:0000dca8       ?getSystem32Dir@SysInfo@@YA?AV?$basic_string@GU?$char_traits@G@std@@V?$allocator@G@2@@std@@XZ 000000018000eca8 f   WinSysInfo.obj
 0001:0000dfb8       Java_jdk_jpackage_internal_WindowsRegistry_closeRegistryKey 000000018000efb8 f   WindowsRegistry.obj
 0001:0000dfc4       Java_jdk_jpackage_internal_WindowsRegistry_comparePaths 000000018000efc4 f   WindowsRegistry.obj
 0001:0000e2c8       Java_jdk_jpackage_internal_WindowsRegistry_enumRegistryValue 000000018000f2c8 f   WindowsRegistry.obj
 0001:0000e4f0       Java_jdk_jpackage_internal_WindowsRegistry_openRegistryKey 000000018000f4f0 f   WindowsRegistry.obj
 0001:0000e5e4       Java_jdk_jpackage_internal_WindowsRegistry_readDwordValue 000000018000f5e4 f   WindowsRegistry.obj
 0001:0000e848       ?lastErrorMsg@app@@YA?AV?$basic_string@DU?$char_traits@D@std@@V?$allocator@D@2@@std@@XZ 000000018000f848 f   app.obj
 0001:0000e8ac       ??0?$basic_istringstream@DU?$char_traits@D@std@@V?$allocator@D@2@@std@@QEAA@AEBV?$basic_string@DU?$char_traits@D@std@@V?$allocator@D@2@@1@H@Z 000000018000f8ac f i jpackage.obj
 0001:0000e94c       ??0?$basic_stringbuf@DU?$char_traits@D@std@@V?$allocator@D@2@@std@@QEAA@AEBV?$basic_string@DU?$char_traits@D@std@@V?$allocator@D@2@@1@H@Z 000000018000f94c f i jpackage.obj
 0001:0000e9dc       ??1?$basic_istringstream@DU?$char_traits@D@std@@V?$allocator@D@2@@std@@UEAA@XZ 000000018000f9dc f i jpackage.obj
 0001:0000ea54       ??1Database@msi@@QEAA@XZ   000000018000fa54 f i jpackage.obj
 0001:0000ea78       ??1VersionInfo@@QEAA@XZ    000000018000fa78 f i jpackage.obj
 0001:0000eaa4       ??_D?$basic_istringstream@DU?$char_traits@D@std@@V?$allocator@D@2@@std@@QEAAXXZ 000000018000faa4 f i jpackage.obj
 0001:0000eac8       ??_E?$basic_istringstream@DU?$char_traits@D@std@@V?$allocator@D@2@@std@@$4PPPPPPPM@A@EAAPEAXI@Z 000000018000fac8 f i jpackage.obj
 0001:0000ead4       ??_E?$basic_istringstream@DU?$char_traits@D@std@@V?$allocator@D@2@@std@@UEAAPEAXI@Z 000000018000fad4 f i jpackage.obj
 0001:0000ead4       ??_G?$basic_istringstream@DU?$char_traits@D@std@@V?$allocator@D@2@@std@@UEAAPEAXI@Z 000000018000fad4 f i jpackage.obj
 0001:0000eb24       ?_Init@?$basic_stringbuf@DU?$char_traits@D@std@@V?$allocator@D@2@@std@@IEAAXPEBD_KH@Z 000000018000fb24 f i jpackage.obj
 0001:0000ec20       Java_jdk_jpackage_internal_ExecutableRebrander_iconSwap 000000018000fc20 f   jpackage.obj
 0001:0000ecc0       Java_jdk_jpackage_internal_ExecutableRebrander_lockResource 000000018000fcc0 f   jpackage.obj
 0001:0000ed2c       Java_jdk_jpackage_internal_ExecutableRebrander_unlockResource 000000018000fd2c f   jpackage.obj
 0001:0000ed6c       Java_jdk_jpackage_internal_ExecutableRebrander_versionSwap 000000018000fd6c f   jpackage.obj
 0001:0000ef88       Java_jdk_jpackage_internal_ShortPathUtils_getShortPath 000000018000ff88 f   jpackage.obj
 0001:0000f000       Java_jdk_jpackage_internal_WinExeBundler_embedMSI 0000000180010000 f   jpackage.obj
 0001:0000f2f0       ??$_Reallocate_grow_by@V<lambda_1>@?1??append@?$basic_string@DU?$char_traits@D@std@@V?$allocator@D@2@@std@@QEAAAEAV34@_KD@Z@_KD@?$basic_string@DU?$char_traits@D@std@@V?$allocator@D@2@@std@@AEAAAEAV01@_KV<lambda_1>@?1??append@01@QEAAAEAV01@0D@Z@_KD@Z 00000001800102f0 f i tstrings.obj
 0001:0000f44c       ??0invalid_argument@std@@QEAA@AEBV01@@Z 000000018001044c f i tstrings.obj
 0001:0000f488       ??0invalid_argument@std@@QEAA@PEBD@Z 0000000180010488 f i tstrings.obj
 0001:0000f4d0       ??0logic_error@std@@QEAA@AEBV01@@Z 00000001800104d0 f i tstrings.obj
 0001:0000f50c       ?append@?$basic_string@DU?$char_traits@D@std@@V?$allocator@D@2@@std@@QEAAAEAV12@_KD@Z 000000018001050c f i tstrings.obj
 0001:0000f588       ?equals@tstrings@@YA_NAEBV?$basic_string@GU?$char_traits@G@std@@V?$allocator@G@2@@std@@0W4CompareType@1@@Z 0000000180010588 f   tstrings.obj
 0001:0000f80c       ?toLower@tstrings@@YA?AV?$basic_string@GU?$char_traits@G@std@@V?$allocator@G@2@@std@@AEBV23@@Z 000000018001080c f   tstrings.obj
 0001:0000fab8       ?toUtf16@tstrings@@YA?AV?$basic_string@GU?$char_traits@G@std@@V?$allocator@G@2@@std@@AEBV?$basic_string@DU?$char_traits@D@std@@V?$allocator@D@2@@3@@Z 0000000180010ab8 f   tstrings.obj
 0001:0000fad8       ?toUtf8@tstrings@@YA?AV?$basic_string@DU?$char_traits@D@std@@V?$allocator@D@2@@std@@AEBV?$basic_string@GU?$char_traits@G@std@@V?$allocator@G@2@@3@@Z 0000000180010ad8 f   tstrings.obj
 0001:0000faf8       ?unsafe_format@tstrings@@YA?AV?$basic_string@GU?$char_traits@G@std@@V?$allocator@G@2@@std@@PEBGZZ 0000000180010af8 f   tstrings.obj
 0001:0000fc28       ?winStringToUtf16@tstrings@@YA?AV?$basic_string@GU?$char_traits@G@std@@V?$allocator@G@2@@std@@AEBV23@@Z 0000000180010c28 f   tstrings.obj
 0001:0000fc63       MsiDatabaseOpenViewW       0000000180010c63 f   msi:msi.dll
 0001:0000fc69       MsiViewExecute             0000000180010c69 f   msi:msi.dll
 0001:0000fc6f       MsiViewFetch               0000000180010c6f f   msi:msi.dll
 0001:0000fc75       MsiOpenDatabaseW           0000000180010c75 f   msi:msi.dll
 0001:0000fc7b       MsiRecordGetFieldCount     0000000180010c7b f   msi:msi.dll
 0001:0000fc81       MsiCloseHandle             0000000180010c81 f   msi:msi.dll
 0001:0000fc87       MsiRecordGetStringW        0000000180010c87 f   msi:msi.dll
 0001:0000fc8d       ??1_Lockit@std@@QEAA@XZ    0000000180010c8d f   msvcprt:MSVCP140.dll
 0001:0000fc93       ?_Xlength_error@std@@YAXPEBD@Z 0000000180010c93 f   msvcprt:MSVCP140.dll
 0001:0000fc99       ?_Xout_of_range@std@@YAXPEBD@Z 0000000180010c99 f   msvcprt:MSVCP140.dll
 0001:0000fc9f       ?uncaught_exception@std@@YA_NXZ 0000000180010c9f f   msvcprt:MSVCP140.dll
 0001:0000fca8       ?_Facet_Register@std@@YAXPEAV_Facet_base@1@@Z 0000000180010ca8 f   msvcprt:locale0_implib.obj
 0001:0000fce5       ?_Getgloballocale@locale@std@@CAPEAV_Locimp@12@XZ 0000000180010ce5 f   msvcprt:MSVCP140.dll
 0001:0000fceb       ??1?$basic_streambuf@DU?$char_traits@D@std@@@std@@UEAA@XZ 0000000180010ceb f   msvcprt:MSVCP140.dll
 0001:0000fcf1       ?imbue@?$basic_streambuf@GU?$char_traits@G@std@@@std@@MEAAXAEBVlocale@2@@Z 0000000180010cf1 f   msvcprt:MSVCP140.dll
 0001:0000fcf7       ?sync@?$basic_streambuf@GU?$char_traits@G@std@@@std@@MEAAHXZ 0000000180010cf7 f   msvcprt:MSVCP140.dll
 0001:0000fcfd       ?setbuf@?$basic_streambuf@GU?$char_traits@G@std@@@std@@MEAAPEAV12@PEAG_J@Z 0000000180010cfd f   msvcprt:MSVCP140.dll
 0001:0000fd03       ?xsputn@?$basic_streambuf@GU?$char_traits@G@std@@@std@@MEAA_JPEBG_J@Z 0000000180010d03 f   msvcprt:MSVCP140.dll
 0001:0000fd09       ?xsgetn@?$basic_streambuf@GU?$char_traits@G@std@@@std@@MEAA_JPEAG_J@Z 0000000180010d09 f   msvcprt:MSVCP140.dll
 0001:0000fd0f       ?uflow@?$basic_streambuf@GU?$char_traits@G@std@@@std@@MEAAGXZ 0000000180010d0f f   msvcprt:MSVCP140.dll
 0001:0000fd15       ?showmanyc@?$basic_streambuf@GU?$char_traits@G@std@@@std@@MEAA_JXZ 0000000180010d15 f   msvcprt:MSVCP140.dll
 0001:0000fd1b       ?_Unlock@?$basic_streambuf@GU?$char_traits@G@std@@@std@@UEAAXXZ 0000000180010d1b f   msvcprt:MSVCP140.dll
 0001:0000fd21       ?_Lock@?$basic_streambuf@GU?$char_traits@G@std@@@std@@UEAAXXZ 0000000180010d21 f   msvcprt:MSVCP140.dll
 0001:0000fd27       ?imbue@?$basic_streambuf@DU?$char_traits@D@std@@@std@@MEAAXAEBVlocale@2@@Z 0000000180010d27 f   msvcprt:MSVCP140.dll
 0001:0000fd2d       ?sync@?$basic_streambuf@DU?$char_traits@D@std@@@std@@MEAAHXZ 0000000180010d2d f   msvcprt:MSVCP140.dll
 0001:0000fd33       ?setbuf@?$basic_streambuf@DU?$char_traits@D@std@@@std@@MEAAPEAV12@PEAD_J@Z 0000000180010d33 f   msvcprt:MSVCP140.dll
 0001:0000fd39       ?xsputn@?$basic_streambuf@DU?$char_traits@D@std@@@std@@MEAA_JPEBD_J@Z 0000000180010d39 f   msvcprt:MSVCP140.dll
 0001:0000fd3f       ?xsgetn@?$basic_streambuf@DU?$char_traits@D@std@@@std@@MEAA_JPEAD_J@Z 0000000180010d3f f   msvcprt:MSVCP140.dll
 0001:0000fd45       ?uflow@?$basic_streambuf@DU?$char_traits@D@std@@@std@@MEAAHXZ 0000000180010d45 f   msvcprt:MSVCP140.dll
 0001:0000fd4b       ?showmanyc@?$basic_streambuf@DU?$char_traits@D@std@@@std@@MEAA_JXZ 0000000180010d4b f   msvcprt:MSVCP140.dll
 0001:0000fd51       ?_Unlock@?$basic_streambuf@DU?$char_traits@D@std@@@std@@UEAAXXZ 0000000180010d51 f   msvcprt:MSVCP140.dll
 0001:0000fd57       ?_Lock@?$basic_streambuf@DU?$char_traits@D@std@@@std@@UEAAXXZ 0000000180010d57 f   msvcprt:MSVCP140.dll
 0001:0000fe70       __std_find_trivial_2       0000000180010e70 f   msvcprt:vector_algorithms.obj
 0001:0000fe75       ?_Fiopen@std@@YAPEAU_iobuf@@PEBGHH@Z 0000000180010e75 f   msvcprt:MSVCP140.dll
 0001:0000fe7b       ?_Xbad_alloc@std@@YAXXZ    0000000180010e7b f   msvcprt:MSVCP140.dll
 0001:0000fe81       ?setw@std@@YA?AU?$_Smanip@_J@1@_J@Z 0000000180010e81 f   msvcprt:MSVCP140.dll
 0001:0000fe88       ??2@YAPEAX_K@Z             0000000180010e88 f   MSVCRT:new_scalar.obj
 0001:0000fec4       ??3@YAXPEAX_K@Z            0000000180010ec4 f   MSVCRT:delete_scalar_size.obj
 0001:0000fec4       ??_V@YAXPEAX@Z             0000000180010ec4 f   MSVCRT:delete_array.obj
 0001:0000fecc       __GSHandlerCheck           0000000180010ecc f   MSVCRT:gshandler.obj
 0001:0000feec       __GSHandlerCheckCommon     0000000180010eec f   MSVCRT:gshandler.obj
 0001:0000ff48       __GSHandlerCheck_EH4       0000000180010f48 f   MSVCRT:gshandlereh4.obj
 0001:0000ffe0       __chkstk                   0000000180010fe0 f   MSVCRT:chkstk.obj
 0001:0000ffe0       _alloca_probe              0000000180010fe0 f   MSVCRT:chkstk.obj
 0001:00010040       __security_check_cookie    0000000180011040 f   MSVCRT:amdsecgs.obj
 0001:00010060       ??_Etype_info@@UEAAPEAXI@Z 0000000180011060 f i MSVCRT:std_type_info_static.obj
 0001:00010060       ??_Gtype_info@@UEAAPEAXI@Z 0000000180011060 f i MSVCRT:std_type_info_static.obj
 0001:0001008c       __raise_securityfailure    000000018001108c f   MSVCRT:gs_report.obj
 0001:000100c0       __report_gsfailure         00000001800110c0 f   MSVCRT:gs_report.obj
 0001:00010194       __report_rangecheckfailure 0000000180011194 f   MSVCRT:gs_report.obj
 0001:000101a8       __report_securityfailure   00000001800111a8 f   MSVCRT:gs_report.obj
 0001:0001032c       ??3@YAXPEAX@Z              000000018001132c f   MSVCRT:delete_scalar.obj
 0001:00010334       ??_U@YAPEAX_K@Z            0000000180011334 f   MSVCRT:new_array.obj
 0001:0001033c       __scrt_acquire_startup_lock 000000018001133c f   MSVCRT:utility.obj
 0001:00010378       __scrt_dllmain_after_initialize_c 0000000180011378 f   MSVCRT:utility.obj
 0001:000103ac       __scrt_dllmain_before_initialize_c 00000001800113ac f   MSVCRT:utility.obj
 0001:000103c4       __scrt_dllmain_crt_thread_attach 00000001800113c4 f   MSVCRT:utility.obj
 0001:000103ec       __scrt_dllmain_crt_thread_detach 00000001800113ec f   MSVCRT:utility.obj
 0001:00010404       __scrt_dllmain_exception_filter 0000000180011404 f   MSVCRT:utility.obj
 0001:00010464       __scrt_dllmain_uninitialize_c 0000000180011464 f   MSVCRT:utility.obj
 0001:00010494       __scrt_dllmain_uninitialize_critical 0000000180011494 f   MSVCRT:utility.obj
 0001:000104a8       __scrt_initialize_crt      00000001800114a8 f   MSVCRT:utility.obj
 0001:000104e4       __scrt_initialize_onexit_tables 00000001800114e4 f   MSVCRT:utility.obj
 0001:00010570       __scrt_is_nonwritable_in_current_image 0000000180011570 f   MSVCRT:utility.obj
 0001:00010608       __scrt_release_startup_lock 0000000180011608 f   MSVCRT:utility.obj
 0001:0001062c       __scrt_uninitialize_crt    000000018001162c f   MSVCRT:utility.obj
 0001:00010658       _onexit                    0000000180011658 f   MSVCRT:utility.obj
 0001:00010694       atexit                     0000000180011694 f   MSVCRT:utility.obj
 0001:000109bc       _DllMainCRTStartup         00000001800119bc f   MSVCRT:dll_dllmain.obj
 0001:000109fc       _guard_check_icall_nop     00000001800119fc f i MSVCRT:guard_support.obj
 0001:00010a00       __isa_available_init       0000000180011a00 f   MSVCRT:cpu_disp.obj
 0001:00010ccc       ??0bad_alloc@std@@QEAA@XZ  0000000180011ccc f i MSVCRT:throw_bad_alloc.obj
 0001:00010cec       ?__scrt_throw_std_bad_alloc@@YAXXZ 0000000180011cec f   MSVCRT:throw_bad_alloc.obj
 0001:00010d0c       _get_startup_argv_mode     0000000180011d0c f   MSVCRT:argv_mode.obj
 0001:00010d14       __scrt_is_ucrt_dll_in_use  0000000180011d14 f   MSVCRT:ucrt_detection.obj
 0001:00010d20       __crt_debugger_hook        0000000180011d20 f   MSVCRT:utility_desktop.obj
 0001:00010d28       __scrt_fastfail            0000000180011d28 f   MSVCRT:utility_desktop.obj
 0001:00010e70       __security_init_cookie     0000000180011e70 f   MSVCRT:gs_support.obj
 0001:00010f1c       DllMain                    0000000180011f1c f   MSVCRT:dll_dllmain_stub.obj
 0001:00010f40       ?__scrt_initialize_type_info@@YAXXZ 0000000180011f40 f   MSVCRT:tncleanup.obj
 0001:00010f50       ?__scrt_uninitialize_type_info@@YAXXZ 0000000180011f50 f   MSVCRT:tncleanup.obj
 0001:00010f5c       __scrt_initialize_default_local_stdio_options 0000000180011f5c f   MSVCRT:default_local_stdio_options.obj
 0001:00010f78       __scrt_get_dyn_tls_init_callback 0000000180011f78 f   MSVCRT:dyn_tls_init.obj
 0001:00010f80       _RTC_Initialize            0000000180011f80 f   MSVCRT:initsect.obj
 0001:00010fbc       _RTC_Terminate             0000000180011fbc f   MSVCRT:initsect.obj
 0001:00011000       __std_terminate            0000000180012000 f   vcruntime:VCRUNTIME140.dll
 0001:00011006       memchr                     0000000180012006 f   vcruntime:VCRUNTIME140.dll
 0001:0001100c       memcpy                     000000018001200c f   vcruntime:VCRUNTIME140.dll
 0001:00011012       memmove                    0000000180012012 f   vcruntime:VCRUNTIME140.dll
 0001:00011018       __std_exception_copy       0000000180012018 f   vcruntime:VCRUNTIME140.dll
 0001:0001101e       __std_exception_destroy    000000018001201e f   vcruntime:VCRUNTIME140.dll
 0001:00011024       _CxxThrowException         0000000180012024 f   vcruntime:VCRUNTIME140.dll
 0001:0001102a       __CxxFrameHandler4         000000018001202a f   vcruntime:VCRUNTIME140_1.dll
 0001:00011030       memset                     0000000180012030 f   vcruntime:VCRUNTIME140.dll
 0001:00011036       _purecall                  0000000180012036 f   vcruntime:VCRUNTIME140.dll
 0001:0001103c       __C_specific_handler       000000018001203c f   vcruntime:VCRUNTIME140.dll
 0001:00011042       __std_type_info_destroy_list 0000000180012042 f   vcruntime:VCRUNTIME140.dll
 0001:00011048       strlen                     0000000180012048 f   ucrt:api-ms-win-crt-string-l1-1-0.dll
 0001:0001104e       free                       000000018001204e f   ucrt:api-ms-win-crt-heap-l1-1-0.dll
 0001:00011054       malloc                     0000000180012054 f   ucrt:api-ms-win-crt-heap-l1-1-0.dll
 0001:0001105a       _callnewh                  000000018001205a f   ucrt:api-ms-win-crt-heap-l1-1-0.dll
 0001:00011060       _seh_filter_dll            0000000180012060 f   ucrt:api-ms-win-crt-runtime-l1-1-0.dll
 0001:00011066       _configure_narrow_argv     0000000180012066 f   ucrt:api-ms-win-crt-runtime-l1-1-0.dll
 0001:0001106c       _initialize_narrow_environment 000000018001206c f   ucrt:api-ms-win-crt-runtime-l1-1-0.dll
 0001:00011072       _initialize_onexit_table   0000000180012072 f   ucrt:api-ms-win-crt-runtime-l1-1-0.dll
 0001:00011078       _register_onexit_function  0000000180012078 f   ucrt:api-ms-win-crt-runtime-l1-1-0.dll
 0001:0001107e       _execute_onexit_table      000000018001207e f   ucrt:api-ms-win-crt-runtime-l1-1-0.dll
 0001:00011084       _crt_atexit                0000000180012084 f   ucrt:api-ms-win-crt-runtime-l1-1-0.dll
 0001:0001108a       _cexit                     000000018001208a f   ucrt:api-ms-win-crt-runtime-l1-1-0.dll
 0001:00011090       _initterm                  0000000180012090 f   ucrt:api-ms-win-crt-runtime-l1-1-0.dll
 0001:00011096       _initterm_e                0000000180012096 f   ucrt:api-ms-win-crt-runtime-l1-1-0.dll
 0001:0001109c       __acrt_initialize          000000018001209c f   MSVCRT:ucrt_stubs.obj
 0001:0001109c       __acrt_thread_attach       000000018001209c f   MSVCRT:ucrt_stubs.obj
 0001:0001109c       __acrt_thread_detach       000000018001209c f   MSVCRT:ucrt_stubs.obj
 0001:0001109c       __acrt_uninitialize        000000018001209c f   MSVCRT:ucrt_stubs.obj
 0001:0001109c       __acrt_uninitialize_critical 000000018001209c f   MSVCRT:ucrt_stubs.obj
 0001:0001109c       __scrt_stub_for_acrt_initialize 000000018001209c f   MSVCRT:ucrt_stubs.obj
 0001:0001109c       __scrt_stub_for_acrt_thread_attach 000000018001209c f   MSVCRT:ucrt_stubs.obj
 0001:0001109c       __scrt_stub_for_acrt_thread_detach 000000018001209c f   MSVCRT:ucrt_stubs.obj
 0001:0001109c       __scrt_stub_for_acrt_uninitialize 000000018001209c f   MSVCRT:ucrt_stubs.obj
 0001:0001109c       __scrt_stub_for_acrt_uninitialize_critical 000000018001209c f   MSVCRT:ucrt_stubs.obj
 0001:0001109c       __vcrt_initialize          000000018001209c f   MSVCRT:ucrt_stubs.obj
 0001:0001109c       __vcrt_thread_attach       000000018001209c f   MSVCRT:ucrt_stubs.obj
 0001:0001109c       __vcrt_thread_detach       000000018001209c f   MSVCRT:ucrt_stubs.obj
 0001:0001109c       __vcrt_uninitialize        000000018001209c f   MSVCRT:ucrt_stubs.obj
 0001:0001109c       __vcrt_uninitialize_critical 000000018001209c f   MSVCRT:ucrt_stubs.obj
 0001:000110a0       __scrt_stub_for_is_c_termination_complete 00000001800120a0 f   MSVCRT:ucrt_stubs.obj
 0001:000110a0       _is_c_termination_complete 00000001800120a0 f   MSVCRT:ucrt_stubs.obj
 0001:000110c0       _guard_dispatch_icall_nop  00000001800120c0 f   MSVCRT:guard_dispatch.obj
 0001:000110e0       _guard_xfg_dispatch_icall_nop 00000001800120e0 f   MSVCRT:guard_xfg_dispatch.obj
 0002:00000000       __imp_RegEnumValueW        0000000180014000     advapi32:ADVAPI32.dll
 0002:00000008       __imp_RegOpenKeyExW        0000000180014008     advapi32:ADVAPI32.dll
 0002:00000010       __imp_RegQueryValueExW     0000000180014010     advapi32:ADVAPI32.dll
 0002:00000018       __imp_RegCloseKey          0000000180014018     advapi32:ADVAPI32.dll
 0002:00000020       \177ADVAPI32_NULL_THUNK_DATA 0000000180014020     advapi32:ADVAPI32.dll
 0002:00000028       __imp_GetModuleHandleExW   0000000180014028     kernel32:KERNEL32.dll
 0002:00000030       __imp_InitializeSListHead  0000000180014030     kernel32:KERNEL32.dll
 0002:00000038       __imp_DisableThreadLibraryCalls 0000000180014038     kernel32:KERNEL32.dll
 0002:00000040       __imp_GetSystemTimeAsFileTime 0000000180014040     kernel32:KERNEL32.dll
 0002:00000048       __imp_QueryPerformanceCounter 0000000180014048     kernel32:KERNEL32.dll
 0002:00000050       __imp_IsDebuggerPresent    0000000180014050     kernel32:KERNEL32.dll
 0002:00000058       __imp_IsProcessorFeaturePresent 0000000180014058     kernel32:KERNEL32.dll
 0002:00000060       __imp_TerminateProcess     0000000180014060     kernel32:KERNEL32.dll
 0002:00000068       __imp_GetCurrentProcess    0000000180014068     kernel32:KERNEL32.dll
 0002:00000070       __imp_SetUnhandledExceptionFilter 0000000180014070     kernel32:KERNEL32.dll
 0002:00000078       __imp_UnhandledExceptionFilter 0000000180014078     kernel32:KERNEL32.dll
 0002:00000080       __imp_RtlVirtualUnwind     0000000180014080     kernel32:KERNEL32.dll
 0002:00000088       __imp_RtlLookupFunctionEntry 0000000180014088     kernel32:KERNEL32.dll
 0002:00000090       __imp_RtlCaptureContext    0000000180014090     kernel32:KERNEL32.dll
 0002:00000098       __imp_WideCharToMultiByte  0000000180014098     kernel32:KERNEL32.dll
 0002:000000a0       __imp_MultiByteToWideChar  00000001800140a0     kernel32:KERNEL32.dll
 0002:000000a8       __imp_GetLongPathNameW     00000001800140a8     kernel32:KERNEL32.dll
 0002:000000b0       __imp_GetModuleFileNameW   00000001800140b0     kernel32:KERNEL32.dll
 0002:000000b8       __imp_GetSystemDirectoryW  00000001800140b8     kernel32:KERNEL32.dll
 0002:000000c0       __imp_GetShortPathNameW    00000001800140c0     kernel32:KERNEL32.dll
 0002:000000c8       __imp_FreeLibrary          00000001800140c8     kernel32:KERNEL32.dll
 0002:000000d0       __imp_FindResourceW        00000001800140d0     kernel32:KERNEL32.dll
 0002:000000d8       __imp_SizeofResource       00000001800140d8     kernel32:KERNEL32.dll
 0002:000000e0       __imp_LockResource         00000001800140e0     kernel32:KERNEL32.dll
 0002:000000e8       __imp_LoadResource         00000001800140e8     kernel32:KERNEL32.dll
 0002:000000f0       __imp_EndUpdateResourceW   00000001800140f0     kernel32:KERNEL32.dll
 0002:000000f8       __imp_BeginUpdateResourceW 00000001800140f8     kernel32:KERNEL32.dll
 0002:00000100       __imp_GetLocalTime         0000000180014100     kernel32:KERNEL32.dll
 0002:00000108       __imp_GetCurrentProcessId  0000000180014108     kernel32:KERNEL32.dll
 0002:00000110       __imp_LoadLibraryExW       0000000180014110     kernel32:KERNEL32.dll
 0002:00000118       __imp_GetCurrentThreadId   0000000180014118     kernel32:KERNEL32.dll
 0002:00000120       __imp_UpdateResourceW      0000000180014120     kernel32:KERNEL32.dll
 0002:00000128       __imp_FormatMessageW       0000000180014128     kernel32:KERNEL32.dll
 0002:00000130       __imp_LocalFree            0000000180014130     kernel32:KERNEL32.dll
 0002:00000138       __imp_SetFilePointer       0000000180014138     kernel32:KERNEL32.dll
 0002:00000140       __imp_ReadFile             0000000180014140     kernel32:KERNEL32.dll
 0002:00000148       __imp_CreateFileW          0000000180014148     kernel32:KERNEL32.dll
 0002:00000150       __imp_GetLastError         0000000180014150     kernel32:KERNEL32.dll
 0002:00000158       __imp_CloseHandle          0000000180014158     kernel32:KERNEL32.dll
 0002:00000160       \177KERNEL32_NULL_THUNK_DATA 0000000180014160     kernel32:KERNEL32.dll
 0002:00000168       __imp_??1?$basic_streambuf@GU?$char_traits@G@std@@@std@@UEAA@XZ 0000000180014168     msvcprt:MSVCP140.dll
 0002:00000170       __imp_?sputc@?$basic_streambuf@GU?$char_traits@G@std@@@std@@QEAAGG@Z 0000000180014170     msvcprt:MSVCP140.dll
 0002:00000178       __imp_?sputn@?$basic_streambuf@GU?$char_traits@G@std@@@std@@QEAA_JPEBG_J@Z 0000000180014178     msvcprt:MSVCP140.dll
 0002:00000180       __imp_?eback@?$basic_streambuf@GU?$char_traits@G@std@@@std@@IEBAPEAGXZ 0000000180014180     msvcprt:MSVCP140.dll
 0002:00000188       __imp_?gptr@?$basic_streambuf@GU?$char_traits@G@std@@@std@@IEBAPEAGXZ 0000000180014188     msvcprt:MSVCP140.dll
 0002:00000190       __imp_?pbase@?$basic_streambuf@GU?$char_traits@G@std@@@std@@IEBAPEAGXZ 0000000180014190     msvcprt:MSVCP140.dll
 0002:00000198       __imp_?pptr@?$basic_streambuf@GU?$char_traits@G@std@@@std@@IEBAPEAGXZ 0000000180014198     msvcprt:MSVCP140.dll
 0002:000001a0       __imp_?egptr@?$basic_streambuf@GU?$char_traits@G@std@@@std@@IEBAPEAGXZ 00000001800141a0     msvcprt:MSVCP140.dll
 0002:000001a8       __imp_?gbump@?$basic_streambuf@GU?$char_traits@G@std@@@std@@IEAAXH@Z 00000001800141a8     msvcprt:MSVCP140.dll
 0002:000001b0       __imp_?setg@?$basic_streambuf@GU?$char_traits@G@std@@@std@@IEAAXPEAG00@Z 00000001800141b0     msvcprt:MSVCP140.dll
 0002:000001b8       __imp_?epptr@?$basic_streambuf@GU?$char_traits@G@std@@@std@@IEBAPEAGXZ 00000001800141b8     msvcprt:MSVCP140.dll
 0002:000001c0       __imp_?setp@?$basic_streambuf@GU?$char_traits@G@std@@@std@@IEAAXPEAG0@Z 00000001800141c0     msvcprt:MSVCP140.dll
 0002:000001c8       __imp_?setp@?$basic_streambuf@GU?$char_traits@G@std@@@std@@IEAAXPEAG00@Z 00000001800141c8     msvcprt:MSVCP140.dll
 0002:000001d0       __imp_?_Pninc@?$basic_streambuf@GU?$char_traits@G@std@@@std@@IEAAPEAGXZ 00000001800141d0     msvcprt:MSVCP140.dll
 0002:000001d8       __imp_??1?$basic_ios@DU?$char_traits@D@std@@@std@@UEAA@XZ 00000001800141d8     msvcprt:MSVCP140.dll
 0002:000001e0       __imp_?setstate@?$basic_ios@DU?$char_traits@D@std@@@std@@QEAAXH_N@Z 00000001800141e0     msvcprt:MSVCP140.dll
 0002:000001e8       __imp_?tie@?$basic_ios@DU?$char_traits@D@std@@@std@@QEBAPEAV?$basic_ostream@DU?$char_traits@D@std@@@2@XZ 00000001800141e8     msvcprt:MSVCP140.dll
 0002:000001f0       __imp_?rdbuf@?$basic_ios@DU?$char_traits@D@std@@@std@@QEBAPEAV?$basic_streambuf@DU?$char_traits@D@std@@@2@XZ 00000001800141f0     msvcprt:MSVCP140.dll
 0002:000001f8       __imp_?fill@?$basic_ios@DU?$char_traits@D@std@@@std@@QEBADXZ 00000001800141f8     msvcprt:MSVCP140.dll
 0002:00000200       __imp_??0?$basic_ios@DU?$char_traits@D@std@@@std@@IEAA@XZ 0000000180014200     msvcprt:MSVCP140.dll
 0002:00000208       __imp_??1?$basic_ios@GU?$char_traits@G@std@@@std@@UEAA@XZ 0000000180014208     msvcprt:MSVCP140.dll
 0002:00000210       __imp_?setstate@?$basic_ios@GU?$char_traits@G@std@@@std@@QEAAXH_N@Z 0000000180014210     msvcprt:MSVCP140.dll
 0002:00000218       __imp_?tie@?$basic_ios@GU?$char_traits@G@std@@@std@@QEBAPEAV?$basic_ostream@GU?$char_traits@G@std@@@2@XZ 0000000180014218     msvcprt:MSVCP140.dll
 0002:00000220       __imp_?rdbuf@?$basic_ios@GU?$char_traits@G@std@@@std@@QEBAPEAV?$basic_streambuf@GU?$char_traits@G@std@@@2@XZ 0000000180014220     msvcprt:MSVCP140.dll
 0002:00000228       __imp_?fill@?$basic_ios@GU?$char_traits@G@std@@@std@@QEBAGXZ 0000000180014228     msvcprt:MSVCP140.dll
 0002:00000230       __imp_??0?$basic_ios@GU?$char_traits@G@std@@@std@@IEAA@XZ 0000000180014230     msvcprt:MSVCP140.dll
 0002:00000238       __imp_??0?$basic_ostream@GU?$char_traits@G@std@@@std@@QEAA@PEAV?$basic_streambuf@GU?$char_traits@G@std@@@1@_N@Z 0000000180014238     msvcprt:MSVCP140.dll
 0002:00000240       __imp_??1?$basic_ostream@GU?$char_traits@G@std@@@std@@UEAA@XZ 0000000180014240     msvcprt:MSVCP140.dll
 0002:00000248       __imp_?_Osfx@?$basic_ostream@GU?$char_traits@G@std@@@std@@QEAAXXZ 0000000180014248     msvcprt:MSVCP140.dll
 0002:00000250       __imp_?flush@?$basic_ostream@GU?$char_traits@G@std@@@std@@QEAAAEAV12@XZ 0000000180014250     msvcprt:MSVCP140.dll
 0002:00000258       __imp_??0?$basic_ostream@DU?$char_traits@D@std@@@std@@QEAA@PEAV?$basic_streambuf@DU?$char_traits@D@std@@@1@_N@Z 0000000180014258     msvcprt:MSVCP140.dll
 0002:00000260       __imp_??1?$basic_ostream@DU?$char_traits@D@std@@@std@@UEAA@XZ 0000000180014260     msvcprt:MSVCP140.dll
 0002:00000268       __imp_?_Pninc@?$basic_streambuf@DU?$char_traits@D@std@@@std@@IEAAPEADXZ 0000000180014268     msvcprt:MSVCP140.dll
 0002:00000270       __imp_??6?$basic_ostream@DU?$char_traits@D@std@@@std@@QEAAAEAV01@H@Z 0000000180014270     msvcprt:MSVCP140.dll
 0002:00000278       __imp_?write@?$basic_ostream@DU?$char_traits@D@std@@@std@@QEAAAEAV12@PEBD_J@Z 0000000180014278     msvcprt:MSVCP140.dll
 0002:00000280       __imp_?flush@?$basic_ostream@DU?$char_traits@D@std@@@std@@QEAAAEAV12@XZ 0000000180014280     msvcprt:MSVCP140.dll
 0002:00000288       __imp_?imbue@?$basic_streambuf@GU?$char_traits@G@std@@@std@@MEAAXAEBVlocale@2@@Z 0000000180014288     msvcprt:MSVCP140.dll
 0002:00000290       __imp_?sync@?$basic_streambuf@GU?$char_traits@G@std@@@std@@MEAAHXZ 0000000180014290     msvcprt:MSVCP140.dll
 0002:00000298       __imp_?setbuf@?$basic_streambuf@GU?$char_traits@G@std@@@std@@MEAAPEAV12@PEAG_J@Z 0000000180014298     msvcprt:MSVCP140.dll
 0002:000002a0       __imp_?xsputn@?$basic_streambuf@GU?$char_traits@G@std@@@std@@MEAA_JPEBG_J@Z 00000001800142a0     msvcprt:MSVCP140.dll
 0002:000002a8       __imp_?xsgetn@?$basic_streambuf@GU?$char_traits@G@std@@@std@@MEAA_JPEAG_J@Z 00000001800142a8     msvcprt:MSVCP140.dll
 0002:000002b0       __imp_?uflow@?$basic_streambuf@GU?$char_traits@G@std@@@std@@MEAAGXZ 00000001800142b0     msvcprt:MSVCP140.dll
 0002:000002b8       __imp_?showmanyc@?$basic_streambuf@GU?$char_traits@G@std@@@std@@MEAA_JXZ 00000001800142b8     msvcprt:MSVCP140.dll
 0002:000002c0       __imp_?_Unlock@?$basic_streambuf@GU?$char_traits@G@std@@@std@@UEAAXXZ 00000001800142c0     msvcprt:MSVCP140.dll
 0002:000002c8       __imp_?_Lock@?$basic_streambuf@GU?$char_traits@G@std@@@std@@UEAAXXZ 00000001800142c8     msvcprt:MSVCP140.dll
 0002:000002d0       __imp_?imbue@?$basic_streambuf@DU?$char_traits@D@std@@@std@@MEAAXAEBVlocale@2@@Z 00000001800142d0     msvcprt:MSVCP140.dll
 0002:000002d8       __imp_?sync@?$basic_streambuf@DU?$char_traits@D@std@@@std@@MEAAHXZ 00000001800142d8     msvcprt:MSVCP140.dll
 0002:000002e0       __imp_?setbuf@?$basic_streambuf@DU?$char_traits@D@std@@@std@@MEAAPEAV12@PEAD_J@Z 00000001800142e0     msvcprt:MSVCP140.dll
 0002:000002e8       __imp_?xsputn@?$basic_streambuf@DU?$char_traits@D@std@@@std@@MEAA_JPEBD_J@Z 00000001800142e8     msvcprt:MSVCP140.dll
 0002:000002f0       __imp_?xsgetn@?$basic_streambuf@DU?$char_traits@D@std@@@std@@MEAA_JPEAD_J@Z 00000001800142f0     msvcprt:MSVCP140.dll
 0002:000002f8       __imp_?uflow@?$basic_streambuf@DU?$char_traits@D@std@@@std@@MEAAHXZ 00000001800142f8     msvcprt:MSVCP140.dll
 0002:00000300       __imp_?showmanyc@?$basic_streambuf@DU?$char_traits@D@std@@@std@@MEAA_JXZ 0000000180014300     msvcprt:MSVCP140.dll
 0002:00000308       __imp_?_Unlock@?$basic_streambuf@DU?$char_traits@D@std@@@std@@UEAAXXZ 0000000180014308     msvcprt:MSVCP140.dll
 0002:00000310       __imp_?_Lock@?$basic_streambuf@DU?$char_traits@D@std@@@std@@UEAAXXZ 0000000180014310     msvcprt:MSVCP140.dll
 0002:00000318       __imp_?id@?$ctype@G@std@@2V0locale@2@A 0000000180014318     msvcprt:MSVCP140.dll
 0002:00000320       __imp_??6?$basic_ostream@GU?$char_traits@G@std@@@std@@QEAAAEAV01@K@Z 0000000180014320     msvcprt:MSVCP140.dll
 0002:00000328       __imp_?widen@?$basic_ios@DU?$char_traits@D@std@@@std@@QEBADD@Z 0000000180014328     msvcprt:MSVCP140.dll
 0002:00000330       __imp_??6?$basic_ostream@GU?$char_traits@G@std@@@std@@QEAAAEAV01@H@Z 0000000180014330     msvcprt:MSVCP140.dll
 0002:00000338       __imp_??6?$basic_ostream@DU?$char_traits@D@std@@@std@@QEAAAEAV01@P6AAEAV01@AEAV01@@Z@Z 0000000180014338     msvcprt:MSVCP140.dll
 0002:00000340       __imp_?put@?$basic_ostream@DU?$char_traits@D@std@@@std@@QEAAAEAV12@D@Z 0000000180014340     msvcprt:MSVCP140.dll
 0002:00000348       __imp_?cout@std@@3V?$basic_ostream@DU?$char_traits@D@std@@@1@A 0000000180014348     msvcprt:MSVCP140.dll
 0002:00000350       __imp_?always_noconv@codecvt_base@std@@QEBA_NXZ 0000000180014350     msvcprt:MSVCP140.dll
 0002:00000358       __imp_?in@?$codecvt@DDU_Mbstatet@@@std@@QEBAHAEAU_Mbstatet@@PEBD1AEAPEBDPEAD3AEAPEAD@Z 0000000180014358     msvcprt:MSVCP140.dll
 0002:00000360       __imp_?out@?$codecvt@DDU_Mbstatet@@@std@@QEBAHAEAU_Mbstatet@@PEBD1AEAPEBDPEAD3AEAPEAD@Z 0000000180014360     msvcprt:MSVCP140.dll
 0002:00000368       __imp_?unshift@?$codecvt@DDU_Mbstatet@@@std@@QEBAHAEAU_Mbstatet@@PEAD1AEAPEAD@Z 0000000180014368     msvcprt:MSVCP140.dll
 0002:00000370       __imp_?_Getcat@?$codecvt@DDU_Mbstatet@@@std@@SA_KPEAPEBVfacet@locale@2@PEBV42@@Z 0000000180014370     msvcprt:MSVCP140.dll
 0002:00000378       __imp_?_Gndec@?$basic_streambuf@DU?$char_traits@D@std@@@std@@IEAAPEADXZ 0000000180014378     msvcprt:MSVCP140.dll
 0002:00000380       __imp_?_Gninc@?$basic_streambuf@DU?$char_traits@D@std@@@std@@IEAAPEADXZ 0000000180014380     msvcprt:MSVCP140.dll
 0002:00000388       __imp_?_Gnavail@?$basic_streambuf@DU?$char_traits@D@std@@@std@@IEBA_JXZ 0000000180014388     msvcprt:MSVCP140.dll
 0002:00000390       __imp_?pbump@?$basic_streambuf@DU?$char_traits@D@std@@@std@@IEAAXH@Z 0000000180014390     msvcprt:MSVCP140.dll
 0002:00000398       __imp_?_Pnavail@?$basic_streambuf@DU?$char_traits@D@std@@@std@@IEBA_JXZ 0000000180014398     msvcprt:MSVCP140.dll
 0002:000003a0       __imp_?_Init@?$basic_streambuf@DU?$char_traits@D@std@@@std@@IEAAXXZ 00000001800143a0     msvcprt:MSVCP140.dll
 0002:000003a8       __imp_?_Init@?$basic_streambuf@DU?$char_traits@D@std@@@std@@IEAAXPEAPEAD0PEAH001@Z 00000001800143a8     msvcprt:MSVCP140.dll
 0002:000003b0       __imp_??6?$basic_ostream@GU?$char_traits@G@std@@@std@@QEAAAEAV01@I@Z 00000001800143b0     msvcprt:MSVCP140.dll
 0002:000003b8       __imp_?id@?$codecvt@DDU_Mbstatet@@@std@@2V0locale@2@A 00000001800143b8     msvcprt:MSVCP140.dll
 0002:000003c0       __imp_??6?$basic_ostream@DU?$char_traits@D@std@@@std@@QEAAAEAV01@I@Z 00000001800143c0     msvcprt:MSVCP140.dll
 0002:000003c8       __imp_?getloc@?$basic_streambuf@DU?$char_traits@D@std@@@std@@QEBA?AVlocale@2@XZ 00000001800143c8     msvcprt:MSVCP140.dll
 0002:000003d0       __imp_?sbumpc@?$basic_streambuf@DU?$char_traits@D@std@@@std@@QEAAHXZ 00000001800143d0     msvcprt:MSVCP140.dll
 0002:000003d8       __imp_?sgetc@?$basic_streambuf@DU?$char_traits@D@std@@@std@@QEAAHXZ 00000001800143d8     msvcprt:MSVCP140.dll
 0002:000003e0       __imp_?_Fiopen@std@@YAPEAU_iobuf@@PEBGHH@Z 00000001800143e0     msvcprt:MSVCP140.dll
 0002:000003e8       __imp_??6?$basic_ostream@GU?$char_traits@G@std@@@std@@QEAAAEAV01@_K@Z 00000001800143e8     msvcprt:MSVCP140.dll
 0002:000003f0       __imp_??6?$basic_ostream@GU?$char_traits@G@std@@@std@@QEAAAEAV01@PEBX@Z 00000001800143f0     msvcprt:MSVCP140.dll
 0002:000003f8       __imp_??0?$basic_istream@DU?$char_traits@D@std@@@std@@QEAA@PEAV?$basic_streambuf@DU?$char_traits@D@std@@@1@_N@Z 00000001800143f8     msvcprt:MSVCP140.dll
 0002:00000400       __imp_??1?$basic_istream@DU?$char_traits@D@std@@@std@@UEAA@XZ 0000000180014400     msvcprt:MSVCP140.dll
 0002:00000408       __imp_?read@?$basic_istream@DU?$char_traits@D@std@@@std@@QEAAAEAV12@PEAD_J@Z 0000000180014408     msvcprt:MSVCP140.dll
 0002:00000410       __imp_?_Xbad_alloc@std@@YAXXZ 0000000180014410     msvcprt:MSVCP140.dll
 0002:00000418       __imp_?setf@ios_base@std@@QEAAHH@Z 0000000180014418     msvcprt:MSVCP140.dll
 0002:00000420       __imp_?setf@ios_base@std@@QEAAHHH@Z 0000000180014420     msvcprt:MSVCP140.dll
 0002:00000428       __imp_?fill@?$basic_ios@GU?$char_traits@G@std@@@std@@QEAAGG@Z 0000000180014428     msvcprt:MSVCP140.dll
 0002:00000430       __imp_??6?$basic_ostream@GU?$char_traits@G@std@@@std@@QEAAAEAV01@P6AAEAVios_base@1@AEAV21@@Z@Z 0000000180014430     msvcprt:MSVCP140.dll
 0002:00000438       __imp_?seekp@?$basic_ostream@DU?$char_traits@D@std@@@std@@QEAAAEAV12@V?$fpos@U_Mbstatet@@@2@@Z 0000000180014438     msvcprt:MSVCP140.dll
 0002:00000440       __imp_?tellp@?$basic_ostream@DU?$char_traits@D@std@@@std@@QEAA?AV?$fpos@U_Mbstatet@@@2@XZ 0000000180014440     msvcprt:MSVCP140.dll
 0002:00000448       __imp_?seekg@?$basic_istream@DU?$char_traits@D@std@@@std@@QEAAAEAV12@V?$fpos@U_Mbstatet@@@2@@Z 0000000180014448     msvcprt:MSVCP140.dll
 0002:00000450       __imp_??0?$basic_iostream@DU?$char_traits@D@std@@@std@@QEAA@PEAV?$basic_streambuf@DU?$char_traits@D@std@@@1@@Z 0000000180014450     msvcprt:MSVCP140.dll
 0002:00000458       __imp_??1?$basic_iostream@DU?$char_traits@D@std@@@std@@UEAA@XZ 0000000180014458     msvcprt:MSVCP140.dll
 0002:00000460       __imp_??0?$basic_iostream@GU?$char_traits@G@std@@@std@@QEAA@PEAV?$basic_streambuf@GU?$char_traits@G@std@@@1@@Z 0000000180014460     msvcprt:MSVCP140.dll
 0002:00000468       __imp_??1?$basic_iostream@GU?$char_traits@G@std@@@std@@UEAA@XZ 0000000180014468     msvcprt:MSVCP140.dll
 0002:00000470       __imp_?setw@std@@YA?AU?$_Smanip@_J@1@_J@Z 0000000180014470     msvcprt:MSVCP140.dll
 0002:00000478       __imp_??6?$basic_ostream@DU?$char_traits@D@std@@@std@@QEAAAEAV01@K@Z 0000000180014478     msvcprt:MSVCP140.dll
 0002:00000480       __imp_?cerr@std@@3V?$basic_ostream@DU?$char_traits@D@std@@@1@A 0000000180014480     msvcprt:MSVCP140.dll
 0002:00000488       __imp_?setp@?$basic_streambuf@DU?$char_traits@D@std@@@std@@IEAAXPEAD00@Z 0000000180014488     msvcprt:MSVCP140.dll
 0002:00000490       __imp_?setp@?$basic_streambuf@DU?$char_traits@D@std@@@std@@IEAAXPEAD0@Z 0000000180014490     msvcprt:MSVCP140.dll
 0002:00000498       __imp_?epptr@?$basic_streambuf@DU?$char_traits@D@std@@@std@@IEBAPEADXZ 0000000180014498     msvcprt:MSVCP140.dll
 0002:000004a0       __imp_?setg@?$basic_streambuf@DU?$char_traits@D@std@@@std@@IEAAXPEAD00@Z 00000001800144a0     msvcprt:MSVCP140.dll
 0002:000004a8       __imp_?gbump@?$basic_streambuf@DU?$char_traits@D@std@@@std@@IEAAXH@Z 00000001800144a8     msvcprt:MSVCP140.dll
 0002:000004b0       __imp_?egptr@?$basic_streambuf@DU?$char_traits@D@std@@@std@@IEBAPEADXZ 00000001800144b0     msvcprt:MSVCP140.dll
 0002:000004b8       __imp_?pptr@?$basic_streambuf@DU?$char_traits@D@std@@@std@@IEBAPEADXZ 00000001800144b8     msvcprt:MSVCP140.dll
 0002:000004c0       __imp_?pbase@?$basic_streambuf@DU?$char_traits@D@std@@@std@@IEBAPEADXZ 00000001800144c0     msvcprt:MSVCP140.dll
 0002:000004c8       __imp_?gptr@?$basic_streambuf@DU?$char_traits@D@std@@@std@@IEBAPEADXZ 00000001800144c8     msvcprt:MSVCP140.dll
 0002:000004d0       __imp_?eback@?$basic_streambuf@DU?$char_traits@D@std@@@std@@IEBAPEADXZ 00000001800144d0     msvcprt:MSVCP140.dll
 0002:000004d8       __imp_?sputn@?$basic_streambuf@DU?$char_traits@D@std@@@std@@QEAA_JPEBD_J@Z 00000001800144d8     msvcprt:MSVCP140.dll
 0002:000004e0       __imp_?sputc@?$basic_streambuf@DU?$char_traits@D@std@@@std@@QEAAHD@Z 00000001800144e0     msvcprt:MSVCP140.dll
 0002:000004e8       __imp_??1?$basic_streambuf@DU?$char_traits@D@std@@@std@@UEAA@XZ 00000001800144e8     msvcprt:MSVCP140.dll
 0002:000004f0       __imp_??0?$basic_streambuf@DU?$char_traits@D@std@@@std@@IEAA@XZ 00000001800144f0     msvcprt:MSVCP140.dll
 0002:000004f8       __imp_?getloc@ios_base@std@@QEBA?AVlocale@2@XZ 00000001800144f8     msvcprt:MSVCP140.dll
 0002:00000500       __imp_?width@ios_base@std@@QEAA_J_J@Z 0000000180014500     msvcprt:MSVCP140.dll
 0002:00000508       __imp_?width@ios_base@std@@QEBA_JXZ 0000000180014508     msvcprt:MSVCP140.dll
 0002:00000510       __imp_?flags@ios_base@std@@QEBAHXZ 0000000180014510     msvcprt:MSVCP140.dll
 0002:00000518       __imp_?exceptions@ios_base@std@@QEAAXH@Z 0000000180014518     msvcprt:MSVCP140.dll
 0002:00000520       __imp_?good@ios_base@std@@QEBA_NXZ 0000000180014520     msvcprt:MSVCP140.dll
 0002:00000528       __imp_?_Getcat@?$ctype@G@std@@SA_KPEAPEBVfacet@locale@2@PEBV42@@Z 0000000180014528     msvcprt:MSVCP140.dll
 0002:00000530       __imp_?widen@?$ctype@G@std@@QEBAGD@Z 0000000180014530     msvcprt:MSVCP140.dll
 0002:00000538       __imp_?_Getgloballocale@locale@std@@CAPEAV_Locimp@12@XZ 0000000180014538     msvcprt:MSVCP140.dll
 0002:00000540       __imp_??Bid@locale@std@@QEAA_KXZ 0000000180014540     msvcprt:MSVCP140.dll
 0002:00000548       __imp_?uncaught_exception@std@@YA_NXZ 0000000180014548     msvcprt:MSVCP140.dll
 0002:00000550       __imp_?_Xout_of_range@std@@YAXPEBD@Z 0000000180014550     msvcprt:MSVCP140.dll
 0002:00000558       __imp_?_Xlength_error@std@@YAXPEBD@Z 0000000180014558     msvcprt:MSVCP140.dll
 0002:00000560       __imp_??1_Lockit@std@@QEAA@XZ 0000000180014560     msvcprt:MSVCP140.dll
 0002:00000568       __imp_??0_Lockit@std@@QEAA@H@Z 0000000180014568     msvcprt:MSVCP140.dll
 0002:00000570       __imp_??0?$basic_streambuf@GU?$char_traits@G@std@@@std@@IEAA@XZ 0000000180014570     msvcprt:MSVCP140.dll
 0002:00000578       __imp_?_Osfx@?$basic_ostream@DU?$char_traits@D@std@@@std@@QEAAXXZ 0000000180014578     msvcprt:MSVCP140.dll
 0002:00000580       \177MSVCP140_NULL_THUNK_DATA 0000000180014580     msvcprt:MSVCP140.dll
 0002:00000588       __imp___std_type_info_destroy_list 0000000180014588     vcruntime:VCRUNTIME140.dll
 0002:00000590       __imp___C_specific_handler 0000000180014590     vcruntime:VCRUNTIME140.dll
 0002:00000598       __imp__purecall            0000000180014598     vcruntime:VCRUNTIME140.dll
 0002:000005a0       __imp_memset               00000001800145a0     vcruntime:VCRUNTIME140.dll
 0002:000005a8       __imp__CxxThrowException   00000001800145a8     vcruntime:VCRUNTIME140.dll
 0002:000005b0       __imp___std_exception_destroy 00000001800145b0     vcruntime:VCRUNTIME140.dll
 0002:000005b8       __imp___std_exception_copy 00000001800145b8     vcruntime:VCRUNTIME140.dll
 0002:000005c0       __imp_memmove              00000001800145c0     vcruntime:VCRUNTIME140.dll
 0002:000005c8       __imp_memcpy               00000001800145c8     vcruntime:VCRUNTIME140.dll
 0002:000005d0       __imp_memchr               00000001800145d0     vcruntime:VCRUNTIME140.dll
 0002:000005d8       __imp___std_terminate      00000001800145d8     vcruntime:VCRUNTIME140.dll
 0002:000005e0       \177VCRUNTIME140_NULL_THUNK_DATA 00000001800145e0     vcruntime:VCRUNTIME140.dll
 0002:000005e8       __imp___CxxFrameHandler4   00000001800145e8     vcruntime:VCRUNTIME140_1.dll
 0002:000005f0       \177VCRUNTIME140_1_NULL_THUNK_DATA 00000001800145f0     vcruntime:VCRUNTIME140_1.dll
 0002:000005f8       __imp__lock_file           00000001800145f8     ucrt:api-ms-win-crt-filesystem-l1-1-0.dll
 0002:00000600       __imp__unlock_file         0000000180014600     ucrt:api-ms-win-crt-filesystem-l1-1-0.dll
 0002:00000608       \177api-ms-win-crt-filesystem-l1-1-0_NULL_THUNK_DATA 0000000180014608     ucrt:api-ms-win-crt-filesystem-l1-1-0.dll
 0002:00000610       __imp_free                 0000000180014610     ucrt:api-ms-win-crt-heap-l1-1-0.dll
 0002:00000618       __imp__callnewh            0000000180014618     ucrt:api-ms-win-crt-heap-l1-1-0.dll
 0002:00000620       __imp_malloc               0000000180014620     ucrt:api-ms-win-crt-heap-l1-1-0.dll
 0002:00000628       \177api-ms-win-crt-heap-l1-1-0_NULL_THUNK_DATA 0000000180014628     ucrt:api-ms-win-crt-heap-l1-1-0.dll
 0002:00000630       __imp__seh_filter_dll      0000000180014630     ucrt:api-ms-win-crt-runtime-l1-1-0.dll
 0002:00000638       __imp__register_onexit_function 0000000180014638     ucrt:api-ms-win-crt-runtime-l1-1-0.dll
 0002:00000640       __imp__configure_narrow_argv 0000000180014640     ucrt:api-ms-win-crt-runtime-l1-1-0.dll
 0002:00000648       __imp__initialize_narrow_environment 0000000180014648     ucrt:api-ms-win-crt-runtime-l1-1-0.dll
 0002:00000650       __imp__execute_onexit_table 0000000180014650     ucrt:api-ms-win-crt-runtime-l1-1-0.dll
 0002:00000658       __imp__crt_atexit          0000000180014658     ucrt:api-ms-win-crt-runtime-l1-1-0.dll
 0002:00000660       __imp__cexit               0000000180014660     ucrt:api-ms-win-crt-runtime-l1-1-0.dll
 0002:00000668       __imp__initterm            0000000180014668     ucrt:api-ms-win-crt-runtime-l1-1-0.dll
 0002:00000670       __imp__initterm_e          0000000180014670     ucrt:api-ms-win-crt-runtime-l1-1-0.dll
 0002:00000678       __imp__invalid_parameter_noinfo_noreturn 0000000180014678     ucrt:api-ms-win-crt-runtime-l1-1-0.dll
 0002:00000680       __imp__initialize_onexit_table 0000000180014680     ucrt:api-ms-win-crt-runtime-l1-1-0.dll
 0002:00000688       \177api-ms-win-crt-runtime-l1-1-0_NULL_THUNK_DATA 0000000180014688     ucrt:api-ms-win-crt-runtime-l1-1-0.dll
 0002:00000690       __imp_fread                0000000180014690     ucrt:api-ms-win-crt-stdio-l1-1-0.dll
 0002:00000698       __imp_fputc                0000000180014698     ucrt:api-ms-win-crt-stdio-l1-1-0.dll
 0002:000006a0       __imp_setvbuf              00000001800146a0     ucrt:api-ms-win-crt-stdio-l1-1-0.dll
 0002:000006a8       __imp_fsetpos              00000001800146a8     ucrt:api-ms-win-crt-stdio-l1-1-0.dll
 0002:000006b0       __imp__fseeki64            00000001800146b0     ucrt:api-ms-win-crt-stdio-l1-1-0.dll
 0002:000006b8       __imp_ungetc               00000001800146b8     ucrt:api-ms-win-crt-stdio-l1-1-0.dll
 0002:000006c0       __imp___stdio_common_vswscanf 00000001800146c0     ucrt:api-ms-win-crt-stdio-l1-1-0.dll
 0002:000006c8       __imp_fgetpos              00000001800146c8     ucrt:api-ms-win-crt-stdio-l1-1-0.dll
 0002:000006d0       __imp_fgetc                00000001800146d0     ucrt:api-ms-win-crt-stdio-l1-1-0.dll
 0002:000006d8       __imp_fflush               00000001800146d8     ucrt:api-ms-win-crt-stdio-l1-1-0.dll
 0002:000006e0       __imp___acrt_iob_func      00000001800146e0     ucrt:api-ms-win-crt-stdio-l1-1-0.dll
 0002:000006e8       __imp___stdio_common_vfprintf 00000001800146e8     ucrt:api-ms-win-crt-stdio-l1-1-0.dll
 0002:000006f0       __imp___stdio_common_vsnwprintf_s 00000001800146f0     ucrt:api-ms-win-crt-stdio-l1-1-0.dll
 0002:000006f8       __imp_fwrite               00000001800146f8     ucrt:api-ms-win-crt-stdio-l1-1-0.dll
 0002:00000700       __imp__get_stream_buffer_pointers 0000000180014700     ucrt:api-ms-win-crt-stdio-l1-1-0.dll
 0002:00000708       __imp_fclose               0000000180014708     ucrt:api-ms-win-crt-stdio-l1-1-0.dll
 0002:00000710       \177api-ms-win-crt-stdio-l1-1-0_NULL_THUNK_DATA 0000000180014710     ucrt:api-ms-win-crt-stdio-l1-1-0.dll
 0002:00000718       __imp_wcslen               0000000180014718     ucrt:api-ms-win-crt-string-l1-1-0.dll
 0002:00000720       __imp_tolower              0000000180014720     ucrt:api-ms-win-crt-string-l1-1-0.dll
 0002:00000728       __imp_strlen               0000000180014728     ucrt:api-ms-win-crt-string-l1-1-0.dll
 0002:00000730       __imp_isspace              0000000180014730     ucrt:api-ms-win-crt-string-l1-1-0.dll
 0002:00000738       \177api-ms-win-crt-string-l1-1-0_NULL_THUNK_DATA 0000000180014738     ucrt:api-ms-win-crt-string-l1-1-0.dll
 0002:00000740       __imp_MsiRecordGetFieldCount 0000000180014740     msi:msi.dll
 0002:00000748       __imp_MsiCloseHandle       0000000180014748     msi:msi.dll
 0002:00000750       __imp_MsiRecordGetStringW  0000000180014750     msi:msi.dll
 0002:00000758       __imp_MsiDatabaseOpenViewW 0000000180014758     msi:msi.dll
 0002:00000760       __imp_MsiViewExecute       0000000180014760     msi:msi.dll
 0002:00000768       __imp_MsiViewFetch         0000000180014768     msi:msi.dll
 0002:00000770       __imp_MsiOpenDatabaseW     0000000180014770     msi:msi.dll
 0002:00000778       \177msi_NULL_THUNK_DATA    0000000180014778     msi:msi.dll
 0002:00000780       __imp_StringFromGUID2      0000000180014780     ole32:ole32.dll
 0002:00000788       __imp_IIDFromString        0000000180014788     ole32:ole32.dll
 0002:00000790       \177ole32_NULL_THUNK_DATA  0000000180014790     ole32:ole32.dll
 0002:00000798       __guard_check_icall_fptr   0000000180014798     MSVCRT:guard_support.obj
 0002:000007a0       __guard_xfg_check_icall_fptr 00000001800147a0     MSVCRT:guard_support.obj
 0002:000007a8       __guard_dispatch_icall_fptr 00000001800147a8     MSVCRT:guard_support.obj
 0002:000007b0       __guard_xfg_dispatch_icall_fptr 00000001800147b0     MSVCRT:guard_support.obj
 0002:000007b8       __guard_xfg_table_dispatch_icall_fptr 00000001800147b8     MSVCRT:guard_support.obj
 0002:000007c0       __castguard_check_failure_os_handled_fptr 00000001800147c0     MSVCRT:guard_support.obj
 0002:000007c8       __guard_memcpy_fptr        00000001800147c8     vcruntime:softmemtag.obj
 0002:000007d0       __xc_a                     00000001800147d0     MSVCRT:initializers.obj
 0002:000007e8       __xc_z                     00000001800147e8     MSVCRT:initializers.obj
 0002:000007f0       __xi_a                     00000001800147f0     MSVCRT:initializers.obj
 0002:000007f8       __xi_z                     00000001800147f8     MSVCRT:initializers.obj
 0002:00000800       __xp_a                     0000000180014800     MSVCRT:initializers.obj
 0002:00000808       __xp_z                     0000000180014808     MSVCRT:initializers.obj
 0002:00000810       __xt_a                     0000000180014810     MSVCRT:initializers.obj
 0002:00000818       __xt_z                     0000000180014818     MSVCRT:initializers.obj
 0002:00000830       ??_7exception@std@@6B@     0000000180014830     ErrorHandling.obj
 0002:00000840       ??_C@_0BC@EOODALEL@Unknown?5exception@ 0000000180014840     ErrorHandling.obj
 0002:00000860       ??_7bad_alloc@std@@6B@     0000000180014860     ErrorHandling.obj
 0002:00000878       ??_7bad_array_new_length@std@@6B@ 0000000180014878     ErrorHandling.obj
 0002:00000888       ??_C@_0BF@KINCDENJ@bad?5array?5new?5length@ 0000000180014888     ErrorHandling.obj
 0002:000008a0       ??_C@_0BA@JFNIOLAK@string?5too?5long@ 00000001800148a0     ErrorHandling.obj
 0002:000008b0       ??_C@_00CNPNBAHC@@         00000001800148b0     ErrorHandling.obj
 0002:000008c0       ??_7bad_cast@std@@6B@      00000001800148c0     ErrorHandling.obj
 0002:000008d0       ??_C@_08EPJLHIJG@bad?5cast@ 00000001800148d0     ErrorHandling.obj
 0002:000008e8       ??_7?$basic_stringbuf@GU?$char_traits@G@std@@V?$allocator@G@2@@std@@6B@ 00000001800148e8     ErrorHandling.obj
 0002:00000968       ??_7?$basic_ostringstream@GU?$char_traits@G@std@@V?$allocator@G@2@@std@@6B@ 0000000180014968     ErrorHandling.obj
 0002:00000970       ??_8?$basic_ostringstream@GU?$char_traits@G@std@@V?$allocator@G@2@@std@@7B@ 0000000180014970     ErrorHandling.obj
 0002:00000978       ??_C@_02HHAEMJFE@?2?1@     0000000180014978     ErrorHandling.obj
 0002:00000980       ??_C@_0BJ@HAJDFNON@Exception?5with?5message?5?8@ 0000000180014980     ErrorHandling.obj
 0002:000009a0       ??_C@_08OFLCGKIF@?8?5caught@ 00000001800149a0     ErrorHandling.obj
 0002:000009b0       ??_C@_1DC@DNLNKJFM@?$AAU?$AAn?$AAk?$AAn?$AAo?$AAw?$AAn?$AA?5?$AAe?$AAx?$AAc?$AAe?$AAp?$AAt?$AAi@ 00000001800149b0     ErrorHandling.obj
 0002:000009f0       ??_7?$basic_stringbuf@DU?$char_traits@D@std@@V?$allocator@D@2@@std@@6B@ 00000001800149f0     ErrorHandling.obj
 0002:00000a70       ??_7?$basic_ostringstream@DU?$char_traits@D@std@@V?$allocator@D@2@@std@@6B@ 0000000180014a70     ErrorHandling.obj
 0002:00000a78       ??_8?$basic_ostringstream@DU?$char_traits@D@std@@V?$allocator@D@2@@std@@7B@ 0000000180014a78     ErrorHandling.obj
 0002:00000a80       ??_C@_04KJCOMIHH@?$CI?$CJ?3?5@ 0000000180014a80     ErrorHandling.obj
 0002:00000a88       ??_C@_05OKLJFBOO@?$CJ?5at?5@ 0000000180014a88     ErrorHandling.obj
 0002:00000a90       ??_C@_01ODHLEDKK@?$CI@     0000000180014a90     ErrorHandling.obj
 0002:00000a94       ??_C@_06PKHGJEE@?$DL?4?0?3?$CB?$DP@ 0000000180014a94     ErrorHandling.obj
 0002:00000a9c       ??_C@_01CLKCMJKC@?5@       0000000180014a9c     ErrorHandling.obj
 0002:00000aa0       ??_C@_02KHOJGJKF@?4?5@     0000000180014aa0     ErrorHandling.obj
 0002:00000aa8       ??_C@_0BI@CFPLBAOH@invalid?5string?5position@ 0000000180014aa8     ErrorHandling.obj
 0002:00000ac0       __xmm@000000000000000f0000000000000000 0000000180014ac0     ErrorHandling.obj
 0002:00000ae0       ??_7runtime_error@std@@6B@ 0000000180014ae0     Executor.obj
 0002:00000af8       ??_7JpErrorBase@@6B@       0000000180014af8     Executor.obj
 0002:00000b08       ??_7SysError@@6B@          0000000180014b08     Executor.obj
 0002:00000b20       ??_7?$JpError@VSysError@@@@6BJpErrorBase@@@ 0000000180014b20     Executor.obj
 0002:00000b30       ??_7?$JpError@VSysError@@@@6BSysError@@@ 0000000180014b30     Executor.obj
 0002:00000b40       ??_C@_0N@LDHCNCJC@System?5error@ 0000000180014b40     Executor.obj
 0002:00000b50       ??_C@_02KEGNLNML@?0?5@     0000000180014b50     Executor.obj
 0002:00000b54       ??_C@_01PKGAHCOL@?$CJ@     0000000180014b54     Executor.obj
 0002:00000b58       ??_C@_07OCDKBNAP@?5failed@ 0000000180014b58     Executor.obj
 0002:00000b60       ??_C@_0BA@FOIKENOD@vector?5too?5long@ 0000000180014b60     Executor.obj
 0002:00000b70       __xmm@00000000000000070000000000000000 0000000180014b70     Executor.obj
 0002:00000b80       ?pathSeparator@FileUtils@@3GB 0000000180014b80     FileUtils.obj
 0002:00000b8c       ??_C@_15MNCACJLI@?$AA?2?$AA?1@ 0000000180014b8c     FileUtils.obj
 0002:00000ba0       ??_7?$JpError@Vruntime_error@std@@@@6BJpErrorBase@@@ 0000000180014ba0     Guid.obj
 0002:00000bb0       ??_7?$JpError@Vruntime_error@std@@@@6Bruntime_error@std@@@ 0000000180014bb0     Guid.obj
 0002:00000bc0       ??_C@_0CA@BMPGLJJN@?$GAanonymous?9namespace?8?3?3initGuid@ 0000000180014bc0     Guid.obj
 0002:00000be0       ??_C@_0DC@KGKIHNFD@s?2src?2jdk?4jpackage?2windows?2nati@ 0000000180014be0     Guid.obj
 0002:00000c18       ??_C@_0P@CINEOJHO@IIDFromString?$CI@ 0000000180014c18     Guid.obj
 0002:00000c28       ??_C@_08EPEDOCDA@?$CJ?5failed@ 0000000180014c28     Guid.obj
 0002:00000c34       ??_C@_13EHOOFIKC@?$AA?$HN@ 0000000180014c34     Guid.obj
 0002:00000c38       ??_C@_13GCIFAHHO@?$AA?$HL@ 0000000180014c38     Guid.obj
 0002:00000c40       ??_C@_0P@ILPPFPKA@Guid?3?3toString@ 0000000180014c40     Guid.obj
 0002:00000c50       ??_C@_0BJ@GPEFFCPB@StringFromGUID2?$CI?$CJ?5failed@ 0000000180014c50     Guid.obj
 0002:00000c6c       ??_C@_02KPKOKMHB@?$CFS@    0000000180014c6c     IconSwap.obj
 0002:00000c70       ??_C@_0CC@PCGMLBAN@Error?3?5Failed?5to?5allocate?5memor@ 0000000180014c70     IconSwap.obj
 0002:00000c98       ??_C@_0BF@FFNHJCPB@jni?3?3toUnicodeString@ 0000000180014c98     JniUtils.obj
 0002:00000cb0       ??_C@_0DL@OIDODNLL@s?2src?2jdk?4jpackage?2windows?2nati@ 0000000180014cb0     JniUtils.obj
 0002:00000cf0       ??_C@_0BI@NCGLOMCE@GetStringChars?$CI?$CJ?5failed@ 0000000180014cf0     JniUtils.obj
 0002:00000d08       ??_C@_0P@BMIEBKCM@jni?3?3toJString@ 0000000180014d08     JniUtils.obj
 0002:00000d18       ??_C@_0BD@OGPAMFEO@NewString?$CI?$CJ?5failed@ 0000000180014d18     JniUtils.obj
 0002:00000d30       ??_C@_0ON@EIBINNHA@AtEndOfScope?$DMclass?5?$GAclass?5std?3?3@ 0000000180014d30     JniUtils.obj
 0002:00000e20       ??_C@_0DB@BLDOPEOL@s?2src?2jdk?4jpackage?2share?2native@ 0000000180014e20     JniUtils.obj
 0002:00000e60       ??_7LogAppender@@6B@       0000000180014e60     Log.obj
 0002:00000e78       ??_7StreamLogAppender@@6B@ 0000000180014e78     Log.obj
 0002:00000e88       ??_C@_1M@MGIHBMCI@?$AAT?$AAR?$AAA?$AAC?$AAE@ 0000000180014e88     Log.obj
 0002:00000e98       ??_C@_19FILLMKCG@?$AAI?$AAN?$AAF?$AAO@ 0000000180014e98     Log.obj
 0002:00000ea8       ??_C@_1BA@KPCCLDOC@?$AAW?$AAA?$AAR?$AAN?$AAI?$AAN?$AAG@ 0000000180014ea8     Log.obj
 0002:00000eb8       ??_C@_1M@BJACCECO@?$AAE?$AAR?$AAR?$AAO?$AAR@ 0000000180014eb8     Log.obj
 0002:00000ec8       ??_C@_1BA@HABJOAEE@?$AAU?$AAN?$AAK?$AAN?$AAO?$AAW?$AAN@ 0000000180014ec8     Log.obj
 0002:00000ed8       ??_C@_15ELOONFKJ@?$AA?3?$AA?5@ 0000000180014ed8     Log.obj
 0002:00000ee0       ??_C@_15CMBHNMLL@?$AA?5?$AA?$CI@ 0000000180014ee0     Log.obj
 0002:00000ee8       ??_C@_0BB@GCADKGJO@map?1set?5too?5long@ 0000000180014ee8     MsiCA.obj
 0002:00000f08       ??_7Error@msi@@6B@         0000000180014f08     MsiCA.obj
 0002:00000f20       ??_7?$JpError@VError@msi@@@@6BJpErrorBase@@@ 0000000180014f20     MsiCA.obj
 0002:00000f30       ??_7?$JpError@VError@msi@@@@6BError@msi@@@ 0000000180014f30     MsiCA.obj
 0002:00000f40       ??_C@_01GEODFPGF@?8@       0000000180014f40     MsiCA.obj
 0002:00000f48       ??_C@_1BI@OOBDCHEH@?$AAP?$AAr?$AAo?$AAd?$AAu?$AAc?$AAt?$AAC?$AAo?$AAd?$AAe@ 0000000180014f48     MsiCA.obj
 0002:00000f60       ??_C@_0CJ@GCOBILED@msi?3?3?$GAanonymous?9namespace?8?3?3ope@ 0000000180014f60     MsiCA.obj
 0002:00000f98       ??_7NoMoreItemsError@msi@@6B@ 0000000180014f98     MsiDb.obj
 0002:00000fb0       ??_7?$basic_filebuf@DU?$char_traits@D@std@@@std@@6B@ 0000000180014fb0     MsiDb.obj
 0002:00001028       ??_C@_0BF@HECCNMNO@?$CJ?5failed?5with?5error?$DN@ 0000000180015028     MsiDb.obj
 0002:00001040       ??_C@_0DD@OMCLKPIE@s?2src?2jdk?4jpackage?2windows?2nati@ 0000000180015040     MsiDb.obj
 0002:00001078       ??_C@_0BB@PGLHLGNP@MsiOpenDatabase?$CI@ 0000000180015078     MsiDb.obj
 0002:00001090       ??_C@_0BN@OKIJDOFB@?0?5MSIDBOPEN_READONLY?$CJ?5failed@ 0000000180015090     MsiDb.obj
 0002:000010b0       ??_C@_0CO@LCNLDDEH@SELECT?5Value?5FROM?5Property?5WHER@ 00000001800150b0     MsiDb.obj
 0002:000010e0       ??_C@_0BL@BEBKODAA@msi?3?3Database?3?3getProperty@ 00000001800150e0     MsiDb.obj
 0002:00001100       ??_C@_0BG@MBCEGHCK@record?4getFieldCount?$CI@ 0000000180015100     MsiDb.obj
 0002:00001118       ??_C@_0BM@HHAOOHHI@?$CJ?5returned?5unexpected?5value@ 0000000180015118     MsiDb.obj
 0002:00001138       ??_C@_0CD@IBMNDFG@msi?3?3DatabaseRecord?3?3getFieldCo@ 0000000180015138     MsiDb.obj
 0002:00001160       ??_C@_0CA@OEIMMPMH@MsiRecordGetFieldCount?$CI?$CJ?5failed@ 0000000180015160     MsiDb.obj
 0002:00001180       ??_C@_0CA@IOLDDDHB@msi?3?3DatabaseView?3?3DatabaseView@ 0000000180015180     MsiDb.obj
 0002:000011a0       ??_C@_0BF@NMGELMFN@MsiDatabaseOpenView?$CI@ 00000001800151a0     MsiDb.obj
 0002:000011b8       ??_C@_0BA@FCCIPHNF@MsiViewExecute?$CI@ 00000001800151b8     MsiDb.obj
 0002:000011d0       ??_7?$JpError@VNoMoreItemsError@msi@@@@6BJpErrorBase@@@ 00000001800151d0     MsiDb.obj
 0002:000011e0       ??_7?$JpError@VNoMoreItemsError@msi@@@@6BNoMoreItemsError@msi@@@ 00000001800151e0     MsiDb.obj
 0002:000011f0       ??_C@_0BJ@FJKBHIAJ@msi?3?3DatabaseView?3?3fetch@ 00000001800151f0     MsiDb.obj
 0002:00001210       ??_C@_0BD@JIBAHKDM@No?5more?5items?5in?5?$FL@ 0000000180015210     MsiDb.obj
 0002:00001228       ??_C@_07MPHPDHHG@?$FN?5query@ 0000000180015228     MsiDb.obj
 0002:00001230       ??_C@_0BM@HAGAJLHK@msi?3?3DatabaseView?3?3tryFetch@ 0000000180015230     MsiDb.obj
 0002:00001250       ??_C@_0O@CGOANHIE@MsiViewFetch?$CI@ 0000000180015250     MsiDb.obj
 0002:00001260       ??_C@_0DG@PCFDMKKJ@s?2src?2jdk?4jpackage?2windows?2nati@ 0000000180015260     MsiUtils.obj
 0002:00001298       ??_C@_0BA@PCHEKKD@MsiCloseHandle?$CI@ 0000000180015298     MsiUtils.obj
 0002:000012a8       ??_C@_1CI@KPCFIJEE@?$AAm?$AAs?$AAi?$AA?3?$AA?3?$AAc?$AAl?$AAo?$AAs?$AAe?$AAM?$AAS?$AAI?$AAH?$AAA@ 00000001800152a8     MsiUtils.obj
 0002:000012d0       ??_C@_1GM@KLMFKHLE@?$AAs?$AA?2?$AAs?$AAr?$AAc?$AA?2?$AAj?$AAd?$AAk?$AA?4?$AAj?$AAp?$AAa?$AAc?$AAk@ 00000001800152d0     MsiUtils.obj
 0002:00001340       ??_C@_0BD@MMKFHCJA@MsiRecordGetString@ 0000000180015340     MsiUtils.obj
 0002:00001354       ??_C@_01LBDDMOBJ@?$FN@     0000000180015354     MsiUtils.obj
 0002:00001358       ??_C@_0M@DFKEBDIB@MSI?5error?5?$FL@ 0000000180015358     MsiUtils.obj
 0002:00001368       ??_C@_1BG@GJFCCOOL@?$AAm?$AAs?$AAi?$AAm?$AAs?$AAg?$AA?4?$AAd?$AAl?$AAl@ 0000000180015368     MsiUtils.obj
 0002:00001380       ??_C@_0CI@PIBEIPJI@msi?3?3?$GAanonymous?9namespace?8?3?3mak@ 0000000180015380     MsiUtils.obj
 0002:000013a8       ??_C@_0BA@HCMFAFI@LoadLibraryExW?$CI@ 00000001800153a8     MsiUtils.obj
 0002:000013b8       ??_C@_1BO@BCJFDHGG@?$AAN?$AAo?$AA?5?$AAd?$AAe?$AAs?$AAc?$AAr?$AAi?$AAp?$AAt?$AAi?$AAo?$AAn@ 00000001800153b8     MsiUtils.obj
 0002:000013d8       ??_C@_02GBLMOEJC@?5?$FL@   00000001800153d8     MsiUtils.obj
 0002:000013e0       ??_C@_0CI@DLOLPNJF@msi?3?3?$GAanonymous?9namespace?8?3?3get@ 00000001800153e0     MsiUtils.obj
 0002:00001410       ??_C@_1BA@LEPJIIOK@?$AAU?$AAn?$AAk?$AAn?$AAo?$AAw?$AAn@ 0000000180015410     PlatformLogEvent.obj
 0002:00001420       ??_C@_1HI@LAPLFCFO@?$AA?$CF?$AA0?$AA4?$AAu?$AA?1?$AA?$CF?$AA0?$AA2?$AAu?$AA?1?$AA?$CF?$AA0?$AA2?$AAu?$AA?5@ 0000000180015420     PlatformLogEvent.obj
 0002:000014a0       ??_C@_0CD@IGBKECFO@ResourceEditor?3?3FileLock?3?3FileL@ 00000001800154a0     ResourceEditor.obj
 0002:000014d0       ??_C@_0EB@PMHIEHM@s?2src?2jdk?4jpackage?2windows?2nati@ 00000001800154d0     ResourceEditor.obj
 0002:00001518       ??_C@_0BF@EEHHJMNO@BeginUpdateResource?$CI@ 0000000180015518     ResourceEditor.obj
 0002:00001530       ??_C@_0CE@BDEPPPPO@ResourceEditor?3?3FileLock?3?3?$HOFile@ 0000000180015530     ResourceEditor.obj
 0002:00001558       ??_C@_0BD@EKOCFJGM@EndUpdateResource?$CI@ 0000000180015558     ResourceEditor.obj
 0002:00001570       ??_C@_09CNJBHKGC@?$CJ?5failed?4@ 0000000180015570     ResourceEditor.obj
 0002:0000157c       ??_C@_13GMDMCADD@?$AA?$CD@ 000000018001557c     ResourceEditor.obj
 0002:00001580       ??_C@_0BG@LIOFEBPP@ResourceEditor?3?3apply@ 0000000180015580     ResourceEditor.obj
 0002:00001598       ??_C@_0BI@OLOABBFD@UpdateResource?$CI?$CJ?5failed@ 0000000180015598     ResourceEditor.obj
 0002:000015b8       ??_7?$basic_ifstream@DU?$char_traits@D@std@@@std@@6B@ 00000001800155b8     ResourceEditor.obj
 0002:000015c0       ??_8?$basic_ifstream@DU?$char_traits@D@std@@@std@@7B@ 00000001800155c0     ResourceEditor.obj
 0002:000015d0       ??_C@_08DCJJILDN@?5?$CIname?$DN?8@ 00000001800155d0     Resources.obj
 0002:000015e0       ??_C@_09BLBBBHKI@?8?0?5type?$DN?8@ 00000001800155e0     Resources.obj
 0002:000015ec       ??_C@_02HJPKOJGD@?8?$CJ@   00000001800155ec     Resources.obj
 0002:000015f0       ??_C@_0BB@IHINCNEI@Resource?3?3getPtr@ 00000001800155f0     Resources.obj
 0002:00001608       ??_C@_0DH@MGEPKFIC@s?2src?2jdk?4jpackage?2windows?2nati@ 0000000180015608     Resources.obj
 0002:00001640       ??_C@_0BF@IIGEHKJO@cannot?5find?5resource@ 0000000180015640     Resources.obj
 0002:00001658       ??_C@_0BF@IICCOAKJ@cannot?5load?5resource@ 0000000180015658     Resources.obj
 0002:000016a0       ??_C@_0DO@FONBEFMI@s?2src?2jdk?4jpackage?2windows?2nati@ 00000001800156a0     VersionInfo.obj
 0002:000016e0       ??_C@_1BI@FCMLLAGN@?$AA?$CF?$AAd?$AA?4?$AA?$CF?$AAd?$AA?4?$AA?$CF?$AAd?$AA?4?$AA?$CF?$AAd@ 00000001800156e0     VersionInfo.obj
 0002:000016f8       ??_C@_0DK@CCIPDNEP@?$GAanonymous?9namespace?8?3?3FixedFil@ 00000001800156f8     VersionInfo.obj
 0002:00001738       ??_C@_0CA@BBEPHEMG@Malformed?5file?5version?5value?3?5?$FL@ 0000000180015738     VersionInfo.obj
 0002:00001758       ??_C@_0CB@DNPOCCOG@?$GAanonymous?9namespace?8?3?3writeWOR@ 0000000180015758     VersionInfo.obj
 0002:00001780       ??_C@_0BD@KNFLMKLN@Invalid?5WORD?5value@ 0000000180015780     VersionInfo.obj
 0002:00001798       ??_C@_0CH@DDHGPDCC@?$GAanonymous?9namespace?8?3?3add32bit@ 0000000180015798     VersionInfo.obj
 0002:000017c0       ??_C@_0CD@PIIDNOPO@Invalid?5data?5written?5in?5the?5str@ 00000001800157c0     VersionInfo.obj
 0002:000017e8       ??_C@_0CP@MFBNHLMG@?$GAanonymous?9namespace?8?3?3StreamSi@ 00000001800157e8     VersionInfo.obj
 0002:00001818       ??_C@_0BM@PFELLINL@Invalid?5negative?5size?5value@ 0000000180015818     VersionInfo.obj
 0002:00001838       ??_C@_1DE@HKLKJHCE@?$AAF?$AAI?$AAX?$AAE?$AAD?$AAF?$AAI?$AAL?$AAE?$AAI?$AAN?$AAF?$AAO?$AA_?$AAF@ 0000000180015838     VersionInfo.obj
 0002:00001878       ??_7?$basic_stringstream@DU?$char_traits@D@std@@V?$allocator@D@2@@std@@6B@ 0000000180015878     VersionInfo.obj
 0002:00001880       ??_8?$basic_stringstream@DU?$char_traits@D@std@@V?$allocator@D@2@@std@@7B?$basic_istream@DU?$char_traits@D@std@@@1@@ 0000000180015880     VersionInfo.obj
 0002:00001888       ??_8?$basic_stringstream@DU?$char_traits@D@std@@V?$allocator@D@2@@std@@7B?$basic_ostream@DU?$char_traits@D@std@@@1@@ 0000000180015888     VersionInfo.obj
 0002:00001890       ??_C@_0BD@LPEGHGBH@VersionInfo?3?3apply@ 0000000180015890     VersionInfo.obj
 0002:000018a8       ??_C@_0CH@NICCFHCM@Missing?5mandatory?5FILEVERSION?5p@ 00000001800158a8     VersionInfo.obj
 0002:000018d8       ??_7?$basic_stringstream@GU?$char_traits@G@std@@V?$allocator@G@2@@std@@6B@ 00000001800158d8     VersionInfo.obj
 0002:000018e0       ??_8?$basic_stringstream@GU?$char_traits@G@std@@V?$allocator@G@2@@std@@7B?$basic_istream@GU?$char_traits@G@std@@@1@@ 00000001800158e0     VersionInfo.obj
 0002:000018e8       ??_8?$basic_stringstream@GU?$char_traits@G@std@@V?$allocator@G@2@@std@@7B?$basic_ostream@GU?$char_traits@G@std@@@1@@ 00000001800158e8     VersionInfo.obj
 0002:000018f0       ??_C@_1BO@HMJELANO@?$AAF?$AAI?$AAX?$AAE?$AAD?$AAF?$AAI?$AAL?$AAE?$AAI?$AAN?$AAF?$AAO?$AA_@ 00000001800158f0     VersionInfo.obj
 0002:00001910       ??_C@_1CA@FOECMPGO@?$AAV?$AAS?$AA_?$AAV?$AAE?$AAR?$AAS?$AAI?$AAO?$AAN?$AA_?$AAI?$AAN?$AAF?$AAO@ 0000000180015910     VersionInfo.obj
 0002:00001930       ??_C@_1BO@PBBNDBNF@?$AAS?$AAt?$AAr?$AAi?$AAn?$AAg?$AAF?$AAi?$AAl?$AAe?$AAI?$AAn?$AAf?$AAo@ 0000000180015930     VersionInfo.obj
 0002:00001950       ??_C@_1BI@LJHFMFCG@?$AAV?$AAa?$AAr?$AAF?$AAi?$AAl?$AAe?$AAI?$AAn?$AAf?$AAo@ 0000000180015950     VersionInfo.obj
 0002:00001968       ??_C@_1BI@OMFAJHAK@?$AAT?$AAr?$AAa?$AAn?$AAs?$AAl?$AAa?$AAt?$AAi?$AAo?$AAn@ 0000000180015968     VersionInfo.obj
 0002:00001980       ??_C@_1DK@JLHDHGFK@?$AAF?$AAI?$AAX?$AAE?$AAD?$AAF?$AAI?$AAL?$AAE?$AAI?$AAN?$AAF?$AAO?$AA_?$AAP@ 0000000180015980     VersionInfo.obj
 0002:000019c0       ??_C@_0L@OLMNIJED@Some?5error@ 00000001800159c0     WinErrorHandling.obj
 0002:000019d0       ??_C@_0CA@GCNKJPPO@GetModuleHandleEx?$CI?$CJ?5failed?5for?5@ 00000001800159d0     WinErrorHandling.obj
 0002:000019f0       ??_C@_09GKEDKJ@?5address?4@ 00000001800159f0     WinErrorHandling.obj
 0002:00001a00       ??_C@_1EG@ONADDMNL@?$AA?$GA?$AAa?$AAn?$AAo?$AAn?$AAy?$AAm?$AAo?$AAu?$AAs?$AA?9?$AAn?$AAa?$AAm?$AAe@ 0000000180015a00     WinErrorHandling.obj
 0002:00001a50       ??_C@_1HM@EKFPGHAD@?$AAs?$AA?2?$AAs?$AAr?$AAc?$AA?2?$AAj?$AAd?$AAk?$AA?4?$AAj?$AAp?$AAa?$AAc?$AAk@ 0000000180015a50     WinErrorHandling.obj
 0002:00001ad0       ??_C@_1DC@DBLHEFGC@?$AAN?$AAo?$AA?5?$AAd?$AAe?$AAs?$AAc?$AAr?$AAi?$AAp?$AAt?$AAi?$AAo?$AAn?$AA?5@ 0000000180015ad0     WinErrorHandling.obj
 0002:00001b08       ??_C@_0O@EGFCNMMA@system?5error?5@ 0000000180015b08     WinErrorHandling.obj
 0002:00001b18       ??_C@_02GFKOMOKH@?5?$CI@   0000000180015b18     WinErrorHandling.obj
 0002:00001b20       ??_C@_0DK@PGDJHLDJ@s?2src?2jdk?4jpackage?2windows?2nati@ 0000000180015b20     WinFileUtils.obj
 0002:00001b60       ??_C@_0BH@FCLNLDKE@FileUtils?3?3toShortPath@ 0000000180015b60     WinFileUtils.obj
 0002:00001b78       ??_C@_0BC@OJHABDJG@GetShortPathName?$CI@ 0000000180015b78     WinFileUtils.obj
 0002:00001b90       ??_C@_0BD@HIJECHKD@GetSystemDirectory@ 0000000180015b90     WinSysInfo.obj
 0002:00001ba8       ??_C@_0CO@MKEKIODH@SysInfo?3?3?$GAanonymous?9namespace?8?3@ 0000000180015ba8     WinSysInfo.obj
 0002:00001bd8       ??_C@_0DI@GLHFKFGD@s?2src?2jdk?4jpackage?2windows?2nati@ 0000000180015bd8     WinSysInfo.obj
 0002:00001c10       ??_C@_0BJ@OHFMJCIO@GetModuleFileName?5failed@ 0000000180015c10     WinSysInfo.obj
 0002:00001c30       ??_C@_0CA@LHHGDJIE@SysInfo?3?3getCurrentModuleHandle@ 0000000180015c30     WinSysInfo.obj
 0002:00001c50       ??_C@_0BK@NEANLJHL@GetModuleHandleExW?5failed@ 0000000180015c50     WinSysInfo.obj
 0002:00001c70       ??_C@_0DB@OADGFLCE@SysInfo?3?3?$GAanonymous?9namespace?8?3@ 0000000180015c70     WinSysInfo.obj
 0002:00001ca8       ??_C@_0BG@GKMJLKJB@Unexpected?5reply?5from@ 0000000180015ca8     WinSysInfo.obj
 0002:00001cc0       ??_C@_0DK@LKGGAEPL@Java_jdk_jpackage_internal_Wind@ 0000000180015cc0     WindowsRegistry.obj
 0002:00001d00       ??_C@_0EC@NPMOIIFN@s?2src?2jdk?4jpackage?2windows?2nati@ 0000000180015d00     WindowsRegistry.obj
 0002:00001d48       ??_C@_0CA@IINBNHIH@Invalid?5Windows?5registry?5key?5id@ 0000000180015d48     WindowsRegistry.obj
 0002:00001d68       ??_C@_0DL@FEEEGFIN@Java_jdk_jpackage_internal_Wind@ 0000000180015d68     WindowsRegistry.obj
 0002:00001da8       ??_C@_0DN@GHOAPCGH@Java_jdk_jpackage_internal_Wind@ 0000000180015da8     WindowsRegistry.obj
 0002:00001de8       ??_C@_0DI@LNIHIHKN@Java_jdk_jpackage_internal_Wind@ 0000000180015de8     WindowsRegistry.obj
 0002:00001e48       ??_C@_0DM@HKFNBGII@Java_jdk_jpackage_internal_Exec@ 0000000180015e48     jpackage.obj
 0002:00001e88       ??_C@_0DL@BGFDHIPP@s?2src?2jdk?4jpackage?2windows?2nati@ 0000000180015e88     jpackage.obj
 0002:00001ec8       ??_C@_0DO@NDGNLHPE@Java_jdk_jpackage_internal_Exec@ 0000000180015ec8     jpackage.obj
 0002:00001f08       ??_C@_0DI@JFLFLAGO@Java_jdk_jpackage_internal_Exec@ 0000000180015f08     jpackage.obj
 0002:00001f40       ??_C@_0DL@KDKICCGN@Java_jdk_jpackage_internal_Exec@ 0000000180015f40     jpackage.obj
 0002:00001f88       ??_7?$basic_istringstream@DU?$char_traits@D@std@@V?$allocator@D@2@@std@@6B@ 0000000180015f88     jpackage.obj
 0002:00001f90       ??_8?$basic_istringstream@DU?$char_traits@D@std@@V?$allocator@D@2@@std@@7B@ 0000000180015f90     jpackage.obj
 0002:00001f98       ??_C@_17BKKLFCBK@?$AAm?$AAs?$AAi@ 0000000180015f98     jpackage.obj
 0002:00001fa0       ??_C@_1BK@BMAHLKDK@?$AAp?$AAr?$AAo?$AAd?$AAu?$AAc?$AAt?$AA_?$AAc?$AAo?$AAd?$AAe@ 0000000180015fa0     jpackage.obj
 0002:00001fc0       ??_C@_0DC@CADNMJOE@Java_jdk_jpackage_internal_WinE@ 0000000180015fc0     jpackage.obj
 0002:00001ff8       ??_C@_0DH@LNAINGFP@Java_jdk_jpackage_internal_Shor@ 0000000180015ff8     jpackage.obj
 0002:00002038       ??_7logic_error@std@@6B@   0000000180016038     tstrings.obj
 0002:00002050       ??_7invalid_argument@std@@6B@ 0000000180016050     tstrings.obj
 0002:00002060       ??_C@_0CB@PKEJGPPE@Destination?5buffer?5can?8t?5be?5NUL@ 0000000180016060     tstrings.obj
 0002:00002088       ??_C@_0CN@LGHLBHHG@tstrings?3?3?$GAanonymous?9namespace?8@ 0000000180016088     tstrings.obj
 0002:000020b8       ??_C@_0DE@PAENJCPL@s?2src?2jdk?4jpackage?2share?2native@ 00000001800160b8     tstrings.obj
 0002:000020f0       ??_C@_0CM@GJHHAJJB@Unexpected?5reply?5from?5WideCharT@ 00000001800160f0     tstrings.obj
 0002:00002120       ??_C@_0CP@CGMDKJBF@tstrings?3?3?$GAanonymous?9namespace?8@ 0000000180016120     tstrings.obj
 0002:00002150       ??_C@_0CM@HMGDIOLF@Unexpected?5reply?5from?5MultiByte@ 0000000180016150     tstrings.obj
 0002:000021c0       __xmm@ffffffffffffffffffffffffffffffff 00000001800161c0     msvcprt:vector_algorithms.obj
 0002:000021d0       ?nothrow@std@@3Unothrow_t@1@B 00000001800161d0     msvcprt:nothrow.obj
 0002:000021e0       ??_7type_info@@6B@         00000001800161e0     MSVCRT:std_type_info_static.obj
 0002:000021f8       _pDefaultRawDllMain        00000001800161f8     MSVCRT:dll_dllmain.obj
 0002:000021f8       _pRawDllMain               00000001800161f8     MSVCRT:dll_dllmain.obj
 0002:00002200       ??_C@_0P@GHFPNOJB@bad?5allocation@ 0000000180016200     MSVCRT:throw_bad_alloc.obj
 0002:00002210       _load_config_used          0000000180016210     MSVCRT:loadcfg.obj
 0002:00002400       ??_R4exception@std@@6B@    0000000180016400     ErrorHandling.obj
 0002:00002428       ??_R3exception@std@@8      0000000180016428     ErrorHandling.obj
 0002:00002440       ??_R2exception@std@@8      0000000180016440     ErrorHandling.obj
 0002:00002450       ??_R1A@?0A@EA@exception@std@@8 0000000180016450     ErrorHandling.obj
 0002:00002478       ??_R4bad_array_new_length@std@@6B@ 0000000180016478     ErrorHandling.obj
 0002:000024a0       ??_R3bad_array_new_length@std@@8 00000001800164a0     ErrorHandling.obj
 0002:000024b8       ??_R2bad_array_new_length@std@@8 00000001800164b8     ErrorHandling.obj
 0002:000024d8       ??_R1A@?0A@EA@bad_array_new_length@std@@8 00000001800164d8     ErrorHandling.obj
 0002:00002500       ??_R1A@?0A@EA@bad_alloc@std@@8 0000000180016500     ErrorHandling.obj
 0002:00002528       ??_R3bad_alloc@std@@8      0000000180016528     ErrorHandling.obj
 0002:00002540       ??_R2bad_alloc@std@@8      0000000180016540     ErrorHandling.obj
 0002:00002558       ??_R4bad_alloc@std@@6B@    0000000180016558     ErrorHandling.obj
 0002:00002580       ??_R4?$basic_stringbuf@DU?$char_traits@D@std@@V?$allocator@D@2@@std@@6B@ 0000000180016580     ErrorHandling.obj
 0002:000025a8       ??_R3?$basic_stringbuf@DU?$char_traits@D@std@@V?$allocator@D@2@@std@@8 00000001800165a8     ErrorHandling.obj
 0002:000025c0       ??_R2?$basic_stringbuf@DU?$char_traits@D@std@@V?$allocator@D@2@@std@@8 00000001800165c0     ErrorHandling.obj
 0002:000025d8       ??_R1A@?0A@EA@?$basic_stringbuf@DU?$char_traits@D@std@@V?$allocator@D@2@@std@@8 00000001800165d8     ErrorHandling.obj
 0002:00002600       ??_R1A@?0A@EA@?$basic_streambuf@DU?$char_traits@D@std@@@std@@8 0000000180016600     ErrorHandling.obj
 0002:00002628       ??_R3?$basic_streambuf@DU?$char_traits@D@std@@@std@@8 0000000180016628     ErrorHandling.obj
 0002:00002640       ??_R2?$basic_streambuf@DU?$char_traits@D@std@@@std@@8 0000000180016640     ErrorHandling.obj
 0002:00002650       ??_R4?$basic_ostringstream@DU?$char_traits@D@std@@V?$allocator@D@2@@std@@6B@ 0000000180016650     ErrorHandling.obj
 0002:00002678       ??_R3?$basic_ostringstream@DU?$char_traits@D@std@@V?$allocator@D@2@@std@@8 0000000180016678     ErrorHandling.obj
 0002:00002690       ??_R2?$basic_ostringstream@DU?$char_traits@D@std@@V?$allocator@D@2@@std@@8 0000000180016690     ErrorHandling.obj
 0002:000026c0       ??_R1A@?0A@EA@?$basic_ostringstream@DU?$char_traits@D@std@@V?$allocator@D@2@@std@@8 00000001800166c0     ErrorHandling.obj
 0002:000026e8       ??_R1A@?0A@EA@?$basic_ostream@DU?$char_traits@D@std@@@std@@8 00000001800166e8     ErrorHandling.obj
 0002:00002710       ??_R3?$basic_ostream@DU?$char_traits@D@std@@@std@@8 0000000180016710     ErrorHandling.obj
 0002:00002728       ??_R2?$basic_ostream@DU?$char_traits@D@std@@@std@@8 0000000180016728     ErrorHandling.obj
 0002:00002750       ??_R1A@A@3FA@?$basic_ios@DU?$char_traits@D@std@@@std@@8 0000000180016750     ErrorHandling.obj
 0002:00002778       ??_R3?$basic_ios@DU?$char_traits@D@std@@@std@@8 0000000180016778     ErrorHandling.obj
 0002:00002790       ??_R2?$basic_ios@DU?$char_traits@D@std@@@std@@8 0000000180016790     ErrorHandling.obj
 0002:000027b0       ??_R1A@?0A@EA@?$basic_ios@DU?$char_traits@D@std@@@std@@8 00000001800167b0     ErrorHandling.obj
 0002:000027d8       ??_R1A@?0A@EA@ios_base@std@@8 00000001800167d8     ErrorHandling.obj
 0002:00002800       ??_R3ios_base@std@@8       0000000180016800     ErrorHandling.obj
 0002:00002818       ??_R2ios_base@std@@8       0000000180016818     ErrorHandling.obj
 0002:00002830       ??_R17?0A@EA@?$_Iosb@H@std@@8 0000000180016830     ErrorHandling.obj
 0002:00002858       ??_R3?$_Iosb@H@std@@8      0000000180016858     ErrorHandling.obj
 0002:00002870       ??_R2?$_Iosb@H@std@@8      0000000180016870     ErrorHandling.obj
 0002:00002880       ??_R1A@?0A@EA@?$_Iosb@H@std@@8 0000000180016880     ErrorHandling.obj
 0002:000028a8       ??_R1A@A@3EA@ios_base@std@@8 00000001800168a8     ErrorHandling.obj
 0002:000028d0       ??_R17A@3EA@?$_Iosb@H@std@@8 00000001800168d0     ErrorHandling.obj
 0002:000028f8       ??_R4?$basic_stringbuf@GU?$char_traits@G@std@@V?$allocator@G@2@@std@@6B@ 00000001800168f8     ErrorHandling.obj
 0002:00002920       ??_R3?$basic_stringbuf@GU?$char_traits@G@std@@V?$allocator@G@2@@std@@8 0000000180016920     ErrorHandling.obj
 0002:00002938       ??_R2?$basic_stringbuf@GU?$char_traits@G@std@@V?$allocator@G@2@@std@@8 0000000180016938     ErrorHandling.obj
 0002:00002950       ??_R1A@?0A@EA@?$basic_stringbuf@GU?$char_traits@G@std@@V?$allocator@G@2@@std@@8 0000000180016950     ErrorHandling.obj
 0002:00002978       ??_R1A@?0A@EA@?$basic_streambuf@GU?$char_traits@G@std@@@std@@8 0000000180016978     ErrorHandling.obj
 0002:000029a0       ??_R3?$basic_streambuf@GU?$char_traits@G@std@@@std@@8 00000001800169a0     ErrorHandling.obj
 0002:000029b8       ??_R2?$basic_streambuf@GU?$char_traits@G@std@@@std@@8 00000001800169b8     ErrorHandling.obj
 0002:000029c8       ??_R4?$basic_ostringstream@GU?$char_traits@G@std@@V?$allocator@G@2@@std@@6B@ 00000001800169c8     ErrorHandling.obj
 0002:000029f0       ??_R3?$basic_ostringstream@GU?$char_traits@G@std@@V?$allocator@G@2@@std@@8 00000001800169f0     ErrorHandling.obj
 0002:00002a08       ??_R2?$basic_ostringstream@GU?$char_traits@G@std@@V?$allocator@G@2@@std@@8 0000000180016a08     ErrorHandling.obj
 0002:00002a38       ??_R1A@?0A@EA@?$basic_ostringstream@GU?$char_traits@G@std@@V?$allocator@G@2@@std@@8 0000000180016a38     ErrorHandling.obj
 0002:00002a60       ??_R1A@?0A@EA@?$basic_ostream@GU?$char_traits@G@std@@@std@@8 0000000180016a60     ErrorHandling.obj
 0002:00002a88       ??_R3?$basic_ostream@GU?$char_traits@G@std@@@std@@8 0000000180016a88     ErrorHandling.obj
 0002:00002aa0       ??_R2?$basic_ostream@GU?$char_traits@G@std@@@std@@8 0000000180016aa0     ErrorHandling.obj
 0002:00002ac8       ??_R1A@A@3FA@?$basic_ios@GU?$char_traits@G@std@@@std@@8 0000000180016ac8     ErrorHandling.obj
 0002:00002af0       ??_R3?$basic_ios@GU?$char_traits@G@std@@@std@@8 0000000180016af0     ErrorHandling.obj
 0002:00002b08       ??_R2?$basic_ios@GU?$char_traits@G@std@@@std@@8 0000000180016b08     ErrorHandling.obj
 0002:00002b28       ??_R1A@?0A@EA@?$basic_ios@GU?$char_traits@G@std@@@std@@8 0000000180016b28     ErrorHandling.obj
 0002:00002b50       ??_R4bad_cast@std@@6B@     0000000180016b50     ErrorHandling.obj
 0002:00002b78       ??_R3bad_cast@std@@8       0000000180016b78     ErrorHandling.obj
 0002:00002b90       ??_R2bad_cast@std@@8       0000000180016b90     ErrorHandling.obj
 0002:00002ba8       ??_R1A@?0A@EA@bad_cast@std@@8 0000000180016ba8     ErrorHandling.obj
 0002:00002bd0       ??_R4runtime_error@std@@6B@ 0000000180016bd0     Executor.obj
 0002:00002bf8       ??_R3runtime_error@std@@8  0000000180016bf8     Executor.obj
 0002:00002c10       ??_R2runtime_error@std@@8  0000000180016c10     Executor.obj
 0002:00002c28       ??_R1A@?0A@EA@runtime_error@std@@8 0000000180016c28     Executor.obj
 0002:00002c50       ??_R4JpErrorBase@@6B@      0000000180016c50     Executor.obj
 0002:00002c78       ??_R3JpErrorBase@@8        0000000180016c78     Executor.obj
 0002:00002c90       ??_R2JpErrorBase@@8        0000000180016c90     Executor.obj
 0002:00002ca0       ??_R1A@?0A@EA@JpErrorBase@@8 0000000180016ca0     Executor.obj
 0002:00002cc8       ??_R17?0A@EA@runtime_error@std@@8 0000000180016cc8     Executor.obj
 0002:00002cf0       ??_R17?0A@EA@exception@std@@8 0000000180016cf0     Executor.obj
 0002:00002d18       ??_R4SysError@@6B@         0000000180016d18     Executor.obj
 0002:00002d40       ??_R3SysError@@8           0000000180016d40     Executor.obj
 0002:00002d58       ??_R2SysError@@8           0000000180016d58     Executor.obj
 0002:00002d78       ??_R1A@?0A@EA@SysError@@8  0000000180016d78     Executor.obj
 0002:00002da0       ??_R4?$JpError@VSysError@@@@6BJpErrorBase@@@ 0000000180016da0     Executor.obj
 0002:00002dc8       ??_R3?$JpError@VSysError@@@@8 0000000180016dc8     Executor.obj
 0002:00002de0       ??_R2?$JpError@VSysError@@@@8 0000000180016de0     Executor.obj
 0002:00002e10       ??_R1A@?0A@EA@?$JpError@VSysError@@@@8 0000000180016e10     Executor.obj
 0002:00002e38       ??_R17?0A@EA@SysError@@8   0000000180016e38     Executor.obj
 0002:00002e60       ??_R4?$JpError@VSysError@@@@6BSysError@@@ 0000000180016e60     Executor.obj
 0002:00002e88       ??_R4?$JpError@Vruntime_error@std@@@@6BJpErrorBase@@@ 0000000180016e88     Guid.obj
 0002:00002eb0       ??_R3?$JpError@Vruntime_error@std@@@@8 0000000180016eb0     Guid.obj
 0002:00002ec8       ??_R2?$JpError@Vruntime_error@std@@@@8 0000000180016ec8     Guid.obj
 0002:00002ef0       ??_R1A@?0A@EA@?$JpError@Vruntime_error@std@@@@8 0000000180016ef0     Guid.obj
 0002:00002f18       ??_R4?$JpError@Vruntime_error@std@@@@6Bruntime_error@std@@@ 0000000180016f18     Guid.obj
 0002:00002f40       ??_R4StreamLogAppender@@6B@ 0000000180016f40     Log.obj
 0002:00002f68       ??_R3StreamLogAppender@@8  0000000180016f68     Log.obj
 0002:00002f80       ??_R2StreamLogAppender@@8  0000000180016f80     Log.obj
 0002:00002f98       ??_R1A@?0A@EA@StreamLogAppender@@8 0000000180016f98     Log.obj
 0002:00002fc0       ??_R1A@?0A@EA@LogAppender@@8 0000000180016fc0     Log.obj
 0002:00002fe8       ??_R3LogAppender@@8        0000000180016fe8     Log.obj
 0002:00003000       ??_R2LogAppender@@8        0000000180017000     Log.obj
 0002:00003010       ??_R4LogAppender@@6B@      0000000180017010     Log.obj
 0002:00003038       ??_R4Error@msi@@6B@        0000000180017038     MsiCA.obj
 0002:00003060       ??_R3Error@msi@@8          0000000180017060     MsiCA.obj
 0002:00003078       ??_R2Error@msi@@8          0000000180017078     MsiCA.obj
 0002:00003098       ??_R1A@?0A@EA@Error@msi@@8 0000000180017098     MsiCA.obj
 0002:000030c0       ??_R4?$JpError@VError@msi@@@@6BJpErrorBase@@@ 00000001800170c0     MsiCA.obj
 0002:000030e8       ??_R3?$JpError@VError@msi@@@@8 00000001800170e8     MsiCA.obj
 0002:00003100       ??_R2?$JpError@VError@msi@@@@8 0000000180017100     MsiCA.obj
 0002:00003130       ??_R1A@?0A@EA@?$JpError@VError@msi@@@@8 0000000180017130     MsiCA.obj
 0002:00003158       ??_R17?0A@EA@Error@msi@@8  0000000180017158     MsiCA.obj
 0002:00003180       ??_R4?$JpError@VError@msi@@@@6BError@msi@@@ 0000000180017180     MsiCA.obj
 0002:000031a8       ??_R4?$basic_filebuf@DU?$char_traits@D@std@@@std@@6B@ 00000001800171a8     MsiDb.obj
 0002:000031d0       ??_R3?$basic_filebuf@DU?$char_traits@D@std@@@std@@8 00000001800171d0     MsiDb.obj
 0002:000031e8       ??_R2?$basic_filebuf@DU?$char_traits@D@std@@@std@@8 00000001800171e8     MsiDb.obj
 0002:00003200       ??_R1A@?0A@EA@?$basic_filebuf@DU?$char_traits@D@std@@@std@@8 0000000180017200     MsiDb.obj
 0002:00003228       ??_R4NoMoreItemsError@msi@@6B@ 0000000180017228     MsiDb.obj
 0002:00003250       ??_R3NoMoreItemsError@msi@@8 0000000180017250     MsiDb.obj
 0002:00003268       ??_R2NoMoreItemsError@msi@@8 0000000180017268     MsiDb.obj
 0002:00003290       ??_R1A@?0A@EA@NoMoreItemsError@msi@@8 0000000180017290     MsiDb.obj
 0002:000032b8       ??_R4?$JpError@VNoMoreItemsError@msi@@@@6BJpErrorBase@@@ 00000001800172b8     MsiDb.obj
 0002:000032e0       ??_R3?$JpError@VNoMoreItemsError@msi@@@@8 00000001800172e0     MsiDb.obj
 0002:000032f8       ??_R2?$JpError@VNoMoreItemsError@msi@@@@8 00000001800172f8     MsiDb.obj
 0002:00003330       ??_R1A@?0A@EA@?$JpError@VNoMoreItemsError@msi@@@@8 0000000180017330     MsiDb.obj
 0002:00003358       ??_R17?0A@EA@NoMoreItemsError@msi@@8 0000000180017358     MsiDb.obj
 0002:00003380       ??_R4?$JpError@VNoMoreItemsError@msi@@@@6BNoMoreItemsError@msi@@@ 0000000180017380     MsiDb.obj
 0002:000033a8       ??_R4?$basic_ifstream@DU?$char_traits@D@std@@@std@@6B@ 00000001800173a8     ResourceEditor.obj
 0002:000033d0       ??_R3?$basic_ifstream@DU?$char_traits@D@std@@@std@@8 00000001800173d0     ResourceEditor.obj
 0002:000033e8       ??_R2?$basic_ifstream@DU?$char_traits@D@std@@@std@@8 00000001800173e8     ResourceEditor.obj
 0002:00003418       ??_R1A@?0A@EA@?$basic_ifstream@DU?$char_traits@D@std@@@std@@8 0000000180017418     ResourceEditor.obj
 0002:00003440       ??_R1A@?0A@EA@?$basic_istream@DU?$char_traits@D@std@@@std@@8 0000000180017440     ResourceEditor.obj
 0002:00003468       ??_R3?$basic_istream@DU?$char_traits@D@std@@@std@@8 0000000180017468     ResourceEditor.obj
 0002:00003480       ??_R2?$basic_istream@DU?$char_traits@D@std@@@std@@8 0000000180017480     ResourceEditor.obj
 0002:000034a8       ??_R4?$basic_stringstream@DU?$char_traits@D@std@@V?$allocator@D@2@@std@@6B@ 00000001800174a8     VersionInfo.obj
 0002:000034d0       ??_R3?$basic_stringstream@DU?$char_traits@D@std@@V?$allocator@D@2@@std@@8 00000001800174d0     VersionInfo.obj
 0002:000034f0       ??_R2?$basic_stringstream@DU?$char_traits@D@std@@V?$allocator@D@2@@std@@8 00000001800174f0     VersionInfo.obj
 0002:00003548       ??_R1A@?0A@EA@?$basic_stringstream@DU?$char_traits@D@std@@V?$allocator@D@2@@std@@8 0000000180017548     VersionInfo.obj
 0002:00003570       ??_R1A@?0A@EA@?$basic_iostream@DU?$char_traits@D@std@@@std@@8 0000000180017570     VersionInfo.obj
 0002:00003598       ??_R3?$basic_iostream@DU?$char_traits@D@std@@@std@@8 0000000180017598     VersionInfo.obj
 0002:000035b0       ??_R2?$basic_iostream@DU?$char_traits@D@std@@@std@@8 00000001800175b0     VersionInfo.obj
 0002:00003600       ??_R1BA@?0A@EA@?$basic_ostream@DU?$char_traits@D@std@@@std@@8 0000000180017600     VersionInfo.obj
 0002:00003628       ??_R4?$basic_stringstream@GU?$char_traits@G@std@@V?$allocator@G@2@@std@@6B@ 0000000180017628     VersionInfo.obj
 0002:00003650       ??_R3?$basic_stringstream@GU?$char_traits@G@std@@V?$allocator@G@2@@std@@8 0000000180017650     VersionInfo.obj
 0002:00003670       ??_R2?$basic_stringstream@GU?$char_traits@G@std@@V?$allocator@G@2@@std@@8 0000000180017670     VersionInfo.obj
 0002:000036c8       ??_R1A@?0A@EA@?$basic_stringstream@GU?$char_traits@G@std@@V?$allocator@G@2@@std@@8 00000001800176c8     VersionInfo.obj
 0002:000036f0       ??_R1A@?0A@EA@?$basic_iostream@GU?$char_traits@G@std@@@std@@8 00000001800176f0     VersionInfo.obj
 0002:00003718       ??_R3?$basic_iostream@GU?$char_traits@G@std@@@std@@8 0000000180017718     VersionInfo.obj
 0002:00003730       ??_R2?$basic_iostream@GU?$char_traits@G@std@@@std@@8 0000000180017730     VersionInfo.obj
 0002:00003780       ??_R1A@?0A@EA@?$basic_istream@GU?$char_traits@G@std@@@std@@8 0000000180017780     VersionInfo.obj
 0002:000037a8       ??_R3?$basic_istream@GU?$char_traits@G@std@@@std@@8 00000001800177a8     VersionInfo.obj
 0002:000037c0       ??_R2?$basic_istream@GU?$char_traits@G@std@@@std@@8 00000001800177c0     VersionInfo.obj
 0002:000037e8       ??_R1BA@?0A@EA@?$basic_ostream@GU?$char_traits@G@std@@@std@@8 00000001800177e8     VersionInfo.obj
 0002:00003890       ??_R4?$basic_istringstream@DU?$char_traits@D@std@@V?$allocator@D@2@@std@@6B@ 0000000180017890     jpackage.obj
 0002:000038b8       ??_R3?$basic_istringstream@DU?$char_traits@D@std@@V?$allocator@D@2@@std@@8 00000001800178b8     jpackage.obj
 0002:000038d0       ??_R2?$basic_istringstream@DU?$char_traits@D@std@@V?$allocator@D@2@@std@@8 00000001800178d0     jpackage.obj
 0002:00003900       ??_R1A@?0A@EA@?$basic_istringstream@DU?$char_traits@D@std@@V?$allocator@D@2@@std@@8 0000000180017900     jpackage.obj
 0002:00003928       ??_R4logic_error@std@@6B@  0000000180017928     tstrings.obj
 0002:00003950       ??_R3logic_error@std@@8    0000000180017950     tstrings.obj
 0002:00003968       ??_R2logic_error@std@@8    0000000180017968     tstrings.obj
 0002:00003980       ??_R1A@?0A@EA@logic_error@std@@8 0000000180017980     tstrings.obj
 0002:000039a8       ??_R4invalid_argument@std@@6B@ 00000001800179a8     tstrings.obj
 0002:000039d0       ??_R3invalid_argument@std@@8 00000001800179d0     tstrings.obj
 0002:000039e8       ??_R2invalid_argument@std@@8 00000001800179e8     tstrings.obj
 0002:00003a08       ??_R1A@?0A@EA@invalid_argument@std@@8 0000000180017a08     tstrings.obj
 0002:00003a30       ??_R4type_info@@6B@        0000000180017a30     MSVCRT:std_type_info_static.obj
 0002:00003a58       ??_R3type_info@@8          0000000180017a58     MSVCRT:std_type_info_static.obj
 0002:00003a70       ??_R2type_info@@8          0000000180017a70     MSVCRT:std_type_info_static.obj
 0002:00003a80       ??_R1A@?0A@EA@type_info@@8 0000000180017a80     MSVCRT:std_type_info_static.obj
 0002:00003aa4       __volatile_metadata        0000000180017aa4     <linker-defined>
 0002:00003f18       __rtc_iaa                  0000000180017f18     MSVCRT:initsect.obj
 0002:00003f20       __rtc_izz                  0000000180017f20     MSVCRT:initsect.obj
 0002:00003f28       __rtc_taa                  0000000180017f28     MSVCRT:initsect.obj
 0002:00003f30       __rtc_tzz                  0000000180017f30     MSVCRT:initsect.obj
 0002:000062b8       _CT??_R0?AVexception@std@@@8??0exception@std@@QEAA@AEBV01@@Z24 000000018001a2b8     ErrorHandling.obj
 0002:000062e0       _TI3?AVbad_array_new_length@std@@ 000000018001a2e0     ErrorHandling.obj
 0002:00006300       _CTA3?AVbad_array_new_length@std@@ 000000018001a300     ErrorHandling.obj
 0002:00006320       _CT??_R0?AVbad_array_new_length@std@@@8??0bad_array_new_length@std@@QEAA@AEBV01@@Z24 000000018001a320     ErrorHandling.obj
 0002:00006348       _CT??_R0?AVbad_alloc@std@@@8??0bad_alloc@std@@QEAA@AEBV01@@Z24 000000018001a348     ErrorHandling.obj
 0002:00006370       _TI2?AVbad_cast@std@@      000000018001a370     ErrorHandling.obj
 0002:00006390       _CTA2?AVbad_cast@std@@     000000018001a390     ErrorHandling.obj
 0002:000063a8       _CT??_R0?AVbad_cast@std@@@8??0bad_cast@std@@QEAA@AEBV01@@Z24 000000018001a3a8     ErrorHandling.obj
 0002:000063d0       _TI5?AV?$JpError@VSysError@@@@ 000000018001a3d0     Executor.obj
 0002:000063f0       _CTA5?AV?$JpError@VSysError@@@@ 000000018001a3f0     Executor.obj
 0002:00006420       _CT??_R0?AV?$JpError@VSysError@@@@@8??0?$JpError@VSysError@@@@QEAA@AEBV0@@Z64 000000018001a420     Executor.obj
 0002:00006448       _CT??_R0?AVJpErrorBase@@@8??0JpErrorBase@@QEAA@AEBV0@@Z8 000000018001a448     Executor.obj
 0002:00006470       _CT??_R0?AVSysError@@@8??0SysError@@QEAA@AEBV0@@Z248 000000018001a470     Executor.obj
 0002:00006498       _CT??_R0?AVruntime_error@std@@@8??0runtime_error@std@@QEAA@AEBV01@@Z248 000000018001a498     Executor.obj
 0002:000064c0       _CT??_R0?AVexception@std@@@8??0exception@std@@QEAA@AEBV01@@Z248 000000018001a4c0     Executor.obj
 0002:000064e8       _TI4?AV?$JpError@Vruntime_error@std@@@@ 000000018001a4e8     Guid.obj
 0002:00006508       _CTA4?AV?$JpError@Vruntime_error@std@@@@ 000000018001a508     Guid.obj
 0002:00006530       _CT??_R0?AV?$JpError@Vruntime_error@std@@@@@8??0?$JpError@Vruntime_error@std@@@@QEAA@AEBV0@@Z64 000000018001a530     Guid.obj
 0002:00006558       _TI5?AV?$JpError@VError@msi@@@@ 000000018001a558     MsiCA.obj
 0002:00006578       _CTA5?AV?$JpError@VError@msi@@@@ 000000018001a578     MsiCA.obj
 0002:000065a8       _CT??_R0?AV?$JpError@VError@msi@@@@@8??0?$JpError@VError@msi@@@@QEAA@AEBV0@@Z72 000000018001a5a8     MsiCA.obj
 0002:000065d0       _CT??_R0?AVError@msi@@@8??0Error@msi@@QEAA@AEBV01@@Z328 000000018001a5d0     MsiCA.obj
 0002:000065f8       _TI6?AV?$JpError@VNoMoreItemsError@msi@@@@ 000000018001a5f8     MsiDb.obj
 0002:00006618       _CTA6?AV?$JpError@VNoMoreItemsError@msi@@@@ 000000018001a618     MsiDb.obj
 0002:00006650       _CT??_R0?AV?$JpError@VNoMoreItemsError@msi@@@@@8??0?$JpError@VNoMoreItemsError@msi@@@@QEAA@AEBV0@@Z72 000000018001a650     MsiDb.obj
 0002:00006678       _CT??_R0?AVNoMoreItemsError@msi@@@8??0NoMoreItemsError@msi@@QEAA@AEBV01@@Z328 000000018001a678     MsiDb.obj
 0002:000066a0       _TI3?AVinvalid_argument@std@@ 000000018001a6a0     tstrings.obj
 0002:000066c0       _CTA3?AVinvalid_argument@std@@ 000000018001a6c0     tstrings.obj
 0002:000066e0       _CT??_R0?AVinvalid_argument@std@@@8??0invalid_argument@std@@QEAA@AEBV01@@Z24 000000018001a6e0     tstrings.obj
 0002:00006708       _CT??_R0?AVlogic_error@std@@@8??0logic_error@std@@QEAA@AEBV01@@Z24 000000018001a708     tstrings.obj
 0002:00006730       _TI2?AVbad_alloc@std@@     000000018001a730     MSVCRT:throw_bad_alloc.obj
 0002:00006750       _CTA2?AVbad_alloc@std@@    000000018001a750     MSVCRT:throw_bad_alloc.obj
 0002:00006a90       __IMPORT_DESCRIPTOR_ADVAPI32 000000018001aa90     advapi32:ADVAPI32.dll
 0002:00006aa4       __IMPORT_DESCRIPTOR_msi    000000018001aaa4     msi:msi.dll
 0002:00006ab8       __IMPORT_DESCRIPTOR_ole32  000000018001aab8     ole32:ole32.dll
 0002:00006acc       __IMPORT_DESCRIPTOR_MSVCP140 000000018001aacc     msvcprt:MSVCP140.dll
 0002:00006ae0       __IMPORT_DESCRIPTOR_KERNEL32 000000018001aae0     kernel32:KERNEL32.dll
 0002:00006af4       __IMPORT_DESCRIPTOR_VCRUNTIME140 000000018001aaf4     vcruntime:VCRUNTIME140.dll
 0002:00006b08       __IMPORT_DESCRIPTOR_VCRUNTIME140_1 000000018001ab08     vcruntime:VCRUNTIME140_1.dll
 0002:00006b1c       __IMPORT_DESCRIPTOR_api-ms-win-crt-runtime-l1-1-0 000000018001ab1c     ucrt:api-ms-win-crt-runtime-l1-1-0.dll
 0002:00006b30       __IMPORT_DESCRIPTOR_api-ms-win-crt-string-l1-1-0 000000018001ab30     ucrt:api-ms-win-crt-string-l1-1-0.dll
 0002:00006b44       __IMPORT_DESCRIPTOR_api-ms-win-crt-stdio-l1-1-0 000000018001ab44     ucrt:api-ms-win-crt-stdio-l1-1-0.dll
 0002:00006b58       __IMPORT_DESCRIPTOR_api-ms-win-crt-heap-l1-1-0 000000018001ab58     ucrt:api-ms-win-crt-heap-l1-1-0.dll
 0002:00006b6c       __IMPORT_DESCRIPTOR_api-ms-win-crt-filesystem-l1-1-0 000000018001ab6c     ucrt:api-ms-win-crt-filesystem-l1-1-0.dll
 0002:00006b80       __NULL_IMPORT_DESCRIPTOR   000000018001ab80     advapi32:ADVAPI32.dll
 0003:00000240       __security_cookie          000000018001e240     MSVCRT:gs_cookie.obj
 0003:00000280       __security_cookie_complement 000000018001e280     MSVCRT:gs_cookie.obj
 0003:00000288       __scrt_native_dllmain_reason 000000018001e288     MSVCRT:utility.obj
 0003:00000290       __isa_inverted             000000018001e290     MSVCRT:cpu_disp.obj
 0003:00000298       __isa_available            000000018001e298     MSVCRT:cpu_disp.obj
 0003:0000029c       __isa_enabled              000000018001e29c     MSVCRT:cpu_disp.obj
 0003:000002a0       __memset_fast_string_threshold 000000018001e2a0     MSVCRT:cpu_disp.obj
 0003:000002a8       __memset_nt_threshold      000000018001e2a8     MSVCRT:cpu_disp.obj
 0003:000002b0       _fltused                   000000018001e2b0     MSVCRT:fltused.obj
 0003:000002c0       __scrt_ucrt_dll_is_in_use  000000018001e2c0     MSVCRT:ucrt_stubs.obj
 0003:000002c8       ??_R0?AVexception@std@@@8  000000018001e2c8     ErrorHandling.obj
 0003:000002f0       ??_R0?AVbad_array_new_length@std@@@8 000000018001e2f0     ErrorHandling.obj
 0003:00000320       ??_R0?AVbad_alloc@std@@@8  000000018001e320     ErrorHandling.obj
 0003:00000348       ??_R0?AVbad_cast@std@@@8   000000018001e348     ErrorHandling.obj
 0003:00000370       ??_R0?AVruntime_error@std@@@8 000000018001e370     Executor.obj
 0003:00000398       ??_R0?AV?$JpError@VSysError@@@@@8 000000018001e398     Executor.obj
 0003:000003c8       ??_R0?AVJpErrorBase@@@8    000000018001e3c8     Executor.obj
 0003:000003f0       ??_R0?AVSysError@@@8       000000018001e3f0     Executor.obj
 0003:00000410       ??_R0?AV?$JpError@Vruntime_error@std@@@@@8 000000018001e410     Guid.obj
 0003:00000448       ??_R0?AV?$JpError@VError@msi@@@@@8 000000018001e448     MsiCA.obj
 0003:00000478       ??_R0?AVError@msi@@@8      000000018001e478     MsiCA.obj
 0003:00000498       ??_R0?AVNoMoreItemsError@msi@@@8 000000018001e498     MsiDb.obj
 0003:000004c8       ??_R0?AV?$JpError@VNoMoreItemsError@msi@@@@@8 000000018001e4c8     MsiDb.obj
 0003:00000500       ??_R0?AVinvalid_argument@std@@@8 000000018001e500     tstrings.obj
 0003:00000530       ??_R0?AVlogic_error@std@@@8 000000018001e530     tstrings.obj
 0003:00000560       ??_R0?AV?$basic_stringbuf@DU?$char_traits@D@std@@V?$allocator@D@2@@std@@@8 000000018001e560     ErrorHandling.obj
 0003:000005c0       ??_R0?AV?$basic_streambuf@DU?$char_traits@D@std@@@std@@@8 000000018001e5c0     ErrorHandling.obj
 0003:00000610       ??_R0?AV?$basic_ostringstream@DU?$char_traits@D@std@@V?$allocator@D@2@@std@@@8 000000018001e610     ErrorHandling.obj
 0003:00000670       ??_R0?AV?$basic_ostream@DU?$char_traits@D@std@@@std@@@8 000000018001e670     ErrorHandling.obj
 0003:000006b8       ??_R0?AV?$basic_ios@DU?$char_traits@D@std@@@std@@@8 000000018001e6b8     ErrorHandling.obj
 0003:000006f8       ??_R0?AVios_base@std@@@8   000000018001e6f8     ErrorHandling.obj
 0003:00000720       ??_R0?AV?$_Iosb@H@std@@@8  000000018001e720     ErrorHandling.obj
 0003:00000750       ??_R0?AV?$basic_stringbuf@GU?$char_traits@G@std@@V?$allocator@G@2@@std@@@8 000000018001e750     ErrorHandling.obj
 0003:000007b0       ??_R0?AV?$basic_streambuf@GU?$char_traits@G@std@@@std@@@8 000000018001e7b0     ErrorHandling.obj
 0003:00000800       ??_R0?AV?$basic_ostringstream@GU?$char_traits@G@std@@V?$allocator@G@2@@std@@@8 000000018001e800     ErrorHandling.obj
 0003:00000860       ??_R0?AV?$basic_ostream@GU?$char_traits@G@std@@@std@@@8 000000018001e860     ErrorHandling.obj
 0003:000008a8       ??_R0?AV?$basic_ios@GU?$char_traits@G@std@@@std@@@8 000000018001e8a8     ErrorHandling.obj
 0003:000008e8       ??_R0?AVStreamLogAppender@@@8 000000018001e8e8     Log.obj
 0003:00000910       ??_R0?AVLogAppender@@@8    000000018001e910     Log.obj
 0003:00000940       ??_R0?AV?$basic_filebuf@DU?$char_traits@D@std@@@std@@@8 000000018001e940     MsiDb.obj
 0003:00000990       ??_R0?AV?$basic_ifstream@DU?$char_traits@D@std@@@std@@@8 000000018001e990     ResourceEditor.obj
 0003:000009e0       ??_R0?AV?$basic_istream@DU?$char_traits@D@std@@@std@@@8 000000018001e9e0     ResourceEditor.obj
 0003:00000a30       ??_R0?AV?$basic_stringstream@DU?$char_traits@D@std@@V?$allocator@D@2@@std@@@8 000000018001ea30     VersionInfo.obj
 0003:00000a90       ??_R0?AV?$basic_iostream@DU?$char_traits@D@std@@@std@@@8 000000018001ea90     VersionInfo.obj
 0003:00000ae0       ??_R0?AV?$basic_stringstream@GU?$char_traits@G@std@@V?$allocator@G@2@@std@@@8 000000018001eae0     VersionInfo.obj
 0003:00000b40       ??_R0?AV?$basic_iostream@GU?$char_traits@G@std@@@std@@@8 000000018001eb40     VersionInfo.obj
 0003:00000b90       ??_R0?AV?$basic_istream@GU?$char_traits@G@std@@@std@@@8 000000018001eb90     VersionInfo.obj
 0003:00000c10       ??_R0?AV?$basic_istringstream@DU?$char_traits@D@std@@V?$allocator@D@2@@std@@@8 000000018001ec10     jpackage.obj
 0003:00000c70       ??_R0?AVtype_info@@@8      000000018001ec70     MSVCRT:std_type_info_static.obj
 0003:00000c90       _Avx2WmemEnabled           000000018001ec90     ErrorHandling.obj
 0003:00000c90       _Avx2WmemEnabledWeakValue  000000018001ec90     ErrorHandling.obj
 0003:00000c98       ?_Psave@?$_Facetptr@V?$ctype@G@std@@@std@@2PEBVfacet@locale@2@EB 000000018001ec98     ErrorHandling.obj
 0003:00000ca0       ?_OptionsStorage@?1??__local_stdio_printf_options@@9@4_KA 000000018001eca0     IconSwap.obj
 0003:00000cd0       ?_Stinit@?1??_Init@?$basic_filebuf@DU?$char_traits@D@std@@@std@@IEAAXPEAU_iobuf@@W4_Initfl@23@@Z@4U_Mbstatet@@A 000000018001ecd0     MsiDb.obj
 0003:00000cd8       ?_Psave@?$_Facetptr@V?$codecvt@DDU_Mbstatet@@@std@@@std@@2PEBVfacet@locale@2@EB 000000018001ecd8     MsiDb.obj
 0003:00000ce0       ?_OptionsStorage@?1??__local_stdio_scanf_options@@9@4_KA 000000018001ece0     VersionInfo.obj
 0003:00001280       __scrt_current_native_startup_state 000000018001f280     MSVCRT:utility.obj
 0003:00001288       __scrt_native_startup_lock 000000018001f288     MSVCRT:utility.obj
 0003:000012cc       __avx10_version            000000018001f2cc     MSVCRT:cpu_disp.obj
 0003:000012d0       __favor                    000000018001f2d0     MSVCRT:cpu_disp.obj
 0003:000012d4       __scrt_debugger_hook_flag  000000018001f2d4     MSVCRT:utility_desktop.obj
 0003:000012e0       ?__type_info_root_node@@3U__type_info_node@@A 000000018001f2e0     MSVCRT:tncleanup.obj
 0003:000012f0       __dyn_tls_init_callback    000000018001f2f0     <common>

 entry point at        0001:000109bc

 Static symbols

 0000:fffdc000       .debug$S                   0000000180000000     jpackage.exp
 0000:fffdc000       .debug$S                   0000000180000000     msvcprt:MSVCP140.dll
 0000:fffdc000       .debug$S                   0000000180000000     msvcprt:MSVCP140.dll
 0000:fffdc000       .debug$S                   0000000180000000     msvcprt:MSVCP140.dll
 0000:fffdc000       .debug$S                   0000000180000000     msvcprt:MSVCP140.dll
 0000:fffdc000       .debug$S                   0000000180000000     msvcprt:MSVCP140.dll
 0000:fffdc000       .debug$S                   0000000180000000     msvcprt:MSVCP140.dll
 0000:fffdc000       .debug$S                   0000000180000000     msvcprt:MSVCP140.dll
 0000:fffdc000       .debug$S                   0000000180000000     msvcprt:MSVCP140.dll
 0000:fffdc000       .debug$S                   0000000180000000     msvcprt:MSVCP140.dll
 0000:fffdc000       .debug$S                   0000000180000000     msvcprt:MSVCP140.dll
 0000:fffdc000       .debug$S                   0000000180000000     msvcprt:MSVCP140.dll
 0000:fffdc000       .debug$S                   0000000180000000     msvcprt:MSVCP140.dll
 0000:fffdc000       .debug$S                   0000000180000000     msvcprt:MSVCP140.dll
 0000:fffdc000       .debug$S                   0000000180000000     msvcprt:MSVCP140.dll
 0000:fffdc000       .debug$S                   0000000180000000     msvcprt:MSVCP140.dll
 0000:fffdc000       .debug$S                   0000000180000000     msvcprt:MSVCP140.dll
 0000:fffdc000       .debug$S                   0000000180000000     msvcprt:MSVCP140.dll
 0000:fffdc000       .debug$S                   0000000180000000     msvcprt:MSVCP140.dll
 0000:fffdc000       .debug$S                   0000000180000000     msvcprt:MSVCP140.dll
 0000:fffdc000       .debug$S                   0000000180000000     msvcprt:MSVCP140.dll
 0000:fffdc000       .debug$S                   0000000180000000     msvcprt:MSVCP140.dll
 0000:fffdc000       .debug$S                   0000000180000000     msvcprt:MSVCP140.dll
 0000:fffdc000       .debug$S                   0000000180000000     msvcprt:MSVCP140.dll
 0000:fffdc000       .debug$S                   0000000180000000     msvcprt:MSVCP140.dll
 0000:fffdc000       .debug$S                   0000000180000000     msvcprt:MSVCP140.dll
 0000:fffdc000       .debug$S                   0000000180000000     msvcprt:MSVCP140.dll
 0000:fffdc000       .debug$S                   0000000180000000     msvcprt:MSVCP140.dll
 0000:fffdc000       .debug$S                   0000000180000000     msvcprt:MSVCP140.dll
 0000:fffdc000       .debug$S                   0000000180000000     msvcprt:MSVCP140.dll
 0000:fffdc000       .debug$S                   0000000180000000     msvcprt:MSVCP140.dll
 0000:fffdc000       .debug$S                   0000000180000000     msvcprt:MSVCP140.dll
 0000:fffdc000       .debug$S                   0000000180000000     msvcprt:MSVCP140.dll
 0000:fffdc000       .debug$S                   0000000180000000     msvcprt:MSVCP140.dll
 0000:fffdc000       .debug$S                   0000000180000000     msvcprt:MSVCP140.dll
 0000:fffdc000       .debug$S                   0000000180000000     msvcprt:MSVCP140.dll
 0000:fffdc000       .debug$S                   0000000180000000     msvcprt:MSVCP140.dll
 0000:fffdc000       .debug$S                   0000000180000000     msvcprt:MSVCP140.dll
 0000:fffdc000       .debug$S                   0000000180000000     msvcprt:MSVCP140.dll
 0000:fffdc000       .debug$S                   0000000180000000     msvcprt:MSVCP140.dll
 0000:fffdc000       .debug$S                   0000000180000000     msvcprt:MSVCP140.dll
 0000:fffdc000       .debug$S                   0000000180000000     msvcprt:MSVCP140.dll
 0000:fffdc000       .debug$S                   0000000180000000     msvcprt:MSVCP140.dll
 0000:fffdc000       .debug$S                   0000000180000000     msvcprt:MSVCP140.dll
 0000:fffdc000       .debug$S                   0000000180000000     msvcprt:MSVCP140.dll
 0000:fffdc000       .debug$S                   0000000180000000     msvcprt:MSVCP140.dll
 0000:fffdc000       .debug$S                   0000000180000000     msvcprt:MSVCP140.dll
 0000:fffdc000       .debug$S                   0000000180000000     msvcprt:MSVCP140.dll
 0000:fffdc000       .debug$S                   0000000180000000     msvcprt:MSVCP140.dll
 0000:fffdc000       .debug$S                   0000000180000000     msvcprt:MSVCP140.dll
 0000:fffdc000       .debug$S                   0000000180000000     msvcprt:MSVCP140.dll
 0000:fffdc000       .debug$S                   0000000180000000     msvcprt:MSVCP140.dll
 0000:fffdc000       .debug$S                   0000000180000000     msvcprt:MSVCP140.dll
 0000:fffdc000       .debug$S                   0000000180000000     msvcprt:MSVCP140.dll
 0000:fffdc000       .debug$S                   0000000180000000     msvcprt:MSVCP140.dll
 0000:fffdc000       .debug$S                   0000000180000000     msvcprt:MSVCP140.dll
 0000:fffdc000       .debug$S                   0000000180000000     msvcprt:MSVCP140.dll
 0000:fffdc000       .debug$S                   0000000180000000     msvcprt:MSVCP140.dll
 0000:fffdc000       .debug$S                   0000000180000000     msvcprt:MSVCP140.dll
 0000:fffdc000       .debug$S                   0000000180000000     msvcprt:MSVCP140.dll
 0000:fffdc000       .debug$S                   0000000180000000     msvcprt:MSVCP140.dll
 0000:fffdc000       .debug$S                   0000000180000000     msvcprt:MSVCP140.dll
 0000:fffdc000       .debug$S                   0000000180000000     msvcprt:MSVCP140.dll
 0000:fffdc000       .debug$S                   0000000180000000     msvcprt:MSVCP140.dll
 0000:fffdc000       .debug$S                   0000000180000000     msvcprt:MSVCP140.dll
 0000:fffdc000       .debug$S                   0000000180000000     msvcprt:MSVCP140.dll
 0000:fffdc000       .debug$S                   0000000180000000     msvcprt:MSVCP140.dll
 0000:fffdc000       .debug$S                   0000000180000000     msvcprt:MSVCP140.dll
 0000:fffdc000       .debug$S                   0000000180000000     msvcprt:MSVCP140.dll
 0000:fffdc000       .debug$S                   0000000180000000     msvcprt:MSVCP140.dll
 0000:fffdc000       .debug$S                   0000000180000000     msvcprt:MSVCP140.dll
 0000:fffdc000       .debug$S                   0000000180000000     msvcprt:MSVCP140.dll
 0000:fffdc000       .debug$S                   0000000180000000     msvcprt:MSVCP140.dll
 0000:fffdc000       .debug$S                   0000000180000000     msvcprt:MSVCP140.dll
 0000:fffdc000       .debug$S                   0000000180000000     msvcprt:MSVCP140.dll
 0000:fffdc000       .debug$S                   0000000180000000     msvcprt:MSVCP140.dll
 0000:fffdc000       .debug$S                   0000000180000000     msvcprt:MSVCP140.dll
 0000:fffdc000       .debug$S                   0000000180000000     msvcprt:MSVCP140.dll
 0000:fffdc000       .debug$S                   0000000180000000     msvcprt:MSVCP140.dll
 0000:fffdc000       .debug$S                   0000000180000000     msvcprt:MSVCP140.dll
 0000:fffdc000       .debug$S                   0000000180000000     msvcprt:MSVCP140.dll
 0000:fffdc000       .debug$S                   0000000180000000     msvcprt:MSVCP140.dll
 0000:fffdc000       .debug$S                   0000000180000000     msvcprt:MSVCP140.dll
 0000:fffdc000       .debug$S                   0000000180000000     msvcprt:MSVCP140.dll
 0000:fffdc000       .debug$S                   0000000180000000     msvcprt:MSVCP140.dll
 0000:fffdc000       .debug$S                   0000000180000000     msvcprt:MSVCP140.dll
 0000:fffdc000       .debug$S                   0000000180000000     msvcprt:MSVCP140.dll
 0000:fffdc000       .debug$S                   0000000180000000     msvcprt:MSVCP140.dll
 0000:fffdc000       .debug$S                   0000000180000000     msvcprt:MSVCP140.dll
 0000:fffdc000       .debug$S                   0000000180000000     msvcprt:MSVCP140.dll
 0000:fffdc000       .debug$S                   0000000180000000     msvcprt:MSVCP140.dll
 0000:fffdc000       .debug$S                   0000000180000000     msvcprt:MSVCP140.dll
 0000:fffdc000       .debug$S                   0000000180000000     msvcprt:MSVCP140.dll
 0000:fffdc000       .debug$S                   0000000180000000     msvcprt:MSVCP140.dll
 0000:fffdc000       .debug$S                   0000000180000000     msvcprt:MSVCP140.dll
 0000:fffdc000       .debug$S                   0000000180000000     msvcprt:MSVCP140.dll
 0000:fffdc000       .debug$S                   0000000180000000     msvcprt:MSVCP140.dll
 0000:fffdc000       .debug$S                   0000000180000000     msvcprt:MSVCP140.dll
 0000:fffdc000       .debug$S                   0000000180000000     msvcprt:MSVCP140.dll
 0000:fffdc000       .debug$S                   0000000180000000     msvcprt:MSVCP140.dll
 0000:fffdc000       .debug$S                   0000000180000000     msvcprt:MSVCP140.dll
 0000:fffdc000       .debug$S                   0000000180000000     msvcprt:MSVCP140.dll
 0000:fffdc000       .debug$S                   0000000180000000     msvcprt:MSVCP140.dll
 0000:fffdc000       .debug$S                   0000000180000000     msvcprt:MSVCP140.dll
 0000:fffdc000       .debug$S                   0000000180000000     msvcprt:MSVCP140.dll
 0000:fffdc000       .debug$S                   0000000180000000     msvcprt:MSVCP140.dll
 0000:fffdc000       .debug$S                   0000000180000000     msvcprt:MSVCP140.dll
 0000:fffdc000       .debug$S                   0000000180000000     msvcprt:MSVCP140.dll
 0000:fffdc000       .debug$S                   0000000180000000     msvcprt:MSVCP140.dll
 0000:fffdc000       .debug$S                   0000000180000000     msvcprt:MSVCP140.dll
 0000:fffdc000       .debug$S                   0000000180000000     msvcprt:MSVCP140.dll
 0000:fffdc000       .debug$S                   0000000180000000     msvcprt:MSVCP140.dll
 0000:fffdc000       .debug$S                   0000000180000000     msvcprt:MSVCP140.dll
 0000:fffdc000       .debug$S                   0000000180000000     msvcprt:MSVCP140.dll
 0000:fffdc000       .debug$S                   0000000180000000     msvcprt:MSVCP140.dll
 0000:fffdc000       .debug$S                   0000000180000000     msvcprt:MSVCP140.dll
 0000:fffdc000       .debug$S                   0000000180000000     msvcprt:MSVCP140.dll
 0000:fffdc000       .debug$S                   0000000180000000     msvcprt:MSVCP140.dll
 0000:fffdc000       .debug$S                   0000000180000000     msvcprt:MSVCP140.dll
 0000:fffdc000       .debug$S                   0000000180000000     msvcprt:MSVCP140.dll
 0000:fffdc000       .debug$S                   0000000180000000     msvcprt:MSVCP140.dll
 0000:fffdc000       .debug$S                   0000000180000000     msvcprt:MSVCP140.dll
 0000:fffdc000       .debug$S                   0000000180000000     msvcprt:MSVCP140.dll
 0000:fffdc000       .debug$S                   0000000180000000     msvcprt:MSVCP140.dll
 0000:fffdc000       .debug$S                   0000000180000000     msvcprt:MSVCP140.dll
 0000:fffdc000       .debug$S                   0000000180000000     msvcprt:MSVCP140.dll
 0000:fffdc000       .debug$S                   0000000180000000     msvcprt:MSVCP140.dll
 0000:fffdc000       .debug$S                   0000000180000000     msvcprt:MSVCP140.dll
 0000:fffdc000       .debug$S                   0000000180000000     msvcprt:MSVCP140.dll
 0000:fffdc000       .debug$S                   0000000180000000     msvcprt:MSVCP140.dll
 0000:fffdc000       .debug$S                   0000000180000000     msvcprt:MSVCP140.dll
 0000:fffdc000       .debug$S                   0000000180000000     msvcprt:MSVCP140.dll
 0000:fffdc000       .debug$S                   0000000180000000     msvcprt:MSVCP140.dll
 0000:fffdc000       .debug$S                   0000000180000000     msvcprt:MSVCP140.dll
 0000:fffdc000       .debug$S                   0000000180000000     msvcprt:MSVCP140.dll
 0000:fffdc000       .debug$S                   0000000180000000     msvcprt:MSVCP140.dll
 0000:fffdc000       .debug$S                   0000000180000000     msvcprt:MSVCP140.dll
 0000:fffdc000       .debug$S                   0000000180000000     msvcprt:MSVCP140.dll
 0000:fffdc000       .debug$S                   0000000180000000     msvcprt:MSVCP140.dll
 0000:fffdc000       .debug$S                   0000000180000000     msvcprt:MSVCP140.dll
 0000:fffdc000       .debug$S                   0000000180000000     vcruntime:VCRUNTIME140.dll
 0000:fffdc000       .debug$S                   0000000180000000     vcruntime:VCRUNTIME140.dll
 0000:fffdc000       .debug$S                   0000000180000000     vcruntime:VCRUNTIME140.dll
 0000:fffdc000       .debug$S                   0000000180000000     vcruntime:VCRUNTIME140.dll
 0000:fffdc000       .debug$S                   0000000180000000     vcruntime:VCRUNTIME140.dll
 0000:fffdc000       .debug$S                   0000000180000000     vcruntime:VCRUNTIME140.dll
 0000:fffdc000       .debug$S                   0000000180000000     vcruntime:VCRUNTIME140.dll
 0000:fffdc000       .debug$S                   0000000180000000     vcruntime:VCRUNTIME140.dll
 0000:fffdc000       .debug$S                   0000000180000000     vcruntime:VCRUNTIME140.dll
 0000:fffdc000       .debug$S                   0000000180000000     vcruntime:VCRUNTIME140.dll
 0000:fffdc000       .debug$S                   0000000180000000     vcruntime:VCRUNTIME140.dll
 0000:fffdc000       .debug$S                   0000000180000000     vcruntime:VCRUNTIME140.dll
 0000:fffdc000       .debug$S                   0000000180000000     vcruntime:VCRUNTIME140.dll
 0000:fffdc000       .debug$S                   0000000180000000     vcruntime:VCRUNTIME140.dll
 0000:fffdc000       .debug$S                   0000000180000000     vcruntime:VCRUNTIME140_1.dll
 0000:fffdc000       .debug$S                   0000000180000000     ucrt:api-ms-win-crt-environment-l1-1-0.dll
 0002:fffec000       .idata$6                   0000000180000000     ucrt:api-ms-win-crt-environment-l1-1-0.dll
 0000:fffdc000       .debug$S                   0000000180000000     ucrt:api-ms-win-crt-filesystem-l1-1-0.dll
 0000:fffdc000       .debug$S                   0000000180000000     ucrt:api-ms-win-crt-filesystem-l1-1-0.dll
 0000:fffdc000       .debug$S                   0000000180000000     ucrt:api-ms-win-crt-filesystem-l1-1-0.dll
 0000:fffdc000       .debug$S                   0000000180000000     ucrt:api-ms-win-crt-heap-l1-1-0.dll
 0000:fffdc000       .debug$S                   0000000180000000     ucrt:api-ms-win-crt-heap-l1-1-0.dll
 0000:fffdc000       .debug$S                   0000000180000000     ucrt:api-ms-win-crt-heap-l1-1-0.dll
 0000:fffdc000       .debug$S                   0000000180000000     ucrt:api-ms-win-crt-heap-l1-1-0.dll
 0000:fffdc000       .debug$S                   0000000180000000     ucrt:api-ms-win-crt-runtime-l1-1-0.dll
 0000:fffdc000       .debug$S                   0000000180000000     ucrt:api-ms-win-crt-runtime-l1-1-0.dll
 0000:fffdc000       .debug$S                   0000000180000000     ucrt:api-ms-win-crt-runtime-l1-1-0.dll
 0000:fffdc000       .debug$S                   0000000180000000     ucrt:api-ms-win-crt-runtime-l1-1-0.dll
 0000:fffdc000       .debug$S                   0000000180000000     ucrt:api-ms-win-crt-runtime-l1-1-0.dll
 0000:fffdc000       .debug$S                   0000000180000000     ucrt:api-ms-win-crt-runtime-l1-1-0.dll
 0000:fffdc000       .debug$S                   0000000180000000     ucrt:api-ms-win-crt-runtime-l1-1-0.dll
 0000:fffdc000       .debug$S                   0000000180000000     ucrt:api-ms-win-crt-runtime-l1-1-0.dll
 0000:fffdc000       .debug$S                   0000000180000000     ucrt:api-ms-win-crt-runtime-l1-1-0.dll
 0000:fffdc000       .debug$S                   0000000180000000     ucrt:api-ms-win-crt-runtime-l1-1-0.dll
 0000:fffdc000       .debug$S                   0000000180000000     ucrt:api-ms-win-crt-runtime-l1-1-0.dll
 0000:fffdc000       .debug$S                   0000000180000000     ucrt:api-ms-win-crt-runtime-l1-1-0.dll
 0000:fffdc000       .debug$S                   0000000180000000     ucrt:api-ms-win-crt-runtime-l1-1-0.dll
 0000:fffdc000       .debug$S                   0000000180000000     ucrt:api-ms-win-crt-runtime-l1-1-0.dll
 0000:fffdc000       .debug$S                   0000000180000000     ucrt:api-ms-win-crt-runtime-l1-1-0.dll
 0000:fffdc000       .debug$S                   0000000180000000     ucrt:api-ms-win-crt-stdio-l1-1-0.dll
 0000:fffdc000       .debug$S                   0000000180000000     ucrt:api-ms-win-crt-stdio-l1-1-0.dll
 0000:fffdc000       .debug$S                   0000000180000000     ucrt:api-ms-win-crt-stdio-l1-1-0.dll
 0000:fffdc000       .debug$S                   0000000180000000     ucrt:api-ms-win-crt-stdio-l1-1-0.dll
 0000:fffdc000       .debug$S                   0000000180000000     ucrt:api-ms-win-crt-stdio-l1-1-0.dll
 0000:fffdc000       .debug$S                   0000000180000000     ucrt:api-ms-win-crt-stdio-l1-1-0.dll
 0000:fffdc000       .debug$S                   0000000180000000     ucrt:api-ms-win-crt-stdio-l1-1-0.dll
 0000:fffdc000       .debug$S                   0000000180000000     ucrt:api-ms-win-crt-stdio-l1-1-0.dll
 0000:fffdc000       .debug$S                   0000000180000000     ucrt:api-ms-win-crt-stdio-l1-1-0.dll
 0000:fffdc000       .debug$S                   0000000180000000     ucrt:api-ms-win-crt-stdio-l1-1-0.dll
 0000:fffdc000       .debug$S                   0000000180000000     ucrt:api-ms-win-crt-stdio-l1-1-0.dll
 0000:fffdc000       .debug$S                   0000000180000000     ucrt:api-ms-win-crt-stdio-l1-1-0.dll
 0000:fffdc000       .debug$S                   0000000180000000     ucrt:api-ms-win-crt-stdio-l1-1-0.dll
 0000:fffdc000       .debug$S                   0000000180000000     ucrt:api-ms-win-crt-stdio-l1-1-0.dll
 0000:fffdc000       .debug$S                   0000000180000000     ucrt:api-ms-win-crt-stdio-l1-1-0.dll
 0000:fffdc000       .debug$S                   0000000180000000     ucrt:api-ms-win-crt-stdio-l1-1-0.dll
 0000:fffdc000       .debug$S                   0000000180000000     ucrt:api-ms-win-crt-stdio-l1-1-0.dll
 0000:fffdc000       .debug$S                   0000000180000000     ucrt:api-ms-win-crt-string-l1-1-0.dll
 0000:fffdc000       .debug$S                   0000000180000000     ucrt:api-ms-win-crt-string-l1-1-0.dll
 0000:fffdc000       .debug$S                   0000000180000000     ucrt:api-ms-win-crt-string-l1-1-0.dll
 0000:fffdc000       .debug$S                   0000000180000000     ucrt:api-ms-win-crt-string-l1-1-0.dll
 0000:fffdc000       .debug$S                   0000000180000000     advapi32:ADVAPI32.dll
 0000:fffdc000       .debug$S                   0000000180000000     advapi32:ADVAPI32.dll
 0000:fffdc000       .debug$S                   0000000180000000     advapi32:ADVAPI32.dll
 0000:fffdc000       .debug$S                   0000000180000000     advapi32:ADVAPI32.dll
 0000:fffdc000       .debug$S                   0000000180000000     kernel32:KERNEL32.dll
 0000:fffdc000       .debug$S                   0000000180000000     kernel32:KERNEL32.dll
 0000:fffdc000       .debug$S                   0000000180000000     kernel32:KERNEL32.dll
 0000:fffdc000       .debug$S                   0000000180000000     kernel32:KERNEL32.dll
 0000:fffdc000       .debug$S                   0000000180000000     kernel32:KERNEL32.dll
 0000:fffdc000       .debug$S                   0000000180000000     kernel32:KERNEL32.dll
 0000:fffdc000       .debug$S                   0000000180000000     kernel32:KERNEL32.dll
 0000:fffdc000       .debug$S                   0000000180000000     kernel32:KERNEL32.dll
 0000:fffdc000       .debug$S                   0000000180000000     kernel32:KERNEL32.dll
 0000:fffdc000       .debug$S                   0000000180000000     kernel32:KERNEL32.dll
 0000:fffdc000       .debug$S                   0000000180000000     kernel32:KERNEL32.dll
 0000:fffdc000       .debug$S                   0000000180000000     kernel32:KERNEL32.dll
 0000:fffdc000       .debug$S                   0000000180000000     kernel32:KERNEL32.dll
 0000:fffdc000       .debug$S                   0000000180000000     kernel32:KERNEL32.dll
 0000:fffdc000       .debug$S                   0000000180000000     kernel32:KERNEL32.dll
 0000:fffdc000       .debug$S                   0000000180000000     kernel32:KERNEL32.dll
 0000:fffdc000       .debug$S                   0000000180000000     kernel32:KERNEL32.dll
 0000:fffdc000       .debug$S                   0000000180000000     kernel32:KERNEL32.dll
 0000:fffdc000       .debug$S                   0000000180000000     kernel32:KERNEL32.dll
 0000:fffdc000       .debug$S                   0000000180000000     kernel32:KERNEL32.dll
 0000:fffdc000       .debug$S                   0000000180000000     kernel32:KERNEL32.dll
 0000:fffdc000       .debug$S                   0000000180000000     kernel32:KERNEL32.dll
 0000:fffdc000       .debug$S                   0000000180000000     kernel32:KERNEL32.dll
 0000:fffdc000       .debug$S                   0000000180000000     kernel32:KERNEL32.dll
 0000:fffdc000       .debug$S                   0000000180000000     kernel32:KERNEL32.dll
 0000:fffdc000       .debug$S                   0000000180000000     kernel32:KERNEL32.dll
 0000:fffdc000       .debug$S                   0000000180000000     kernel32:KERNEL32.dll
 0000:fffdc000       .debug$S                   0000000180000000     kernel32:KERNEL32.dll
 0000:fffdc000       .debug$S                   0000000180000000     kernel32:KERNEL32.dll
 0000:fffdc000       .debug$S                   0000000180000000     kernel32:KERNEL32.dll
 0000:fffdc000       .debug$S                   0000000180000000     kernel32:KERNEL32.dll
 0000:fffdc000       .debug$S                   0000000180000000     kernel32:KERNEL32.dll
 0000:fffdc000       .debug$S                   0000000180000000     kernel32:KERNEL32.dll
 0000:fffdc000       .debug$S                   0000000180000000     kernel32:KERNEL32.dll
 0000:fffdc000       .debug$S                   0000000180000000     kernel32:KERNEL32.dll
 0000:fffdc000       .debug$S                   0000000180000000     kernel32:KERNEL32.dll
 0000:fffdc000       .debug$S                   0000000180000000     kernel32:KERNEL32.dll
 0000:fffdc000       .debug$S                   0000000180000000     kernel32:KERNEL32.dll
 0000:fffdc000       .debug$S                   0000000180000000     kernel32:KERNEL32.dll
 0000:fffdc000       .debug$S                   0000000180000000     kernel32:KERNEL32.dll
 0000:fffdc000       .debug$S                   0000000180000000     kernel32:KERNEL32.dll
 0000:fffdc000       .debug$S                   0000000180000000     kernel32:KERNEL32.dll
 0000:fffdc000       .debug$S                   0000000180000000     kernel32:KERNEL32.dll
 0000:fffdc000       .debug$S                   0000000180000000     kernel32:KERNEL32.dll
 0000:fffdc000       .debug$S                   0000000180000000     kernel32:KERNEL32.dll
 0000:fffdc000       .debug$S                   0000000180000000     kernel32:KERNEL32.dll
 0000:fffdc000       .debug$S                   0000000180000000     kernel32:KERNEL32.dll
 0000:fffdc000       .debug$S                   0000000180000000     kernel32:KERNEL32.dll
 0000:fffdc000       .debug$S                   0000000180000000     kernel32:KERNEL32.dll
 0000:fffdc000       .debug$S                   0000000180000000     kernel32:KERNEL32.dll
 0000:fffdc000       .debug$S                   0000000180000000     kernel32:KERNEL32.dll
 0000:fffdc000       .debug$S                   0000000180000000     kernel32:KERNEL32.dll
 0000:fffdc000       .debug$S                   0000000180000000     kernel32:KERNEL32.dll
 0000:fffdc000       .debug$S                   0000000180000000     kernel32:KERNEL32.dll
 0000:fffdc000       .debug$S                   0000000180000000     kernel32:KERNEL32.dll
 0000:fffdc000       .debug$S                   0000000180000000     kernel32:KERNEL32.dll
 0000:fffdc000       .debug$S                   0000000180000000     kernel32:KERNEL32.dll
 0000:fffdc000       .debug$S                   0000000180000000     kernel32:KERNEL32.dll
 0000:fffdc000       .debug$S                   0000000180000000     kernel32:KERNEL32.dll
 0000:fffdc000       .debug$S                   0000000180000000     kernel32:KERNEL32.dll
 0000:fffdc000       .debug$S                   0000000180000000     kernel32:KERNEL32.dll
 0000:fffdc000       .debug$S                   0000000180000000     kernel32:KERNEL32.dll
 0000:fffdc000       .debug$S                   0000000180000000     kernel32:KERNEL32.dll
 0000:fffdc000       .debug$S                   0000000180000000     kernel32:KERNEL32.dll
 0000:fffdc000       .debug$S                   0000000180000000     kernel32:KERNEL32.dll
 0000:fffdc000       .debug$S                   0000000180000000     kernel32:KERNEL32.dll
 0000:fffdc000       .debug$S                   0000000180000000     kernel32:KERNEL32.dll
 0000:fffdc000       .debug$S                   0000000180000000     kernel32:KERNEL32.dll
 0000:fffdc000       .debug$S                   0000000180000000     msi:msi.dll
 0000:fffdc000       .debug$S                   0000000180000000     msi:msi.dll
 0000:fffdc000       .debug$S                   0000000180000000     msi:msi.dll
 0000:fffdc000       .debug$S                   0000000180000000     msi:msi.dll
 0000:fffdc000       .debug$S                   0000000180000000     msi:msi.dll
 0000:fffdc000       .debug$S                   0000000180000000     msi:msi.dll
 0000:fffdc000       .debug$S                   0000000180000000     msi:msi.dll
 0000:fffdc000       .debug$S                   0000000180000000     msi:msi.dll
 0000:fffdc000       .debug$S                   0000000180000000     msi:msi.dll
 0000:fffdc000       .debug$S                   0000000180000000     msi:msi.dll
 0000:fffdc000       .debug$S                   0000000180000000     msi:msi.dll
 0000:fffdc000       .debug$S                   0000000180000000     msi:msi.dll
 0000:fffdc000       .debug$S                   0000000180000000     msi:msi.dll
 0000:fffdc000       .debug$S                   0000000180000000     msi:msi.dll
 0000:fffdc000       .debug$S                   0000000180000000     msi:msi.dll
 0000:fffdc000       .debug$S                   0000000180000000     msi:msi.dll
 0000:fffdc000       .debug$S                   0000000180000000     msi:msi.dll
 0000:fffdc000       .debug$S                   0000000180000000     msi:msi.dll
 0000:fffdc000       .debug$S                   0000000180000000     msi:msi.dll
 0000:fffdc000       .debug$S                   0000000180000000     msi:msi.dll
 0000:fffdc000       .debug$S                   0000000180000000     msi:msi.dll
 0000:fffdc000       .debug$S                   0000000180000000     msi:msi.dll
 0000:fffdc000       .debug$S                   0000000180000000     msi:msi.dll
 0000:fffdc000       .debug$S                   0000000180000000     msi:msi.dll
 0000:fffdc000       .debug$S                   0000000180000000     msi:msi.dll
 0000:fffdc000       .debug$S                   0000000180000000     msi:msi.dll
 0000:fffdc000       .debug$S                   0000000180000000     msi:msi.dll
 0000:fffdc000       .debug$S                   0000000180000000     ole32:ole32.dll
 0000:fffdc000       .debug$S                   0000000180000000     ole32:ole32.dll
 0000:fffdc000       .debug$S                   0000000180000000     ole32:ole32.dll
 0000:fffdc000       .debug$S                   0000000180000000     shell32:SHELL32.dll
 0002:fffec000       .idata$6                   0000000180000000     shell32:SHELL32.dll
 0000:fffdc000       .debug$S                   0000000180000000     shlwapi:SHLWAPI.dll
 0002:fffec000       .idata$6                   0000000180000000     shlwapi:SHLWAPI.dll
 0000:fffdc000       .debug$S                   0000000180000000     user32:USER32.dll
 0002:fffec000       .idata$6                   0000000180000000     user32:USER32.dll
 0001:00000000       ??__ElastErrorLogAppender@?A0xd3578678@@YAXXZ 0000000180001000 f   app.obj
 0001:0000000c       ??__E_Fac_tidy_reg@std@@YAXXZ 000000018000100c f   msvcprt:locale0_implib.obj
 0001:00001d80       ?getFilename@?A0xd1a094c7@@YA?AV?$basic_string@GU?$char_traits@G@std@@V?$allocator@G@2@@std@@AEBUSourceCodePos@@@Z 0000000180002d80 f   ErrorHandling.obj
 0001:00002918       ?printWithoutWhitespaces@?A0xd1a094c7@@YA_KAEAV?$basic_ostream@DU?$char_traits@D@std@@@std@@AEBV?$basic_string@DU?$char_traits@D@std@@V?$allocator@D@2@@3@W4TrimMode@1@@Z 0000000180003918 f   ErrorHandling.obj
 0001:00002a0c       ?reportError@?A0xd1a094c7@@YAXAEBUSourceCodePos@@AEBV?$basic_string@GU?$char_traits@G@std@@V?$allocator@G@2@@std@@@Z 0000000180003a0c f   ErrorHandling.obj
 0001:00005298       ?initGuid@?A0x2459fff0@@YAXAEBV?$basic_string@GU?$char_traits@G@std@@V?$allocator@G@2@@std@@AEAU_GUID@@@Z 0000000180006298 f   Guid.obj
 0001:000061bc       ??1?$AtEndOfScope@V<lambda_1>@?1??toUnicodeString@jni@@YA?AV?$basic_string@GU?$char_traits@G@std@@V?$allocator@G@2@@std@@PEAUJNIEnv_@@PEAV_jstring@@@Z@@@QEAA@XZ 00000001800071bc f   JniUtils.obj
 0001:000086a8       ?openDatabase@?A0x6ccb95c8@msi@@YAKAEBV?$basic_string@GU?$char_traits@G@std@@V?$allocator@G@2@@std@@@Z 00000001800096a8 f   MsiDb.obj
 0001:00009484       ??$getProperty@P6AIKIPEAGPEAK@ZKI@?A0x0e70828c@msi@@YA?AV?$basic_string@GU?$char_traits@G@std@@V?$allocator@G@2@@std@@P6AIKIPEAGPEAK@ZQEBDKI@Z 000000018000a484 f   MsiUtils.obj
 0001:00009a10       ?makeMessage@?A0x0e70828c@msi@@YA?AV?$basic_string@DU?$char_traits@D@std@@V?$allocator@D@2@@std@@AEBV34@I@Z 000000018000aa10 f   MsiUtils.obj
 0001:0000a134       ?retrieveModuleName@?A0x40e1fcfd@@YA?AV?$basic_string@GU?$char_traits@G@std@@V?$allocator@G@2@@std@@XZ 000000018000b134 f   PlatformLogEvent.obj
 0001:0000ba50       ??0FixedFileVersion@?A0xcb1fbc16@@QEAA@AEBV?$basic_string@GU?$char_traits@G@std@@V?$allocator@G@2@@std@@@Z 000000018000ca50 f   VersionInfo.obj
 0001:0000bca4       ??1StreamSize@?A0xcb1fbc16@@QEAA@XZ 000000018000cca4 f   VersionInfo.obj
 0001:0000beb8       ?add32bitPadding@?A0xcb1fbc16@@YAXAEAV?$basic_ostream@DU?$char_traits@D@std@@@std@@@Z 000000018000ceb8 f   VersionInfo.obj
 0001:0000cb6c       ?writeWORD@?A0xcb1fbc16@@YAAEAV?$basic_ostream@DU?$char_traits@D@std@@@std@@AEAV23@_K@Z 000000018000db6c f   VersionInfo.obj
 0001:0000cec0       ?getSystemMessageDescription@?A0xd5983087@@YA?AV?$basic_string@GU?$char_traits@G@std@@V?$allocator@G@2@@std@@KPEAUHINSTANCE__@@@Z 000000018000dec0 f   WinErrorHandling.obj
 0001:0000d004       ?makeMessage@?A0xd5983087@@YA?AV?$basic_string@DU?$char_traits@D@std@@V?$allocator@D@2@@std@@AEBV23@PEBDPEBXK@Z 000000018000e004 f   WinErrorHandling.obj
 0001:0000d644       ??$getSystemDirImpl@P6AIPEAGI@Z@?A0x7970c2a6@SysInfo@@YA?AV?$basic_string@GU?$char_traits@G@std@@V?$allocator@G@2@@std@@P6AIPEAGI@ZAEBV?$basic_string@DU?$char_traits@D@std@@V?$allocator@D@2@@3@@Z 000000018000e644 f   WinSysInfo.obj
 0001:0000dae0       ?getModulePath@?A0x7970c2a6@SysInfo@@YA?AV?$basic_string@GU?$char_traits@G@std@@V?$allocator@G@2@@std@@PEAUHINSTANCE__@@@Z 000000018000eae0 f   WinSysInfo.obj
 0001:0000dd64       ?GetLongPath@?A0x764c93a3@@YA?AV?$basic_string@GU?$char_traits@G@std@@V?$allocator@G@2@@std@@AEBV23@@Z 000000018000ed64 f   WindowsRegistry.obj
 0001:0000e77c       ?append@LastErrorLogAppender@?A0xd3578678@@UEAAXAEBULogEvent@@@Z 000000018000f77c f   app.obj
 0001:0000e81c       ??_GLastErrorLogAppender@?A0xd3578678@@UEAAPEAXI@Z 000000018000f81c f   app.obj
 0001:0000f670       ?fromMultiByte@?A0xf04d92fb@tstrings@@YA?AV?$basic_string@GU?$char_traits@G@std@@V?$allocator@G@2@@std@@AEBV?$basic_string@DU?$char_traits@D@std@@V?$allocator@D@2@@4@H@Z 0000000180010670 f   tstrings.obj
 0001:0000f904       ?toMultiByte@?A0xf04d92fb@tstrings@@YA?AV?$basic_string@DU?$char_traits@D@std@@V?$allocator@D@2@@std@@AEBV?$basic_string@GU?$char_traits@G@std@@V?$allocator@G@2@@4@H@Z 0000000180010904 f   tstrings.obj
 0001:0000fd60       ??$__std_find_trivial_impl@U_Find_traits_2@?A0x8417fefe@@G@?A0x8417fefe@@YAPEBXPEBX0G@Z 0000000180010d60 f   msvcprt:vector_algorithms.obj
 0001:0000ffd0       $$000000                   0000000180010fd0     MSVCRT:chkstk.obj
 0001:00010030       $$000000                   0000000180011030     MSVCRT:amdsecgs.obj
 0001:00010248       capture_current_context    0000000180011248 f   MSVCRT:gs_report.obj
 0001:000102b8       capture_previous_context   00000001800112b8 f   MSVCRT:gs_report.obj
 0001:000106ac       ?dllmain_crt_dispatch@@YAHQEAUHINSTANCE__@@KQEAX@Z 00000001800116ac f   MSVCRT:dll_dllmain.obj
 0001:000106fc       ?dllmain_crt_process_attach@@YAHQEAUHINSTANCE__@@QEAX@Z 00000001800116fc f   MSVCRT:dll_dllmain.obj
 0001:00010814       ?dllmain_crt_process_detach@@YAH_N@Z 0000000180011814 f   MSVCRT:dll_dllmain.obj
 0001:00010894       ?dllmain_dispatch@@YAHQEAUHINSTANCE__@@KQEAX@Z 0000000180011894 f   MSVCRT:dll_dllmain.obj
 0001:000110b0       $$000000                   00000001800120b0     MSVCRT:guard_dispatch.obj
 0001:000110d0       $$000000                   00000001800120d0     MSVCRT:guard_xfg_dispatch.obj
 0001:000110e6       ?dtor$0@?0???$?6GU?$char_traits@G@std@@@std@@YAAEAV?$basic_ostream@GU?$char_traits@G@std@@@0@AEAV10@PEBD@Z@4HA 00000001800120e6 f   ErrorHandling.obj
 0001:000110e6       ?dtor$0@?0???$?6GU?$char_traits@G@std@@@std@@YAAEAV?$basic_ostream@GU?$char_traits@G@std@@@0@AEAV10@PEBG@Z@4HA 00000001800120e6 f   ErrorHandling.obj
 0001:000110e6       ?dtor$0@?0???$_Insert_string@GU?$char_traits@G@std@@_K@std@@YAAEAV?$basic_ostream@GU?$char_traits@G@std@@@0@AEAV10@QEBG_K@Z@4HA 00000001800120e6 f   ErrorHandling.obj
 0001:000110e6       ?dtor$0@?0???6?$basic_ostream@GU?$char_traits@G@std@@@std@@QEAAAEAV01@G@Z@4HA 00000001800120e6 f   Log.obj
 0001:000110f2       ?dtor$1@?0???$?6GU?$char_traits@G@std@@@std@@YAAEAV?$basic_ostream@GU?$char_traits@G@std@@@0@AEAV10@PEBD@Z@4HA 00000001800120f2 f   ErrorHandling.obj
 0001:000110fe       ?catch$4@?0???$?6GU?$char_traits@G@std@@@std@@YAAEAV?$basic_ostream@GU?$char_traits@G@std@@@0@AEAV10@PEBD@Z@4HA 00000001800120fe f   ErrorHandling.obj
 0001:0001110b       __catch$??$?6GU?$char_traits@G@std@@@std@@YAAEAV?$basic_ostream@GU?$char_traits@G@std@@@0@AEAV10@PEBD@Z$0 000000018001210b f   ErrorHandling.obj
 0001:0001113c       ?catch$3@?0???$?6GU?$char_traits@G@std@@@std@@YAAEAV?$basic_ostream@GU?$char_traits@G@std@@@0@AEAV10@PEBG@Z@4HA 000000018001213c f   ErrorHandling.obj
 0001:0001113c       ?catch$3@?0???$_Insert_string@GU?$char_traits@G@std@@_K@std@@YAAEAV?$basic_ostream@GU?$char_traits@G@std@@@0@AEAV10@QEBG_K@Z@4HA 000000018001213c f   ErrorHandling.obj
 0001:0001113c       ?catch$3@?0???6?$basic_ostream@GU?$char_traits@G@std@@@std@@QEAAAEAV01@G@Z@4HA 000000018001213c f   Log.obj
 0001:00011149       __catch$??$?6GU?$char_traits@G@std@@@std@@YAAEAV?$basic_ostream@GU?$char_traits@G@std@@@0@AEAV10@PEBG@Z$0 0000000180012149 f   ErrorHandling.obj
 0001:00011149       __catch$??$_Insert_string@GU?$char_traits@G@std@@_K@std@@YAAEAV?$basic_ostream@GU?$char_traits@G@std@@@0@AEAV10@QEBG_K@Z$0 0000000180012149 f   ErrorHandling.obj
 0001:00011149       __catch$??6?$basic_ostream@GU?$char_traits@G@std@@@std@@QEAAAEAV01@G@Z$0 0000000180012149 f   Log.obj
 0001:00011177       ?dtor$0@?0???$?6U?$char_traits@D@std@@@std@@YAAEAV?$basic_ostream@DU?$char_traits@D@std@@@0@AEAV10@PEBD@Z@4HA 0000000180012177 f   ErrorHandling.obj
 0001:00011177       ?dtor$0@?0???$_Insert_string@DU?$char_traits@D@std@@_K@std@@YAAEAV?$basic_ostream@DU?$char_traits@D@std@@@0@AEAV10@QEBD_K@Z@4HA 0000000180012177 f   ErrorHandling.obj
 0001:00011183       ?catch$3@?0???$?6U?$char_traits@D@std@@@std@@YAAEAV?$basic_ostream@DU?$char_traits@D@std@@@0@AEAV10@PEBD@Z@4HA 0000000180012183 f   ErrorHandling.obj
 0001:00011183       ?catch$3@?0???$_Insert_string@DU?$char_traits@D@std@@_K@std@@YAAEAV?$basic_ostream@DU?$char_traits@D@std@@@0@AEAV10@QEBD_K@Z@4HA 0000000180012183 f   ErrorHandling.obj
 0001:00011190       __catch$??$?6U?$char_traits@D@std@@@std@@YAAEAV?$basic_ostream@DU?$char_traits@D@std@@@0@AEAV10@PEBD@Z$0 0000000180012190 f   ErrorHandling.obj
 0001:00011190       __catch$??$_Insert_string@DU?$char_traits@D@std@@_K@std@@YAAEAV?$basic_ostream@DU?$char_traits@D@std@@@0@AEAV10@QEBD_K@Z$0 0000000180012190 f   ErrorHandling.obj
 0001:000111be       ?dtor$0@?0???$use_facet@V?$ctype@G@std@@@std@@YAAEBV?$ctype@G@0@AEBVlocale@0@@Z@4HA 00000001800121be f   ErrorHandling.obj
 0001:000111be       ?dtor$0@?0???$use_facet@V?$codecvt@DDU_Mbstatet@@@std@@@std@@YAAEBV?$codecvt@DDU_Mbstatet@@@0@AEBVlocale@0@@Z@4HA 00000001800121be f   MsiDb.obj
 0001:000111cc       ?dtor$1@?0???$use_facet@V?$ctype@G@std@@@std@@YAAEBV?$ctype@G@0@AEBVlocale@0@@Z@4HA 00000001800121cc f   ErrorHandling.obj
 0001:000111cc       ?dtor$1@?0???$use_facet@V?$codecvt@DDU_Mbstatet@@@std@@@std@@YAAEBV?$codecvt@DDU_Mbstatet@@@0@AEBVlocale@0@@Z@4HA 00000001800121cc f   MsiDb.obj
 0001:000111d8       ?dtor$0@?0???0?$basic_ostringstream@DU?$char_traits@D@std@@V?$allocator@D@2@@std@@QEAA@XZ@4HA 00000001800121d8 f   ErrorHandling.obj
 0001:00011206       ?dtor$1@?0???0?$basic_ostringstream@DU?$char_traits@D@std@@V?$allocator@D@2@@std@@QEAA@XZ@4HA 0000000180012206 f   ErrorHandling.obj
 0001:00011218       ?dtor$0@?0???0?$basic_ostringstream@GU?$char_traits@G@std@@V?$allocator@G@2@@std@@QEAA@XZ@4HA 0000000180012218 f   ErrorHandling.obj
 0001:00011246       ?dtor$1@?0???0?$basic_ostringstream@GU?$char_traits@G@std@@V?$allocator@G@2@@std@@QEAA@XZ@4HA 0000000180012246 f   ErrorHandling.obj
 0001:00011258       ?dtor$0@?0???0sentry@?$basic_ostream@DU?$char_traits@D@std@@@std@@QEAA@AEAV12@@Z@4HA 0000000180012258 f   ErrorHandling.obj
 0001:00011264       ?dtor$0@?0???0sentry@?$basic_ostream@GU?$char_traits@G@std@@@std@@QEAA@AEAV12@@Z@4HA 0000000180012264 f   ErrorHandling.obj
 0001:00011270       ?dtor$0@?0???6@YAAEAV?$basic_ostream@DU?$char_traits@D@std@@@std@@AEAV01@AEBVany@tstrings@@@Z@4HA 0000000180012270 f   ErrorHandling.obj
 0001:0001127c       ?dtor$1@?0???6@YAAEAV?$basic_ostream@DU?$char_traits@D@std@@@std@@AEAV01@AEBVany@tstrings@@@Z@4HA 000000018001227c f   ErrorHandling.obj
 0001:0001127c       Java_jdk_jpackage_internal_WindowsRegistry_comparePaths$dtor$0 000000018001227c f   WindowsRegistry.obj
 0001:0001127c       Java_jdk_jpackage_internal_ShortPathUtils_getShortPath$dtor$0 000000018001227c f   jpackage.obj
 0001:00011288       ?dtor$0@?0??getFilename@?A0xd1a094c7@@YA?AV?$basic_string@GU?$char_traits@G@std@@V?$allocator@G@2@@std@@AEBUSourceCodePos@@@Z@4HA 0000000180012288 f   ErrorHandling.obj
 0001:00011294       ?dtor$2@?0??getFilename@?A0xd1a094c7@@YA?AV?$basic_string@GU?$char_traits@G@std@@V?$allocator@G@2@@std@@AEBUSourceCodePos@@@Z@4HA 0000000180012294 f   ErrorHandling.obj
 0001:00011294       ?dtor$0@?0???0Error@msi@@QEAA@AEBVany@tstrings@@I@Z@4HA 0000000180012294 f   MsiUtils.obj
 0001:000112a0       ?dtor$0@?0??joinErrorMessages@@YA?AV?$basic_string@DU?$char_traits@D@std@@V?$allocator@D@2@@std@@AEBV12@0@Z@4HA 00000001800122a0 f   ErrorHandling.obj
 0001:000112a0       ?dtor$1@?0???$getSystemDirImpl@P6AIPEAGI@Z@?A0x7970c2a6@SysInfo@@YA?AV?$basic_string@GU?$char_traits@G@std@@V?$allocator@G@2@@std@@P6AIPEAGI@ZAEBV?$basic_string@DU?$char_traits@D@std@@V?$allocator@D@2@@3@@Z@4HA 00000001800122a0 f   WinSysInfo.obj
 0001:000112ac       ?dtor$1@?0??joinErrorMessages@@YA?AV?$basic_string@DU?$char_traits@D@std@@V?$allocator@D@2@@std@@AEBV12@0@Z@4HA 00000001800122ac f   ErrorHandling.obj
 0001:000112ac       ?dtor$6@?0???$getSystemDirImpl@P6AIPEAGI@Z@?A0x7970c2a6@SysInfo@@YA?AV?$basic_string@GU?$char_traits@G@std@@V?$allocator@G@2@@std@@P6AIPEAGI@ZAEBV?$basic_string@DU?$char_traits@D@std@@V?$allocator@D@2@@3@@Z@4HA 00000001800122ac f   WinSysInfo.obj
 0001:000112b8       ?dtor$2@?0??joinErrorMessages@@YA?AV?$basic_string@DU?$char_traits@D@std@@V?$allocator@D@2@@std@@AEBV12@0@Z@4HA 00000001800122b8 f   ErrorHandling.obj
 0001:000112b8       ?dtor$3@?0??append@StreamLogAppender@@UEAAXAEBULogEvent@@@Z@4HA 00000001800122b8 f   Log.obj
 0001:000112c4       ?dtor$3@?0??joinErrorMessages@@YA?AV?$basic_string@DU?$char_traits@D@std@@V?$allocator@D@2@@std@@AEBV12@0@Z@4HA 00000001800122c4 f   ErrorHandling.obj
 0001:000112d0       ?dtor$4@?0??joinErrorMessages@@YA?AV?$basic_string@DU?$char_traits@D@std@@V?$allocator@D@2@@std@@AEBV12@0@Z@4HA 00000001800122d0 f   ErrorHandling.obj
 0001:000112dc       ?dtor$0@?0??makeMessage@@YA?AV?$basic_string@DU?$char_traits@D@std@@V?$allocator@D@2@@std@@AEBVruntime_error@2@AEBUSourceCodePos@@@Z@4HA 00000001800122dc f   ErrorHandling.obj
 0001:000112e8       ?dtor$1@?0??makeMessage@@YA?AV?$basic_string@DU?$char_traits@D@std@@V?$allocator@D@2@@std@@AEBVruntime_error@2@AEBUSourceCodePos@@@Z@4HA 00000001800122e8 f   ErrorHandling.obj
 0001:000112f4       ?dtor$2@?0??makeMessage@@YA?AV?$basic_string@DU?$char_traits@D@std@@V?$allocator@D@2@@std@@AEBVruntime_error@2@AEBUSourceCodePos@@@Z@4HA 00000001800122f4 f   ErrorHandling.obj
 0001:000112f4       ?dtor$4@?0??makeMessage@@YA?AV?$basic_string@DU?$char_traits@D@std@@V?$allocator@D@2@@std@@AEBVruntime_error@2@AEBUSourceCodePos@@@Z@4HA 00000001800122f4 f   ErrorHandling.obj
 0001:000112f4       ?dtor$1@?0??append@StreamLogAppender@@UEAAXAEBULogEvent@@@Z@4HA 00000001800122f4 f   Log.obj
 0001:000112f4       ?dtor$0@?0??closeMSIHANDLE@msi@@YAXK@Z@4HA 00000001800122f4 f   MsiUtils.obj
 0001:000112f4       ?dtor$0@?0??id@ResourceEditor@@QEAAAEAV1@PEBG@Z@4HA 00000001800122f4 f   ResourceEditor.obj
 0001:000112f4       ?dtor$0@?0??type@ResourceEditor@@QEAAAEAV1@PEBG@Z@4HA 00000001800122f4 f   ResourceEditor.obj
 0001:000112f4       ?dtor$0@?0??getErrMsg@Resource@@AEBA?AV?$basic_string@DU?$char_traits@D@std@@V?$allocator@D@2@@std@@AEBV23@@Z@4HA 00000001800122f4 f   Resources.obj
 0001:000112f4       ?dtor$0@?0??init@Resource@@AEAAXPEBG0PEAUHINSTANCE__@@@Z@4HA 00000001800122f4 f   Resources.obj
 0001:000112f4       ?dtor$2@?0??init@Resource@@AEAAXPEBG0PEAUHINSTANCE__@@@Z@4HA 00000001800122f4 f   Resources.obj
 0001:000112f4       ?dtor$0@?0??getSysErrorMessage@SysError@@SA?AV?$basic_string@GU?$char_traits@G@std@@V?$allocator@G@2@@std@@KPEAUHINSTANCE__@@@Z@4HA 00000001800122f4 f   WinErrorHandling.obj
 0001:00011300       ?dtor$0@?0??reportError@?A0xd1a094c7@@YAXAEBUSourceCodePos@@AEBV?$basic_string@GU?$char_traits@G@std@@V?$allocator@G@2@@std@@@Z@4HA 0000000180012300 f   ErrorHandling.obj
 0001:0001130c       ?dtor$1@?0??reportError@?A0xd1a094c7@@YAXAEBUSourceCodePos@@AEBV?$basic_string@GU?$char_traits@G@std@@V?$allocator@G@2@@std@@@Z@4HA 000000018001230c f   ErrorHandling.obj
 0001:00011318       ?dtor$2@?0??reportError@?A0xd1a094c7@@YAXAEBUSourceCodePos@@AEBV?$basic_string@GU?$char_traits@G@std@@V?$allocator@G@2@@std@@@Z@4HA 0000000180012318 f   ErrorHandling.obj
 0001:00011324       ?dtor$0@?0??reportError@@YAXAEBUSourceCodePos@@AEBVruntime_error@std@@@Z@4HA 0000000180012324 f   ErrorHandling.obj
 0001:00011330       ?dtor$1@?0??reportError@@YAXAEBUSourceCodePos@@AEBVruntime_error@std@@@Z@4HA 0000000180012330 f   ErrorHandling.obj
 0001:0001133c       ?dtor$0@?0??reportUnknownError@@YAXAEBUSourceCodePos@@@Z@4HA 000000018001233c f   ErrorHandling.obj
 0001:0001133c       ?dtor$0@?0???0Guid@@QEAA@AEBV?$basic_string@GU?$char_traits@G@std@@V?$allocator@G@2@@std@@@Z@4HA 000000018001233c f   Guid.obj
 0001:0001133c       ?dtor$1@?0??log@Logger@@QEBAXW4LogLevel@1@PEBGH1AEBV?$basic_string@GU?$char_traits@G@std@@V?$allocator@G@2@@std@@@Z@4HA 000000018001233c f   Log.obj
 0001:0001133c       ?dtor$3@?0???0Error@msi@@QEAA@AEBVany@tstrings@@I@Z@4HA 000000018001233c f   MsiUtils.obj
 0001:0001133c       ?dtor$0@?0??initializeLogging@Logger@@CAXXZ@4HA 000000018001233c f   PlatformLogEvent.obj
 0001:00011348       ?dtor$0@?0??str@?$basic_stringbuf@DU?$char_traits@D@std@@V?$allocator@D@2@@std@@QEBA?AV?$basic_string@DU?$char_traits@D@std@@V?$allocator@D@2@@2@XZ@4HA 0000000180012348 f   ErrorHandling.obj
 0001:0001136e       ?dtor$0@?0??str@?$basic_stringbuf@GU?$char_traits@G@std@@V?$allocator@G@2@@std@@QEBA?AV?$basic_string@GU?$char_traits@G@std@@V?$allocator@G@2@@2@XZ@4HA 000000018001236e f   ErrorHandling.obj
 0001:00011394       ?dtor$0@?0???0?$JpError@VSysError@@@@QEAA@AEBV0@@Z@4HA 0000000180012394 f   Executor.obj
 0001:00011394       ?dtor$0@?0???0?$JpError@VSysError@@@@QEAA@AEBVSysError@@AEBUSourceCodePos@@@Z@4HA 0000000180012394 f   Executor.obj
 0001:00011394       ?dtor$0@?0???0?$JpError@Vruntime_error@std@@@@QEAA@AEBV0@@Z@4HA 0000000180012394 f   Guid.obj
 0001:00011394       ?dtor$0@?0???0?$JpError@Vruntime_error@std@@@@QEAA@AEBVruntime_error@std@@AEBUSourceCodePos@@@Z@4HA 0000000180012394 f   Guid.obj
 0001:00011394       ?dtor$0@?0???0?$JpError@VError@msi@@@@QEAA@AEBV0@@Z@4HA 0000000180012394 f   MsiCA.obj
 0001:00011394       ?dtor$0@?0???0?$JpError@VError@msi@@@@QEAA@AEBVError@msi@@AEBUSourceCodePos@@@Z@4HA 0000000180012394 f   MsiCA.obj
 0001:00011394       ?dtor$0@?0???0?$JpError@VNoMoreItemsError@msi@@@@QEAA@AEBV0@@Z@4HA 0000000180012394 f   MsiDb.obj
 0001:00011394       ?dtor$0@?0???0?$JpError@VNoMoreItemsError@msi@@@@QEAA@AEBVNoMoreItemsError@msi@@AEBUSourceCodePos@@@Z@4HA 0000000180012394 f   MsiDb.obj
 0001:000113a4       ?dtor$0@?0???0any@tstrings@@QEAA@PEBD@Z@4HA 00000001800123a4 f   Executor.obj
 0001:000113a4       ?dtor$0@?0???0any@tstrings@@QEAA@AEBV?$basic_string@DU?$char_traits@D@std@@V?$allocator@D@2@@std@@@Z@4HA 00000001800123a4 f   Resources.obj
 0001:000113b0       ?dtor$1@?0???0any@tstrings@@QEAA@PEBD@Z@4HA 00000001800123b0 f   Executor.obj
 0001:000113bc       ?dtor$2@?0???0any@tstrings@@QEAA@PEBD@Z@4HA 00000001800123bc f   Executor.obj
 0001:000113bc       ?dtor$4@?0??combinePath@FileUtils@@YA?AV?$basic_string@GU?$char_traits@G@std@@V?$allocator@G@2@@std@@AEBV23@0@Z@4HA 00000001800123bc f   FileUtils.obj
 0001:000113bc       ?dtor$0@?0??toString@Guid@@QEBA?AV?$basic_string@GU?$char_traits@G@std@@V?$allocator@G@2@@std@@H@Z@4HA 00000001800123bc f   Guid.obj
 0001:000113bc       ?dtor$0@?0??retrieveModuleName@?A0x40e1fcfd@@YA?AV?$basic_string@GU?$char_traits@G@std@@V?$allocator@G@2@@std@@XZ@4HA 00000001800123bc f   PlatformLogEvent.obj
 0001:000113bc       ?dtor$0@?0??string@StringResource@@QEBA?AV?$basic_string@GU?$char_traits@G@std@@V?$allocator@G@2@@std@@XZ@4HA 00000001800123bc f   Resources.obj
 0001:000113bc       ?dtor$1@?0???0any@tstrings@@QEAA@AEBV?$basic_string@DU?$char_traits@D@std@@V?$allocator@D@2@@std@@@Z@4HA 00000001800123bc f   Resources.obj
 0001:000113bc       ?dtor$3@?0???0SysError@@QEAA@AEBVany@tstrings@@PEBXKPEBD@Z@4HA 00000001800123bc f   WinErrorHandling.obj
 0001:000113bc       ?dtor$2@?0??GetLongPath@?A0x764c93a3@@YA?AV?$basic_string@GU?$char_traits@G@std@@V?$allocator@G@2@@std@@AEBV23@@Z@4HA 00000001800123bc f   WindowsRegistry.obj
 0001:000113c8       ?dtor$0@?0??log@Logger@@QEBAXW4LogLevel@1@PEBGH1AEBVany@tstrings@@@Z@4HA 00000001800123c8 f   Executor.obj
 0001:000113d4       ?dtor$1@?0??combinePath@FileUtils@@YA?AV?$basic_string@GU?$char_traits@G@std@@V?$allocator@G@2@@std@@AEBV23@0@Z@4HA 00000001800123d4 f   FileUtils.obj
 0001:000113e0       ?dtor$2@?0??combinePath@FileUtils@@YA?AV?$basic_string@GU?$char_traits@G@std@@V?$allocator@G@2@@std@@AEBV23@0@Z@4HA 00000001800123e0 f   FileUtils.obj
 0001:00011406       ?dtor$3@?0??combinePath@FileUtils@@YA?AV?$basic_string@GU?$char_traits@G@std@@V?$allocator@G@2@@std@@AEBV23@0@Z@4HA 0000000180012406 f   FileUtils.obj
 0001:0001142c       ?dtor$1@?0???0Guid@@QEAA@AEBV?$basic_string@GU?$char_traits@G@std@@V?$allocator@G@2@@std@@@Z@4HA 000000018001242c f   Guid.obj
 0001:0001142c       ?dtor$2@?0??toUnicodeStringArray@jni@@YA?AV?$vector@V?$basic_string@GU?$char_traits@G@std@@V?$allocator@G@2@@std@@V?$allocator@V?$basic_string@GU?$char_traits@G@std@@V?$allocator@G@2@@std@@@2@@std@@PEAUJNIEnv_@@PEAV_jobjectArray@@@Z@4HA 000000018001242c f   JniUtils.obj
 0001:0001142c       ?dtor$0@?0??appendFormatted@LogEvent@@CAXAEBUPlatformLogEvent@@AEAV?$basic_string@GU?$char_traits@G@std@@V?$allocator@G@2@@std@@@Z@4HA 000000018001242c f   PlatformLogEvent.obj
 0001:00011438       ?dtor$0@?0??initGuid@?A0x2459fff0@@YAXAEBV?$basic_string@GU?$char_traits@G@std@@V?$allocator@G@2@@std@@AEAU_GUID@@@Z@4HA 0000000180012438 f   Guid.obj
 0001:00011444       ?dtor$0@?0??makeException@@YA?AV?$JpError@Vruntime_error@std@@@@AEBV?$basic_string@DU?$char_traits@D@std@@V?$allocator@D@2@@std@@AEBUSourceCodePos@@@Z@4HA 0000000180012444 f   Guid.obj
 0001:00011444       ?dtor$1@?0??getFieldCount@DatabaseRecord@msi@@QEBAIXZ@4HA 0000000180012444 f   MsiDb.obj
 0001:00011444       ?dtor$1@?0??toShortPath@FileUtils@@YA?AV?$basic_string@GU?$char_traits@G@std@@V?$allocator@G@2@@std@@AEBV23@@Z@4HA 0000000180012444 f   WinFileUtils.obj
 0001:00011444       ?dtor$1@?0??getCurrentModuleHandle@SysInfo@@YAPEAUHINSTANCE__@@XZ@4HA 0000000180012444 f   WinSysInfo.obj
 0001:00011450       ?dtor$0@?0??makeException@@YA?AV?$JpError@Vruntime_error@std@@@@AEBVany@tstrings@@AEBUSourceCodePos@@@Z@4HA 0000000180012450 f   Guid.obj
 0001:00011450       ?dtor$0@?0??makeException@@YA?AV?$JpError@Vruntime_error@std@@@@PEBDAEBUSourceCodePos@@@Z@4HA 0000000180012450 f   Guid.obj
 0001:00011450       ?dtor$0@?0??getSystem32Dir@SysInfo@@YA?AV?$basic_string@GU?$char_traits@G@std@@V?$allocator@G@2@@std@@XZ@4HA 0000000180012450 f   WinSysInfo.obj
 0001:0001145c       ?dtor$2@?0??makeException@@YA?AV?$JpError@Vruntime_error@std@@@@AEBVany@tstrings@@AEBUSourceCodePos@@@Z@4HA 000000018001245c f   Guid.obj
 0001:0001145c       Java_jdk_jpackage_internal_WindowsRegistry_enumRegistryValue$dtor$0 000000018001245c f   WindowsRegistry.obj
 0001:00011468       ?dtor$1@?0??toString@Guid@@QEBA?AV?$basic_string@GU?$char_traits@G@std@@V?$allocator@G@2@@std@@H@Z@4HA 0000000180012468 f   Guid.obj
 0001:0001148e       ?catch$3@?0???$_Emplace_reallocate@V?$basic_string@GU?$char_traits@G@std@@V?$allocator@G@2@@std@@@?$vector@V?$basic_string@GU?$char_traits@G@std@@V?$allocator@G@2@@std@@V?$allocator@V?$basic_string@GU?$char_traits@G@std@@V?$allocator@G@2@@std@@@2@@std@@AEAAPEAV?$basic_string@GU?$char_traits@G@std@@V?$allocator@G@2@@1@QEAV21@$$QEAV21@@Z@4HA 000000018001248e f   JniUtils.obj
 0001:0001149b       __catch$??$_Emplace_reallocate@V?$basic_string@GU?$char_traits@G@std@@V?$allocator@G@2@@std@@@?$vector@V?$basic_string@GU?$char_traits@G@std@@V?$allocator@G@2@@std@@V?$allocator@V?$basic_string@GU?$char_traits@G@std@@V?$allocator@G@2@@std@@@2@@std@@AEAAPEAV?$basic_string@GU?$char_traits@G@std@@V?$allocator@G@2@@1@QEAV21@$$QEAV21@@Z$0 000000018001249b f   JniUtils.obj
 0001:000114d3       ?catch$0@?0???1?$AtEndOfScope@V<lambda_1>@?1??toUnicodeString@jni@@YA?AV?$basic_string@GU?$char_traits@G@std@@V?$allocator@G@2@@std@@PEAUJNIEnv_@@PEAV_jstring@@@Z@@@QEAA@XZ@4HA 00000001800124d3 f   JniUtils.obj
 0001:000114e0       __catch$??1?$AtEndOfScope@V<lambda_1>@?1??toUnicodeString@jni@@YA?AV?$basic_string@GU?$char_traits@G@std@@V?$allocator@G@2@@std@@PEAUJNIEnv_@@PEAV_jstring@@@Z@@@QEAA@XZ$0 00000001800124e0 f   JniUtils.obj
 0001:0001151c       ?catch$1@?0???1?$AtEndOfScope@V<lambda_1>@?1??toUnicodeString@jni@@YA?AV?$basic_string@GU?$char_traits@G@std@@V?$allocator@G@2@@std@@PEAUJNIEnv_@@PEAV_jstring@@@Z@@@QEAA@XZ@4HA 000000018001251c f   JniUtils.obj
 0001:00011529       __catch$??1?$AtEndOfScope@V<lambda_1>@?1??toUnicodeString@jni@@YA?AV?$basic_string@GU?$char_traits@G@std@@V?$allocator@G@2@@std@@PEAUJNIEnv_@@PEAV_jstring@@@Z@@@QEAA@XZ$1 0000000180012529 f   JniUtils.obj
 0001:00011561       ?dtor$0@?0??toUnicodeString@jni@@YA?AV?$basic_string@GU?$char_traits@G@std@@V?$allocator@G@2@@std@@PEAUJNIEnv_@@PEAV_jstring@@@Z@4HA 0000000180012561 f   JniUtils.obj
 0001:0001156d       ?dtor$0@?0??toUnicodeStringArray@jni@@YA?AV?$vector@V?$basic_string@GU?$char_traits@G@std@@V?$allocator@G@2@@std@@V?$allocator@V?$basic_string@GU?$char_traits@G@std@@V?$allocator@G@2@@std@@@2@@std@@PEAUJNIEnv_@@PEAV_jobjectArray@@@Z@4HA 000000018001256d f   JniUtils.obj
 0001:00011593       ?dtor$1@?0??toUnicodeStringArray@jni@@YA?AV?$vector@V?$basic_string@GU?$char_traits@G@std@@V?$allocator@G@2@@std@@V?$allocator@V?$basic_string@GU?$char_traits@G@std@@V?$allocator@G@2@@std@@@2@@std@@PEAUJNIEnv_@@PEAV_jobjectArray@@@Z@4HA 0000000180012593 f   JniUtils.obj
 0001:0001159f       ?dtor$0@?0??append@StreamLogAppender@@UEAAXAEBULogEvent@@@Z@4HA 000000018001259f f   Log.obj
 0001:0001159f       ?dtor$1@?0??getSysErrorMessage@SysError@@SA?AV?$basic_string@GU?$char_traits@G@std@@V?$allocator@G@2@@std@@KPEAUHINSTANCE__@@@Z@4HA 000000018001259f f   WinErrorHandling.obj
 0001:000115ab       ?dtor$2@?0??append@StreamLogAppender@@UEAAXAEBULogEvent@@@Z@4HA 00000001800125ab f   Log.obj
 0001:000115ab       ?dtor$4@?0???$getSystemDirImpl@P6AIPEAGI@Z@?A0x7970c2a6@SysInfo@@YA?AV?$basic_string@GU?$char_traits@G@std@@V?$allocator@G@2@@std@@P6AIPEAGI@ZAEBV?$basic_string@DU?$char_traits@D@std@@V?$allocator@D@2@@3@@Z@4HA 00000001800125ab f   WinSysInfo.obj
 0001:000115ab       Java_jdk_jpackage_internal_WinExeBundler_embedMSI$dtor$0 00000001800125ab f   jpackage.obj
 0001:000115b7       ?dtor$0@?0??log@Logger@@QEBAXW4LogLevel@1@PEBGH1AEBV?$basic_string@GU?$char_traits@G@std@@V?$allocator@G@2@@std@@@Z@4HA 00000001800125b7 f   Log.obj
 0001:000115c3       ?dtor$0@?0???$?0AEBUpiecewise_construct_t@std@@V?$tuple@AEBV?$basic_string@GU?$char_traits@G@std@@V?$allocator@G@2@@std@@@1@V?$tuple@$$V@1@@?$_Tree_temp_node@V?$allocator@U?$_Tree_node@U?$pair@$$CBV?$basic_string@GU?$char_traits@G@std@@V?$allocator@G@2@@std@@V12@@std@@PEAX@std@@@std@@@std@@QEAA@AEAV?$allocator@U?$_Tree_node@U?$pair@$$CBV?$basic_string@GU?$char_traits@G@std@@V?$allocator@G@2@@std@@V12@@std@@PEAX@std@@@1@PEAU?$_Tree_node@U?$pair@$$CBV?$basic_string@GU?$char_traits@G@std@@V?$allocator@G@2@@std@@V12@@std@@PEAX@1@AEBUpiecewise_construct_t@1@$$QEAV?$tuple@AEBV?$basic_string@GU?$char_traits@G@std@@V?$allocator@G@2@@std@@@1@$$QEAV?$tuple@$$V@1@@Z@4HA 00000001800125c3 f   MsiCA.obj
 0001:000115c3       ?dtor$1@?0???$?0AEBUpiecewise_construct_t@std@@V?$tuple@AEBV?$basic_string@GU?$char_traits@G@std@@V?$allocator@G@2@@std@@@1@V?$tuple@$$V@1@@?$_Tree_temp_node@V?$allocator@U?$_Tree_node@U?$pair@$$CBV?$basic_string@GU?$char_traits@G@std@@V?$allocator@G@2@@std@@V12@@std@@PEAX@std@@@std@@@std@@QEAA@AEAV?$allocator@U?$_Tree_node@U?$pair@$$CBV?$basic_string@GU?$char_traits@G@std@@V?$allocator@G@2@@std@@V12@@std@@PEAX@std@@@1@PEAU?$_Tree_node@U?$pair@$$CBV?$basic_string@GU?$char_traits@G@std@@V?$allocator@G@2@@std@@V12@@std@@PEAX@1@AEBUpiecewise_construct_t@1@$$QEAV?$tuple@AEBV?$basic_string@GU?$char_traits@G@std@@V?$allocator@G@2@@std@@@1@$$QEAV?$tuple@$$V@1@@Z@4HA 00000001800125c3 f   MsiCA.obj
 0001:000115cf       ?dtor$0@?0???0Database@msi@@QEAA@AEBV?$basic_string@GU?$char_traits@G@std@@V?$allocator@G@2@@std@@@Z@4HA 00000001800125cf f   MsiDb.obj
 0001:000115cf       ?dtor$0@?0???0Resource@@QEAA@IPEBGPEAUHINSTANCE__@@@Z@4HA 00000001800125cf f   Resources.obj
 0001:000115db       ?dtor$0@?0???0DatabaseView@msi@@QEAA@AEBVDatabase@1@AEBV?$basic_string@GU?$char_traits@G@std@@V?$allocator@G@2@@std@@AEBVDatabaseRecord@1@@Z@4HA 00000001800125db f   MsiDb.obj
 0001:000115e7       ?dtor$1@?0???0DatabaseView@msi@@QEAA@AEBVDatabase@1@AEBV?$basic_string@GU?$char_traits@G@std@@V?$allocator@G@2@@std@@AEBVDatabaseRecord@1@@Z@4HA 00000001800125e7 f   MsiDb.obj
 0001:000115e7       ?dtor$1@?0??fetch@DatabaseView@msi@@QEAA?AVDatabaseRecord@2@XZ@4HA 00000001800125e7 f   MsiDb.obj
 0001:000115e7       ?dtor$1@?0??tryFetch@DatabaseView@msi@@QEAA?AVDatabaseRecord@2@XZ@4HA 00000001800125e7 f   MsiDb.obj
 0001:000115e7       ?dtor$3@?0???0DatabaseView@msi@@QEAA@AEBVDatabase@1@AEBV?$basic_string@GU?$char_traits@G@std@@V?$allocator@G@2@@std@@AEBVDatabaseRecord@1@@Z@4HA 00000001800125e7 f   MsiDb.obj
 0001:000115e7       ?dtor$0@?0???1FileLock@ResourceEditor@@QEAA@XZ@4HA 00000001800125e7 f   ResourceEditor.obj
 0001:000115e7       ?dtor$0@?0??getCurrentModuleHandle@SysInfo@@YAPEAUHINSTANCE__@@XZ@4HA 00000001800125e7 f   WinSysInfo.obj
 0001:000115f3       ?dtor$2@?0???0DatabaseView@msi@@QEAA@AEBVDatabase@1@AEBV?$basic_string@GU?$char_traits@G@std@@V?$allocator@G@2@@std@@AEBVDatabaseRecord@1@@Z@4HA 00000001800125f3 f   MsiDb.obj
 0001:000115f3       ?dtor$2@?0??fetch@DatabaseView@msi@@QEAA?AVDatabaseRecord@2@XZ@4HA 00000001800125f3 f   MsiDb.obj
 0001:000115f3       ?dtor$2@?0??tryFetch@DatabaseView@msi@@QEAA?AVDatabaseRecord@2@XZ@4HA 00000001800125f3 f   MsiDb.obj
 0001:000115f3       ?dtor$4@?0???0DatabaseView@msi@@QEAA@AEBVDatabase@1@AEBV?$basic_string@GU?$char_traits@G@std@@V?$allocator@G@2@@std@@AEBVDatabaseRecord@1@@Z@4HA 00000001800125f3 f   MsiDb.obj
 0001:000115f3       ?dtor$7@?0??getPtr@Resource@@AEBAPEAXAEAK@Z@4HA 00000001800125f3 f   Resources.obj
 0001:000115ff       ?dtor$0@?0??fetch@DatabaseView@msi@@QEAA?AVDatabaseRecord@2@XZ@4HA 00000001800125ff f   MsiDb.obj
 0001:00011625       ?dtor$0@?0??getFieldCount@DatabaseRecord@msi@@QEBAIXZ@4HA 0000000180012625 f   MsiDb.obj
 0001:00011625       ?dtor$0@?0??uflow@?$basic_filebuf@DU?$char_traits@D@std@@@std@@MEAAHXZ@4HA 0000000180012625 f   MsiDb.obj
 0001:00011631       ?dtor$0@?0??getProperty@Database@msi@@QEBA?AV?$basic_string@GU?$char_traits@G@std@@V?$allocator@G@2@@std@@AEBV34@@Z@4HA 0000000180012631 f   MsiDb.obj
 0001:00011631       ?dtor$5@?0??getProperty@Database@msi@@QEBA?AV?$basic_string@GU?$char_traits@G@std@@V?$allocator@G@2@@std@@AEBV34@@Z@4HA 0000000180012631 f   MsiDb.obj
 0001:0001163d       ?dtor$1@?0??getProperty@Database@msi@@QEBA?AV?$basic_string@GU?$char_traits@G@std@@V?$allocator@G@2@@std@@AEBV34@@Z@4HA 000000018001263d f   MsiDb.obj
 0001:00011649       ?dtor$2@?0??getProperty@Database@msi@@QEBA?AV?$basic_string@GU?$char_traits@G@std@@V?$allocator@G@2@@std@@AEBV34@@Z@4HA 0000000180012649 f   MsiDb.obj
 0001:00011655       ?dtor$3@?0??getProperty@Database@msi@@QEBA?AV?$basic_string@GU?$char_traits@G@std@@V?$allocator@G@2@@std@@AEBV34@@Z@4HA 0000000180012655 f   MsiDb.obj
 0001:00011661       ?dtor$4@?0??getProperty@Database@msi@@QEBA?AV?$basic_string@GU?$char_traits@G@std@@V?$allocator@G@2@@std@@AEBV34@@Z@4HA 0000000180012661 f   MsiDb.obj
 0001:0001166d       ?dtor$6@?0??getProperty@Database@msi@@QEBA?AV?$basic_string@GU?$char_traits@G@std@@V?$allocator@G@2@@std@@AEBV34@@Z@4HA 000000018001266d f   MsiDb.obj
 0001:00011679       ?dtor$0@?0??openDatabase@?A0x6ccb95c8@msi@@YAKAEBV?$basic_string@GU?$char_traits@G@std@@V?$allocator@G@2@@std@@@Z@4HA 0000000180012679 f   MsiDb.obj
 0001:00011679       ?dtor$0@?0???0FileLock@ResourceEditor@@QEAA@AEBV?$basic_string@GU?$char_traits@G@std@@V?$allocator@G@2@@std@@@Z@4HA 0000000180012679 f   ResourceEditor.obj
 0001:00011679       ?dtor$2@?0??getPtr@Resource@@AEBAPEAXAEAK@Z@4HA 0000000180012679 f   Resources.obj
 0001:00011679       ?dtor$6@?0??getPtr@Resource@@AEBAPEAXAEAK@Z@4HA 0000000180012679 f   Resources.obj
 0001:00011685       ?dtor$1@?0??openDatabase@?A0x6ccb95c8@msi@@YAKAEBV?$basic_string@GU?$char_traits@G@std@@V?$allocator@G@2@@std@@@Z@4HA 0000000180012685 f   MsiDb.obj
 0001:00011691       ?catch$0@?0???$_Resize_reallocate@U_Value_init_tag@std@@@?$vector@GV?$allocator@G@std@@@std@@AEAAX_KAEBU_Value_init_tag@1@@Z@4HA 0000000180012691 f   MsiUtils.obj
 0001:0001169e       __catch$??$_Resize_reallocate@U_Value_init_tag@std@@@?$vector@GV?$allocator@G@std@@@std@@AEAAX_KAEBU_Value_init_tag@1@@Z$0 000000018001269e f   MsiUtils.obj
 0001:000116b9       ?dtor$0@?0???$getProperty@P6AIKIPEAGPEAK@ZKI@?A0x0e70828c@msi@@YA?AV?$basic_string@GU?$char_traits@G@std@@V?$allocator@G@2@@std@@P6AIKIPEAGPEAK@ZQEBDKI@Z@4HA 00000001800126b9 f   MsiUtils.obj
 0001:000116c5       ?dtor$1@?0???$getProperty@P6AIKIPEAGPEAK@ZKI@?A0x0e70828c@msi@@YA?AV?$basic_string@GU?$char_traits@G@std@@V?$allocator@G@2@@std@@P6AIKIPEAGPEAK@ZQEBDKI@Z@4HA 00000001800126c5 f   MsiUtils.obj
 0001:000116d1       ?dtor$2@?0???$getProperty@P6AIKIPEAGPEAK@ZKI@?A0x0e70828c@msi@@YA?AV?$basic_string@GU?$char_traits@G@std@@V?$allocator@G@2@@std@@P6AIKIPEAGPEAK@ZQEBDKI@Z@4HA 00000001800126d1 f   MsiUtils.obj
 0001:000116dd       ?dtor$0@?0??makeMessage@?A0x0e70828c@msi@@YA?AV?$basic_string@DU?$char_traits@D@std@@V?$allocator@D@2@@std@@AEBV34@I@Z@4HA 00000001800126dd f   MsiUtils.obj
 0001:000116e9       ?dtor$1@?0??makeMessage@?A0x0e70828c@msi@@YA?AV?$basic_string@DU?$char_traits@D@std@@V?$allocator@D@2@@std@@AEBV34@I@Z@4HA 00000001800126e9 f   MsiUtils.obj
 0001:000116f5       ?dtor$2@?0??makeMessage@?A0x0e70828c@msi@@YA?AV?$basic_string@DU?$char_traits@D@std@@V?$allocator@D@2@@std@@AEBV34@I@Z@4HA 00000001800126f5 f   MsiUtils.obj
 0001:00011701       ?dtor$3@?0??makeMessage@?A0x0e70828c@msi@@YA?AV?$basic_string@DU?$char_traits@D@std@@V?$allocator@D@2@@std@@AEBV34@I@Z@4HA 0000000180012701 f   MsiUtils.obj
 0001:0001170d       ?dtor$4@?0??makeMessage@?A0x0e70828c@msi@@YA?AV?$basic_string@DU?$char_traits@D@std@@V?$allocator@D@2@@std@@AEBV34@I@Z@4HA 000000018001270d f   MsiUtils.obj
 0001:00011719       ?dtor$5@?0??makeMessage@?A0x0e70828c@msi@@YA?AV?$basic_string@DU?$char_traits@D@std@@V?$allocator@D@2@@std@@AEBV34@I@Z@4HA 0000000180012719 f   MsiUtils.obj
 0001:00011725       ?dtor$11@?0??makeMessage@?A0x0e70828c@msi@@YA?AV?$basic_string@DU?$char_traits@D@std@@V?$allocator@D@2@@std@@AEBV34@I@Z@4HA 0000000180012725 f   MsiUtils.obj
 0001:00011725       ?dtor$28@?0??makeMessage@?A0x0e70828c@msi@@YA?AV?$basic_string@DU?$char_traits@D@std@@V?$allocator@D@2@@std@@AEBV34@I@Z@4HA 0000000180012725 f   MsiUtils.obj
 0001:00011725       ?dtor$6@?0??makeMessage@?A0x0e70828c@msi@@YA?AV?$basic_string@DU?$char_traits@D@std@@V?$allocator@D@2@@std@@AEBV34@I@Z@4HA 0000000180012725 f   MsiUtils.obj
 0001:00011731       ?dtor$7@?0??makeMessage@?A0x0e70828c@msi@@YA?AV?$basic_string@DU?$char_traits@D@std@@V?$allocator@D@2@@std@@AEBV34@I@Z@4HA 0000000180012731 f   MsiUtils.obj
 0001:0001173d       ?dtor$8@?0??makeMessage@?A0x0e70828c@msi@@YA?AV?$basic_string@DU?$char_traits@D@std@@V?$allocator@D@2@@std@@AEBV34@I@Z@4HA 000000018001273d f   MsiUtils.obj
 0001:00011749       ?dtor$9@?0??makeMessage@?A0x0e70828c@msi@@YA?AV?$basic_string@DU?$char_traits@D@std@@V?$allocator@D@2@@std@@AEBV34@I@Z@4HA 0000000180012749 f   MsiUtils.obj
 0001:00011755       ?dtor$12@?0??makeMessage@?A0x0e70828c@msi@@YA?AV?$basic_string@DU?$char_traits@D@std@@V?$allocator@D@2@@std@@AEBV34@I@Z@4HA 0000000180012755 f   MsiUtils.obj
 0001:00011761       ?catch$38@?0??makeMessage@?A0x0e70828c@msi@@YA?AV?$basic_string@DU?$char_traits@D@std@@V?$allocator@D@2@@std@@AEBV34@I@Z@4HA 0000000180012761 f   MsiUtils.obj
 0001:0001176e       __catch$?makeMessage@?A0x0e70828c@msi@@YA?AV?$basic_string@DU?$char_traits@D@std@@V?$allocator@D@2@@std@@AEBV34@I@Z$0 000000018001276e f   MsiUtils.obj
 0001:00011793       ?catch$5@?0??retrieveModuleName@?A0x40e1fcfd@@YA?AV?$basic_string@GU?$char_traits@G@std@@V?$allocator@G@2@@std@@XZ@4HA 0000000180012793 f   PlatformLogEvent.obj
 0001:000117a1       __catch$?retrieveModuleName@?A0x40e1fcfd@@YA?AV?$basic_string@GU?$char_traits@G@std@@V?$allocator@G@2@@std@@XZ$0 00000001800127a1 f   PlatformLogEvent.obj
 0001:000117e7       ?catch$0@?0???$_Emplace_reallocate@D@?$vector@EV?$allocator@E@std@@@std@@AEAAPEAEQEAE$$QEAD@Z@4HA 00000001800127e7 f   ResourceEditor.obj
 0001:000117f4       __catch$??$_Emplace_reallocate@D@?$vector@EV?$allocator@E@std@@@std@@AEAAPEAEQEAE$$QEAD@Z$0 00000001800127f4 f   ResourceEditor.obj
 0001:0001180f       ?catch$0@?0???$_Resize_reallocate@U_Value_init_tag@std@@@?$vector@EV?$allocator@E@std@@@std@@AEAAX_KAEBU_Value_init_tag@1@@Z@4HA 000000018001280f f   ResourceEditor.obj
 0001:0001181c       __catch$??$_Resize_reallocate@U_Value_init_tag@std@@@?$vector@EV?$allocator@E@std@@@std@@AEAAX_KAEBU_Value_init_tag@1@@Z$0 000000018001281c f   ResourceEditor.obj
 0001:00011837       ?dtor$0@?0???0?$basic_ifstream@DU?$char_traits@D@std@@@std@@QEAA@PEBGHH@Z@4HA 0000000180012837 f   ResourceEditor.obj
 0001:00011865       ?dtor$1@?0???0?$basic_ifstream@DU?$char_traits@D@std@@@std@@QEAA@PEBGHH@Z@4HA 0000000180012865 f   ResourceEditor.obj
 0001:00011877       ?dtor$2@?0???0?$basic_ifstream@DU?$char_traits@D@std@@@std@@QEAA@PEBGHH@Z@4HA 0000000180012877 f   ResourceEditor.obj
 0001:00011887       ?dtor$1@?0???0FileLock@ResourceEditor@@QEAA@AEBV?$basic_string@GU?$char_traits@G@std@@V?$allocator@G@2@@std@@@Z@4HA 0000000180012887 f   ResourceEditor.obj
 0001:00011887       ?dtor$1@?0???1FileLock@ResourceEditor@@QEAA@XZ@4HA 0000000180012887 f   ResourceEditor.obj
 0001:00011887       ?dtor$3@?0??getPtr@Resource@@AEBAPEAXAEAK@Z@4HA 0000000180012887 f   Resources.obj
 0001:00011893       ?dtor$0@?0???0ResourceEditor@@QEAA@XZ@4HA 0000000180012893 f   ResourceEditor.obj
 0001:000118a3       ?dtor$1@?0???0ResourceEditor@@QEAA@XZ@4HA 00000001800128a3 f   ResourceEditor.obj
 0001:000118b3       ?catch$5@?0???1FileLock@ResourceEditor@@QEAA@XZ@4HA 00000001800128b3 f   ResourceEditor.obj
 0001:000118c0       __catch$??1FileLock@ResourceEditor@@QEAA@XZ$0 00000001800128c0 f   ResourceEditor.obj
 0001:000118fc       ?catch$6@?0???1FileLock@ResourceEditor@@QEAA@XZ@4HA 00000001800128fc f   ResourceEditor.obj
 0001:00011909       __catch$??1FileLock@ResourceEditor@@QEAA@XZ$1 0000000180012909 f   ResourceEditor.obj
 0001:00011941       ?dtor$0@?0??apply@ResourceEditor@@QEAAAEAV1@AEBVFileLock@1@AEAV?$basic_istream@DU?$char_traits@D@std@@@std@@_J@Z@4HA 0000000180012941 f   ResourceEditor.obj
 0001:0001194d       ?dtor$2@?0??apply@ResourceEditor@@QEAAAEAV1@AEBVFileLock@1@AEAV?$basic_istream@DU?$char_traits@D@std@@@std@@_J@Z@4HA 000000018001294d f   ResourceEditor.obj
 0001:00011959       ?dtor$3@?0??apply@ResourceEditor@@QEAAAEAV1@AEBVFileLock@1@AEAV?$basic_istream@DU?$char_traits@D@std@@@std@@_J@Z@4HA 0000000180012959 f   ResourceEditor.obj
 0001:00011965       ?dtor$4@?0??apply@ResourceEditor@@QEAAAEAV1@AEBVFileLock@1@AEAV?$basic_istream@DU?$char_traits@D@std@@@std@@_J@Z@4HA 0000000180012965 f   ResourceEditor.obj
 0001:00011971       ?dtor$0@?0??apply@ResourceEditor@@QEAAAEAV1@AEBVFileLock@1@AEBV?$basic_string@GU?$char_traits@G@std@@V?$allocator@G@2@@std@@@Z@4HA 0000000180012971 f   ResourceEditor.obj
 0001:0001197d       ?dtor$0@?0??open@?$basic_filebuf@DU?$char_traits@D@std@@@std@@QEAAPEAV12@PEBGHH@Z@4HA 000000018001297d f   ResourceEditor.obj
 0001:00011989       ?dtor$1@?0???0Resource@@QEAA@IPEBGPEAUHINSTANCE__@@@Z@4HA 0000000180012989 f   Resources.obj
 0001:00011999       ?dtor$3@?0??getErrMsg@Resource@@AEBA?AV?$basic_string@DU?$char_traits@D@std@@V?$allocator@D@2@@std@@AEBV23@@Z@4HA 0000000180012999 f   Resources.obj
 0001:00011999       ?dtor$6@?0??getErrMsg@Resource@@AEBA?AV?$basic_string@DU?$char_traits@D@std@@V?$allocator@D@2@@std@@AEBV23@@Z@4HA 0000000180012999 f   Resources.obj
 0001:000119a5       ?dtor$0@?0??getPtr@Resource@@AEBAPEAXAEAK@Z@4HA 00000001800129a5 f   Resources.obj
 0001:000119a5       ?dtor$4@?0??getPtr@Resource@@AEBAPEAXAEAK@Z@4HA 00000001800129a5 f   Resources.obj
 0001:000119b1       ?dtor$1@?0??getPtr@Resource@@AEBAPEAXAEAK@Z@4HA 00000001800129b1 f   Resources.obj
 0001:000119b1       ?dtor$5@?0??getPtr@Resource@@AEBAPEAXAEAK@Z@4HA 00000001800129b1 f   Resources.obj
 0001:000119bd       ?dtor$0@?0???0?$basic_stringstream@DU?$char_traits@D@std@@V?$allocator@D@2@@std@@QEAA@H@Z@4HA 00000001800129bd f   VersionInfo.obj
 0001:000119eb       ?dtor$1@?0???0?$basic_stringstream@DU?$char_traits@D@std@@V?$allocator@D@2@@std@@QEAA@H@Z@4HA 00000001800129eb f   VersionInfo.obj
 0001:000119fd       ?dtor$0@?0???0?$basic_stringstream@GU?$char_traits@G@std@@V?$allocator@G@2@@std@@QEAA@XZ@4HA 00000001800129fd f   VersionInfo.obj
 0001:00011a2b       ?dtor$1@?0???0?$basic_stringstream@GU?$char_traits@G@std@@V?$allocator@G@2@@std@@QEAA@XZ@4HA 0000000180012a2b f   VersionInfo.obj
 0001:00011a3d       ?dtor$0@?0???0FixedFileVersion@?A0xcb1fbc16@@QEAA@AEBV?$basic_string@GU?$char_traits@G@std@@V?$allocator@G@2@@std@@@Z@4HA 0000000180012a3d f   VersionInfo.obj
 0001:00011a49       ?catch$0@?0???1StreamSize@?A0xcb1fbc16@@QEAA@XZ@4HA 0000000180012a49 f   VersionInfo.obj
 0001:00011a56       __catch$??1StreamSize@?A0xcb1fbc16@@QEAA@XZ$0 0000000180012a56 f   VersionInfo.obj
 0001:00011a92       ?catch$1@?0???1StreamSize@?A0xcb1fbc16@@QEAA@XZ@4HA 0000000180012a92 f   VersionInfo.obj
 0001:00011a9f       __catch$??1StreamSize@?A0xcb1fbc16@@QEAA@XZ$1 0000000180012a9f f   VersionInfo.obj
 0001:00011ad7       ?dtor$1@?0??apply@VersionInfo@@QEBAAEBV1@AEBVFileLock@ResourceEditor@@@Z@4HA 0000000180012ad7 f   VersionInfo.obj
 0001:00011ae3       ?dtor$2@?0??apply@VersionInfo@@QEBAAEBV1@AEBVFileLock@ResourceEditor@@@Z@4HA 0000000180012ae3 f   VersionInfo.obj
 0001:00011aef       ?dtor$0@?0??createFIXEDFILEINFO@VersionInfo@@AEBA?AUtagVS_FIXEDFILEINFO@@XZ@4HA 0000000180012aef f   VersionInfo.obj
 0001:00011aef       Java_jdk_jpackage_internal_ExecutableRebrander_iconSwap$dtor$1 0000000180012aef f   jpackage.obj
 0001:00011aef       Java_jdk_jpackage_internal_ExecutableRebrander_lockResource$dtor$0 0000000180012aef f   jpackage.obj
 0001:00011aef       ?dtor$0@?0??equals@tstrings@@YA_NAEBV?$basic_string@GU?$char_traits@G@std@@V?$allocator@G@2@@std@@0W4CompareType@1@@Z@4HA 0000000180012aef f   tstrings.obj
 0001:00011afb       ?catch$8@?0??createFIXEDFILEINFO@VersionInfo@@AEBA?AUtagVS_FIXEDFILEINFO@@XZ@4HA 0000000180012afb f   VersionInfo.obj
 0001:00011b08       __catch$?createFIXEDFILEINFO@VersionInfo@@AEBA?AUtagVS_FIXEDFILEINFO@@XZ$0 0000000180012b08 f   VersionInfo.obj
 0001:00011b4d       ?dtor$0@?0??fillBuffer@VersionInfo@@AEBAXAEAV?$basic_ostream@DU?$char_traits@D@std@@@std@@@Z@4HA 0000000180012b4d f   VersionInfo.obj
 0001:00011b59       ?dtor$10@?0??fillBuffer@VersionInfo@@AEBAXAEAV?$basic_ostream@DU?$char_traits@D@std@@@std@@@Z@4HA 0000000180012b59 f   VersionInfo.obj
 0001:00011b59       ?dtor$1@?0??fillBuffer@VersionInfo@@AEBAXAEAV?$basic_ostream@DU?$char_traits@D@std@@@std@@@Z@4HA 0000000180012b59 f   VersionInfo.obj
 0001:00011b59       ?dtor$3@?0??fillBuffer@VersionInfo@@AEBAXAEAV?$basic_ostream@DU?$char_traits@D@std@@@std@@@Z@4HA 0000000180012b59 f   VersionInfo.obj
 0001:00011b59       ?dtor$8@?0??fillBuffer@VersionInfo@@AEBAXAEAV?$basic_ostream@DU?$char_traits@D@std@@@std@@@Z@4HA 0000000180012b59 f   VersionInfo.obj
 0001:00011b65       ?dtor$2@?0??fillBuffer@VersionInfo@@AEBAXAEAV?$basic_ostream@DU?$char_traits@D@std@@@std@@@Z@4HA 0000000180012b65 f   VersionInfo.obj
 0001:00011b71       ?dtor$4@?0??fillBuffer@VersionInfo@@AEBAXAEAV?$basic_ostream@DU?$char_traits@D@std@@@std@@@Z@4HA 0000000180012b71 f   VersionInfo.obj
 0001:00011b7d       ?dtor$5@?0??fillBuffer@VersionInfo@@AEBAXAEAV?$basic_ostream@DU?$char_traits@D@std@@@std@@@Z@4HA 0000000180012b7d f   VersionInfo.obj
 0001:00011b89       ?dtor$6@?0??fillBuffer@VersionInfo@@AEBAXAEAV?$basic_ostream@DU?$char_traits@D@std@@@std@@@Z@4HA 0000000180012b89 f   VersionInfo.obj
 0001:00011b95       ?dtor$7@?0??fillBuffer@VersionInfo@@AEBAXAEAV?$basic_ostream@DU?$char_traits@D@std@@@std@@@Z@4HA 0000000180012b95 f   VersionInfo.obj
 0001:00011ba1       ?dtor$9@?0??fillBuffer@VersionInfo@@AEBAXAEAV?$basic_ostream@DU?$char_traits@D@std@@@std@@@Z@4HA 0000000180012ba1 f   VersionInfo.obj
 0001:00011bad       ?dtor$15@?0??fillBuffer@VersionInfo@@AEBAXAEAV?$basic_ostream@DU?$char_traits@D@std@@@std@@@Z@4HA 0000000180012bad f   VersionInfo.obj
 0001:00011bb9       ?dtor$0@?0???0SysError@@QEAA@AEBVany@tstrings@@PEBXKPEBD@Z@4HA 0000000180012bb9 f   WinErrorHandling.obj
 0001:00011bc5       ?dtor$0@?0??getSystemMessageDescription@?A0xd5983087@@YA?AV?$basic_string@GU?$char_traits@G@std@@V?$allocator@G@2@@std@@KPEAUHINSTANCE__@@@Z@4HA 0000000180012bc5 f   WinErrorHandling.obj
 0001:00011beb       ?dtor$0@?0??makeMessage@?A0xd5983087@@YA?AV?$basic_string@DU?$char_traits@D@std@@V?$allocator@D@2@@std@@AEBV23@PEBDPEBXK@Z@4HA 0000000180012beb f   WinErrorHandling.obj
 0001:00011bf7       ?dtor$10@?0??makeMessage@?A0xd5983087@@YA?AV?$basic_string@DU?$char_traits@D@std@@V?$allocator@D@2@@std@@AEBV23@PEBDPEBXK@Z@4HA 0000000180012bf7 f   WinErrorHandling.obj
 0001:00011bf7       ?dtor$1@?0??makeMessage@?A0xd5983087@@YA?AV?$basic_string@DU?$char_traits@D@std@@V?$allocator@D@2@@std@@AEBV23@PEBDPEBXK@Z@4HA 0000000180012bf7 f   WinErrorHandling.obj
 0001:00011bf7       ?dtor$3@?0??makeMessage@?A0xd5983087@@YA?AV?$basic_string@DU?$char_traits@D@std@@V?$allocator@D@2@@std@@AEBV23@PEBDPEBXK@Z@4HA 0000000180012bf7 f   WinErrorHandling.obj
 0001:00011c03       ?dtor$2@?0??makeMessage@?A0xd5983087@@YA?AV?$basic_string@DU?$char_traits@D@std@@V?$allocator@D@2@@std@@AEBV23@PEBDPEBXK@Z@4HA 0000000180012c03 f   WinErrorHandling.obj
 0001:00011c0f       ?dtor$4@?0??makeMessage@?A0xd5983087@@YA?AV?$basic_string@DU?$char_traits@D@std@@V?$allocator@D@2@@std@@AEBV23@PEBDPEBXK@Z@4HA 0000000180012c0f f   WinErrorHandling.obj
 0001:00011c1b       ?dtor$0@?0??toShortPath@FileUtils@@YA?AV?$basic_string@GU?$char_traits@G@std@@V?$allocator@G@2@@std@@AEBV23@@Z@4HA 0000000180012c1b f   WinFileUtils.obj
 0001:00011c1b       ?dtor$3@?0??toShortPath@FileUtils@@YA?AV?$basic_string@GU?$char_traits@G@std@@V?$allocator@G@2@@std@@AEBV23@@Z@4HA 0000000180012c1b f   WinFileUtils.obj
 0001:00011c1b       ?dtor$1@?0??getModulePath@?A0x7970c2a6@SysInfo@@YA?AV?$basic_string@GU?$char_traits@G@std@@V?$allocator@G@2@@std@@PEAUHINSTANCE__@@@Z@4HA 0000000180012c1b f   WinSysInfo.obj
 0001:00011c27       ?dtor$2@?0??toShortPath@FileUtils@@YA?AV?$basic_string@GU?$char_traits@G@std@@V?$allocator@G@2@@std@@AEBV23@@Z@4HA 0000000180012c27 f   WinFileUtils.obj
 0001:00011c27       ?dtor$0@?0???$getSystemDirImpl@P6AIPEAGI@Z@?A0x7970c2a6@SysInfo@@YA?AV?$basic_string@GU?$char_traits@G@std@@V?$allocator@G@2@@std@@P6AIPEAGI@ZAEBV?$basic_string@DU?$char_traits@D@std@@V?$allocator@D@2@@3@@Z@4HA 0000000180012c27 f   WinSysInfo.obj
 0001:00011c27       ?dtor$0@?0??getModulePath@?A0x7970c2a6@SysInfo@@YA?AV?$basic_string@GU?$char_traits@G@std@@V?$allocator@G@2@@std@@PEAUHINSTANCE__@@@Z@4HA 0000000180012c27 f   WinSysInfo.obj
 0001:00011c33       ?dtor$4@?0??toShortPath@FileUtils@@YA?AV?$basic_string@GU?$char_traits@G@std@@V?$allocator@G@2@@std@@AEBV23@@Z@4HA 0000000180012c33 f   WinFileUtils.obj
 0001:00011c33       ?dtor$2@?0??getModulePath@?A0x7970c2a6@SysInfo@@YA?AV?$basic_string@GU?$char_traits@G@std@@V?$allocator@G@2@@std@@PEAUHINSTANCE__@@@Z@4HA 0000000180012c33 f   WinSysInfo.obj
 0001:00011c33       ?dtor$3@?0???$getSystemDirImpl@P6AIPEAGI@Z@?A0x7970c2a6@SysInfo@@YA?AV?$basic_string@GU?$char_traits@G@std@@V?$allocator@G@2@@std@@P6AIPEAGI@ZAEBV?$basic_string@DU?$char_traits@D@std@@V?$allocator@D@2@@3@@Z@4HA 0000000180012c33 f   WinSysInfo.obj
 0001:00011c3f       ?dtor$2@?0???$getSystemDirImpl@P6AIPEAGI@Z@?A0x7970c2a6@SysInfo@@YA?AV?$basic_string@GU?$char_traits@G@std@@V?$allocator@G@2@@std@@P6AIPEAGI@ZAEBV?$basic_string@DU?$char_traits@D@std@@V?$allocator@D@2@@3@@Z@4HA 0000000180012c3f f   WinSysInfo.obj
 0001:00011c4b       ?dtor$0@?0??GetLongPath@?A0x764c93a3@@YA?AV?$basic_string@GU?$char_traits@G@std@@V?$allocator@G@2@@std@@AEBV23@@Z@4HA 0000000180012c4b f   WindowsRegistry.obj
 0001:00011c57       Java_jdk_jpackage_internal_WindowsRegistry_comparePaths$dtor$1 0000000180012c57 f   WindowsRegistry.obj
 0001:00011c57       Java_jdk_jpackage_internal_ShortPathUtils_getShortPath$dtor$1 0000000180012c57 f   jpackage.obj
 0001:00011c63       Java_jdk_jpackage_internal_WindowsRegistry_comparePaths$catch$12 0000000180012c63 f   WindowsRegistry.obj
 0001:00011c70       __catch$Java_jdk_jpackage_internal_WindowsRegistry_comparePaths$0 0000000180012c70 f   WindowsRegistry.obj
 0001:00011cac       Java_jdk_jpackage_internal_WindowsRegistry_comparePaths$catch$13 0000000180012cac f   WindowsRegistry.obj
 0001:00011cb9       __catch$Java_jdk_jpackage_internal_WindowsRegistry_comparePaths$1 0000000180012cb9 f   WindowsRegistry.obj
 0001:00011cf1       Java_jdk_jpackage_internal_WindowsRegistry_enumRegistryValue$catch$4 0000000180012cf1 f   WindowsRegistry.obj
 0001:00011cfe       __catch$Java_jdk_jpackage_internal_WindowsRegistry_enumRegistryValue$1 0000000180012cfe f   WindowsRegistry.obj
 0001:00011d36       Java_jdk_jpackage_internal_WindowsRegistry_enumRegistryValue$catch$5 0000000180012d36 f   WindowsRegistry.obj
 0001:00011d43       __catch$Java_jdk_jpackage_internal_WindowsRegistry_enumRegistryValue$0 0000000180012d43 f   WindowsRegistry.obj
 0001:00011d7f       Java_jdk_jpackage_internal_WindowsRegistry_openRegistryKey$catch$3 0000000180012d7f f   WindowsRegistry.obj
 0001:00011d8c       __catch$Java_jdk_jpackage_internal_WindowsRegistry_openRegistryKey$0 0000000180012d8c f   WindowsRegistry.obj
 0001:00011dc8       Java_jdk_jpackage_internal_WindowsRegistry_openRegistryKey$catch$4 0000000180012dc8 f   WindowsRegistry.obj
 0001:00011dd5       __catch$Java_jdk_jpackage_internal_WindowsRegistry_openRegistryKey$1 0000000180012dd5 f   WindowsRegistry.obj
 0001:00011e0d       Java_jdk_jpackage_internal_WindowsRegistry_readDwordValue$dtor$0 0000000180012e0d f   WindowsRegistry.obj
 0001:00011e0d       Java_jdk_jpackage_internal_ExecutableRebrander_versionSwap$dtor$2 0000000180012e0d f   jpackage.obj
 0001:00011e19       Java_jdk_jpackage_internal_WindowsRegistry_readDwordValue$catch$4 0000000180012e19 f   WindowsRegistry.obj
 0001:00011e26       __catch$Java_jdk_jpackage_internal_WindowsRegistry_readDwordValue$0 0000000180012e26 f   WindowsRegistry.obj
 0001:00011e62       Java_jdk_jpackage_internal_WindowsRegistry_readDwordValue$catch$5 0000000180012e62 f   WindowsRegistry.obj
 0001:00011e6f       __catch$Java_jdk_jpackage_internal_WindowsRegistry_readDwordValue$1 0000000180012e6f f   WindowsRegistry.obj
 0001:00011ea7       ?dtor$0@?0??append@LastErrorLogAppender@?A0xd3578678@@UEAAXAEBULogEvent@@@Z@4HA 0000000180012ea7 f   app.obj
 0001:00011eb3       ?dtor$0@?0???0?$basic_istringstream@DU?$char_traits@D@std@@V?$allocator@D@2@@std@@QEAA@AEBV?$basic_string@DU?$char_traits@D@std@@V?$allocator@D@2@@1@H@Z@4HA 0000000180012eb3 f   jpackage.obj
 0001:00011ee1       ?dtor$1@?0???0?$basic_istringstream@DU?$char_traits@D@std@@V?$allocator@D@2@@std@@QEAA@AEBV?$basic_string@DU?$char_traits@D@std@@V?$allocator@D@2@@1@H@Z@4HA 0000000180012ee1 f   jpackage.obj
 0001:00011ef3       ?dtor$0@?0???0?$basic_stringbuf@DU?$char_traits@D@std@@V?$allocator@D@2@@std@@QEAA@AEBV?$basic_string@DU?$char_traits@D@std@@V?$allocator@D@2@@1@H@Z@4HA 0000000180012ef3 f   jpackage.obj
 0001:00011f01       Java_jdk_jpackage_internal_ExecutableRebrander_iconSwap$dtor$0 0000000180012f01 f   jpackage.obj
 0001:00011f01       Java_jdk_jpackage_internal_WinExeBundler_embedMSI$dtor$1 0000000180012f01 f   jpackage.obj
 0001:00011f0d       Java_jdk_jpackage_internal_ExecutableRebrander_iconSwap$catch$4 0000000180012f0d f   jpackage.obj
 0001:00011f1a       __catch$Java_jdk_jpackage_internal_ExecutableRebrander_iconSwap$0 0000000180012f1a f   jpackage.obj
 0001:00011f56       Java_jdk_jpackage_internal_ExecutableRebrander_iconSwap$catch$5 0000000180012f56 f   jpackage.obj
 0001:00011f63       __catch$Java_jdk_jpackage_internal_ExecutableRebrander_iconSwap$1 0000000180012f63 f   jpackage.obj
 0001:00011f9b       Java_jdk_jpackage_internal_ExecutableRebrander_lockResource$catch$3 0000000180012f9b f   jpackage.obj
 0001:00011fa8       __catch$Java_jdk_jpackage_internal_ExecutableRebrander_lockResource$0 0000000180012fa8 f   jpackage.obj
 0001:00011fe4       Java_jdk_jpackage_internal_ExecutableRebrander_lockResource$catch$4 0000000180012fe4 f   jpackage.obj
 0001:00011ff1       __catch$Java_jdk_jpackage_internal_ExecutableRebrander_lockResource$1 0000000180012ff1 f   jpackage.obj
 0001:00012029       Java_jdk_jpackage_internal_ExecutableRebrander_unlockResource$catch$1 0000000180013029 f   jpackage.obj
 0001:00012036       __catch$Java_jdk_jpackage_internal_ExecutableRebrander_unlockResource$0 0000000180013036 f   jpackage.obj
 0001:00012072       Java_jdk_jpackage_internal_ExecutableRebrander_unlockResource$catch$2 0000000180013072 f   jpackage.obj
 0001:0001207f       __catch$Java_jdk_jpackage_internal_ExecutableRebrander_unlockResource$1 000000018001307f f   jpackage.obj
 0001:000120b7       Java_jdk_jpackage_internal_ExecutableRebrander_versionSwap$dtor$0 00000001800130b7 f   jpackage.obj
 0001:000120c3       Java_jdk_jpackage_internal_ExecutableRebrander_versionSwap$dtor$1 00000001800130c3 f   jpackage.obj
 0001:000120cf       Java_jdk_jpackage_internal_ExecutableRebrander_versionSwap$dtor$3 00000001800130cf f   jpackage.obj
 0001:000120db       Java_jdk_jpackage_internal_ExecutableRebrander_versionSwap$dtor$4 00000001800130db f   jpackage.obj
 0001:000120e7       Java_jdk_jpackage_internal_ExecutableRebrander_versionSwap$catch$13 00000001800130e7 f   jpackage.obj
 0001:000120f4       __catch$Java_jdk_jpackage_internal_ExecutableRebrander_versionSwap$0 00000001800130f4 f   jpackage.obj
 0001:00012130       Java_jdk_jpackage_internal_ExecutableRebrander_versionSwap$catch$14 0000000180013130 f   jpackage.obj
 0001:0001213d       __catch$Java_jdk_jpackage_internal_ExecutableRebrander_versionSwap$1 000000018001313d f   jpackage.obj
 0001:00012175       Java_jdk_jpackage_internal_ShortPathUtils_getShortPath$catch$4 0000000180013175 f   jpackage.obj
 0001:00012182       __catch$Java_jdk_jpackage_internal_ShortPathUtils_getShortPath$0 0000000180013182 f   jpackage.obj
 0001:000121be       Java_jdk_jpackage_internal_ShortPathUtils_getShortPath$catch$5 00000001800131be f   jpackage.obj
 0001:000121cb       __catch$Java_jdk_jpackage_internal_ShortPathUtils_getShortPath$1 00000001800131cb f   jpackage.obj
 0001:00012203       Java_jdk_jpackage_internal_WinExeBundler_embedMSI$dtor$2 0000000180013203 f   jpackage.obj
 0001:00012203       Java_jdk_jpackage_internal_WinExeBundler_embedMSI$dtor$9 0000000180013203 f   jpackage.obj
 0001:0001220f       Java_jdk_jpackage_internal_WinExeBundler_embedMSI$dtor$3 000000018001320f f   jpackage.obj
 0001:0001221b       Java_jdk_jpackage_internal_WinExeBundler_embedMSI$dtor$4 000000018001321b f   jpackage.obj
 0001:00012227       Java_jdk_jpackage_internal_WinExeBundler_embedMSI$dtor$5 0000000180013227 f   jpackage.obj
 0001:00012227       Java_jdk_jpackage_internal_WinExeBundler_embedMSI$dtor$6 0000000180013227 f   jpackage.obj
 0001:00012233       Java_jdk_jpackage_internal_WinExeBundler_embedMSI$dtor$7 0000000180013233 f   jpackage.obj
 0001:0001223f       Java_jdk_jpackage_internal_WinExeBundler_embedMSI$dtor$8 000000018001323f f   jpackage.obj
 0001:0001224b       Java_jdk_jpackage_internal_WinExeBundler_embedMSI$catch$25 000000018001324b f   jpackage.obj
 0001:00012258       __catch$Java_jdk_jpackage_internal_WinExeBundler_embedMSI$0 0000000180013258 f   jpackage.obj
 0001:00012294       Java_jdk_jpackage_internal_WinExeBundler_embedMSI$catch$26 0000000180013294 f   jpackage.obj
 0001:000122a1       __catch$Java_jdk_jpackage_internal_WinExeBundler_embedMSI$1 00000001800132a1 f   jpackage.obj
 0001:000122d9       ?dtor$0@?0??fromMultiByte@?A0xf04d92fb@tstrings@@YA?AV?$basic_string@GU?$char_traits@G@std@@V?$allocator@G@2@@std@@AEBV?$basic_string@DU?$char_traits@D@std@@V?$allocator@D@2@@4@H@Z@4HA 00000001800132d9 f   tstrings.obj
 0001:000122ff       ?dtor$0@?0??toLower@tstrings@@YA?AV?$basic_string@GU?$char_traits@G@std@@V?$allocator@G@2@@std@@AEBV23@@Z@4HA 00000001800132ff f   tstrings.obj
 0001:00012325       ?dtor$0@?0??toMultiByte@?A0xf04d92fb@tstrings@@YA?AV?$basic_string@DU?$char_traits@D@std@@V?$allocator@D@2@@std@@AEBV?$basic_string@GU?$char_traits@G@std@@V?$allocator@G@2@@4@H@Z@4HA 0000000180013325 f   tstrings.obj
 0001:0001234b       ?dtor$0@?0??unsafe_format@tstrings@@YA?AV?$basic_string@GU?$char_traits@G@std@@V?$allocator@G@2@@std@@PEBGZZ@4HA 000000018001334b f   tstrings.obj
 0001:00012374       __scrt_is_nonwritable_in_current_image$filt$0 0000000180013374 f   MSVCRT:utility.obj
 0001:0001238c       ?fin$0@?0??dllmain_crt_process_attach@@YAHQEAUHINSTANCE__@@QEAX@Z@4HA 000000018001338c f   MSVCRT:dll_dllmain.obj
 0001:000123a3       ?fin$0@?0??dllmain_crt_process_detach@@YAH_N@Z@4HA 00000001800133a3 f   MSVCRT:dll_dllmain.obj
 0001:000123bc       ?fin$1@?0??dllmain_crt_process_detach@@YAH_N@Z@4HA 00000001800133bc f   MSVCRT:dll_dllmain.obj
 0001:000123d0       ?filt$0@?0??dllmain_dispatch@@YAHQEAUHINSTANCE__@@KQEAX@Z@4HA 00000001800133d0 f   MSVCRT:dll_dllmain.obj
 0001:00012408       ??__FlastErrorLogAppender@?A0xd3578678@@YAXXZ 0000000180013408 f   app.obj
 0001:00012418       ??__F_Fac_tidy_reg@std@@YAXXZ 0000000180013418 f   msvcprt:locale0_implib.obj
 0002:000007d8       ?_Fac_tidy_reg$initializer$@std@@3P6AXXZEA 00000001800147d8     msvcprt:locale0_implib.obj
 0002:000007e0       ?lastErrorLogAppender$initializer$@?A0xd3578678@@3P6AXXZEA 00000001800147e0     app.obj
 0002:00000820       ?_Fake_alloc@std@@3U_Fake_allocator@1@B 0000000180014820     ErrorHandling.obj
 0002:00000ad0       ?_Fake_alloc@std@@3U_Fake_allocator@1@B 0000000180014ad0     Executor.obj
 0002:00000b82       ?_Fake_alloc@std@@3U_Fake_allocator@1@B 0000000180014b82     FileUtils.obj
 0002:00000b84       ?dirSeparator@?A0x534245bb@FileUtils@@3GB 0000000180014b84     FileUtils.obj
 0002:00000b88       ?alianDirSeparator@?A0x534245bb@FileUtils@@3GB 0000000180014b88     FileUtils.obj
 0002:00000b92       ?_Fake_alloc@std@@3U_Fake_allocator@1@B 0000000180014b92     Guid.obj
 0002:00000c69       ?_Fake_alloc@std@@3U_Fake_allocator@1@B 0000000180014c69     IconSwap.obj
 0002:00000c92       ?_Fake_alloc@std@@3U_Fake_allocator@1@B 0000000180014c92     JniUtils.obj
 0002:00000e51       ?_Fake_alloc@std@@3U_Fake_allocator@1@B 0000000180014e51     Log.obj
 0002:00000ee6       ?_Fake_alloc@std@@3U_Fake_allocator@1@B 0000000180014ee6     MsiCA.obj
 0002:00000ee7       ?piecewise_construct@std@@3Upiecewise_construct_t@1@B 0000000180014ee7     MsiCA.obj
 0002:00000f89       ?_Fake_alloc@std@@3U_Fake_allocator@1@B 0000000180014f89     MsiDb.obj
 0002:0000125e       ?_Fake_alloc@std@@3U_Fake_allocator@1@B 000000018001525e     MsiUtils.obj
 0002:0000125f       ?piecewise_construct@std@@3Upiecewise_construct_t@1@B 000000018001525f     MsiUtils.obj
 0002:00001408       ?_Fake_alloc@std@@3U_Fake_allocator@1@B 0000000180015408     PlatformLogEvent.obj
 0002:00001498       ?_Fake_alloc@std@@3U_Fake_allocator@1@B 0000000180015498     ResourceEditor.obj
 0002:000015c8       ?_Fake_alloc@std@@3U_Fake_allocator@1@B 00000001800155c8     Resources.obj
 0002:00001670       ?_Fake_alloc@std@@3U_Fake_allocator@1@B 0000000180015670     VersionInfo.obj
 0002:00001671       ?piecewise_construct@std@@3Upiecewise_construct_t@1@B 0000000180015671     VersionInfo.obj
 0002:00001678       ?_Valid_strftime_specifiers@std@@3QBDB 0000000180015678     VersionInfo.obj
 0002:000019ba       ?_Fake_alloc@std@@3U_Fake_allocator@1@B 00000001800159ba     WinApp.obj
 0002:000019bb       ?_Fake_alloc@std@@3U_Fake_allocator@1@B 00000001800159bb     WinDll.obj
 0002:000019bc       ?_Fake_alloc@std@@3U_Fake_allocator@1@B 00000001800159bc     WinErrorHandling.obj
 0002:00001b1b       ?_Fake_alloc@std@@3U_Fake_allocator@1@B 0000000180015b1b     WinFileUtils.obj
 0002:00001b8a       ?_Fake_alloc@std@@3U_Fake_allocator@1@B 0000000180015b8a     WinSysInfo.obj
 0002:00001cbe       ?_Fake_alloc@std@@3U_Fake_allocator@1@B 0000000180015cbe     WindowsRegistry.obj
 0002:00001e20       ?_Fake_alloc@std@@3U_Fake_allocator@1@B 0000000180015e20     app.obj
 0002:00001e30       ??_7LastErrorLogAppender@?A0xd3578678@@6B@ 0000000180015e30     app.obj
 0002:00001e40       ?_Fake_alloc@std@@3U_Fake_allocator@1@B 0000000180015e40     jpackage.obj
 0002:0000202f       ?_Fake_alloc@std@@3U_Fake_allocator@1@B 000000018001602f     tstrings.obj
 0002:00002180       ?_Tail_masks@?1??_Avx2_tail_mask_32@?A0x8417fefe@@YA?AT__m256i@@_K@Z@4QBIB 0000000180016180     msvcprt:vector_algorithms.obj
 0002:000021e8       GS_ExceptionPointers       00000001800161e8     MSVCRT:gs_report.obj
 0002:00003810       ??_R4LastErrorLogAppender@?A0xd3578678@@6B@ 0000000180017810     app.obj
 0002:00003838       ??_R3LastErrorLogAppender@?A0xd3578678@@8 0000000180017838     app.obj
 0002:00003850       ??_R2LastErrorLogAppender@?A0xd3578678@@8 0000000180017850     app.obj
 0002:00003868       ??_R1A@?0A@EA@LastErrorLogAppender@?A0xd3578678@@8 0000000180017868     app.obj
 0002:00003f38       $unwind$??0bad_alloc@std@@QEAA@AEBV01@@Z 0000000180017f38     ErrorHandling.obj
 0002:00003f38       $unwind$??0bad_array_new_length@std@@QEAA@AEBV01@@Z 0000000180017f38     ErrorHandling.obj
 0002:00003f38       $unwind$??0bad_cast@std@@QEAA@AEBV01@@Z 0000000180017f38     ErrorHandling.obj
 0002:00003f38       $unwind$??0exception@std@@QEAA@AEBV01@@Z 0000000180017f38     ErrorHandling.obj
 0002:00003f38       $unwind$??1?$basic_string@DU?$char_traits@D@std@@V?$allocator@D@2@@std@@QEAA@XZ 0000000180017f38     ErrorHandling.obj
 0002:00003f38       $unwind$??1any@tstrings@@QEAA@XZ 0000000180017f38     ErrorHandling.obj
 0002:00003f38       $unwind$??_D?$basic_ostringstream@DU?$char_traits@D@std@@V?$allocator@D@2@@std@@QEAAXXZ 0000000180017f38     ErrorHandling.obj
 0002:00003f38       $unwind$??_D?$basic_ostringstream@GU?$char_traits@G@std@@V?$allocator@G@2@@std@@QEAAXXZ 0000000180017f38     ErrorHandling.obj
 0002:00003f38       $unwind$?_Tidy_deallocate@?$basic_string@GU?$char_traits@G@std@@V?$allocator@G@2@@std@@AEAAXXZ 0000000180017f38     ErrorHandling.obj
 0002:00003f38       $unwind$??$?6PEBD@any@tstrings@@QEAAAEAV01@PEBD@Z 0000000180017f38     Executor.obj
 0002:00003f38       $unwind$??0SysError@@QEAA@AEBV0@@Z 0000000180017f38     Executor.obj
 0002:00003f38       $unwind$??0any@tstrings@@QEAA@XZ 0000000180017f38     Executor.obj
 0002:00003f38       $unwind$??0runtime_error@std@@QEAA@AEBV01@@Z 0000000180017f38     Executor.obj
 0002:00003f38       $unwind$??1?$JpError@VSysError@@@@UEAA@XZ 0000000180017f38     Executor.obj
 0002:00003f38       $unwind$??1?$_Tidy_guard@V?$vector@GV?$allocator@G@std@@@std@@@std@@QEAA@XZ 0000000180017f38     Executor.obj
 0002:00003f38       $unwind$??1?$vector@GV?$allocator@G@std@@@std@@QEAA@XZ 0000000180017f38     Executor.obj
 0002:00003f38       $unwind$??1?$JpError@Vruntime_error@std@@@@UEAA@XZ 0000000180017f38     Guid.obj
 0002:00003f38       $unwind$??6any@tstrings@@QEAAAEAV01@AEBV?$basic_string@GU?$char_traits@G@std@@V?$allocator@G@2@@std@@@Z 0000000180017f38     Guid.obj
 0002:00003f38       $unwind$??$endl@DU?$char_traits@D@std@@@std@@YAAEAV?$basic_ostream@DU?$char_traits@D@std@@@0@AEAV10@@Z 0000000180017f38     Log.obj
 0002:00003f38       $unwind$??1LogEvent@@QEAA@XZ 0000000180017f38     Log.obj
 0002:00003f38       $unwind$??_GLogAppender@@UEAAPEAXI@Z 0000000180017f38     Log.obj
 0002:00003f38       $unwind$??_GStreamLogAppender@@UEAAPEAXI@Z 0000000180017f38     Log.obj
 0002:00003f38       $unwind$??1?$JpError@VError@msi@@@@UEAA@XZ 0000000180017f38     MsiCA.obj
 0002:00003f38       $unwind$??$?6I@any@tstrings@@QEAAAEAV01@I@Z 0000000180017f38     MsiDb.obj
 0002:00003f38       $unwind$??0NoMoreItemsError@msi@@QEAA@AEBVany@tstrings@@@Z 0000000180017f38     MsiDb.obj
 0002:00003f38       $unwind$??1?$JpError@VNoMoreItemsError@msi@@@@UEAA@XZ 0000000180017f38     MsiDb.obj
 0002:00003f38       $unwind$?setbuf@?$basic_filebuf@DU?$char_traits@D@std@@@std@@MEAAPEAV?$basic_streambuf@DU?$char_traits@D@std@@@2@PEAD_J@Z 0000000180017f38     MsiDb.obj
 0002:00003f38       $unwind$??$?6K@any@tstrings@@QEAAAEAV01@K@Z 0000000180017f38     MsiUtils.obj
 0002:00003f38       $unwind$??1StringResource@@QEAA@XZ 0000000180017f38     MsiUtils.obj
 0002:00003f38       $unwind$??0PlatformLogEvent@@QEAA@XZ 0000000180017f38     PlatformLogEvent.obj
 0002:00003f38       $unwind$?init@LogEvent@@CAXAEAUPlatformLogEvent@@@Z 0000000180017f38     PlatformLogEvent.obj
 0002:00003f38       $unwind$??$?6PEAX@any@tstrings@@QEAAAEAV01@PEAX@Z 0000000180017f38     ResourceEditor.obj
 0002:00003f38       $unwind$??1?$_Tidy_guard@V?$vector@EV?$allocator@E@std@@@std@@@std@@QEAA@XZ 0000000180017f38     ResourceEditor.obj
 0002:00003f38       $unwind$??1?$vector@EV?$allocator@E@std@@@std@@QEAA@XZ 0000000180017f38     ResourceEditor.obj
 0002:00003f38       $unwind$??_D?$basic_ifstream@DU?$char_traits@D@std@@@std@@QEAAXXZ 0000000180017f38     ResourceEditor.obj
 0002:00003f38       $unwind$??0VersionInfo@@QEAA@XZ 0000000180017f38     VersionInfo.obj
 0002:00003f38       $unwind$??1ResourceEditor@@QEAA@XZ 0000000180017f38     VersionInfo.obj
 0002:00003f38       $unwind$??_D?$basic_stringstream@DU?$char_traits@D@std@@V?$allocator@D@2@@std@@QEAAXXZ 0000000180017f38     VersionInfo.obj
 0002:00003f38       $unwind$??_D?$basic_stringstream@GU?$char_traits@G@std@@V?$allocator@G@2@@std@@QEAAXXZ 0000000180017f38     VersionInfo.obj
 0002:00003f38       $unwind$?hex@std@@YAAEAVios_base@1@AEAV21@@Z 0000000180017f38     VersionInfo.obj
 0002:00003f38       $unwind$?uppercase@std@@YAAEAVios_base@1@AEAV21@@Z 0000000180017f38     VersionInfo.obj
 0002:00003f38       $unwind$??_GLastErrorLogAppender@?A0xd3578678@@UEAAPEAXI@Z 0000000180017f38     app.obj
 0002:00003f38       $unwind$??1VersionInfo@@QEAA@XZ 0000000180017f38     jpackage.obj
 0002:00003f38       $unwind$??_D?$basic_istringstream@DU?$char_traits@D@std@@V?$allocator@D@2@@std@@QEAAXXZ 0000000180017f38     jpackage.obj
 0002:00003f38       $unwind$??0invalid_argument@std@@QEAA@AEBV01@@Z 0000000180017f38     tstrings.obj
 0002:00003f38       $unwind$??0logic_error@std@@QEAA@AEBV01@@Z 0000000180017f38     tstrings.obj
 0002:00003f38       $unwind$__raise_securityfailure 0000000180017f38     MSVCRT:gs_report.obj
 0002:00003f38       $unwind$??2@YAPEAX_K@Z     0000000180017f38     MSVCRT:new_scalar.obj
 0002:00003f38       $unwind$??_Gtype_info@@UEAAPEAXI@Z 0000000180017f38     MSVCRT:std_type_info_static.obj
 0002:00003f38       $unwind$__scrt_initialize_onexit_tables 0000000180017f38     MSVCRT:utility.obj
 0002:00003f38       $unwind$__scrt_release_startup_lock 0000000180017f38     MSVCRT:utility.obj
 0002:00003f38       $unwind$__scrt_uninitialize_crt 0000000180017f38     MSVCRT:utility.obj
 0002:00003f38       $unwind$_onexit            0000000180017f38     MSVCRT:utility.obj
 0002:00003f38       $unwind$??__F_Fac_tidy_reg@std@@YAXXZ 0000000180017f38     msvcprt:locale0_implib.obj
 0002:00003f38       $unwind$?_Facet_Register@std@@YAXPEAV_Facet_base@1@@Z 0000000180017f38     msvcprt:locale0_implib.obj
 0002:00003f40       $unwind$??1?$basic_ostringstream@DU?$char_traits@D@std@@V?$allocator@D@2@@std@@UEAA@XZ 0000000180017f40     ErrorHandling.obj
 0002:00003f40       $unwind$??1?$basic_ostringstream@GU?$char_traits@G@std@@V?$allocator@G@2@@std@@UEAA@XZ 0000000180017f40     ErrorHandling.obj
 0002:00003f40       $unwind$??_G?$basic_stringbuf@DU?$char_traits@D@std@@V?$allocator@D@2@@std@@UEAAPEAXI@Z 0000000180017f40     ErrorHandling.obj
 0002:00003f40       $unwind$??_G?$basic_stringbuf@GU?$char_traits@G@std@@V?$allocator@G@2@@std@@UEAAPEAXI@Z 0000000180017f40     ErrorHandling.obj
 0002:00003f40       $unwind$??_Gbad_alloc@std@@UEAAPEAXI@Z 0000000180017f40     ErrorHandling.obj
 0002:00003f40       $unwind$??_Gbad_array_new_length@std@@UEAAPEAXI@Z 0000000180017f40     ErrorHandling.obj
 0002:00003f40       $unwind$??_Gbad_cast@std@@UEAAPEAXI@Z 0000000180017f40     ErrorHandling.obj
 0002:00003f40       $unwind$??_Gexception@std@@UEAAPEAXI@Z 0000000180017f40     ErrorHandling.obj
 0002:00003f40       $unwind$??$_Copy_memmove@PEAGPEAG@std@@YAPEAGPEAG00@Z 0000000180017f40     Executor.obj
 0002:00003f40       $unwind$??_G?$JpError@VSysError@@@@UEAAPEAXI@Z 0000000180017f40     Executor.obj
 0002:00003f40       $unwind$??_GSysError@@UEAAPEAXI@Z 0000000180017f40     Executor.obj
 0002:00003f40       $unwind$??_Gruntime_error@std@@UEAAPEAXI@Z 0000000180017f40     Executor.obj
 0002:00003f40       $unwind$??$?MGU?$char_traits@G@std@@V?$allocator@G@1@@std@@YA_NAEBV?$basic_string@GU?$char_traits@G@std@@V?$allocator@G@2@@0@0@Z 0000000180017f40     Guid.obj
 0002:00003f40       $unwind$??_G?$JpError@Vruntime_error@std@@@@UEAAPEAXI@Z 0000000180017f40     Guid.obj
 0002:00003f40       $unwind$??0?$basic_string@DU?$char_traits@D@std@@V?$allocator@D@2@@std@@QEAA@QEBD@Z 0000000180017f40     MsiCA.obj
 0002:00003f40       $unwind$??0Error@msi@@QEAA@AEBV01@@Z 0000000180017f40     MsiCA.obj
 0002:00003f40       $unwind$??_G?$JpError@VError@msi@@@@UEAAPEAXI@Z 0000000180017f40     MsiCA.obj
 0002:00003f40       $unwind$??_GError@msi@@UEAAPEAXI@Z 0000000180017f40     MsiCA.obj
 0002:00003f40       $unwind$??0NoMoreItemsError@msi@@QEAA@AEBV01@@Z 0000000180017f40     MsiDb.obj
 0002:00003f40       $unwind$??_G?$JpError@VNoMoreItemsError@msi@@@@UEAAPEAXI@Z 0000000180017f40     MsiDb.obj
 0002:00003f40       $unwind$??_G?$basic_filebuf@DU?$char_traits@D@std@@@std@@UEAAPEAXI@Z 0000000180017f40     MsiDb.obj
 0002:00003f40       $unwind$??_GNoMoreItemsError@msi@@UEAAPEAXI@Z 0000000180017f40     MsiDb.obj
 0002:00003f40       $unwind$?imbue@?$basic_filebuf@DU?$char_traits@D@std@@@std@@MEAAXAEBVlocale@2@@Z 0000000180017f40     MsiDb.obj
 0002:00003f40       $unwind$?sync@?$basic_filebuf@DU?$char_traits@D@std@@@std@@MEAAHXZ 0000000180017f40     MsiDb.obj
 0002:00003f40       $unwind$?underflow@?$basic_filebuf@DU?$char_traits@D@std@@@std@@MEAAHXZ 0000000180017f40     MsiDb.obj
 0002:00003f40       $unwind$??$_Copy_memmove@PEAEPEAE@std@@YAPEAEPEAE00@Z 0000000180017f40     ResourceEditor.obj
 0002:00003f40       $unwind$??_G?$basic_ifstream@DU?$char_traits@D@std@@@std@@UEAAPEAXI@Z 0000000180017f40     ResourceEditor.obj
 0002:00003f40       $unwind$??1?$basic_stringstream@DU?$char_traits@D@std@@V?$allocator@D@2@@std@@UEAA@XZ 0000000180017f40     VersionInfo.obj
 0002:00003f40       $unwind$??1?$basic_stringstream@GU?$char_traits@G@std@@V?$allocator@G@2@@std@@UEAA@XZ 0000000180017f40     VersionInfo.obj
 0002:00003f40       $unwind$??1?$basic_istringstream@DU?$char_traits@D@std@@V?$allocator@D@2@@std@@UEAA@XZ 0000000180017f40     jpackage.obj
 0002:00003f40       $unwind$??_Ginvalid_argument@std@@UEAAPEAXI@Z 0000000180017f40     tstrings.obj
 0002:00003f40       $unwind$??_Glogic_error@std@@UEAAPEAXI@Z 0000000180017f40     tstrings.obj
 0002:00003f40       $unwind$_RTC_Initialize    0000000180017f40     MSVCRT:initsect.obj
 0002:00003f40       $unwind$_RTC_Terminate     0000000180017f40     MSVCRT:initsect.obj
 0002:00003f4c       $unwind$?_Throw_bad_array_new_length@std@@YAXXZ 0000000180017f4c     ErrorHandling.obj
 0002:00003f4c       $unwind$?_Throw_bad_cast@std@@YAXXZ 0000000180017f4c     ErrorHandling.obj
 0002:00003f4c       $unwind$?PrintError@@YAXXZ 0000000180017f4c     IconSwap.obj
 0002:00003f4c       $unwind$?__scrt_throw_std_bad_alloc@@YAXXZ 0000000180017f4c     MSVCRT:throw_bad_alloc.obj
 0002:00003f4c       $unwind$?__scrt_throw_std_bad_array_new_length@@YAXXZ 0000000180017f4c     MSVCRT:throw_bad_alloc.obj
 0002:00003f54       $unwind$??$_Allocate_manually_vector_aligned@U_Default_allocate_traits@std@@@std@@YAPEAX_K@Z 0000000180017f54     ErrorHandling.obj
 0002:00003f54       $unwind$??1?$unique_ptr@V_Facet_base@std@@U?$default_delete@V_Facet_base@std@@@2@@std@@QEAA@XZ 0000000180017f54     ErrorHandling.obj
 0002:00003f54       $unwind$??1locale@std@@QEAA@XZ 0000000180017f54     ErrorHandling.obj
 0002:00003f54       $unwind$?_Xlen_string@std@@YAXXZ 0000000180017f54     ErrorHandling.obj
 0002:00003f54       $unwind$?_Xran@?$_String_val@U?$_Simple_types@D@std@@@std@@SAXXZ 0000000180017f54     ErrorHandling.obj
 0002:00003f54       $unwind$?_Xlength@?$vector@GV?$allocator@G@std@@@std@@CAXXZ 0000000180017f54     Executor.obj
 0002:00003f54       $unwind$?_Xlength@?$vector@V?$basic_string@GU?$char_traits@G@std@@V?$allocator@G@2@@std@@V?$allocator@V?$basic_string@GU?$char_traits@G@std@@V?$allocator@G@2@@std@@@2@@std@@CAXXZ 0000000180017f54     Executor.obj
 0002:00003f54       $unwind$?deallocate@?$allocator@G@std@@QEAAXQEAG_K@Z 0000000180017f54     Executor.obj
 0002:00003f54       $unwind$?deallocate@?$allocator@V?$basic_string@GU?$char_traits@G@std@@V?$allocator@G@2@@std@@@std@@QEAAXQEAV?$basic_string@GU?$char_traits@G@std@@V?$allocator@G@2@@2@_K@Z 0000000180017f54     Executor.obj
 0002:00003f54       $unwind$?_Xran@?$_String_val@U?$_Simple_types@G@std@@@std@@SAXXZ 0000000180017f54     FileUtils.obj
 0002:00003f54       $unwind$?defaultLogger@Logger@@SAAEAV1@XZ 0000000180017f54     Log.obj
 0002:00003f54       $unwind$??1?$_Alloc_construct_ptr@V?$allocator@U?$_Tree_node@U?$pair@$$CBV?$basic_string@GU?$char_traits@G@std@@V?$allocator@G@2@@std@@V12@@std@@PEAX@std@@@std@@@std@@QEAA@XZ 0000000180017f54     MsiCA.obj
 0002:00003f54       $unwind$??1?$_Tree_temp_node_alloc@V?$allocator@U?$_Tree_node@U?$pair@$$CBV?$basic_string@GU?$char_traits@G@std@@V?$allocator@G@2@@std@@V12@@std@@PEAX@std@@@std@@@std@@QEAA@XZ 0000000180017f54     MsiCA.obj
 0002:00003f54       $unwind$?_Throw_tree_length_error@std@@YAXXZ 0000000180017f54     MsiCA.obj
 0002:00003f54       $unwind$?_Lock@?$basic_filebuf@DU?$char_traits@D@std@@@std@@UEAAXXZ 0000000180017f54     MsiDb.obj
 0002:00003f54       $unwind$?_Unlock@?$basic_filebuf@DU?$char_traits@D@std@@@std@@UEAAXXZ 0000000180017f54     MsiDb.obj
 0002:00003f54       $unwind$?_Xlength@?$vector@EV?$allocator@E@std@@@std@@CAXXZ 0000000180017f54     ResourceEditor.obj
 0002:00003f54       $unwind$?deallocate@?$allocator@E@std@@QEAAXQEAE_K@Z 0000000180017f54     ResourceEditor.obj
 0002:00003f54       $unwind$?freeLibrary@Dll@@SAXPEAUHINSTANCE__@@@Z 0000000180017f54     WinDll.obj
 0002:00003f54       $unwind$__scrt_initialize_default_local_stdio_options 0000000180017f54     MSVCRT:default_local_stdio_options.obj
 0002:00003f54       $unwind$?dllmain_crt_dispatch@@YAHQEAUHINSTANCE__@@KQEAX@Z 0000000180017f54     MSVCRT:dll_dllmain.obj
 0002:00003f54       $unwind$DllMain            0000000180017f54     MSVCRT:dll_dllmain_stub.obj
 0002:00003f54       $unwind$__report_rangecheckfailure 0000000180017f54     MSVCRT:gs_report.obj
 0002:00003f54       $unwind$__GSHandlerCheck   0000000180017f54     MSVCRT:gshandler.obj
 0002:00003f54       $unwind$__scrt_acquire_startup_lock 0000000180017f54     MSVCRT:utility.obj
 0002:00003f54       $unwind$__scrt_dllmain_after_initialize_c 0000000180017f54     MSVCRT:utility.obj
 0002:00003f54       $unwind$__scrt_dllmain_before_initialize_c 0000000180017f54     MSVCRT:utility.obj
 0002:00003f54       $unwind$__scrt_dllmain_crt_thread_attach 0000000180017f54     MSVCRT:utility.obj
 0002:00003f54       $unwind$__scrt_dllmain_crt_thread_detach 0000000180017f54     MSVCRT:utility.obj
 0002:00003f54       $unwind$__scrt_dllmain_uninitialize_c 0000000180017f54     MSVCRT:utility.obj
 0002:00003f54       $unwind$__scrt_dllmain_uninitialize_critical 0000000180017f54     MSVCRT:utility.obj
 0002:00003f54       $unwind$__scrt_initialize_crt 0000000180017f54     MSVCRT:utility.obj
 0002:00003f54       $unwind$atexit             0000000180017f54     MSVCRT:utility.obj
 0002:00003f5c       $unwind$??1_Sentry_base@?$basic_ostream@DU?$char_traits@D@std@@@std@@QEAA@XZ 0000000180017f5c     ErrorHandling.obj
 0002:00003f5c       $unwind$??1_Sentry_base@?$basic_ostream@GU?$char_traits@G@std@@@std@@QEAA@XZ 0000000180017f5c     ErrorHandling.obj
 0002:00003f6c       $cppxdata$??1_Sentry_base@?$basic_ostream@DU?$char_traits@D@std@@@std@@QEAA@XZ 0000000180017f6c     ErrorHandling.obj
 0002:00003f6c       $cppxdata$??1_Sentry_base@?$basic_ostream@GU?$char_traits@G@std@@@std@@QEAA@XZ 0000000180017f6c     ErrorHandling.obj
 0002:00003f71       $ip2state$??1_Sentry_base@?$basic_ostream@DU?$char_traits@D@std@@@std@@QEAA@XZ 0000000180017f71     ErrorHandling.obj
 0002:00003f71       $ip2state$??1_Sentry_base@?$basic_ostream@GU?$char_traits@G@std@@@std@@QEAA@XZ 0000000180017f71     ErrorHandling.obj
 0002:00003f74       $unwind$??0sentry@?$basic_ostream@GU?$char_traits@G@std@@@std@@QEAA@AEAV12@@Z 0000000180017f74     ErrorHandling.obj
 0002:00003f8c       $cppxdata$??0sentry@?$basic_ostream@GU?$char_traits@G@std@@@std@@QEAA@AEAV12@@Z 0000000180017f8c     ErrorHandling.obj
 0002:00003f95       $stateUnwindMap$??0sentry@?$basic_ostream@GU?$char_traits@G@std@@@std@@QEAA@AEAV12@@Z 0000000180017f95     ErrorHandling.obj
 0002:00003f9c       $ip2state$??0sentry@?$basic_ostream@DU?$char_traits@D@std@@@std@@QEAA@AEAV12@@Z 0000000180017f9c     ErrorHandling.obj
 0002:00003f9c       $ip2state$??0sentry@?$basic_ostream@GU?$char_traits@G@std@@@std@@QEAA@AEAV12@@Z 0000000180017f9c     ErrorHandling.obj
 0002:00003fa4       $unwind$??1sentry@?$basic_ostream@DU?$char_traits@D@std@@@std@@QEAA@XZ 0000000180017fa4     ErrorHandling.obj
 0002:00003fa4       $unwind$??1sentry@?$basic_ostream@GU?$char_traits@G@std@@@std@@QEAA@XZ 0000000180017fa4     ErrorHandling.obj
 0002:00003fb4       $cppxdata$??1sentry@?$basic_ostream@DU?$char_traits@D@std@@@std@@QEAA@XZ 0000000180017fb4     ErrorHandling.obj
 0002:00003fb4       $cppxdata$??1sentry@?$basic_ostream@GU?$char_traits@G@std@@@std@@QEAA@XZ 0000000180017fb4     ErrorHandling.obj
 0002:00003fbd       $stateUnwindMap$??1sentry@?$basic_ostream@DU?$char_traits@D@std@@@std@@QEAA@XZ 0000000180017fbd     ErrorHandling.obj
 0002:00003fbd       $stateUnwindMap$??1sentry@?$basic_ostream@GU?$char_traits@G@std@@@std@@QEAA@XZ 0000000180017fbd     ErrorHandling.obj
 0002:00003fbd       $stateUnwindMap$?fetch@DatabaseRecord@msi@@QEAAAEAV12@AEAVDatabaseView@2@@Z 0000000180017fbd     MsiDb.obj
 0002:00003fc3       $ip2state$??1sentry@?$basic_ostream@DU?$char_traits@D@std@@@std@@QEAA@XZ 0000000180017fc3     ErrorHandling.obj
 0002:00003fc3       $ip2state$??1sentry@?$basic_ostream@GU?$char_traits@G@std@@@std@@QEAA@XZ 0000000180017fc3     ErrorHandling.obj
 0002:00003fc8       $unwind$??0?$basic_ostringstream@GU?$char_traits@G@std@@V?$allocator@G@2@@std@@QEAA@XZ 0000000180017fc8     ErrorHandling.obj
 0002:00003fdc       $cppxdata$??0?$basic_ostringstream@GU?$char_traits@G@std@@V?$allocator@G@2@@std@@QEAA@XZ 0000000180017fdc     ErrorHandling.obj
 0002:00003fe5       $stateUnwindMap$??0?$basic_ostringstream@GU?$char_traits@G@std@@V?$allocator@G@2@@std@@QEAA@XZ 0000000180017fe5     ErrorHandling.obj
 0002:00003ff0       $ip2state$??0?$basic_ostringstream@DU?$char_traits@D@std@@V?$allocator@D@2@@std@@QEAA@XZ 0000000180017ff0     ErrorHandling.obj
 0002:00003ff0       $ip2state$??0?$basic_ostringstream@GU?$char_traits@G@std@@V?$allocator@G@2@@std@@QEAA@XZ 0000000180017ff0     ErrorHandling.obj
 0002:00003ff8       $unwind$?dtor$0@?0???0?$basic_ostringstream@DU?$char_traits@D@std@@V?$allocator@D@2@@std@@QEAA@XZ@4HA 0000000180017ff8     ErrorHandling.obj
 0002:00003ff8       $unwind$?dtor$0@?0???0?$basic_ostringstream@GU?$char_traits@G@std@@V?$allocator@G@2@@std@@QEAA@XZ@4HA 0000000180017ff8     ErrorHandling.obj
 0002:00003ff8       $unwind$?dtor$0@?0??str@?$basic_stringbuf@DU?$char_traits@D@std@@V?$allocator@D@2@@std@@QEBA?AV?$basic_string@DU?$char_traits@D@std@@V?$allocator@D@2@@2@XZ@4HA 0000000180017ff8     ErrorHandling.obj
 0002:00003ff8       $unwind$?dtor$0@?0??str@?$basic_stringbuf@GU?$char_traits@G@std@@V?$allocator@G@2@@std@@QEBA?AV?$basic_string@GU?$char_traits@G@std@@V?$allocator@G@2@@2@XZ@4HA 0000000180017ff8     ErrorHandling.obj
 0002:00003ff8       $unwind$?dtor$2@?0??combinePath@FileUtils@@YA?AV?$basic_string@GU?$char_traits@G@std@@V?$allocator@G@2@@std@@AEBV23@0@Z@4HA 0000000180017ff8     FileUtils.obj
 0002:00003ff8       $unwind$?dtor$3@?0??combinePath@FileUtils@@YA?AV?$basic_string@GU?$char_traits@G@std@@V?$allocator@G@2@@std@@AEBV23@0@Z@4HA 0000000180017ff8     FileUtils.obj
 0002:00003ff8       $unwind$?dtor$1@?0??toString@Guid@@QEBA?AV?$basic_string@GU?$char_traits@G@std@@V?$allocator@G@2@@std@@H@Z@4HA 0000000180017ff8     Guid.obj
 0002:00003ff8       $unwind$?dtor$0@?0??toUnicodeStringArray@jni@@YA?AV?$vector@V?$basic_string@GU?$char_traits@G@std@@V?$allocator@G@2@@std@@V?$allocator@V?$basic_string@GU?$char_traits@G@std@@V?$allocator@G@2@@std@@@2@@std@@PEAUJNIEnv_@@PEAV_jobjectArray@@@Z@4HA 0000000180017ff8     JniUtils.obj
 0002:00003ff8       $unwind$?dtor$0@?0??fetch@DatabaseView@msi@@QEAA?AVDatabaseRecord@2@XZ@4HA 0000000180017ff8     MsiDb.obj
 0002:00003ff8       $unwind$?dtor$0@?0???0?$basic_ifstream@DU?$char_traits@D@std@@@std@@QEAA@PEBGHH@Z@4HA 0000000180017ff8     ResourceEditor.obj
 0002:00003ff8       $unwind$?dtor$0@?0???0?$basic_stringstream@DU?$char_traits@D@std@@V?$allocator@D@2@@std@@QEAA@H@Z@4HA 0000000180017ff8     VersionInfo.obj
 0002:00003ff8       $unwind$?dtor$0@?0???0?$basic_stringstream@GU?$char_traits@G@std@@V?$allocator@G@2@@std@@QEAA@XZ@4HA 0000000180017ff8     VersionInfo.obj
 0002:00003ff8       $unwind$?dtor$0@?0??getSystemMessageDescription@?A0xd5983087@@YA?AV?$basic_string@GU?$char_traits@G@std@@V?$allocator@G@2@@std@@KPEAUHINSTANCE__@@@Z@4HA 0000000180017ff8     WinErrorHandling.obj
 0002:00003ff8       $unwind$?dtor$0@?0???0?$basic_istringstream@DU?$char_traits@D@std@@V?$allocator@D@2@@std@@QEAA@AEBV?$basic_string@DU?$char_traits@D@std@@V?$allocator@D@2@@1@H@Z@4HA 0000000180017ff8     jpackage.obj
 0002:00003ff8       $unwind$?dtor$0@?0??fromMultiByte@?A0xf04d92fb@tstrings@@YA?AV?$basic_string@GU?$char_traits@G@std@@V?$allocator@G@2@@std@@AEBV?$basic_string@DU?$char_traits@D@std@@V?$allocator@D@2@@4@H@Z@4HA 0000000180017ff8     tstrings.obj
 0002:00003ff8       $unwind$?dtor$0@?0??toLower@tstrings@@YA?AV?$basic_string@GU?$char_traits@G@std@@V?$allocator@G@2@@std@@AEBV23@@Z@4HA 0000000180017ff8     tstrings.obj
 0002:00003ff8       $unwind$?dtor$0@?0??toMultiByte@?A0xf04d92fb@tstrings@@YA?AV?$basic_string@DU?$char_traits@D@std@@V?$allocator@D@2@@std@@AEBV?$basic_string@GU?$char_traits@G@std@@V?$allocator@G@2@@4@H@Z@4HA 0000000180017ff8     tstrings.obj
 0002:00003ff8       $unwind$?dtor$0@?0??unsafe_format@tstrings@@YA?AV?$basic_string@GU?$char_traits@G@std@@V?$allocator@G@2@@std@@PEBGZZ@4HA 0000000180017ff8     tstrings.obj
 0002:00003ff8       $unwind$?fin$0@?0??dllmain_crt_process_attach@@YAHQEAUHINSTANCE__@@QEAX@Z@4HA 0000000180017ff8     MSVCRT:dll_dllmain.obj
 0002:00003ff8       $unwind$?fin$0@?0??dllmain_crt_process_detach@@YAH_N@Z@4HA 0000000180017ff8     MSVCRT:dll_dllmain.obj
 0002:00003ff8       $unwind$?fin$1@?0??dllmain_crt_process_detach@@YAH_N@Z@4HA 0000000180017ff8     MSVCRT:dll_dllmain.obj
 0002:00004000       $unwind$??_G?$basic_ostringstream@DU?$char_traits@D@std@@V?$allocator@D@2@@std@@UEAAPEAXI@Z 0000000180018000     ErrorHandling.obj
 0002:00004000       $unwind$??_G?$basic_ostringstream@GU?$char_traits@G@std@@V?$allocator@G@2@@std@@UEAAPEAXI@Z 0000000180018000     ErrorHandling.obj
 0002:00004000       $unwind$?_Get_buffer_view@?$basic_stringbuf@DU?$char_traits@D@std@@V?$allocator@D@2@@std@@QEBA?AU_Buffer_view@12@XZ 0000000180018000     ErrorHandling.obj
 0002:00004000       $unwind$?_Get_buffer_view@?$basic_stringbuf@GU?$char_traits@G@std@@V?$allocator@G@2@@std@@QEBA?AU_Buffer_view@12@XZ 0000000180018000     ErrorHandling.obj
 0002:00004000       $unwind$?_Tidy@?$basic_stringbuf@DU?$char_traits@D@std@@V?$allocator@D@2@@std@@IEAAXXZ 0000000180018000     ErrorHandling.obj
 0002:00004000       $unwind$?_Tidy@?$basic_stringbuf@GU?$char_traits@G@std@@V?$allocator@G@2@@std@@IEAAXXZ 0000000180018000     ErrorHandling.obj
 0002:00004000       $unwind$?underflow@?$basic_stringbuf@DU?$char_traits@D@std@@V?$allocator@D@2@@std@@MEAAHXZ 0000000180018000     ErrorHandling.obj
 0002:00004000       $unwind$?underflow@?$basic_stringbuf@GU?$char_traits@G@std@@V?$allocator@G@2@@std@@MEAAGXZ 0000000180018000     ErrorHandling.obj
 0002:00004000       $unwind$?_Tidy@?$vector@V?$basic_string@GU?$char_traits@G@std@@V?$allocator@G@2@@std@@V?$allocator@V?$basic_string@GU?$char_traits@G@std@@V?$allocator@G@2@@std@@@2@@std@@AEAAXXZ 0000000180018000     Executor.obj
 0002:00004000       $unwind$??4?$basic_string@GU?$char_traits@G@std@@V?$allocator@G@2@@std@@QEAAAEAV01@AEBV01@@Z 0000000180018000     Guid.obj
 0002:00004000       $unwind$??$_Find_lower_bound@V?$basic_string@GU?$char_traits@G@std@@V?$allocator@G@2@@std@@@?$_Tree@V?$_Tmap_traits@V?$basic_string@GU?$char_traits@G@std@@V?$allocator@G@2@@std@@V12@U?$less@V?$basic_string@GU?$char_traits@G@std@@V?$allocator@G@2@@std@@@2@V?$allocator@U?$pair@$$CBV?$basic_string@GU?$char_traits@G@std@@V?$allocator@G@2@@std@@V12@@std@@@2@$0A@@std@@@std@@IEBA?AU?$_Tree_find_result@PEAU?$_Tree_node@U?$pair@$$CBV?$basic_string@GU?$char_traits@G@std@@V?$allocator@G@2@@std@@V12@@std@@PEAX@std@@@1@AEBV?$basic_string@GU?$char_traits@G@std@@V?$allocator@G@2@@1@@Z 0000000180018000     MsiCA.obj
 0002:00004000       $unwind$?close@?$basic_filebuf@DU?$char_traits@D@std@@@std@@QEAAPEAV12@XZ 0000000180018000     MsiDb.obj
 0002:00004000       $unwind$??$_Resize@U_Value_init_tag@std@@@?$vector@GV?$allocator@G@std@@@std@@AEAAX_KAEBU_Value_init_tag@1@@Z 0000000180018000     MsiUtils.obj
 0002:00004000       $unwind$??$_Resize@U_Value_init_tag@std@@@?$vector@EV?$allocator@E@std@@@std@@AEAAX_KAEBU_Value_init_tag@1@@Z 0000000180018000     ResourceEditor.obj
 0002:00004000       $unwind$??_G?$basic_stringstream@DU?$char_traits@D@std@@V?$allocator@D@2@@std@@UEAAPEAXI@Z 0000000180018000     VersionInfo.obj
 0002:00004000       $unwind$??_G?$basic_stringstream@GU?$char_traits@G@std@@V?$allocator@G@2@@std@@UEAAPEAXI@Z 0000000180018000     VersionInfo.obj
 0002:00004000       $unwind$??_G?$basic_istringstream@DU?$char_traits@D@std@@V?$allocator@D@2@@std@@UEAAPEAXI@Z 0000000180018000     jpackage.obj
 0002:00004000       $unwind$_DllMainCRTStartup 0000000180018000     MSVCRT:dll_dllmain.obj
 0002:00004010       $unwind$?str@?$basic_stringbuf@GU?$char_traits@G@std@@V?$allocator@G@2@@std@@QEBA?AV?$basic_string@GU?$char_traits@G@std@@V?$allocator@G@2@@2@XZ 0000000180018010     ErrorHandling.obj
 0002:0000402c       $cppxdata$?str@?$basic_stringbuf@GU?$char_traits@G@std@@V?$allocator@G@2@@std@@QEBA?AV?$basic_string@GU?$char_traits@G@std@@V?$allocator@G@2@@2@XZ 000000018001802c     ErrorHandling.obj
 0002:00004035       $stateUnwindMap$?str@?$basic_stringbuf@GU?$char_traits@G@std@@V?$allocator@G@2@@std@@QEBA?AV?$basic_string@GU?$char_traits@G@std@@V?$allocator@G@2@@2@XZ 0000000180018035     ErrorHandling.obj
 0002:0000403b       $ip2state$?str@?$basic_stringbuf@DU?$char_traits@D@std@@V?$allocator@D@2@@std@@QEBA?AV?$basic_string@DU?$char_traits@D@std@@V?$allocator@D@2@@2@XZ 000000018001803b     ErrorHandling.obj
 0002:0000403b       $ip2state$?str@?$basic_stringbuf@GU?$char_traits@G@std@@V?$allocator@G@2@@std@@QEBA?AV?$basic_string@GU?$char_traits@G@std@@V?$allocator@G@2@@2@XZ 000000018001803b     ErrorHandling.obj
 0002:00004040       $unwind$?overflow@?$basic_stringbuf@GU?$char_traits@G@std@@V?$allocator@G@2@@std@@MEAAGG@Z 0000000180018040     ErrorHandling.obj
 0002:00004040       $unwind$?seekoff@?$basic_stringbuf@DU?$char_traits@D@std@@V?$allocator@D@2@@std@@MEAA?AV?$fpos@U_Mbstatet@@@2@_JHH@Z 0000000180018040     ErrorHandling.obj
 0002:00004040       $unwind$?seekoff@?$basic_stringbuf@GU?$char_traits@G@std@@V?$allocator@G@2@@std@@MEAA?AV?$fpos@U_Mbstatet@@@2@_JHH@Z 0000000180018040     ErrorHandling.obj
 0002:00004040       $unwind$?seekpos@?$basic_stringbuf@DU?$char_traits@D@std@@V?$allocator@D@2@@std@@MEAA?AV?$fpos@U_Mbstatet@@@2@V32@H@Z 0000000180018040     ErrorHandling.obj
 0002:00004040       $unwind$?seekpos@?$basic_stringbuf@GU?$char_traits@G@std@@V?$allocator@G@2@@std@@MEAA?AV?$fpos@U_Mbstatet@@@2@V32@H@Z 0000000180018040     ErrorHandling.obj
 0002:00004040       $unwind$??0?$basic_string@GU?$char_traits@G@std@@V?$allocator@G@2@@std@@QEAA@U_String_constructor_concat_tag@1@AEBV01@QEBG_K23@Z 0000000180018040     Executor.obj
 0002:00004040       $unwind$??$_Reallocate_grow_by@V<lambda_1>@?1??append@?$basic_string@GU?$char_traits@G@std@@V?$allocator@G@2@@std@@QEAAAEAV34@QEBG_K@Z@PEBG_K@?$basic_string@GU?$char_traits@G@std@@V?$allocator@G@2@@std@@AEAAAEAV01@_KV<lambda_1>@?1??append@01@QEAAAEAV01@QEBG0@Z@PEBG_K@Z 0000000180018040     FileUtils.obj
 0002:00004040       $unwind$??$_Reallocate_grow_by@V<lambda_1>@?1??append@?$basic_string@GU?$char_traits@G@std@@V?$allocator@G@2@@std@@QEAAAEAV34@_KG@Z@_KG@?$basic_string@GU?$char_traits@G@std@@V?$allocator@G@2@@std@@AEAAAEAV01@_KV<lambda_1>@?1??append@01@QEAAAEAV01@0G@Z@_KG@Z 0000000180018040     FileUtils.obj
 0002:00004040       $unwind$??$_Reallocate_grow_by@V<lambda_1>@?1??append@?$basic_string@DU?$char_traits@D@std@@V?$allocator@D@2@@std@@QEAAAEAV34@_KD@Z@_KD@?$basic_string@DU?$char_traits@D@std@@V?$allocator@D@2@@std@@AEAAAEAV01@_KV<lambda_1>@?1??append@01@QEAAAEAV01@0D@Z@_KD@Z 0000000180018040     tstrings.obj
 0002:0000405c       $unwind$??$_Construct@$00PEBD@?$basic_string@DU?$char_traits@D@std@@V?$allocator@D@2@@std@@AEAAXQEBD_K@Z 000000018001805c     ErrorHandling.obj
 0002:0000405c       $unwind$?pbackfail@?$basic_stringbuf@GU?$char_traits@G@std@@V?$allocator@G@2@@std@@MEAAGG@Z 000000018001805c     ErrorHandling.obj
 0002:0000405c       $unwind$??$_Erase_tree@V?$allocator@U?$_Tree_node@U?$pair@$$CBV?$basic_string@GU?$char_traits@G@std@@V?$allocator@G@2@@std@@V12@@std@@PEAX@std@@@std@@@?$_Tree_val@U?$_Tree_simple_types@U?$pair@$$CBV?$basic_string@GU?$char_traits@G@std@@V?$allocator@G@2@@std@@V12@@std@@@std@@@std@@QEAAXAEAV?$allocator@U?$_Tree_node@U?$pair@$$CBV?$basic_string@GU?$char_traits@G@std@@V?$allocator@G@2@@std@@V12@@std@@PEAX@std@@@1@PEAU?$_Tree_node@U?$pair@$$CBV?$basic_string@GU?$char_traits@G@std@@V?$allocator@G@2@@std@@V12@@std@@PEAX@1@@Z 000000018001805c     MsiCA.obj
 0002:0000405c       $unwind$?xsgetn@?$basic_filebuf@DU?$char_traits@D@std@@@std@@MEAA_JPEAD_J@Z 000000018001805c     MsiDb.obj
 0002:0000405c       $unwind$?_Init@?$basic_stringbuf@DU?$char_traits@D@std@@V?$allocator@D@2@@std@@IEAAXPEBD_KH@Z 000000018001805c     jpackage.obj
 0002:0000405c       $unwind$__GSHandlerCheck_EH4 000000018001805c     MSVCRT:gshandlereh4.obj
 0002:00004074       $unwind$??$?6GU?$char_traits@G@std@@@std@@YAAEAV?$basic_ostream@GU?$char_traits@G@std@@@0@AEAV10@PEBG@Z 0000000180018074     ErrorHandling.obj
 0002:00004094       $cppxdata$??$?6GU?$char_traits@G@std@@@std@@YAAEAV?$basic_ostream@GU?$char_traits@G@std@@@0@AEAV10@PEBG@Z 0000000180018094     ErrorHandling.obj
 0002:000040a1       $stateUnwindMap$??$?6GU?$char_traits@G@std@@@std@@YAAEAV?$basic_ostream@GU?$char_traits@G@std@@@0@AEAV10@PEBG@Z 00000001800180a1     ErrorHandling.obj
 0002:000040a1       $stateUnwindMap$??$_Insert_string@GU?$char_traits@G@std@@_K@std@@YAAEAV?$basic_ostream@GU?$char_traits@G@std@@@0@AEAV10@QEBG_K@Z 00000001800180a1     ErrorHandling.obj
 0002:000040a1       $stateUnwindMap$??6?$basic_ostream@GU?$char_traits@G@std@@@std@@QEAAAEAV01@G@Z 00000001800180a1     Log.obj
 0002:000040af       $tryMap$??$?6GU?$char_traits@G@std@@@std@@YAAEAV?$basic_ostream@GU?$char_traits@G@std@@@0@AEAV10@PEBG@Z 00000001800180af     ErrorHandling.obj
 0002:000040b7       $handlerMap$??$?6GU?$char_traits@G@std@@@std@@YAAEAV?$basic_ostream@GU?$char_traits@G@std@@@0@AEAV10@PEBG@Z 00000001800180b7     ErrorHandling.obj
 0002:000040c0       $ip2state$??$?6GU?$char_traits@G@std@@@std@@YAAEAV?$basic_ostream@GU?$char_traits@G@std@@@0@AEAV10@PEBG@Z 00000001800180c0     ErrorHandling.obj
 0002:000040d0       $unwind$?catch$3@?0???$?6GU?$char_traits@G@std@@@std@@YAAEAV?$basic_ostream@GU?$char_traits@G@std@@@0@AEAV10@PEBG@Z@4HA 00000001800180d0     ErrorHandling.obj
 0002:000040d0       $unwind$?catch$3@?0???$?6U?$char_traits@D@std@@@std@@YAAEAV?$basic_ostream@DU?$char_traits@D@std@@@0@AEAV10@PEBD@Z@4HA 00000001800180d0     ErrorHandling.obj
 0002:000040d0       $unwind$?catch$3@?0???$_Insert_string@DU?$char_traits@D@std@@_K@std@@YAAEAV?$basic_ostream@DU?$char_traits@D@std@@@0@AEAV10@QEBD_K@Z@4HA 00000001800180d0     ErrorHandling.obj
 0002:000040d0       $unwind$?catch$3@?0???$_Insert_string@GU?$char_traits@G@std@@_K@std@@YAAEAV?$basic_ostream@GU?$char_traits@G@std@@@0@AEAV10@QEBG_K@Z@4HA 00000001800180d0     ErrorHandling.obj
 0002:000040d0       $unwind$?catch$4@?0???$?6GU?$char_traits@G@std@@@std@@YAAEAV?$basic_ostream@GU?$char_traits@G@std@@@0@AEAV10@PEBD@Z@4HA 00000001800180d0     ErrorHandling.obj
 0002:000040d0       $unwind$?catch$3@?0???$_Emplace_reallocate@V?$basic_string@GU?$char_traits@G@std@@V?$allocator@G@2@@std@@@?$vector@V?$basic_string@GU?$char_traits@G@std@@V?$allocator@G@2@@std@@V?$allocator@V?$basic_string@GU?$char_traits@G@std@@V?$allocator@G@2@@std@@@2@@std@@AEAAPEAV?$basic_string@GU?$char_traits@G@std@@V?$allocator@G@2@@1@QEAV21@$$QEAV21@@Z@4HA 00000001800180d0     JniUtils.obj
 0002:000040d0       $unwind$?catch$3@?0???6?$basic_ostream@GU?$char_traits@G@std@@@std@@QEAAAEAV01@G@Z@4HA 00000001800180d0     Log.obj
 0002:000040d0       $unwind$?catch$0@?0???$_Resize_reallocate@U_Value_init_tag@std@@@?$vector@GV?$allocator@G@std@@@std@@AEAAX_KAEBU_Value_init_tag@1@@Z@4HA 00000001800180d0     MsiUtils.obj
 0002:000040d0       $unwind$?catch$0@?0???$_Emplace_reallocate@D@?$vector@EV?$allocator@E@std@@@std@@AEAAPEAEQEAE$$QEAD@Z@4HA 00000001800180d0     ResourceEditor.obj
 0002:000040d0       $unwind$?catch$0@?0???$_Resize_reallocate@U_Value_init_tag@std@@@?$vector@EV?$allocator@E@std@@@std@@AEAAX_KAEBU_Value_init_tag@1@@Z@4HA 00000001800180d0     ResourceEditor.obj
 0002:000040d0       $unwind$?catch$8@?0??createFIXEDFILEINFO@VersionInfo@@AEBA?AUtagVS_FIXEDFILEINFO@@XZ@4HA 00000001800180d0     VersionInfo.obj
 0002:000040d0       $unwind$Java_jdk_jpackage_internal_WindowsRegistry_comparePaths$catch$12 00000001800180d0     WindowsRegistry.obj
 0002:000040d0       $unwind$Java_jdk_jpackage_internal_WindowsRegistry_comparePaths$catch$13 00000001800180d0     WindowsRegistry.obj
 0002:000040d0       $unwind$Java_jdk_jpackage_internal_ExecutableRebrander_iconSwap$catch$4 00000001800180d0     jpackage.obj
 0002:000040d0       $unwind$Java_jdk_jpackage_internal_ExecutableRebrander_iconSwap$catch$5 00000001800180d0     jpackage.obj
 0002:000040d0       $unwind$Java_jdk_jpackage_internal_ExecutableRebrander_lockResource$catch$3 00000001800180d0     jpackage.obj
 0002:000040d0       $unwind$Java_jdk_jpackage_internal_ExecutableRebrander_lockResource$catch$4 00000001800180d0     jpackage.obj
 0002:000040d0       $unwind$Java_jdk_jpackage_internal_ExecutableRebrander_unlockResource$catch$1 00000001800180d0     jpackage.obj
 0002:000040d0       $unwind$Java_jdk_jpackage_internal_ExecutableRebrander_unlockResource$catch$2 00000001800180d0     jpackage.obj
 0002:000040d0       $unwind$Java_jdk_jpackage_internal_ExecutableRebrander_versionSwap$catch$13 00000001800180d0     jpackage.obj
 0002:000040d0       $unwind$Java_jdk_jpackage_internal_ExecutableRebrander_versionSwap$catch$14 00000001800180d0     jpackage.obj
 0002:000040d0       $unwind$Java_jdk_jpackage_internal_ShortPathUtils_getShortPath$catch$4 00000001800180d0     jpackage.obj
 0002:000040d0       $unwind$Java_jdk_jpackage_internal_ShortPathUtils_getShortPath$catch$5 00000001800180d0     jpackage.obj
 0002:000040d0       $unwind$Java_jdk_jpackage_internal_WinExeBundler_embedMSI$catch$25 00000001800180d0     jpackage.obj
 0002:000040d0       $unwind$Java_jdk_jpackage_internal_WinExeBundler_embedMSI$catch$26 00000001800180d0     jpackage.obj
 0002:000040d8       $unwind$??6@YAAEAV?$basic_ostream@DU?$char_traits@D@std@@@std@@AEAV01@AEBVany@tstrings@@@Z 00000001800180d8     ErrorHandling.obj
 0002:000040ec       $cppxdata$??6@YAAEAV?$basic_ostream@DU?$char_traits@D@std@@@std@@AEAV01@AEBVany@tstrings@@@Z 00000001800180ec     ErrorHandling.obj
 0002:000040f5       $stateUnwindMap$??6@YAAEAV?$basic_ostream@DU?$char_traits@D@std@@@std@@AEAV01@AEBVany@tstrings@@@Z 00000001800180f5     ErrorHandling.obj
 0002:00004102       $ip2state$??6@YAAEAV?$basic_ostream@DU?$char_traits@D@std@@@std@@AEAV01@AEBVany@tstrings@@@Z 0000000180018102     ErrorHandling.obj
 0002:0000410c       $unwind$?reportError@@YAXAEBUSourceCodePos@@AEBVruntime_error@std@@@Z 000000018001810c     ErrorHandling.obj
 0002:00004128       $cppxdata$?reportError@@YAXAEBUSourceCodePos@@AEBVruntime_error@std@@@Z 0000000180018128     ErrorHandling.obj
 0002:00004131       $stateUnwindMap$?reportError@@YAXAEBUSourceCodePos@@AEBVruntime_error@std@@@Z 0000000180018131     ErrorHandling.obj
 0002:0000413f       $ip2state$?reportError@@YAXAEBUSourceCodePos@@AEBVruntime_error@std@@@Z 000000018001813f     ErrorHandling.obj
 0002:0000414c       $unwind$?reportUnknownError@@YAXAEBUSourceCodePos@@@Z 000000018001814c     ErrorHandling.obj
 0002:00004160       $cppxdata$?reportUnknownError@@YAXAEBUSourceCodePos@@@Z 0000000180018160     ErrorHandling.obj
 0002:00004169       $stateUnwindMap$?reportUnknownError@@YAXAEBUSourceCodePos@@@Z 0000000180018169     ErrorHandling.obj
 0002:00004169       $stateUnwindMap$?initializeLogging@Logger@@CAXXZ 0000000180018169     PlatformLogEvent.obj
 0002:00004170       $ip2state$?reportUnknownError@@YAXAEBUSourceCodePos@@@Z 0000000180018170     ErrorHandling.obj
 0002:00004178       $unwind$?makeMessage@@YA?AV?$basic_string@DU?$char_traits@D@std@@V?$allocator@D@2@@std@@AEBVruntime_error@2@AEBUSourceCodePos@@@Z 0000000180018178     ErrorHandling.obj
 0002:00004198       $cppxdata$?makeMessage@@YA?AV?$basic_string@DU?$char_traits@D@std@@V?$allocator@D@2@@std@@AEBVruntime_error@2@AEBUSourceCodePos@@@Z 0000000180018198     ErrorHandling.obj
 0002:000041a1       $stateUnwindMap$?makeMessage@@YA?AV?$basic_string@DU?$char_traits@D@std@@V?$allocator@D@2@@std@@AEBVruntime_error@2@AEBUSourceCodePos@@@Z 00000001800181a1     ErrorHandling.obj
 0002:000041bc       $ip2state$?makeMessage@@YA?AV?$basic_string@DU?$char_traits@D@std@@V?$allocator@D@2@@std@@AEBVruntime_error@2@AEBUSourceCodePos@@@Z 00000001800181bc     ErrorHandling.obj
 0002:000041d0       $unwind$?joinErrorMessages@@YA?AV?$basic_string@DU?$char_traits@D@std@@V?$allocator@D@2@@std@@AEBV12@0@Z 00000001800181d0     ErrorHandling.obj
 0002:000041f8       $cppxdata$?joinErrorMessages@@YA?AV?$basic_string@DU?$char_traits@D@std@@V?$allocator@D@2@@std@@AEBV12@0@Z 00000001800181f8     ErrorHandling.obj
 0002:00004201       $stateUnwindMap$?joinErrorMessages@@YA?AV?$basic_string@DU?$char_traits@D@std@@V?$allocator@D@2@@std@@AEBV12@0@Z 0000000180018201     ErrorHandling.obj
 0002:00004224       $ip2state$?joinErrorMessages@@YA?AV?$basic_string@DU?$char_traits@D@std@@V?$allocator@D@2@@std@@AEBV12@0@Z 0000000180018224     ErrorHandling.obj
 0002:0000423c       $unwind$?getFilename@?A0xd1a094c7@@YA?AV?$basic_string@GU?$char_traits@G@std@@V?$allocator@G@2@@std@@AEBUSourceCodePos@@@Z 000000018001823c     ErrorHandling.obj
 0002:0000425c       $cppxdata$?getFilename@?A0xd1a094c7@@YA?AV?$basic_string@GU?$char_traits@G@std@@V?$allocator@G@2@@std@@AEBUSourceCodePos@@@Z 000000018001825c     ErrorHandling.obj
 0002:00004265       $stateUnwindMap$?getFilename@?A0xd1a094c7@@YA?AV?$basic_string@GU?$char_traits@G@std@@V?$allocator@G@2@@std@@AEBUSourceCodePos@@@Z 0000000180018265     ErrorHandling.obj
 0002:00004272       $ip2state$?getFilename@?A0xd1a094c7@@YA?AV?$basic_string@GU?$char_traits@G@std@@V?$allocator@G@2@@std@@AEBUSourceCodePos@@@Z 0000000180018272     ErrorHandling.obj
 0002:00004284       $unwind$?reportError@?A0xd1a094c7@@YAXAEBUSourceCodePos@@AEBV?$basic_string@GU?$char_traits@G@std@@V?$allocator@G@2@@std@@@Z 0000000180018284     ErrorHandling.obj
 0002:000042a8       $cppxdata$?reportError@?A0xd1a094c7@@YAXAEBUSourceCodePos@@AEBV?$basic_string@GU?$char_traits@G@std@@V?$allocator@G@2@@std@@@Z 00000001800182a8     ErrorHandling.obj
 0002:000042b1       $stateUnwindMap$?reportError@?A0xd1a094c7@@YAXAEBUSourceCodePos@@AEBV?$basic_string@GU?$char_traits@G@std@@V?$allocator@G@2@@std@@@Z 00000001800182b1     ErrorHandling.obj
 0002:000042c4       $ip2state$?reportError@?A0xd1a094c7@@YAXAEBUSourceCodePos@@AEBV?$basic_string@GU?$char_traits@G@std@@V?$allocator@G@2@@std@@@Z 00000001800182c4     ErrorHandling.obj
 0002:000042d4       $unwind$??0?$basic_ostringstream@DU?$char_traits@D@std@@V?$allocator@D@2@@std@@QEAA@XZ 00000001800182d4     ErrorHandling.obj
 0002:000042e8       $cppxdata$??0?$basic_ostringstream@DU?$char_traits@D@std@@V?$allocator@D@2@@std@@QEAA@XZ 00000001800182e8     ErrorHandling.obj
 0002:000042f1       $stateUnwindMap$??0?$basic_ostringstream@DU?$char_traits@D@std@@V?$allocator@D@2@@std@@QEAA@XZ 00000001800182f1     ErrorHandling.obj
 0002:000042fc       $unwind$?str@?$basic_stringbuf@DU?$char_traits@D@std@@V?$allocator@D@2@@std@@QEBA?AV?$basic_string@DU?$char_traits@D@std@@V?$allocator@D@2@@2@XZ 00000001800182fc     ErrorHandling.obj
 0002:00004314       $cppxdata$?str@?$basic_stringbuf@DU?$char_traits@D@std@@V?$allocator@D@2@@std@@QEBA?AV?$basic_string@DU?$char_traits@D@std@@V?$allocator@D@2@@2@XZ 0000000180018314     ErrorHandling.obj
 0002:0000431d       $stateUnwindMap$?str@?$basic_stringbuf@DU?$char_traits@D@std@@V?$allocator@D@2@@std@@QEBA?AV?$basic_string@DU?$char_traits@D@std@@V?$allocator@D@2@@2@XZ 000000018001831d     ErrorHandling.obj
 0002:00004324       $unwind$?overflow@?$basic_stringbuf@DU?$char_traits@D@std@@V?$allocator@D@2@@std@@MEAAHH@Z 0000000180018324     ErrorHandling.obj
 0002:0000433c       $unwind$?pbackfail@?$basic_stringbuf@DU?$char_traits@D@std@@V?$allocator@D@2@@std@@MEAAHH@Z 000000018001833c     ErrorHandling.obj
 0002:0000433c       $unwind$?pbackfail@?$basic_filebuf@DU?$char_traits@D@std@@@std@@MEAAHH@Z 000000018001833c     MsiDb.obj
 0002:00004350       $unwind$??$?6U?$char_traits@D@std@@@std@@YAAEAV?$basic_ostream@DU?$char_traits@D@std@@@0@AEAV10@PEBD@Z 0000000180018350     ErrorHandling.obj
 0002:0000436c       $cppxdata$??$?6U?$char_traits@D@std@@@std@@YAAEAV?$basic_ostream@DU?$char_traits@D@std@@@0@AEAV10@PEBD@Z 000000018001836c     ErrorHandling.obj
 0002:00004379       $stateUnwindMap$??$?6U?$char_traits@D@std@@@std@@YAAEAV?$basic_ostream@DU?$char_traits@D@std@@@0@AEAV10@PEBD@Z 0000000180018379     ErrorHandling.obj
 0002:00004379       $stateUnwindMap$??$_Insert_string@DU?$char_traits@D@std@@_K@std@@YAAEAV?$basic_ostream@DU?$char_traits@D@std@@@0@AEAV10@QEBD_K@Z 0000000180018379     ErrorHandling.obj
 0002:00004387       $tryMap$??$?6U?$char_traits@D@std@@@std@@YAAEAV?$basic_ostream@DU?$char_traits@D@std@@@0@AEAV10@PEBD@Z 0000000180018387     ErrorHandling.obj
 0002:0000438f       $handlerMap$??$?6U?$char_traits@D@std@@@std@@YAAEAV?$basic_ostream@DU?$char_traits@D@std@@@0@AEAV10@PEBD@Z 000000018001838f     ErrorHandling.obj
 0002:00004398       $ip2state$??$?6U?$char_traits@D@std@@@std@@YAAEAV?$basic_ostream@DU?$char_traits@D@std@@@0@AEAV10@PEBD@Z 0000000180018398     ErrorHandling.obj
 0002:000043a4       $unwind$??$_Construct@$00PEBG@?$basic_string@GU?$char_traits@G@std@@V?$allocator@G@2@@std@@AEAAXQEBG_K@Z 00000001800183a4     ErrorHandling.obj
 0002:000043a4       $unwind$??$_Reallocate_for@V<lambda_1>@?1??assign@?$basic_string@DU?$char_traits@D@std@@V?$allocator@D@2@@std@@QEAAAEAV34@QEBD_K@Z@PEBD@?$basic_string@DU?$char_traits@D@std@@V?$allocator@D@2@@std@@AEAAAEAV01@_KV<lambda_1>@?1??assign@01@QEAAAEAV01@QEBD0@Z@PEBD@Z 00000001800183a4     ErrorHandling.obj
 0002:000043a4       $unwind$?printWithoutWhitespaces@?A0xd1a094c7@@YA_KAEAV?$basic_ostream@DU?$char_traits@D@std@@@std@@AEBV?$basic_string@DU?$char_traits@D@std@@V?$allocator@D@2@@3@W4TrimMode@1@@Z 00000001800183a4     ErrorHandling.obj
 0002:000043a4       $unwind$??$_Uninitialized_move@PEAV?$basic_string@GU?$char_traits@G@std@@V?$allocator@G@2@@std@@V?$allocator@V?$basic_string@GU?$char_traits@G@std@@V?$allocator@G@2@@std@@@2@@std@@YAPEAV?$basic_string@GU?$char_traits@G@std@@V?$allocator@G@2@@0@QEAV10@0PEAV10@AEAV?$allocator@V?$basic_string@GU?$char_traits@G@std@@V?$allocator@G@2@@std@@@0@@Z 00000001800183a4     Executor.obj
 0002:000043a4       $unwind$?_Change_array@?$vector@V?$basic_string@GU?$char_traits@G@std@@V?$allocator@G@2@@std@@V?$allocator@V?$basic_string@GU?$char_traits@G@std@@V?$allocator@G@2@@std@@@2@@std@@AEAAXQEAV?$basic_string@GU?$char_traits@G@std@@V?$allocator@G@2@@2@_K1@Z 00000001800183a4     Executor.obj
 0002:000043a4       $unwind$??$_Construct@$00PEAG@?$basic_string@GU?$char_traits@G@std@@V?$allocator@G@2@@std@@AEAAXQEAG_K@Z 00000001800183a4     Guid.obj
 0002:000043a4       $unwind$??R<lambda_1>@?1??insert@?$basic_string@GU?$char_traits@G@std@@V?$allocator@G@2@@std@@QEAAAEAV23@_K0G@Z@QEBA@QEAGQEBG000G@Z 00000001800183a4     Guid.obj
 0002:000043bc       $unwind$??0sentry@?$basic_ostream@DU?$char_traits@D@std@@@std@@QEAA@AEAV12@@Z 00000001800183bc     ErrorHandling.obj
 0002:000043d4       $cppxdata$??0sentry@?$basic_ostream@DU?$char_traits@D@std@@@std@@QEAA@AEAV12@@Z 00000001800183d4     ErrorHandling.obj
 0002:000043dd       $stateUnwindMap$??0sentry@?$basic_ostream@DU?$char_traits@D@std@@@std@@QEAA@AEAV12@@Z 00000001800183dd     ErrorHandling.obj
 0002:000043e4       $unwind$??$_Traits_find_last_of@U?$char_traits@D@std@@$00@std@@YA_KQEBD_K101@Z 00000001800183e4     ErrorHandling.obj
 0002:00004400       $unwind$??$_Construct@$01PEBD@?$basic_string@DU?$char_traits@D@std@@V?$allocator@D@2@@std@@AEAAXQEBD_K@Z 0000000180018400     ErrorHandling.obj
 0002:00004400       $unwind$??$_Construct@$01PEBG@?$basic_string@GU?$char_traits@G@std@@V?$allocator@G@2@@std@@AEAAXQEBG_K@Z 0000000180018400     Executor.obj
 0002:00004400       $unwind$?_Change_array@?$vector@GV?$allocator@G@std@@@std@@AEAAXQEAG_K1@Z 0000000180018400     Executor.obj
 0002:00004400       $unwind$?assign@?$basic_string@GU?$char_traits@G@std@@V?$allocator@G@2@@std@@QEAAAEAV12@QEBG@Z 0000000180018400     Log.obj
 0002:00004400       $unwind$?_Change_array@?$vector@EV?$allocator@E@std@@@std@@AEAAXQEAE_K1@Z 0000000180018400     ResourceEditor.obj
 0002:00004400       $unwind$__scrt_dllmain_exception_filter 0000000180018400     MSVCRT:utility.obj
 0002:00004414       $unwind$??$use_facet@V?$ctype@G@std@@@std@@YAAEBV?$ctype@G@0@AEBVlocale@0@@Z 0000000180018414     ErrorHandling.obj
 0002:00004414       $unwind$??$use_facet@V?$codecvt@DDU_Mbstatet@@@std@@@std@@YAAEBV?$codecvt@DDU_Mbstatet@@@0@AEBVlocale@0@@Z 0000000180018414     MsiDb.obj
 0002:0000442c       $cppxdata$??$use_facet@V?$ctype@G@std@@@std@@YAAEBV?$ctype@G@0@AEBVlocale@0@@Z 000000018001842c     ErrorHandling.obj
 0002:0000442c       $cppxdata$??$use_facet@V?$codecvt@DDU_Mbstatet@@@std@@@std@@YAAEBV?$codecvt@DDU_Mbstatet@@@0@AEBVlocale@0@@Z 000000018001842c     MsiDb.obj
 0002:00004435       $stateUnwindMap$??$use_facet@V?$ctype@G@std@@@std@@YAAEBV?$ctype@G@0@AEBVlocale@0@@Z 0000000180018435     ErrorHandling.obj
 0002:00004435       $stateUnwindMap$??$use_facet@V?$codecvt@DDU_Mbstatet@@@std@@@std@@YAAEBV?$codecvt@DDU_Mbstatet@@@0@AEBVlocale@0@@Z 0000000180018435     MsiDb.obj
 0002:00004442       $ip2state$??$use_facet@V?$ctype@G@std@@@std@@YAAEBV?$ctype@G@0@AEBVlocale@0@@Z 0000000180018442     ErrorHandling.obj
 0002:00004442       $ip2state$??$use_facet@V?$codecvt@DDU_Mbstatet@@@std@@@std@@YAAEBV?$codecvt@DDU_Mbstatet@@@0@AEBVlocale@0@@Z 0000000180018442     MsiDb.obj
 0002:0000444c       $unwind$??$_Reallocate_for@V<lambda_1>@?1??assign@?$basic_string@GU?$char_traits@G@std@@V?$allocator@G@2@@std@@QEAAAEAV34@QEBG_K@Z@PEBG@?$basic_string@GU?$char_traits@G@std@@V?$allocator@G@2@@std@@AEAAAEAV01@_KV<lambda_1>@?1??assign@01@QEAAAEAV01@QEBG0@Z@PEBG@Z 000000018001844c     ErrorHandling.obj
 0002:0000444c       $unwind$??$_Reallocate_grow_by@V<lambda_1>@?1??push_back@?$basic_string@DU?$char_traits@D@std@@V?$allocator@D@2@@std@@QEAAXD@Z@D@?$basic_string@DU?$char_traits@D@std@@V?$allocator@D@2@@std@@AEAAAEAV01@_KV<lambda_1>@?1??push_back@01@QEAAXD@Z@D@Z 000000018001844c     MsiDb.obj
 0002:0000444c       $unwind$??0?$basic_string@DU?$char_traits@D@std@@V?$allocator@D@2@@std@@QEAA@U_String_constructor_concat_tag@1@AEBV01@QEBD_K23@Z 000000018001844c     WinSysInfo.obj
 0002:00004468       $unwind$??$_Insert_string@GU?$char_traits@G@std@@_K@std@@YAAEAV?$basic_ostream@GU?$char_traits@G@std@@@0@AEAV10@QEBG_K@Z 0000000180018468     ErrorHandling.obj
 0002:00004488       $cppxdata$??$_Insert_string@GU?$char_traits@G@std@@_K@std@@YAAEAV?$basic_ostream@GU?$char_traits@G@std@@@0@AEAV10@QEBG_K@Z 0000000180018488     ErrorHandling.obj
 0002:00004495       $tryMap$??$_Insert_string@GU?$char_traits@G@std@@_K@std@@YAAEAV?$basic_ostream@GU?$char_traits@G@std@@@0@AEAV10@QEBG_K@Z 0000000180018495     ErrorHandling.obj
 0002:0000449d       $handlerMap$??$_Insert_string@GU?$char_traits@G@std@@_K@std@@YAAEAV?$basic_ostream@GU?$char_traits@G@std@@@0@AEAV10@QEBG_K@Z 000000018001849d     ErrorHandling.obj
 0002:000044a6       $ip2state$??$_Insert_string@GU?$char_traits@G@std@@_K@std@@YAAEAV?$basic_ostream@GU?$char_traits@G@std@@@0@AEAV10@QEBG_K@Z 00000001800184a6     ErrorHandling.obj
 0002:000044b4       $unwind$??$_Insert_string@DU?$char_traits@D@std@@_K@std@@YAAEAV?$basic_ostream@DU?$char_traits@D@std@@@0@AEAV10@QEBD_K@Z 00000001800184b4     ErrorHandling.obj
 0002:000044d0       $cppxdata$??$_Insert_string@DU?$char_traits@D@std@@_K@std@@YAAEAV?$basic_ostream@DU?$char_traits@D@std@@@0@AEAV10@QEBD_K@Z 00000001800184d0     ErrorHandling.obj
 0002:000044dd       $tryMap$??$_Insert_string@DU?$char_traits@D@std@@_K@std@@YAAEAV?$basic_ostream@DU?$char_traits@D@std@@@0@AEAV10@QEBD_K@Z 00000001800184dd     ErrorHandling.obj
 0002:000044e5       $handlerMap$??$_Insert_string@DU?$char_traits@D@std@@_K@std@@YAAEAV?$basic_ostream@DU?$char_traits@D@std@@@0@AEAV10@QEBD_K@Z 00000001800184e5     ErrorHandling.obj
 0002:000044ee       $ip2state$??$_Insert_string@DU?$char_traits@D@std@@_K@std@@YAAEAV?$basic_ostream@DU?$char_traits@D@std@@@0@AEAV10@QEBD_K@Z 00000001800184ee     ErrorHandling.obj
 0002:000044fc       $unwind$??$?6GU?$char_traits@G@std@@@std@@YAAEAV?$basic_ostream@GU?$char_traits@G@std@@@0@AEAV10@PEBD@Z 00000001800184fc     ErrorHandling.obj
 0002:00004518       $cppxdata$??$?6GU?$char_traits@G@std@@@std@@YAAEAV?$basic_ostream@GU?$char_traits@G@std@@@0@AEAV10@PEBD@Z 0000000180018518     ErrorHandling.obj
 0002:00004525       $stateUnwindMap$??$?6GU?$char_traits@G@std@@@std@@YAAEAV?$basic_ostream@GU?$char_traits@G@std@@@0@AEAV10@PEBD@Z 0000000180018525     ErrorHandling.obj
 0002:00004539       $tryMap$??$?6GU?$char_traits@G@std@@@std@@YAAEAV?$basic_ostream@GU?$char_traits@G@std@@@0@AEAV10@PEBD@Z 0000000180018539     ErrorHandling.obj
 0002:00004541       $handlerMap$??$?6GU?$char_traits@G@std@@@std@@YAAEAV?$basic_ostream@GU?$char_traits@G@std@@@0@AEAV10@PEBD@Z 0000000180018541     ErrorHandling.obj
 0002:0000454a       $ip2state$??$?6GU?$char_traits@G@std@@@std@@YAAEAV?$basic_ostream@GU?$char_traits@G@std@@@0@AEAV10@PEBD@Z 000000018001854a     ErrorHandling.obj
 0002:0000455c       $unwind$wmemchr            000000018001855c     Executor.obj
 0002:00004568       $unwind$??0any@tstrings@@QEAA@PEBD@Z 0000000180018568     Executor.obj
 0002:00004584       $cppxdata$??0any@tstrings@@QEAA@PEBD@Z 0000000180018584     Executor.obj
 0002:0000458d       $stateUnwindMap$??0any@tstrings@@QEAA@PEBD@Z 000000018001858d     Executor.obj
 0002:000045a0       $ip2state$??0any@tstrings@@QEAA@PEBD@Z 00000001800185a0     Executor.obj
 0002:000045ac       $unwind$?log@Logger@@QEBAXW4LogLevel@1@PEBGH1AEBVany@tstrings@@@Z 00000001800185ac     Executor.obj
 0002:000045c8       $cppxdata$?log@Logger@@QEBAXW4LogLevel@1@PEBGH1AEBVany@tstrings@@@Z 00000001800185c8     Executor.obj
 0002:000045d1       $stateUnwindMap$?log@Logger@@QEBAXW4LogLevel@1@PEBGH1AEBVany@tstrings@@@Z 00000001800185d1     Executor.obj
 0002:000045d8       $ip2state$?log@Logger@@QEBAXW4LogLevel@1@PEBGH1AEBVany@tstrings@@@Z 00000001800185d8     Executor.obj
 0002:000045e0       $unwind$??$makeException@VSysError@@@@YA?AV?$JpError@VSysError@@@@AEBVSysError@@AEBUSourceCodePos@@@Z 00000001800185e0     Executor.obj
 0002:000045e0       $unwind$?removeTrailingSlash@FileUtils@@YA?AV?$basic_string@GU?$char_traits@G@std@@V?$allocator@G@2@@std@@AEBV23@@Z 00000001800185e0     FileUtils.obj
 0002:000045e0       $unwind$??$makeException@VError@msi@@@@YA?AV?$JpError@VError@msi@@@@AEBVError@msi@@AEBUSourceCodePos@@@Z 00000001800185e0     MsiCA.obj
 0002:000045e0       $unwind$??$makeException@VNoMoreItemsError@msi@@@@YA?AV?$JpError@VNoMoreItemsError@msi@@@@AEBVNoMoreItemsError@msi@@AEBUSourceCodePos@@@Z 00000001800185e0     MsiDb.obj
 0002:000045e0       $unwind$?getCurrentModulePath@SysInfo@@YA?AV?$basic_string@GU?$char_traits@G@std@@V?$allocator@G@2@@std@@XZ 00000001800185e0     WinSysInfo.obj
 0002:000045e0       $unwind$?lastErrorMsg@app@@YA?AV?$basic_string@DU?$char_traits@D@std@@V?$allocator@D@2@@std@@XZ 00000001800185e0     app.obj
 0002:000045e0       $unwind$??0invalid_argument@std@@QEAA@PEBD@Z 00000001800185e0     tstrings.obj
 0002:000045e0       $unwind$?toUtf16@tstrings@@YA?AV?$basic_string@GU?$char_traits@G@std@@V?$allocator@G@2@@std@@AEBV?$basic_string@DU?$char_traits@D@std@@V?$allocator@D@2@@3@@Z 00000001800185e0     tstrings.obj
 0002:000045e0       $unwind$?toUtf8@tstrings@@YA?AV?$basic_string@DU?$char_traits@D@std@@V?$allocator@D@2@@std@@AEBV?$basic_string@GU?$char_traits@G@std@@V?$allocator@G@2@@3@@Z 00000001800185e0     tstrings.obj
 0002:000045e0       $unwind$?winStringToUtf16@tstrings@@YA?AV?$basic_string@GU?$char_traits@G@std@@V?$allocator@G@2@@std@@AEBV23@@Z 00000001800185e0     tstrings.obj
 0002:000045e8       $unwind$??0?$JpError@VSysError@@@@QEAA@AEBVSysError@@AEBUSourceCodePos@@@Z 00000001800185e8     Executor.obj
 0002:000045e8       $unwind$??0?$JpError@Vruntime_error@std@@@@QEAA@AEBVruntime_error@std@@AEBUSourceCodePos@@@Z 00000001800185e8     Guid.obj
 0002:00004600       $cppxdata$??0?$JpError@VSysError@@@@QEAA@AEBVSysError@@AEBUSourceCodePos@@@Z 0000000180018600     Executor.obj
 0002:00004600       $cppxdata$??0?$JpError@Vruntime_error@std@@@@QEAA@AEBVruntime_error@std@@AEBUSourceCodePos@@@Z 0000000180018600     Guid.obj
 0002:00004609       $stateUnwindMap$??0?$JpError@VSysError@@@@QEAA@AEBV0@@Z 0000000180018609     Executor.obj
 0002:00004609       $stateUnwindMap$??0?$JpError@VSysError@@@@QEAA@AEBVSysError@@AEBUSourceCodePos@@@Z 0000000180018609     Executor.obj
 0002:00004609       $stateUnwindMap$??0?$JpError@Vruntime_error@std@@@@QEAA@AEBV0@@Z 0000000180018609     Guid.obj
 0002:00004609       $stateUnwindMap$??0?$JpError@Vruntime_error@std@@@@QEAA@AEBVruntime_error@std@@AEBUSourceCodePos@@@Z 0000000180018609     Guid.obj
 0002:00004609       $stateUnwindMap$??0?$JpError@VError@msi@@@@QEAA@AEBV0@@Z 0000000180018609     MsiCA.obj
 0002:00004609       $stateUnwindMap$??0?$JpError@VError@msi@@@@QEAA@AEBVError@msi@@AEBUSourceCodePos@@@Z 0000000180018609     MsiCA.obj
 0002:00004609       $stateUnwindMap$??0?$JpError@VNoMoreItemsError@msi@@@@QEAA@AEBV0@@Z 0000000180018609     MsiDb.obj
 0002:00004609       $stateUnwindMap$??0?$JpError@VNoMoreItemsError@msi@@@@QEAA@AEBVNoMoreItemsError@msi@@AEBUSourceCodePos@@@Z 0000000180018609     MsiDb.obj
 0002:0000460f       $ip2state$??0?$JpError@VSysError@@@@QEAA@AEBVSysError@@AEBUSourceCodePos@@@Z 000000018001860f     Executor.obj
 0002:0000460f       $ip2state$??0?$JpError@Vruntime_error@std@@@@QEAA@AEBVruntime_error@std@@AEBUSourceCodePos@@@Z 000000018001860f     Guid.obj
 0002:00004614       $unwind$??0?$JpError@VSysError@@@@QEAA@AEBV0@@Z 0000000180018614     Executor.obj
 0002:00004614       $unwind$??0?$JpError@Vruntime_error@std@@@@QEAA@AEBV0@@Z 0000000180018614     Guid.obj
 0002:00004628       $cppxdata$??0?$JpError@VSysError@@@@QEAA@AEBV0@@Z 0000000180018628     Executor.obj
 0002:00004628       $cppxdata$??0?$JpError@Vruntime_error@std@@@@QEAA@AEBV0@@Z 0000000180018628     Guid.obj
 0002:00004631       $ip2state$??0?$JpError@VSysError@@@@QEAA@AEBV0@@Z 0000000180018631     Executor.obj
 0002:00004631       $ip2state$??0?$JpError@Vruntime_error@std@@@@QEAA@AEBV0@@Z 0000000180018631     Guid.obj
 0002:00004634       $unwind$??$_Destroy_range@V?$allocator@V?$basic_string@GU?$char_traits@G@std@@V?$allocator@G@2@@std@@@std@@@std@@YAXPEAV?$basic_string@GU?$char_traits@G@std@@V?$allocator@G@2@@0@QEAV10@AEAV?$allocator@V?$basic_string@GU?$char_traits@G@std@@V?$allocator@G@2@@std@@@0@@Z 0000000180018634     Executor.obj
 0002:00004640       $unwind$?append@?$basic_string@GU?$char_traits@G@std@@V?$allocator@G@2@@std@@QEAAAEAV12@QEBG_K@Z 0000000180018640     FileUtils.obj
 0002:00004640       $unwind$?append@?$basic_string@DU?$char_traits@D@std@@V?$allocator@D@2@@std@@QEAAAEAV12@_KD@Z 0000000180018640     tstrings.obj
 0002:00004650       $unwind$?append@?$basic_string@GU?$char_traits@G@std@@V?$allocator@G@2@@std@@QEAAAEAV12@_KG@Z 0000000180018650     FileUtils.obj
 0002:0000465c       $unwind$?basename@FileUtils@@YA?AV?$basic_string@GU?$char_traits@G@std@@V?$allocator@G@2@@std@@AEBV23@@Z 000000018001865c     FileUtils.obj
 0002:00004670       $unwind$?combinePath@FileUtils@@YA?AV?$basic_string@GU?$char_traits@G@std@@V?$allocator@G@2@@std@@AEBV23@0@Z 0000000180018670     FileUtils.obj
 0002:00004698       $cppxdata$?combinePath@FileUtils@@YA?AV?$basic_string@GU?$char_traits@G@std@@V?$allocator@G@2@@std@@AEBV23@0@Z 0000000180018698     FileUtils.obj
 0002:000046a1       $stateUnwindMap$?combinePath@FileUtils@@YA?AV?$basic_string@GU?$char_traits@G@std@@V?$allocator@G@2@@std@@AEBV23@0@Z 00000001800186a1     FileUtils.obj
 0002:000046c5       $ip2state$?combinePath@FileUtils@@YA?AV?$basic_string@GU?$char_traits@G@std@@V?$allocator@G@2@@std@@AEBV23@0@Z 00000001800186c5     FileUtils.obj
 0002:000046dc       $unwind$??$_Traits_find_last_of@U?$char_traits@G@std@@$00@std@@YA_KQEBG_K101@Z 00000001800186dc     FileUtils.obj
 0002:000046f8       $unwind$wmemcmp            00000001800186f8     Guid.obj
 0002:00004704       $unwind$??$?HGU?$char_traits@G@std@@V?$allocator@G@1@@std@@YA?AV?$basic_string@GU?$char_traits@G@std@@V?$allocator@G@2@@0@$$QEAV10@QEBG@Z 0000000180018704     Guid.obj
 0002:00004704       $unwind$?insert@?$basic_string@GU?$char_traits@G@std@@V?$allocator@G@2@@std@@QEAAAEAV12@_K0G@Z 0000000180018704     Guid.obj
 0002:00004718       $unwind$??0Guid@@QEAA@AEBV?$basic_string@GU?$char_traits@G@std@@V?$allocator@G@2@@std@@@Z 0000000180018718     Guid.obj
 0002:0000473c       $cppxdata$??0Guid@@QEAA@AEBV?$basic_string@GU?$char_traits@G@std@@V?$allocator@G@2@@std@@@Z 000000018001873c     Guid.obj
 0002:00004745       $stateUnwindMap$??0Guid@@QEAA@AEBV?$basic_string@GU?$char_traits@G@std@@V?$allocator@G@2@@std@@@Z 0000000180018745     Guid.obj
 0002:00004752       $ip2state$??0Guid@@QEAA@AEBV?$basic_string@GU?$char_traits@G@std@@V?$allocator@G@2@@std@@@Z 0000000180018752     Guid.obj
 0002:00004760       $unwind$?toString@Guid@@QEBA?AV?$basic_string@GU?$char_traits@G@std@@V?$allocator@G@2@@std@@H@Z 0000000180018760     Guid.obj
 0002:00004788       $cppxdata$?toString@Guid@@QEBA?AV?$basic_string@GU?$char_traits@G@std@@V?$allocator@G@2@@std@@H@Z 0000000180018788     Guid.obj
 0002:00004791       $stateUnwindMap$?toString@Guid@@QEBA?AV?$basic_string@GU?$char_traits@G@std@@V?$allocator@G@2@@std@@H@Z 0000000180018791     Guid.obj
 0002:0000479d       $ip2state$?toString@Guid@@QEBA?AV?$basic_string@GU?$char_traits@G@std@@V?$allocator@G@2@@std@@H@Z 000000018001879d     Guid.obj
 0002:000047a8       $unwind$?makeException@@YA?AV?$JpError@Vruntime_error@std@@@@AEBV?$basic_string@DU?$char_traits@D@std@@V?$allocator@D@2@@std@@AEBUSourceCodePos@@@Z 00000001800187a8     Guid.obj
 0002:000047c0       $cppxdata$?makeException@@YA?AV?$JpError@Vruntime_error@std@@@@AEBV?$basic_string@DU?$char_traits@D@std@@V?$allocator@D@2@@std@@AEBUSourceCodePos@@@Z 00000001800187c0     Guid.obj
 0002:000047c9       $stateUnwindMap$?makeException@@YA?AV?$JpError@Vruntime_error@std@@@@AEBV?$basic_string@DU?$char_traits@D@std@@V?$allocator@D@2@@std@@AEBUSourceCodePos@@@Z 00000001800187c9     Guid.obj
 0002:000047d0       $ip2state$?makeException@@YA?AV?$JpError@Vruntime_error@std@@@@AEBV?$basic_string@DU?$char_traits@D@std@@V?$allocator@D@2@@std@@AEBUSourceCodePos@@@Z 00000001800187d0     Guid.obj
 0002:000047d4       $unwind$?makeException@@YA?AV?$JpError@Vruntime_error@std@@@@AEBVany@tstrings@@AEBUSourceCodePos@@@Z 00000001800187d4     Guid.obj
 0002:000047ec       $cppxdata$?makeException@@YA?AV?$JpError@Vruntime_error@std@@@@AEBVany@tstrings@@AEBUSourceCodePos@@@Z 00000001800187ec     Guid.obj
 0002:000047f5       $stateUnwindMap$?makeException@@YA?AV?$JpError@Vruntime_error@std@@@@AEBVany@tstrings@@AEBUSourceCodePos@@@Z 00000001800187f5     Guid.obj
 0002:00004802       $ip2state$?makeException@@YA?AV?$JpError@Vruntime_error@std@@@@AEBVany@tstrings@@AEBUSourceCodePos@@@Z 0000000180018802     Guid.obj
 0002:0000480c       $unwind$?makeException@@YA?AV?$JpError@Vruntime_error@std@@@@PEBDAEBUSourceCodePos@@@Z 000000018001880c     Guid.obj
 0002:00004824       $cppxdata$?makeException@@YA?AV?$JpError@Vruntime_error@std@@@@PEBDAEBUSourceCodePos@@@Z 0000000180018824     Guid.obj
 0002:0000482d       $stateUnwindMap$?makeException@@YA?AV?$JpError@Vruntime_error@std@@@@PEBDAEBUSourceCodePos@@@Z 000000018001882d     Guid.obj
 0002:0000482d       $stateUnwindMap$?getSystem32Dir@SysInfo@@YA?AV?$basic_string@GU?$char_traits@G@std@@V?$allocator@G@2@@std@@XZ 000000018001882d     WinSysInfo.obj
 0002:00004834       $ip2state$?makeException@@YA?AV?$JpError@Vruntime_error@std@@@@PEBDAEBUSourceCodePos@@@Z 0000000180018834     Guid.obj
 0002:0000483c       $unwind$?initGuid@?A0x2459fff0@@YAXAEBV?$basic_string@GU?$char_traits@G@std@@V?$allocator@G@2@@std@@AEAU_GUID@@@Z 000000018001883c     Guid.obj
 0002:0000485c       $cppxdata$?initGuid@?A0x2459fff0@@YAXAEBV?$basic_string@GU?$char_traits@G@std@@V?$allocator@G@2@@std@@AEAU_GUID@@@Z 000000018001885c     Guid.obj
 0002:00004865       $stateUnwindMap$?initGuid@?A0x2459fff0@@YAXAEBV?$basic_string@GU?$char_traits@G@std@@V?$allocator@G@2@@std@@AEAU_GUID@@@Z 0000000180018865     Guid.obj
 0002:0000486c       $ip2state$?initGuid@?A0x2459fff0@@YAXAEBV?$basic_string@GU?$char_traits@G@std@@V?$allocator@G@2@@std@@AEAU_GUID@@@Z 000000018001886c     Guid.obj
 0002:00004874       $unwind$??$?HGU?$char_traits@G@std@@V?$allocator@G@1@@std@@YA?AV?$basic_string@GU?$char_traits@G@std@@V?$allocator@G@2@@0@QEBGAEBV10@@Z 0000000180018874     Guid.obj
 0002:00004874       $unwind$??$?HDU?$char_traits@D@std@@V?$allocator@D@1@@std@@YA?AV?$basic_string@DU?$char_traits@D@std@@V?$allocator@D@2@@0@QEBDAEBV10@@Z 0000000180018874     WinSysInfo.obj
 0002:00004884       $unwind$??$_Reallocate_grow_by@V<lambda_1>@?1??insert@?$basic_string@GU?$char_traits@G@std@@V?$allocator@G@2@@std@@QEAAAEAV34@_K0G@Z@_K_KG@?$basic_string@GU?$char_traits@G@std@@V?$allocator@G@2@@std@@AEAAAEAV01@_KV<lambda_1>@?1??insert@01@QEAAAEAV01@00G@Z@_K2G@Z 0000000180018884     Guid.obj
 0002:0000489c       $unwind$printf             000000018001889c     IconSwap.obj
 0002:000048a8       $unwind$?ChangeIcon@@YA_NPEAXAEBV?$basic_string@GU?$char_traits@G@std@@V?$allocator@G@2@@std@@@Z 00000001800188a8     IconSwap.obj
 0002:000048c0       $unwind$?toUnicodeString@jni@@YA?AV?$basic_string@GU?$char_traits@G@std@@V?$allocator@G@2@@std@@PEAUJNIEnv_@@PEAV_jstring@@@Z 00000001800188c0     JniUtils.obj
 0002:000048e0       $cppxdata$?toUnicodeString@jni@@YA?AV?$basic_string@GU?$char_traits@G@std@@V?$allocator@G@2@@std@@PEAUJNIEnv_@@PEAV_jstring@@@Z 00000001800188e0     JniUtils.obj
 0002:000048e9       $stateUnwindMap$?toUnicodeString@jni@@YA?AV?$basic_string@GU?$char_traits@G@std@@V?$allocator@G@2@@std@@PEAUJNIEnv_@@PEAV_jstring@@@Z 00000001800188e9     JniUtils.obj
 0002:000048f0       $ip2state$?toUnicodeString@jni@@YA?AV?$basic_string@GU?$char_traits@G@std@@V?$allocator@G@2@@std@@PEAUJNIEnv_@@PEAV_jstring@@@Z 00000001800188f0     JniUtils.obj
 0002:000048f8       $unwind$?toJString@jni@@YAPEAV_jstring@@PEAUJNIEnv_@@AEBV?$basic_string@GU?$char_traits@G@std@@V?$allocator@G@2@@std@@@Z 00000001800188f8     JniUtils.obj
 0002:000048f8       $unwind$?writeWORD@?A0xcb1fbc16@@YAAEAV?$basic_ostream@DU?$char_traits@D@std@@@std@@AEAV23@_K@Z 00000001800188f8     VersionInfo.obj
 0002:00004908       $unwind$?toUnicodeStringArray@jni@@YA?AV?$vector@V?$basic_string@GU?$char_traits@G@std@@V?$allocator@G@2@@std@@V?$allocator@V?$basic_string@GU?$char_traits@G@std@@V?$allocator@G@2@@std@@@2@@std@@PEAUJNIEnv_@@PEAV_jobjectArray@@@Z 0000000180018908     JniUtils.obj
 0002:00004930       $cppxdata$?toUnicodeStringArray@jni@@YA?AV?$vector@V?$basic_string@GU?$char_traits@G@std@@V?$allocator@G@2@@std@@V?$allocator@V?$basic_string@GU?$char_traits@G@std@@V?$allocator@G@2@@std@@@2@@std@@PEAUJNIEnv_@@PEAV_jobjectArray@@@Z 0000000180018930     JniUtils.obj
 0002:00004939       $stateUnwindMap$?toUnicodeStringArray@jni@@YA?AV?$vector@V?$basic_string@GU?$char_traits@G@std@@V?$allocator@G@2@@std@@V?$allocator@V?$basic_string@GU?$char_traits@G@std@@V?$allocator@G@2@@std@@@2@@std@@PEAUJNIEnv_@@PEAV_jobjectArray@@@Z 0000000180018939     JniUtils.obj
 0002:00004950       $ip2state$?toUnicodeStringArray@jni@@YA?AV?$vector@V?$basic_string@GU?$char_traits@G@std@@V?$allocator@G@2@@std@@V?$allocator@V?$basic_string@GU?$char_traits@G@std@@V?$allocator@G@2@@std@@@2@@std@@PEAUJNIEnv_@@PEAV_jobjectArray@@@Z 0000000180018950     JniUtils.obj
 0002:00004960       $unwind$??1?$AtEndOfScope@V<lambda_1>@?1??toUnicodeString@jni@@YA?AV?$basic_string@GU?$char_traits@G@std@@V?$allocator@G@2@@std@@PEAUJNIEnv_@@PEAV_jstring@@@Z@@@QEAA@XZ 0000000180018960     JniUtils.obj
 0002:00004970       $cppxdata$??1?$AtEndOfScope@V<lambda_1>@?1??toUnicodeString@jni@@YA?AV?$basic_string@GU?$char_traits@G@std@@V?$allocator@G@2@@std@@PEAUJNIEnv_@@PEAV_jstring@@@Z@@@QEAA@XZ 0000000180018970     JniUtils.obj
 0002:0000497d       $stateUnwindMap$??$_Emplace_reallocate@V?$basic_string@GU?$char_traits@G@std@@V?$allocator@G@2@@std@@@?$vector@V?$basic_string@GU?$char_traits@G@std@@V?$allocator@G@2@@std@@V?$allocator@V?$basic_string@GU?$char_traits@G@std@@V?$allocator@G@2@@std@@@2@@std@@AEAAPEAV?$basic_string@GU?$char_traits@G@std@@V?$allocator@G@2@@1@QEAV21@$$QEAV21@@Z 000000018001897d     JniUtils.obj
 0002:0000497d       $stateUnwindMap$??1?$AtEndOfScope@V<lambda_1>@?1??toUnicodeString@jni@@YA?AV?$basic_string@GU?$char_traits@G@std@@V?$allocator@G@2@@std@@PEAUJNIEnv_@@PEAV_jstring@@@Z@@@QEAA@XZ 000000018001897d     JniUtils.obj
 0002:0000497d       $stateUnwindMap$??$_Resize_reallocate@U_Value_init_tag@std@@@?$vector@GV?$allocator@G@std@@@std@@AEAAX_KAEBU_Value_init_tag@1@@Z 000000018001897d     MsiUtils.obj
 0002:0000497d       $stateUnwindMap$??$_Emplace_reallocate@D@?$vector@EV?$allocator@E@std@@@std@@AEAAPEAEQEAE$$QEAD@Z 000000018001897d     ResourceEditor.obj
 0002:0000497d       $stateUnwindMap$??$_Resize_reallocate@U_Value_init_tag@std@@@?$vector@EV?$allocator@E@std@@@std@@AEAAX_KAEBU_Value_init_tag@1@@Z 000000018001897d     ResourceEditor.obj
 0002:0000497d       $stateUnwindMap$??1StreamSize@?A0xcb1fbc16@@QEAA@XZ 000000018001897d     VersionInfo.obj
 0002:0000497d       $stateUnwindMap$Java_jdk_jpackage_internal_WindowsRegistry_openRegistryKey 000000018001897d     WindowsRegistry.obj
 0002:0000497d       $stateUnwindMap$Java_jdk_jpackage_internal_ExecutableRebrander_unlockResource 000000018001897d     jpackage.obj
 0002:00004980       $tryMap$??1?$AtEndOfScope@V<lambda_1>@?1??toUnicodeString@jni@@YA?AV?$basic_string@GU?$char_traits@G@std@@V?$allocator@G@2@@std@@PEAUJNIEnv_@@PEAV_jstring@@@Z@@@QEAA@XZ 0000000180018980     JniUtils.obj
 0002:00004988       $handlerMap$??1?$AtEndOfScope@V<lambda_1>@?1??toUnicodeString@jni@@YA?AV?$basic_string@GU?$char_traits@G@std@@V?$allocator@G@2@@std@@PEAUJNIEnv_@@PEAV_jstring@@@Z@@@QEAA@XZ 0000000180018988     JniUtils.obj
 0002:0000499c       $ip2state$??1?$AtEndOfScope@V<lambda_1>@?1??toUnicodeString@jni@@YA?AV?$basic_string@GU?$char_traits@G@std@@V?$allocator@G@2@@std@@PEAUJNIEnv_@@PEAV_jstring@@@Z@@@QEAA@XZ 000000018001899c     JniUtils.obj
 0002:000049a0       $unwind$?catch$0@?0???1?$AtEndOfScope@V<lambda_1>@?1??toUnicodeString@jni@@YA?AV?$basic_string@GU?$char_traits@G@std@@V?$allocator@G@2@@std@@PEAUJNIEnv_@@PEAV_jstring@@@Z@@@QEAA@XZ@4HA 00000001800189a0     JniUtils.obj
 0002:000049a0       $unwind$?catch$0@?0???1StreamSize@?A0xcb1fbc16@@QEAA@XZ@4HA 00000001800189a0     VersionInfo.obj
 0002:000049b0       $cppxdata$?catch$0@?0???1?$AtEndOfScope@V<lambda_1>@?1??toUnicodeString@jni@@YA?AV?$basic_string@GU?$char_traits@G@std@@V?$allocator@G@2@@std@@PEAUJNIEnv_@@PEAV_jstring@@@Z@@@QEAA@XZ@4HA 00000001800189b0     JniUtils.obj
 0002:000049b0       $cppxdata$?catch$0@?0???1StreamSize@?A0xcb1fbc16@@QEAA@XZ@4HA 00000001800189b0     VersionInfo.obj
 0002:000049ba       $stateUnwindMap$?catch$0@?0???1?$AtEndOfScope@V<lambda_1>@?1??toUnicodeString@jni@@YA?AV?$basic_string@GU?$char_traits@G@std@@V?$allocator@G@2@@std@@PEAUJNIEnv_@@PEAV_jstring@@@Z@@@QEAA@XZ@4HA 00000001800189ba     JniUtils.obj
 0002:000049ba       $stateUnwindMap$?catch$1@?0???1?$AtEndOfScope@V<lambda_1>@?1??toUnicodeString@jni@@YA?AV?$basic_string@GU?$char_traits@G@std@@V?$allocator@G@2@@std@@PEAUJNIEnv_@@PEAV_jstring@@@Z@@@QEAA@XZ@4HA 00000001800189ba     JniUtils.obj
 0002:000049ba       $stateUnwindMap$?catch$5@?0???1FileLock@ResourceEditor@@QEAA@XZ@4HA 00000001800189ba     ResourceEditor.obj
 0002:000049ba       $stateUnwindMap$?catch$6@?0???1FileLock@ResourceEditor@@QEAA@XZ@4HA 00000001800189ba     ResourceEditor.obj
 0002:000049ba       $stateUnwindMap$?catch$0@?0???1StreamSize@?A0xcb1fbc16@@QEAA@XZ@4HA 00000001800189ba     VersionInfo.obj
 0002:000049ba       $stateUnwindMap$?catch$1@?0???1StreamSize@?A0xcb1fbc16@@QEAA@XZ@4HA 00000001800189ba     VersionInfo.obj
 0002:000049bc       $ip2state$?catch$0@?0???1?$AtEndOfScope@V<lambda_1>@?1??toUnicodeString@jni@@YA?AV?$basic_string@GU?$char_traits@G@std@@V?$allocator@G@2@@std@@PEAUJNIEnv_@@PEAV_jstring@@@Z@@@QEAA@XZ@4HA 00000001800189bc     JniUtils.obj
 0002:000049bc       $ip2state$?catch$5@?0???1FileLock@ResourceEditor@@QEAA@XZ@4HA 00000001800189bc     ResourceEditor.obj
 0002:000049bc       $ip2state$?catch$0@?0???1StreamSize@?A0xcb1fbc16@@QEAA@XZ@4HA 00000001800189bc     VersionInfo.obj
 0002:000049c0       $unwind$?catch$1@?0???1?$AtEndOfScope@V<lambda_1>@?1??toUnicodeString@jni@@YA?AV?$basic_string@GU?$char_traits@G@std@@V?$allocator@G@2@@std@@PEAUJNIEnv_@@PEAV_jstring@@@Z@@@QEAA@XZ@4HA 00000001800189c0     JniUtils.obj
 0002:000049c0       $unwind$?catch$1@?0???1StreamSize@?A0xcb1fbc16@@QEAA@XZ@4HA 00000001800189c0     VersionInfo.obj
 0002:000049d0       $cppxdata$?catch$1@?0???1?$AtEndOfScope@V<lambda_1>@?1??toUnicodeString@jni@@YA?AV?$basic_string@GU?$char_traits@G@std@@V?$allocator@G@2@@std@@PEAUJNIEnv_@@PEAV_jstring@@@Z@@@QEAA@XZ@4HA 00000001800189d0     JniUtils.obj
 0002:000049d0       $cppxdata$?catch$1@?0???1StreamSize@?A0xcb1fbc16@@QEAA@XZ@4HA 00000001800189d0     VersionInfo.obj
 0002:000049da       $ip2state$?catch$1@?0???1?$AtEndOfScope@V<lambda_1>@?1??toUnicodeString@jni@@YA?AV?$basic_string@GU?$char_traits@G@std@@V?$allocator@G@2@@std@@PEAUJNIEnv_@@PEAV_jstring@@@Z@@@QEAA@XZ@4HA 00000001800189da     JniUtils.obj
 0002:000049da       $ip2state$?catch$6@?0???1FileLock@ResourceEditor@@QEAA@XZ@4HA 00000001800189da     ResourceEditor.obj
 0002:000049da       $ip2state$?catch$1@?0???1StreamSize@?A0xcb1fbc16@@QEAA@XZ@4HA 00000001800189da     VersionInfo.obj
 0002:000049e0       $unwind$??1?$unique_ptr@UJniObjWithEnv@jni@@ULocalRefDeleter@12@@std@@QEAA@XZ 00000001800189e0     JniUtils.obj
 0002:000049f0       $cppxdata$??1?$unique_ptr@UJniObjWithEnv@jni@@ULocalRefDeleter@12@@std@@QEAA@XZ 00000001800189f0     JniUtils.obj
 0002:000049f5       $ip2state$??1?$unique_ptr@UJniObjWithEnv@jni@@ULocalRefDeleter@12@@std@@QEAA@XZ 00000001800189f5     JniUtils.obj
 0002:000049f8       $unwind$??$_Emplace_reallocate@V?$basic_string@GU?$char_traits@G@std@@V?$allocator@G@2@@std@@@?$vector@V?$basic_string@GU?$char_traits@G@std@@V?$allocator@G@2@@std@@V?$allocator@V?$basic_string@GU?$char_traits@G@std@@V?$allocator@G@2@@std@@@2@@std@@AEAAPEAV?$basic_string@GU?$char_traits@G@std@@V?$allocator@G@2@@1@QEAV21@$$QEAV21@@Z 00000001800189f8     JniUtils.obj
 0002:00004a14       $cppxdata$??$_Emplace_reallocate@V?$basic_string@GU?$char_traits@G@std@@V?$allocator@G@2@@std@@@?$vector@V?$basic_string@GU?$char_traits@G@std@@V?$allocator@G@2@@std@@V?$allocator@V?$basic_string@GU?$char_traits@G@std@@V?$allocator@G@2@@std@@@2@@std@@AEAAPEAV?$basic_string@GU?$char_traits@G@std@@V?$allocator@G@2@@1@QEAV21@$$QEAV21@@Z 0000000180018a14     JniUtils.obj
 0002:00004a21       $tryMap$??$_Emplace_reallocate@V?$basic_string@GU?$char_traits@G@std@@V?$allocator@G@2@@std@@@?$vector@V?$basic_string@GU?$char_traits@G@std@@V?$allocator@G@2@@std@@V?$allocator@V?$basic_string@GU?$char_traits@G@std@@V?$allocator@G@2@@std@@@2@@std@@AEAAPEAV?$basic_string@GU?$char_traits@G@std@@V?$allocator@G@2@@1@QEAV21@$$QEAV21@@Z 0000000180018a21     JniUtils.obj
 0002:00004a29       $handlerMap$??$_Emplace_reallocate@V?$basic_string@GU?$char_traits@G@std@@V?$allocator@G@2@@std@@@?$vector@V?$basic_string@GU?$char_traits@G@std@@V?$allocator@G@2@@std@@V?$allocator@V?$basic_string@GU?$char_traits@G@std@@V?$allocator@G@2@@std@@@2@@std@@AEAAPEAV?$basic_string@GU?$char_traits@G@std@@V?$allocator@G@2@@1@QEAV21@$$QEAV21@@Z 0000000180018a29     JniUtils.obj
 0002:00004a30       $ip2state$??$_Emplace_reallocate@V?$basic_string@GU?$char_traits@G@std@@V?$allocator@G@2@@std@@@?$vector@V?$basic_string@GU?$char_traits@G@std@@V?$allocator@G@2@@std@@V?$allocator@V?$basic_string@GU?$char_traits@G@std@@V?$allocator@G@2@@std@@@2@@std@@AEAAPEAV?$basic_string@GU?$char_traits@G@std@@V?$allocator@G@2@@1@QEAV21@$$QEAV21@@Z 0000000180018a30     JniUtils.obj
 0002:00004a3c       $unwind$??6?$basic_ostream@GU?$char_traits@G@std@@@std@@QEAAAEAV01@G@Z 0000000180018a3c     Log.obj
 0002:00004a5c       $cppxdata$??6?$basic_ostream@GU?$char_traits@G@std@@@std@@QEAAAEAV01@G@Z 0000000180018a5c     Log.obj
 0002:00004a69       $tryMap$??6?$basic_ostream@GU?$char_traits@G@std@@@std@@QEAAAEAV01@G@Z 0000000180018a69     Log.obj
 0002:00004a71       $handlerMap$??6?$basic_ostream@GU?$char_traits@G@std@@@std@@QEAAAEAV01@G@Z 0000000180018a71     Log.obj
 0002:00004a7a       $ip2state$??6?$basic_ostream@GU?$char_traits@G@std@@@std@@QEAAAEAV01@G@Z 0000000180018a7a     Log.obj
 0002:00004a88       $unwind$??0LogEvent@@QEAA@XZ 0000000180018a88     Log.obj
 0002:00004ab0       $unwind$?append@StreamLogAppender@@UEAAXAEBULogEvent@@@Z 0000000180018ab0     Log.obj
 0002:00004ad8       $cppxdata$?append@StreamLogAppender@@UEAAXAEBULogEvent@@@Z 0000000180018ad8     Log.obj
 0002:00004ae1       $stateUnwindMap$?append@StreamLogAppender@@UEAAXAEBULogEvent@@@Z 0000000180018ae1     Log.obj
 0002:00004afd       $ip2state$?append@StreamLogAppender@@UEAAXAEBULogEvent@@@Z 0000000180018afd     Log.obj
 0002:00004b0c       $unwind$?log@Logger@@QEBAXW4LogLevel@1@PEBGH1AEBV?$basic_string@GU?$char_traits@G@std@@V?$allocator@G@2@@std@@@Z 0000000180018b0c     Log.obj
 0002:00004b34       $cppxdata$?log@Logger@@QEBAXW4LogLevel@1@PEBGH1AEBV?$basic_string@GU?$char_traits@G@std@@V?$allocator@G@2@@std@@@Z 0000000180018b34     Log.obj
 0002:00004b3d       $stateUnwindMap$?log@Logger@@QEBAXW4LogLevel@1@PEBGH1AEBV?$basic_string@GU?$char_traits@G@std@@V?$allocator@G@2@@std@@@Z 0000000180018b3d     Log.obj
 0002:00004b4a       $ip2state$?log@Logger@@QEBAXW4LogLevel@1@PEBGH1AEBV?$basic_string@GU?$char_traits@G@std@@V?$allocator@G@2@@std@@@Z 0000000180018b4a     Log.obj
 0002:00004b58       $unwind$?_Insert_node@?$_Tree_val@U?$_Tree_simple_types@U?$pair@$$CBV?$basic_string@GU?$char_traits@G@std@@V?$allocator@G@2@@std@@V12@@std@@@std@@@std@@QEAAPEAU?$_Tree_node@U?$pair@$$CBV?$basic_string@GU?$char_traits@G@std@@V?$allocator@G@2@@std@@V12@@std@@PEAX@2@U?$_Tree_id@PEAU?$_Tree_node@U?$pair@$$CBV?$basic_string@GU?$char_traits@G@std@@V?$allocator@G@2@@std@@V12@@std@@PEAX@std@@@2@QEAU32@@Z 0000000180018b58     MsiCA.obj
 0002:00004b60       $unwind$??1DatabaseRecord@msi@@QEAA@XZ 0000000180018b60     MsiCA.obj
 0002:00004b70       $cppxdata$??1DatabaseRecord@msi@@QEAA@XZ 0000000180018b70     MsiCA.obj
 0002:00004b75       $ip2state$??1DatabaseRecord@msi@@QEAA@XZ 0000000180018b75     MsiCA.obj
 0002:00004b78       $unwind$??0?$JpError@VError@msi@@@@QEAA@AEBVError@msi@@AEBUSourceCodePos@@@Z 0000000180018b78     MsiCA.obj
 0002:00004b78       $unwind$??0?$JpError@VNoMoreItemsError@msi@@@@QEAA@AEBVNoMoreItemsError@msi@@AEBUSourceCodePos@@@Z 0000000180018b78     MsiDb.obj
 0002:00004b90       $cppxdata$??0?$JpError@VError@msi@@@@QEAA@AEBVError@msi@@AEBUSourceCodePos@@@Z 0000000180018b90     MsiCA.obj
 0002:00004b90       $cppxdata$??0?$JpError@VNoMoreItemsError@msi@@@@QEAA@AEBVNoMoreItemsError@msi@@AEBUSourceCodePos@@@Z 0000000180018b90     MsiDb.obj
 0002:00004b99       $ip2state$??0?$JpError@VError@msi@@@@QEAA@AEBVError@msi@@AEBUSourceCodePos@@@Z 0000000180018b99     MsiCA.obj
 0002:00004b99       $ip2state$??0?$JpError@VNoMoreItemsError@msi@@@@QEAA@AEBVNoMoreItemsError@msi@@AEBUSourceCodePos@@@Z 0000000180018b99     MsiDb.obj
 0002:00004b9c       $unwind$??0?$JpError@VError@msi@@@@QEAA@AEBV0@@Z 0000000180018b9c     MsiCA.obj
 0002:00004b9c       $unwind$??0?$JpError@VNoMoreItemsError@msi@@@@QEAA@AEBV0@@Z 0000000180018b9c     MsiDb.obj
 0002:00004bb0       $cppxdata$??0?$JpError@VError@msi@@@@QEAA@AEBV0@@Z 0000000180018bb0     MsiCA.obj
 0002:00004bb0       $cppxdata$??0?$JpError@VNoMoreItemsError@msi@@@@QEAA@AEBV0@@Z 0000000180018bb0     MsiDb.obj
 0002:00004bb9       $ip2state$??0?$JpError@VError@msi@@@@QEAA@AEBV0@@Z 0000000180018bb9     MsiCA.obj
 0002:00004bb9       $ip2state$??0?$JpError@VNoMoreItemsError@msi@@@@QEAA@AEBV0@@Z 0000000180018bb9     MsiDb.obj
 0002:00004bb9       $ip2state$?unsafe_format@tstrings@@YA?AV?$basic_string@GU?$char_traits@G@std@@V?$allocator@G@2@@std@@PEBGZZ 0000000180018bb9     tstrings.obj
 0002:00004bc0       $unwind$??$_Try_emplace@AEBV?$basic_string@GU?$char_traits@G@std@@V?$allocator@G@2@@std@@$$V@?$map@V?$basic_string@GU?$char_traits@G@std@@V?$allocator@G@2@@std@@V12@U?$less@V?$basic_string@GU?$char_traits@G@std@@V?$allocator@G@2@@std@@@2@V?$allocator@U?$pair@$$CBV?$basic_string@GU?$char_traits@G@std@@V?$allocator@G@2@@std@@V12@@std@@@2@@std@@AEAA?AU?$pair@PEAU?$_Tree_node@U?$pair@$$CBV?$basic_string@GU?$char_traits@G@std@@V?$allocator@G@2@@std@@V12@@std@@PEAX@std@@_N@1@AEBV?$basic_string@GU?$char_traits@G@std@@V?$allocator@G@2@@1@@Z 0000000180018bc0     MsiCA.obj
 0002:00004bd4       $unwind$??$?0AEBUpiecewise_construct_t@std@@V?$tuple@AEBV?$basic_string@GU?$char_traits@G@std@@V?$allocator@G@2@@std@@@1@V?$tuple@$$V@1@@?$_Tree_temp_node@V?$allocator@U?$_Tree_node@U?$pair@$$CBV?$basic_string@GU?$char_traits@G@std@@V?$allocator@G@2@@std@@V12@@std@@PEAX@std@@@std@@@std@@QEAA@AEAV?$allocator@U?$_Tree_node@U?$pair@$$CBV?$basic_string@GU?$char_traits@G@std@@V?$allocator@G@2@@std@@V12@@std@@PEAX@std@@@1@PEAU?$_Tree_node@U?$pair@$$CBV?$basic_string@GU?$char_traits@G@std@@V?$allocator@G@2@@std@@V12@@std@@PEAX@1@AEBUpiecewise_construct_t@1@$$QEAV?$tuple@AEBV?$basic_string@GU?$char_traits@G@std@@V?$allocator@G@2@@std@@@1@$$QEAV?$tuple@$$V@1@@Z 0000000180018bd4     MsiCA.obj
 0002:00004bf0       $cppxdata$??$?0AEBUpiecewise_construct_t@std@@V?$tuple@AEBV?$basic_string@GU?$char_traits@G@std@@V?$allocator@G@2@@std@@@1@V?$tuple@$$V@1@@?$_Tree_temp_node@V?$allocator@U?$_Tree_node@U?$pair@$$CBV?$basic_string@GU?$char_traits@G@std@@V?$allocator@G@2@@std@@V12@@std@@PEAX@std@@@std@@@std@@QEAA@AEAV?$allocator@U?$_Tree_node@U?$pair@$$CBV?$basic_string@GU?$char_traits@G@std@@V?$allocator@G@2@@std@@V12@@std@@PEAX@std@@@1@PEAU?$_Tree_node@U?$pair@$$CBV?$basic_string@GU?$char_traits@G@std@@V?$allocator@G@2@@std@@V12@@std@@PEAX@1@AEBUpiecewise_construct_t@1@$$QEAV?$tuple@AEBV?$basic_string@GU?$char_traits@G@std@@V?$allocator@G@2@@std@@@1@$$QEAV?$tuple@$$V@1@@Z 0000000180018bf0     MsiCA.obj
 0002:00004bf9       $stateUnwindMap$??$?0AEBUpiecewise_construct_t@std@@V?$tuple@AEBV?$basic_string@GU?$char_traits@G@std@@V?$allocator@G@2@@std@@@1@V?$tuple@$$V@1@@?$_Tree_temp_node@V?$allocator@U?$_Tree_node@U?$pair@$$CBV?$basic_string@GU?$char_traits@G@std@@V?$allocator@G@2@@std@@V12@@std@@PEAX@std@@@std@@@std@@QEAA@AEAV?$allocator@U?$_Tree_node@U?$pair@$$CBV?$basic_string@GU?$char_traits@G@std@@V?$allocator@G@2@@std@@V12@@std@@PEAX@std@@@1@PEAU?$_Tree_node@U?$pair@$$CBV?$basic_string@GU?$char_traits@G@std@@V?$allocator@G@2@@std@@V12@@std@@PEAX@1@AEBUpiecewise_construct_t@1@$$QEAV?$tuple@AEBV?$basic_string@GU?$char_traits@G@std@@V?$allocator@G@2@@std@@@1@$$QEAV?$tuple@$$V@1@@Z 0000000180018bf9     MsiCA.obj
 0002:00004c06       $ip2state$??$?0AEBUpiecewise_construct_t@std@@V?$tuple@AEBV?$basic_string@GU?$char_traits@G@std@@V?$allocator@G@2@@std@@@1@V?$tuple@$$V@1@@?$_Tree_temp_node@V?$allocator@U?$_Tree_node@U?$pair@$$CBV?$basic_string@GU?$char_traits@G@std@@V?$allocator@G@2@@std@@V12@@std@@PEAX@std@@@std@@@std@@QEAA@AEAV?$allocator@U?$_Tree_node@U?$pair@$$CBV?$basic_string@GU?$char_traits@G@std@@V?$allocator@G@2@@std@@V12@@std@@PEAX@std@@@1@PEAU?$_Tree_node@U?$pair@$$CBV?$basic_string@GU?$char_traits@G@std@@V?$allocator@G@2@@std@@V12@@std@@PEAX@1@AEBUpiecewise_construct_t@1@$$QEAV?$tuple@AEBV?$basic_string@GU?$char_traits@G@std@@V?$allocator@G@2@@std@@@1@$$QEAV?$tuple@$$V@1@@Z 0000000180018c06     MsiCA.obj
 0002:00004c0c       $unwind$??0Database@msi@@QEAA@AEBV?$basic_string@GU?$char_traits@G@std@@V?$allocator@G@2@@std@@@Z 0000000180018c0c     MsiDb.obj
 0002:00004c20       $cppxdata$??0Database@msi@@QEAA@AEBV?$basic_string@GU?$char_traits@G@std@@V?$allocator@G@2@@std@@@Z 0000000180018c20     MsiDb.obj
 0002:00004c29       $stateUnwindMap$??0Database@msi@@QEAA@AEBV?$basic_string@GU?$char_traits@G@std@@V?$allocator@G@2@@std@@@Z 0000000180018c29     MsiDb.obj
 0002:00004c30       $ip2state$??0Database@msi@@QEAA@AEBV?$basic_string@GU?$char_traits@G@std@@V?$allocator@G@2@@std@@@Z 0000000180018c30     MsiDb.obj
 0002:00004c38       $unwind$?getProperty@Database@msi@@QEBA?AV?$basic_string@GU?$char_traits@G@std@@V?$allocator@G@2@@std@@AEBV34@@Z 0000000180018c38     MsiDb.obj
 0002:00004c58       $cppxdata$?getProperty@Database@msi@@QEBA?AV?$basic_string@GU?$char_traits@G@std@@V?$allocator@G@2@@std@@AEBV34@@Z 0000000180018c58     MsiDb.obj
 0002:00004c61       $stateUnwindMap$?getProperty@Database@msi@@QEBA?AV?$basic_string@GU?$char_traits@G@std@@V?$allocator@G@2@@std@@AEBV34@@Z 0000000180018c61     MsiDb.obj
 0002:00004ca8       $ip2state$?getProperty@Database@msi@@QEBA?AV?$basic_string@GU?$char_traits@G@std@@V?$allocator@G@2@@std@@AEBV34@@Z 0000000180018ca8     MsiDb.obj
 0002:00004cc4       $unwind$?fetch@DatabaseRecord@msi@@QEAAAEAV12@AEAVDatabaseView@2@@Z 0000000180018cc4     MsiDb.obj
 0002:00004cd4       $cppxdata$?fetch@DatabaseRecord@msi@@QEAAAEAV12@AEAVDatabaseView@2@@Z 0000000180018cd4     MsiDb.obj
 0002:00004cdd       $ip2state$?fetch@DatabaseRecord@msi@@QEAAAEAV12@AEAVDatabaseView@2@@Z 0000000180018cdd     MsiDb.obj
 0002:00004ce4       $unwind$?getFieldCount@DatabaseRecord@msi@@QEBAIXZ 0000000180018ce4     MsiDb.obj
 0002:00004cfc       $cppxdata$?getFieldCount@DatabaseRecord@msi@@QEBAIXZ 0000000180018cfc     MsiDb.obj
 0002:00004d05       $stateUnwindMap$?getFieldCount@DatabaseRecord@msi@@QEBAIXZ 0000000180018d05     MsiDb.obj
 0002:00004d12       $ip2state$?getFieldCount@DatabaseRecord@msi@@QEBAIXZ 0000000180018d12     MsiDb.obj
 0002:00004d1c       $unwind$??0DatabaseView@msi@@QEAA@AEBVDatabase@1@AEBV?$basic_string@GU?$char_traits@G@std@@V?$allocator@G@2@@std@@AEBVDatabaseRecord@1@@Z 0000000180018d1c     MsiDb.obj
 0002:00004d3c       $cppxdata$??0DatabaseView@msi@@QEAA@AEBVDatabase@1@AEBV?$basic_string@GU?$char_traits@G@std@@V?$allocator@G@2@@std@@AEBVDatabaseRecord@1@@Z 0000000180018d3c     MsiDb.obj
 0002:00004d45       $stateUnwindMap$??0DatabaseView@msi@@QEAA@AEBVDatabase@1@AEBV?$basic_string@GU?$char_traits@G@std@@V?$allocator@G@2@@std@@AEBVDatabaseRecord@1@@Z 0000000180018d45     MsiDb.obj
 0002:00004d58       $ip2state$??0DatabaseView@msi@@QEAA@AEBVDatabase@1@AEBV?$basic_string@GU?$char_traits@G@std@@V?$allocator@G@2@@std@@AEBVDatabaseRecord@1@@Z 0000000180018d58     MsiDb.obj
 0002:00004d68       $unwind$??1DatabaseView@msi@@QEAA@XZ 0000000180018d68     MsiDb.obj
 0002:00004d68       $unwind$??1Database@msi@@QEAA@XZ 0000000180018d68     jpackage.obj
 0002:00004d78       $cppxdata$??1DatabaseView@msi@@QEAA@XZ 0000000180018d78     MsiDb.obj
 0002:00004d78       $cppxdata$??1Database@msi@@QEAA@XZ 0000000180018d78     jpackage.obj
 0002:00004d7d       $ip2state$??1DatabaseView@msi@@QEAA@XZ 0000000180018d7d     MsiDb.obj
 0002:00004d7d       $ip2state$??1Database@msi@@QEAA@XZ 0000000180018d7d     jpackage.obj
 0002:00004d80       $unwind$?fetch@DatabaseView@msi@@QEAA?AVDatabaseRecord@2@XZ 0000000180018d80     MsiDb.obj
 0002:00004d9c       $cppxdata$?fetch@DatabaseView@msi@@QEAA?AVDatabaseRecord@2@XZ 0000000180018d9c     MsiDb.obj
 0002:00004da5       $stateUnwindMap$?fetch@DatabaseView@msi@@QEAA?AVDatabaseRecord@2@XZ 0000000180018da5     MsiDb.obj
 0002:00004db7       $ip2state$?fetch@DatabaseView@msi@@QEAA?AVDatabaseRecord@2@XZ 0000000180018db7     MsiDb.obj
 0002:00004dc0       $unwind$?tryFetch@DatabaseView@msi@@QEAA?AVDatabaseRecord@2@XZ 0000000180018dc0     MsiDb.obj
 0002:00004de0       $cppxdata$?tryFetch@DatabaseView@msi@@QEAA?AVDatabaseRecord@2@XZ 0000000180018de0     MsiDb.obj
 0002:00004de9       $stateUnwindMap$?tryFetch@DatabaseView@msi@@QEAA?AVDatabaseRecord@2@XZ 0000000180018de9     MsiDb.obj
 0002:00004dfb       $ip2state$?tryFetch@DatabaseView@msi@@QEAA?AVDatabaseRecord@2@XZ 0000000180018dfb     MsiDb.obj
 0002:00004e04       $unwind$??1?$basic_filebuf@DU?$char_traits@D@std@@@std@@UEAA@XZ 0000000180018e04     MsiDb.obj
 0002:00004e14       $cppxdata$??1?$basic_filebuf@DU?$char_traits@D@std@@@std@@UEAA@XZ 0000000180018e14     MsiDb.obj
 0002:00004e19       $ip2state$??1?$basic_filebuf@DU?$char_traits@D@std@@@std@@UEAA@XZ 0000000180018e19     MsiDb.obj
 0002:00004e1c       $unwind$?overflow@?$basic_filebuf@DU?$char_traits@D@std@@@std@@MEAAHH@Z 0000000180018e1c     MsiDb.obj
 0002:00004e38       $unwind$?uflow@?$basic_filebuf@DU?$char_traits@D@std@@@std@@MEAAHXZ 0000000180018e38     MsiDb.obj
 0002:00004e58       $cppxdata$?uflow@?$basic_filebuf@DU?$char_traits@D@std@@@std@@MEAAHXZ 0000000180018e58     MsiDb.obj
 0002:00004e61       $stateUnwindMap$?uflow@?$basic_filebuf@DU?$char_traits@D@std@@@std@@MEAAHXZ 0000000180018e61     MsiDb.obj
 0002:00004e68       $ip2state$?uflow@?$basic_filebuf@DU?$char_traits@D@std@@@std@@MEAAHXZ 0000000180018e68     MsiDb.obj
 0002:00004e70       $unwind$?xsputn@?$basic_filebuf@DU?$char_traits@D@std@@@std@@MEAA_JPEBD_J@Z 0000000180018e70     MsiDb.obj
 0002:00004e84       $unwind$?seekoff@?$basic_filebuf@DU?$char_traits@D@std@@@std@@MEAA?AV?$fpos@U_Mbstatet@@@2@_JHH@Z 0000000180018e84     MsiDb.obj
 0002:00004e98       $unwind$?seekpos@?$basic_filebuf@DU?$char_traits@D@std@@@std@@MEAA?AV?$fpos@U_Mbstatet@@@2@V32@H@Z 0000000180018e98     MsiDb.obj
 0002:00004ea8       $unwind$?_Init@?$basic_filebuf@DU?$char_traits@D@std@@@std@@IEAAXPEAU_iobuf@@W4_Initfl@12@@Z 0000000180018ea8     MsiDb.obj
 0002:00004eb4       $unwind$?_Endwrite@?$basic_filebuf@DU?$char_traits@D@std@@@std@@IEAA_NXZ 0000000180018eb4     MsiDb.obj
 0002:00004ec8       $unwind$?openDatabase@?A0x6ccb95c8@msi@@YAKAEBV?$basic_string@GU?$char_traits@G@std@@V?$allocator@G@2@@std@@@Z 0000000180018ec8     MsiDb.obj
 0002:00004ee4       $cppxdata$?openDatabase@?A0x6ccb95c8@msi@@YAKAEBV?$basic_string@GU?$char_traits@G@std@@V?$allocator@G@2@@std@@@Z 0000000180018ee4     MsiDb.obj
 0002:00004eed       $stateUnwindMap$?openDatabase@?A0x6ccb95c8@msi@@YAKAEBV?$basic_string@GU?$char_traits@G@std@@V?$allocator@G@2@@std@@@Z 0000000180018eed     MsiDb.obj
 0002:00004efa       $ip2state$?openDatabase@?A0x6ccb95c8@msi@@YAKAEBV?$basic_string@GU?$char_traits@G@std@@V?$allocator@G@2@@std@@@Z 0000000180018efa     MsiDb.obj
 0002:00004f04       $unwind$?closeMSIHANDLE@msi@@YAXK@Z 0000000180018f04     MsiUtils.obj
 0002:00004f1c       $cppxdata$?closeMSIHANDLE@msi@@YAXK@Z 0000000180018f1c     MsiUtils.obj
 0002:00004f25       $stateUnwindMap$?closeMSIHANDLE@msi@@YAXK@Z 0000000180018f25     MsiUtils.obj
 0002:00004f25       $stateUnwindMap$?id@ResourceEditor@@QEAAAEAV1@PEBG@Z 0000000180018f25     ResourceEditor.obj
 0002:00004f25       $stateUnwindMap$?type@ResourceEditor@@QEAAAEAV1@PEBG@Z 0000000180018f25     ResourceEditor.obj
 0002:00004f25       $stateUnwindMap$?init@Resource@@AEAAXPEBG0PEAUHINSTANCE__@@@Z 0000000180018f25     Resources.obj
 0002:00004f2c       $ip2state$?closeMSIHANDLE@msi@@YAXK@Z 0000000180018f2c     MsiUtils.obj
 0002:00004f34       $unwind$??0Error@msi@@QEAA@AEBVany@tstrings@@I@Z 0000000180018f34     MsiUtils.obj
 0002:00004f50       $cppxdata$??0Error@msi@@QEAA@AEBVany@tstrings@@I@Z 0000000180018f50     MsiUtils.obj
 0002:00004f59       $stateUnwindMap$??0Error@msi@@QEAA@AEBVany@tstrings@@I@Z 0000000180018f59     MsiUtils.obj
 0002:00004f66       $ip2state$??0Error@msi@@QEAA@AEBVany@tstrings@@I@Z 0000000180018f66     MsiUtils.obj
 0002:00004f70       $unwind$??0Error@msi@@QEAA@AEBV?$basic_string@DU?$char_traits@D@std@@V?$allocator@D@2@@std@@I@Z 0000000180018f70     MsiUtils.obj
 0002:00004f84       $unwind$?getString@DatabaseRecord@msi@@QEBA?AV?$basic_string@GU?$char_traits@G@std@@V?$allocator@G@2@@std@@I@Z 0000000180018f84     MsiUtils.obj
 0002:00004f8c       $unwind$??1?$unique_ptr@PEAUHINSTANCE__@@ULibraryReleaser@Dll@@@std@@QEAA@XZ 0000000180018f8c     MsiUtils.obj
 0002:00004f9c       $cppxdata$??1?$unique_ptr@PEAUHINSTANCE__@@ULibraryReleaser@Dll@@@std@@QEAA@XZ 0000000180018f9c     MsiUtils.obj
 0002:00004fa1       $ip2state$??1?$unique_ptr@PEAUHINSTANCE__@@ULibraryReleaser@Dll@@@std@@QEAA@XZ 0000000180018fa1     MsiUtils.obj
 0002:00004fa4       $unwind$??$getProperty@P6AIKIPEAGPEAK@ZKI@?A0x0e70828c@msi@@YA?AV?$basic_string@GU?$char_traits@G@std@@V?$allocator@G@2@@std@@P6AIKIPEAGPEAK@ZQEBDKI@Z 0000000180018fa4     MsiUtils.obj
 0002:00004fc8       $cppxdata$??$getProperty@P6AIKIPEAGPEAK@ZKI@?A0x0e70828c@msi@@YA?AV?$basic_string@GU?$char_traits@G@std@@V?$allocator@G@2@@std@@P6AIKIPEAGPEAK@ZQEBDKI@Z 0000000180018fc8     MsiUtils.obj
 0002:00004fd1       $stateUnwindMap$??$getProperty@P6AIKIPEAGPEAK@ZKI@?A0x0e70828c@msi@@YA?AV?$basic_string@GU?$char_traits@G@std@@V?$allocator@G@2@@std@@P6AIKIPEAGPEAK@ZQEBDKI@Z 0000000180018fd1     MsiUtils.obj
 0002:00004fe5       $ip2state$??$getProperty@P6AIKIPEAGPEAK@ZKI@?A0x0e70828c@msi@@YA?AV?$basic_string@GU?$char_traits@G@std@@V?$allocator@G@2@@std@@P6AIKIPEAGPEAK@ZQEBDKI@Z 0000000180018fe5     MsiUtils.obj
 0002:00004ff4       $unwind$?makeMessage@?A0x0e70828c@msi@@YA?AV?$basic_string@DU?$char_traits@D@std@@V?$allocator@D@2@@std@@AEBV34@I@Z 0000000180018ff4     MsiUtils.obj
 0002:00005018       $cppxdata$?makeMessage@?A0x0e70828c@msi@@YA?AV?$basic_string@DU?$char_traits@D@std@@V?$allocator@D@2@@std@@AEBV34@I@Z 0000000180019018     MsiUtils.obj
 0002:00005025       $stateUnwindMap$?makeMessage@?A0x0e70828c@msi@@YA?AV?$basic_string@DU?$char_traits@D@std@@V?$allocator@D@2@@std@@AEBV34@I@Z 0000000180019025     MsiUtils.obj
 0002:0000509f       $tryMap$?makeMessage@?A0x0e70828c@msi@@YA?AV?$basic_string@DU?$char_traits@D@std@@V?$allocator@D@2@@std@@AEBV34@I@Z 000000018001909f     MsiUtils.obj
 0002:000050a7       $handlerMap$?makeMessage@?A0x0e70828c@msi@@YA?AV?$basic_string@DU?$char_traits@D@std@@V?$allocator@D@2@@std@@AEBV34@I@Z 00000001800190a7     MsiUtils.obj
 0002:000050b4       $ip2state$?makeMessage@?A0x0e70828c@msi@@YA?AV?$basic_string@DU?$char_traits@D@std@@V?$allocator@D@2@@std@@AEBV34@I@Z 00000001800190b4     MsiUtils.obj
 0002:000050e0       $unwind$?catch$38@?0??makeMessage@?A0x0e70828c@msi@@YA?AV?$basic_string@DU?$char_traits@D@std@@V?$allocator@D@2@@std@@AEBV34@I@Z@4HA 00000001800190e0     MsiUtils.obj
 0002:000050e0       $unwind$Java_jdk_jpackage_internal_WindowsRegistry_openRegistryKey$catch$3 00000001800190e0     WindowsRegistry.obj
 0002:000050e0       $unwind$Java_jdk_jpackage_internal_WindowsRegistry_openRegistryKey$catch$4 00000001800190e0     WindowsRegistry.obj
 0002:000050e0       $unwind$Java_jdk_jpackage_internal_WindowsRegistry_readDwordValue$catch$4 00000001800190e0     WindowsRegistry.obj
 0002:000050e0       $unwind$Java_jdk_jpackage_internal_WindowsRegistry_readDwordValue$catch$5 00000001800190e0     WindowsRegistry.obj
 0002:000050e8       $unwind$??$_Construct_n@$$V@?$vector@GV?$allocator@G@std@@@std@@AEAAX_K@Z 00000001800190e8     MsiUtils.obj
 0002:000050f8       $unwind$??$_Resize_reallocate@U_Value_init_tag@std@@@?$vector@GV?$allocator@G@std@@@std@@AEAAX_KAEBU_Value_init_tag@1@@Z 00000001800190f8     MsiUtils.obj
 0002:00005110       $cppxdata$??$_Resize_reallocate@U_Value_init_tag@std@@@?$vector@GV?$allocator@G@std@@@std@@AEAAX_KAEBU_Value_init_tag@1@@Z 0000000180019110     MsiUtils.obj
 0002:0000511d       $tryMap$??$_Resize_reallocate@U_Value_init_tag@std@@@?$vector@GV?$allocator@G@std@@@std@@AEAAX_KAEBU_Value_init_tag@1@@Z 000000018001911d     MsiUtils.obj
 0002:00005125       $handlerMap$??$_Resize_reallocate@U_Value_init_tag@std@@@?$vector@GV?$allocator@G@std@@@std@@AEAAX_KAEBU_Value_init_tag@1@@Z 0000000180019125     MsiUtils.obj
 0002:0000512c       $ip2state$??$_Resize_reallocate@U_Value_init_tag@std@@@?$vector@GV?$allocator@G@std@@@std@@AEAAX_KAEBU_Value_init_tag@1@@Z 000000018001912c     MsiUtils.obj
 0002:00005134       $unwind$?appendFormatted@LogEvent@@CAXAEBUPlatformLogEvent@@AEAV?$basic_string@GU?$char_traits@G@std@@V?$allocator@G@2@@std@@@Z 0000000180019134     PlatformLogEvent.obj
 0002:00005154       $cppxdata$?appendFormatted@LogEvent@@CAXAEBUPlatformLogEvent@@AEAV?$basic_string@GU?$char_traits@G@std@@V?$allocator@G@2@@std@@@Z 0000000180019154     PlatformLogEvent.obj
 0002:0000515d       $stateUnwindMap$?appendFormatted@LogEvent@@CAXAEBUPlatformLogEvent@@AEAV?$basic_string@GU?$char_traits@G@std@@V?$allocator@G@2@@std@@@Z 000000018001915d     PlatformLogEvent.obj
 0002:00005164       $ip2state$?appendFormatted@LogEvent@@CAXAEBUPlatformLogEvent@@AEAV?$basic_string@GU?$char_traits@G@std@@V?$allocator@G@2@@std@@@Z 0000000180019164     PlatformLogEvent.obj
 0002:0000516c       $unwind$?initializeLogging@Logger@@CAXXZ 000000018001916c     PlatformLogEvent.obj
 0002:00005188       $cppxdata$?initializeLogging@Logger@@CAXXZ 0000000180019188     PlatformLogEvent.obj
 0002:00005191       $ip2state$?initializeLogging@Logger@@CAXXZ 0000000180019191     PlatformLogEvent.obj
 0002:00005198       $unwind$?retrieveModuleName@?A0x40e1fcfd@@YA?AV?$basic_string@GU?$char_traits@G@std@@V?$allocator@G@2@@std@@XZ 0000000180019198     PlatformLogEvent.obj
 0002:000051ac       $cppxdata$?retrieveModuleName@?A0x40e1fcfd@@YA?AV?$basic_string@GU?$char_traits@G@std@@V?$allocator@G@2@@std@@XZ 00000001800191ac     PlatformLogEvent.obj
 0002:000051b9       $stateUnwindMap$?retrieveModuleName@?A0x40e1fcfd@@YA?AV?$basic_string@GU?$char_traits@G@std@@V?$allocator@G@2@@std@@XZ 00000001800191b9     PlatformLogEvent.obj
 0002:000051c2       $tryMap$?retrieveModuleName@?A0x40e1fcfd@@YA?AV?$basic_string@GU?$char_traits@G@std@@V?$allocator@G@2@@std@@XZ 00000001800191c2     PlatformLogEvent.obj
 0002:000051ca       $handlerMap$?retrieveModuleName@?A0x40e1fcfd@@YA?AV?$basic_string@GU?$char_traits@G@std@@V?$allocator@G@2@@std@@XZ 00000001800191ca     PlatformLogEvent.obj
 0002:000051d6       $ip2state$?retrieveModuleName@?A0x40e1fcfd@@YA?AV?$basic_string@GU?$char_traits@G@std@@V?$allocator@G@2@@std@@XZ 00000001800191d6     PlatformLogEvent.obj
 0002:000051e0       $unwind$?catch$5@?0??retrieveModuleName@?A0x40e1fcfd@@YA?AV?$basic_string@GU?$char_traits@G@std@@V?$allocator@G@2@@std@@XZ@4HA 00000001800191e0     PlatformLogEvent.obj
 0002:000051ec       $unwind$??0FileLock@ResourceEditor@@QEAA@AEBV?$basic_string@GU?$char_traits@G@std@@V?$allocator@G@2@@std@@@Z 00000001800191ec     ResourceEditor.obj
 0002:0000520c       $cppxdata$??0FileLock@ResourceEditor@@QEAA@AEBV?$basic_string@GU?$char_traits@G@std@@V?$allocator@G@2@@std@@@Z 000000018001920c     ResourceEditor.obj
 0002:00005215       $stateUnwindMap$??0FileLock@ResourceEditor@@QEAA@AEBV?$basic_string@GU?$char_traits@G@std@@V?$allocator@G@2@@std@@@Z 0000000180019215     ResourceEditor.obj
 0002:00005222       $ip2state$??0FileLock@ResourceEditor@@QEAA@AEBV?$basic_string@GU?$char_traits@G@std@@V?$allocator@G@2@@std@@@Z 0000000180019222     ResourceEditor.obj
 0002:0000522c       $unwind$??1FileLock@ResourceEditor@@QEAA@XZ 000000018001922c     ResourceEditor.obj
 0002:00005244       $cppxdata$??1FileLock@ResourceEditor@@QEAA@XZ 0000000180019244     ResourceEditor.obj
 0002:00005251       $stateUnwindMap$??1FileLock@ResourceEditor@@QEAA@XZ 0000000180019251     ResourceEditor.obj
 0002:00005260       $tryMap$??1FileLock@ResourceEditor@@QEAA@XZ 0000000180019260     ResourceEditor.obj
 0002:00005268       $handlerMap$??1FileLock@ResourceEditor@@QEAA@XZ 0000000180019268     ResourceEditor.obj
 0002:0000527c       $ip2state$??1FileLock@ResourceEditor@@QEAA@XZ 000000018001927c     ResourceEditor.obj
 0002:00005288       $unwind$?catch$5@?0???1FileLock@ResourceEditor@@QEAA@XZ@4HA 0000000180019288     ResourceEditor.obj
 0002:00005298       $cppxdata$?catch$5@?0???1FileLock@ResourceEditor@@QEAA@XZ@4HA 0000000180019298     ResourceEditor.obj
 0002:000052a4       $unwind$?catch$6@?0???1FileLock@ResourceEditor@@QEAA@XZ@4HA 00000001800192a4     ResourceEditor.obj
 0002:000052b4       $cppxdata$?catch$6@?0???1FileLock@ResourceEditor@@QEAA@XZ@4HA 00000001800192b4     ResourceEditor.obj
 0002:000052c0       $unwind$??0ResourceEditor@@QEAA@XZ 00000001800192c0     ResourceEditor.obj
 0002:000052d0       $cppxdata$??0ResourceEditor@@QEAA@XZ 00000001800192d0     ResourceEditor.obj
 0002:000052d9       $stateUnwindMap$??0ResourceEditor@@QEAA@XZ 00000001800192d9     ResourceEditor.obj
 0002:000052e4       $ip2state$??0ResourceEditor@@QEAA@XZ 00000001800192e4     ResourceEditor.obj
 0002:000052ec       $unwind$?type@ResourceEditor@@QEAAAEAV1@PEBG@Z 00000001800192ec     ResourceEditor.obj
 0002:0000530c       $cppxdata$?type@ResourceEditor@@QEAAAEAV1@PEBG@Z 000000018001930c     ResourceEditor.obj
 0002:00005315       $ip2state$?type@ResourceEditor@@QEAAAEAV1@PEBG@Z 0000000180019315     ResourceEditor.obj
 0002:0000531c       $unwind$?id@ResourceEditor@@QEAAAEAV1@PEBG@Z 000000018001931c     ResourceEditor.obj
 0002:0000533c       $cppxdata$?id@ResourceEditor@@QEAAAEAV1@PEBG@Z 000000018001933c     ResourceEditor.obj
 0002:00005345       $ip2state$?id@ResourceEditor@@QEAAAEAV1@PEBG@Z 0000000180019345     ResourceEditor.obj
 0002:0000534c       $unwind$?apply@ResourceEditor@@QEAAAEAV1@AEBVFileLock@1@AEAV?$basic_istream@DU?$char_traits@D@std@@@std@@_J@Z 000000018001934c     ResourceEditor.obj
 0002:0000536c       $cppxdata$?apply@ResourceEditor@@QEAAAEAV1@AEBVFileLock@1@AEAV?$basic_istream@DU?$char_traits@D@std@@@std@@_J@Z 000000018001936c     ResourceEditor.obj
 0002:00005375       $stateUnwindMap$?apply@ResourceEditor@@QEAAAEAV1@AEBVFileLock@1@AEAV?$basic_istream@DU?$char_traits@D@std@@@std@@_J@Z 0000000180019375     ResourceEditor.obj
 0002:00005391       $ip2state$?apply@ResourceEditor@@QEAAAEAV1@AEBVFileLock@1@AEAV?$basic_istream@DU?$char_traits@D@std@@@std@@_J@Z 0000000180019391     ResourceEditor.obj
 0002:000053a0       $unwind$?apply@ResourceEditor@@QEAAAEAV1@AEBVFileLock@1@AEBV?$basic_string@GU?$char_traits@G@std@@V?$allocator@G@2@@std@@@Z 00000001800193a0     ResourceEditor.obj
 0002:000053b8       $cppxdata$?apply@ResourceEditor@@QEAAAEAV1@AEBVFileLock@1@AEBV?$basic_string@GU?$char_traits@G@std@@V?$allocator@G@2@@std@@@Z 00000001800193b8     ResourceEditor.obj
 0002:000053c1       $stateUnwindMap$?apply@ResourceEditor@@QEAAAEAV1@AEBVFileLock@1@AEBV?$basic_string@GU?$char_traits@G@std@@V?$allocator@G@2@@std@@@Z 00000001800193c1     ResourceEditor.obj
 0002:000053c8       $ip2state$?apply@ResourceEditor@@QEAAAEAV1@AEBVFileLock@1@AEBV?$basic_string@GU?$char_traits@G@std@@V?$allocator@G@2@@std@@@Z 00000001800193c8     ResourceEditor.obj
 0002:000053d0       $unwind$??0?$basic_ifstream@DU?$char_traits@D@std@@@std@@QEAA@PEBGHH@Z 00000001800193d0     ResourceEditor.obj
 0002:000053ec       $cppxdata$??0?$basic_ifstream@DU?$char_traits@D@std@@@std@@QEAA@PEBGHH@Z 00000001800193ec     ResourceEditor.obj
 0002:000053f5       $stateUnwindMap$??0?$basic_ifstream@DU?$char_traits@D@std@@@std@@QEAA@PEBGHH@Z 00000001800193f5     ResourceEditor.obj
 0002:00005405       $ip2state$??0?$basic_ifstream@DU?$char_traits@D@std@@@std@@QEAA@PEBGHH@Z 0000000180019405     ResourceEditor.obj
 0002:00005410       $unwind$?open@?$basic_filebuf@DU?$char_traits@D@std@@@std@@QEAAPEAV12@PEBGHH@Z 0000000180019410     ResourceEditor.obj
 0002:00005424       $cppxdata$?open@?$basic_filebuf@DU?$char_traits@D@std@@@std@@QEAAPEAV12@PEBGHH@Z 0000000180019424     ResourceEditor.obj
 0002:0000542d       $stateUnwindMap$?open@?$basic_filebuf@DU?$char_traits@D@std@@@std@@QEAAPEAV12@PEBGHH@Z 000000018001942d     ResourceEditor.obj
 0002:00005434       $ip2state$?open@?$basic_filebuf@DU?$char_traits@D@std@@@std@@QEAAPEAV12@PEBGHH@Z 0000000180019434     ResourceEditor.obj
 0002:0000543c       $unwind$??$_Append_uncounted_range@V?$istreambuf_iterator@DU?$char_traits@D@std@@@std@@V12@@?$vector@EV?$allocator@E@std@@@std@@AEAAXV?$istreambuf_iterator@DU?$char_traits@D@std@@@1@V21@@Z 000000018001943c     ResourceEditor.obj
 0002:00005454       $unwind$??$_Resize_reallocate@U_Value_init_tag@std@@@?$vector@EV?$allocator@E@std@@@std@@AEAAX_KAEBU_Value_init_tag@1@@Z 0000000180019454     ResourceEditor.obj
 0002:00005470       $cppxdata$??$_Resize_reallocate@U_Value_init_tag@std@@@?$vector@EV?$allocator@E@std@@@std@@AEAAX_KAEBU_Value_init_tag@1@@Z 0000000180019470     ResourceEditor.obj
 0002:0000547d       $tryMap$??$_Resize_reallocate@U_Value_init_tag@std@@@?$vector@EV?$allocator@E@std@@@std@@AEAAX_KAEBU_Value_init_tag@1@@Z 000000018001947d     ResourceEditor.obj
 0002:00005485       $handlerMap$??$_Resize_reallocate@U_Value_init_tag@std@@@?$vector@EV?$allocator@E@std@@@std@@AEAAX_KAEBU_Value_init_tag@1@@Z 0000000180019485     ResourceEditor.obj
 0002:0000548c       $ip2state$??$_Resize_reallocate@U_Value_init_tag@std@@@?$vector@EV?$allocator@E@std@@@std@@AEAAX_KAEBU_Value_init_tag@1@@Z 000000018001948c     ResourceEditor.obj
 0002:00005494       $unwind$??$_Emplace_reallocate@D@?$vector@EV?$allocator@E@std@@@std@@AEAAPEAEQEAE$$QEAD@Z 0000000180019494     ResourceEditor.obj
 0002:000054b0       $cppxdata$??$_Emplace_reallocate@D@?$vector@EV?$allocator@E@std@@@std@@AEAAPEAEQEAE$$QEAD@Z 00000001800194b0     ResourceEditor.obj
 0002:000054bd       $tryMap$??$_Emplace_reallocate@D@?$vector@EV?$allocator@E@std@@@std@@AEAAPEAEQEAE$$QEAD@Z 00000001800194bd     ResourceEditor.obj
 0002:000054c5       $handlerMap$??$_Emplace_reallocate@D@?$vector@EV?$allocator@E@std@@@std@@AEAAPEAEQEAE$$QEAD@Z 00000001800194c5     ResourceEditor.obj
 0002:000054cc       $ip2state$??$_Emplace_reallocate@D@?$vector@EV?$allocator@E@std@@@std@@AEAAPEAEQEAE$$QEAD@Z 00000001800194cc     ResourceEditor.obj
 0002:000054d4       $unwind$??0any@tstrings@@QEAA@AEBV?$basic_string@DU?$char_traits@D@std@@V?$allocator@D@2@@std@@@Z 00000001800194d4     Resources.obj
 0002:000054ec       $cppxdata$??0any@tstrings@@QEAA@AEBV?$basic_string@DU?$char_traits@D@std@@V?$allocator@D@2@@std@@@Z 00000001800194ec     Resources.obj
 0002:000054f5       $stateUnwindMap$??0any@tstrings@@QEAA@AEBV?$basic_string@DU?$char_traits@D@std@@V?$allocator@D@2@@std@@@Z 00000001800194f5     Resources.obj
 0002:00005502       $ip2state$??0any@tstrings@@QEAA@AEBV?$basic_string@DU?$char_traits@D@std@@V?$allocator@D@2@@std@@@Z 0000000180019502     Resources.obj
 0002:0000550c       $unwind$??0Resource@@QEAA@IPEBGPEAUHINSTANCE__@@@Z 000000018001950c     Resources.obj
 0002:0000551c       $cppxdata$??0Resource@@QEAA@IPEBGPEAUHINSTANCE__@@@Z 000000018001951c     Resources.obj
 0002:00005525       $stateUnwindMap$??0Resource@@QEAA@IPEBGPEAUHINSTANCE__@@@Z 0000000180019525     Resources.obj
 0002:00005531       $ip2state$??0Resource@@QEAA@IPEBGPEAUHINSTANCE__@@@Z 0000000180019531     Resources.obj
 0002:00005534       $unwind$?init@Resource@@AEAAXPEBG0PEAUHINSTANCE__@@@Z 0000000180019534     Resources.obj
 0002:00005558       $cppxdata$?init@Resource@@AEAAXPEBG0PEAUHINSTANCE__@@@Z 0000000180019558     Resources.obj
 0002:00005561       $ip2state$?init@Resource@@AEAAXPEBG0PEAUHINSTANCE__@@@Z 0000000180019561     Resources.obj
 0002:0000556c       $unwind$?getErrMsg@Resource@@AEBA?AV?$basic_string@DU?$char_traits@D@std@@V?$allocator@D@2@@std@@AEBV23@@Z 000000018001956c     Resources.obj
 0002:0000558c       $cppxdata$?getErrMsg@Resource@@AEBA?AV?$basic_string@DU?$char_traits@D@std@@V?$allocator@D@2@@std@@AEBV23@@Z 000000018001958c     Resources.obj
 0002:00005595       $stateUnwindMap$?getErrMsg@Resource@@AEBA?AV?$basic_string@DU?$char_traits@D@std@@V?$allocator@D@2@@std@@AEBV23@@Z 0000000180019595     Resources.obj
 0002:000055a3       $ip2state$?getErrMsg@Resource@@AEBA?AV?$basic_string@DU?$char_traits@D@std@@V?$allocator@D@2@@std@@AEBV23@@Z 00000001800195a3     Resources.obj
 0002:000055b4       $unwind$?getPtr@Resource@@AEBAPEAXAEAK@Z 00000001800195b4     Resources.obj
 0002:000055d8       $cppxdata$?getPtr@Resource@@AEBAPEAXAEAK@Z 00000001800195d8     Resources.obj
 0002:000055e1       $stateUnwindMap$?getPtr@Resource@@AEBAPEAXAEAK@Z 00000001800195e1     Resources.obj
 0002:00005607       $ip2state$?getPtr@Resource@@AEBAPEAXAEAK@Z 0000000180019607     Resources.obj
 0002:00005620       $unwind$?string@StringResource@@QEBA?AV?$basic_string@GU?$char_traits@G@std@@V?$allocator@G@2@@std@@XZ 0000000180019620     Resources.obj
 0002:00005644       $cppxdata$?string@StringResource@@QEBA?AV?$basic_string@GU?$char_traits@G@std@@V?$allocator@G@2@@std@@XZ 0000000180019644     Resources.obj
 0002:0000564d       $stateUnwindMap$?string@StringResource@@QEBA?AV?$basic_string@GU?$char_traits@G@std@@V?$allocator@G@2@@std@@XZ 000000018001964d     Resources.obj
 0002:00005654       $ip2state$?string@StringResource@@QEBA?AV?$basic_string@GU?$char_traits@G@std@@V?$allocator@G@2@@std@@XZ 0000000180019654     Resources.obj
 0002:0000565c       $unwind$swscanf_s          000000018001965c     VersionInfo.obj
 0002:00005668       $unwind$?setProperty@VersionInfo@@QEAAAEAV1@AEBV?$basic_string@GU?$char_traits@G@std@@V?$allocator@G@2@@std@@0@Z 0000000180019668     VersionInfo.obj
 0002:0000567c       $unwind$?apply@VersionInfo@@QEBAAEBV1@AEBVFileLock@ResourceEditor@@@Z 000000018001967c     VersionInfo.obj
 0002:000056a0       $cppxdata$?apply@VersionInfo@@QEBAAEBV1@AEBVFileLock@ResourceEditor@@@Z 00000001800196a0     VersionInfo.obj
 0002:000056a9       $stateUnwindMap$?apply@VersionInfo@@QEBAAEBV1@AEBVFileLock@ResourceEditor@@@Z 00000001800196a9     VersionInfo.obj
 0002:000056b7       $ip2state$?apply@VersionInfo@@QEBAAEBV1@AEBVFileLock@ResourceEditor@@@Z 00000001800196b7     VersionInfo.obj
 0002:000056c4       $unwind$?fillBuffer@VersionInfo@@AEBAXAEAV?$basic_ostream@DU?$char_traits@D@std@@@std@@@Z 00000001800196c4     VersionInfo.obj
 0002:000056e8       $cppxdata$?fillBuffer@VersionInfo@@AEBAXAEAV?$basic_ostream@DU?$char_traits@D@std@@@std@@@Z 00000001800196e8     VersionInfo.obj
 0002:000056f1       $stateUnwindMap$?fillBuffer@VersionInfo@@AEBAXAEAV?$basic_ostream@DU?$char_traits@D@std@@@std@@@Z 00000001800196f1     VersionInfo.obj
 0002:00005744       $ip2state$?fillBuffer@VersionInfo@@AEBAXAEAV?$basic_ostream@DU?$char_traits@D@std@@@std@@@Z 0000000180019744     VersionInfo.obj
 0002:00005774       $unwind$?createFIXEDFILEINFO@VersionInfo@@AEBA?AUtagVS_FIXEDFILEINFO@@XZ 0000000180019774     VersionInfo.obj
 0002:00005790       $cppxdata$?createFIXEDFILEINFO@VersionInfo@@AEBA?AUtagVS_FIXEDFILEINFO@@XZ 0000000180019790     VersionInfo.obj
 0002:0000579d       $stateUnwindMap$?createFIXEDFILEINFO@VersionInfo@@AEBA?AUtagVS_FIXEDFILEINFO@@XZ 000000018001979d     VersionInfo.obj
 0002:000057a6       $tryMap$?createFIXEDFILEINFO@VersionInfo@@AEBA?AUtagVS_FIXEDFILEINFO@@XZ 00000001800197a6     VersionInfo.obj
 0002:000057ae       $handlerMap$?createFIXEDFILEINFO@VersionInfo@@AEBA?AUtagVS_FIXEDFILEINFO@@XZ 00000001800197ae     VersionInfo.obj
 0002:000057bb       $ip2state$?createFIXEDFILEINFO@VersionInfo@@AEBA?AUtagVS_FIXEDFILEINFO@@XZ 00000001800197bb     VersionInfo.obj
 0002:000057c8       $unwind$??0FixedFileVersion@?A0xcb1fbc16@@QEAA@AEBV?$basic_string@GU?$char_traits@G@std@@V?$allocator@G@2@@std@@@Z 00000001800197c8     VersionInfo.obj
 0002:000057e8       $cppxdata$??0FixedFileVersion@?A0xcb1fbc16@@QEAA@AEBV?$basic_string@GU?$char_traits@G@std@@V?$allocator@G@2@@std@@@Z 00000001800197e8     VersionInfo.obj
 0002:000057f1       $stateUnwindMap$??0FixedFileVersion@?A0xcb1fbc16@@QEAA@AEBV?$basic_string@GU?$char_traits@G@std@@V?$allocator@G@2@@std@@@Z 00000001800197f1     VersionInfo.obj
 0002:000057f8       $ip2state$??0FixedFileVersion@?A0xcb1fbc16@@QEAA@AEBV?$basic_string@GU?$char_traits@G@std@@V?$allocator@G@2@@std@@@Z 00000001800197f8     VersionInfo.obj
 0002:00005800       $unwind$?add32bitPadding@?A0xcb1fbc16@@YAXAEAV?$basic_ostream@DU?$char_traits@D@std@@@std@@@Z 0000000180019800     VersionInfo.obj
 0002:00005818       $unwind$??1StreamSize@?A0xcb1fbc16@@QEAA@XZ 0000000180019818     VersionInfo.obj
 0002:00005838       $cppxdata$??1StreamSize@?A0xcb1fbc16@@QEAA@XZ 0000000180019838     VersionInfo.obj
 0002:00005845       $tryMap$??1StreamSize@?A0xcb1fbc16@@QEAA@XZ 0000000180019845     VersionInfo.obj
 0002:0000584d       $handlerMap$??1StreamSize@?A0xcb1fbc16@@QEAA@XZ 000000018001984d     VersionInfo.obj
 0002:00005863       $ip2state$??1StreamSize@?A0xcb1fbc16@@QEAA@XZ 0000000180019863     VersionInfo.obj
 0002:0000586c       $unwind$??0?$basic_stringstream@DU?$char_traits@D@std@@V?$allocator@D@2@@std@@QEAA@H@Z 000000018001986c     VersionInfo.obj
 0002:00005880       $cppxdata$??0?$basic_stringstream@DU?$char_traits@D@std@@V?$allocator@D@2@@std@@QEAA@H@Z 0000000180019880     VersionInfo.obj
 0002:00005889       $stateUnwindMap$??0?$basic_stringstream@DU?$char_traits@D@std@@V?$allocator@D@2@@std@@QEAA@H@Z 0000000180019889     VersionInfo.obj
 0002:00005894       $ip2state$??0?$basic_stringstream@DU?$char_traits@D@std@@V?$allocator@D@2@@std@@QEAA@H@Z 0000000180019894     VersionInfo.obj
 0002:00005894       $ip2state$??0?$basic_stringstream@GU?$char_traits@G@std@@V?$allocator@G@2@@std@@QEAA@XZ 0000000180019894     VersionInfo.obj
 0002:0000589c       $unwind$??0?$basic_stringstream@GU?$char_traits@G@std@@V?$allocator@G@2@@std@@QEAA@XZ 000000018001989c     VersionInfo.obj
 0002:000058b0       $cppxdata$??0?$basic_stringstream@GU?$char_traits@G@std@@V?$allocator@G@2@@std@@QEAA@XZ 00000001800198b0     VersionInfo.obj
 0002:000058b9       $stateUnwindMap$??0?$basic_stringstream@GU?$char_traits@G@std@@V?$allocator@G@2@@std@@QEAA@XZ 00000001800198b9     VersionInfo.obj
 0002:000058c4       $unwind$??$_Traits_rfind@U?$char_traits@G@std@@@std@@YA_KQEBG_K101@Z 00000001800198c4     VersionInfo.obj
 0002:000058d4       $unwind$??0SysError@@QEAA@AEBVany@tstrings@@PEBXKPEBD@Z 00000001800198d4     WinErrorHandling.obj
 0002:000058f4       $cppxdata$??0SysError@@QEAA@AEBVany@tstrings@@PEBXKPEBD@Z 00000001800198f4     WinErrorHandling.obj
 0002:000058fd       $stateUnwindMap$??0SysError@@QEAA@AEBVany@tstrings@@PEBXKPEBD@Z 00000001800198fd     WinErrorHandling.obj
 0002:0000590a       $ip2state$??0SysError@@QEAA@AEBVany@tstrings@@PEBXKPEBD@Z 000000018001990a     WinErrorHandling.obj
 0002:00005914       $unwind$?getSysErrorMessage@SysError@@SA?AV?$basic_string@GU?$char_traits@G@std@@V?$allocator@G@2@@std@@KPEAUHINSTANCE__@@@Z 0000000180019914     WinErrorHandling.obj
 0002:00005934       $cppxdata$?getSysErrorMessage@SysError@@SA?AV?$basic_string@GU?$char_traits@G@std@@V?$allocator@G@2@@std@@KPEAUHINSTANCE__@@@Z 0000000180019934     WinErrorHandling.obj
 0002:0000593d       $stateUnwindMap$?getSysErrorMessage@SysError@@SA?AV?$basic_string@GU?$char_traits@G@std@@V?$allocator@G@2@@std@@KPEAUHINSTANCE__@@@Z 000000018001993d     WinErrorHandling.obj
 0002:0000594b       $ip2state$?getSysErrorMessage@SysError@@SA?AV?$basic_string@GU?$char_traits@G@std@@V?$allocator@G@2@@std@@KPEAUHINSTANCE__@@@Z 000000018001994b     WinErrorHandling.obj
 0002:00005958       $unwind$?makeMessage@?A0xd5983087@@YA?AV?$basic_string@DU?$char_traits@D@std@@V?$allocator@D@2@@std@@AEBV23@PEBDPEBXK@Z 0000000180019958     WinErrorHandling.obj
 0002:00005978       $cppxdata$?makeMessage@?A0xd5983087@@YA?AV?$basic_string@DU?$char_traits@D@std@@V?$allocator@D@2@@std@@AEBV23@PEBDPEBXK@Z 0000000180019978     WinErrorHandling.obj
 0002:00005981       $stateUnwindMap$?makeMessage@?A0xd5983087@@YA?AV?$basic_string@DU?$char_traits@D@std@@V?$allocator@D@2@@std@@AEBV23@PEBDPEBXK@Z 0000000180019981     WinErrorHandling.obj
 0002:000059aa       $ip2state$?makeMessage@?A0xd5983087@@YA?AV?$basic_string@DU?$char_traits@D@std@@V?$allocator@D@2@@std@@AEBV23@PEBDPEBXK@Z 00000001800199aa     WinErrorHandling.obj
 0002:000059c4       $unwind$?getSystemMessageDescription@?A0xd5983087@@YA?AV?$basic_string@GU?$char_traits@G@std@@V?$allocator@G@2@@std@@KPEAUHINSTANCE__@@@Z 00000001800199c4     WinErrorHandling.obj
 0002:000059dc       $cppxdata$?getSystemMessageDescription@?A0xd5983087@@YA?AV?$basic_string@GU?$char_traits@G@std@@V?$allocator@G@2@@std@@KPEAUHINSTANCE__@@@Z 00000001800199dc     WinErrorHandling.obj
 0002:000059e5       $stateUnwindMap$?getSystemMessageDescription@?A0xd5983087@@YA?AV?$basic_string@GU?$char_traits@G@std@@V?$allocator@G@2@@std@@KPEAUHINSTANCE__@@@Z 00000001800199e5     WinErrorHandling.obj
 0002:000059eb       $ip2state$?getSystemMessageDescription@?A0xd5983087@@YA?AV?$basic_string@GU?$char_traits@G@std@@V?$allocator@G@2@@std@@KPEAUHINSTANCE__@@@Z 00000001800199eb     WinErrorHandling.obj
 0002:000059f0       $unwind$?toShortPath@FileUtils@@YA?AV?$basic_string@GU?$char_traits@G@std@@V?$allocator@G@2@@std@@AEBV23@@Z 00000001800199f0     WinFileUtils.obj
 0002:00005a14       $cppxdata$?toShortPath@FileUtils@@YA?AV?$basic_string@GU?$char_traits@G@std@@V?$allocator@G@2@@std@@AEBV23@@Z 0000000180019a14     WinFileUtils.obj
 0002:00005a1d       $stateUnwindMap$?toShortPath@FileUtils@@YA?AV?$basic_string@GU?$char_traits@G@std@@V?$allocator@G@2@@std@@AEBV23@@Z 0000000180019a1d     WinFileUtils.obj
 0002:00005a3e       $ip2state$?toShortPath@FileUtils@@YA?AV?$basic_string@GU?$char_traits@G@std@@V?$allocator@G@2@@std@@AEBV23@@Z 0000000180019a3e     WinFileUtils.obj
 0002:00005a50       $unwind$?getSystem32Dir@SysInfo@@YA?AV?$basic_string@GU?$char_traits@G@std@@V?$allocator@G@2@@std@@XZ 0000000180019a50     WinSysInfo.obj
 0002:00005a64       $cppxdata$?getSystem32Dir@SysInfo@@YA?AV?$basic_string@GU?$char_traits@G@std@@V?$allocator@G@2@@std@@XZ 0000000180019a64     WinSysInfo.obj
 0002:00005a6d       $ip2state$?getSystem32Dir@SysInfo@@YA?AV?$basic_string@GU?$char_traits@G@std@@V?$allocator@G@2@@std@@XZ 0000000180019a6d     WinSysInfo.obj
 0002:00005a74       $unwind$?getCurrentModuleHandle@SysInfo@@YAPEAUHINSTANCE__@@XZ 0000000180019a74     WinSysInfo.obj
 0002:00005a90       $cppxdata$?getCurrentModuleHandle@SysInfo@@YAPEAUHINSTANCE__@@XZ 0000000180019a90     WinSysInfo.obj
 0002:00005a99       $stateUnwindMap$?getCurrentModuleHandle@SysInfo@@YAPEAUHINSTANCE__@@XZ 0000000180019a99     WinSysInfo.obj
 0002:00005aa6       $ip2state$?getCurrentModuleHandle@SysInfo@@YAPEAUHINSTANCE__@@XZ 0000000180019aa6     WinSysInfo.obj
 0002:00005ab0       $unwind$??$?HDU?$char_traits@D@std@@V?$allocator@D@1@@std@@YA?AV?$basic_string@DU?$char_traits@D@std@@V?$allocator@D@2@@0@AEBV10@QEBD@Z 0000000180019ab0     WinSysInfo.obj
 0002:00005ac4       $unwind$??$getSystemDirImpl@P6AIPEAGI@Z@?A0x7970c2a6@SysInfo@@YA?AV?$basic_string@GU?$char_traits@G@std@@V?$allocator@G@2@@std@@P6AIPEAGI@ZAEBV?$basic_string@DU?$char_traits@D@std@@V?$allocator@D@2@@3@@Z 0000000180019ac4     WinSysInfo.obj
 0002:00005ae8       $cppxdata$??$getSystemDirImpl@P6AIPEAGI@Z@?A0x7970c2a6@SysInfo@@YA?AV?$basic_string@GU?$char_traits@G@std@@V?$allocator@G@2@@std@@P6AIPEAGI@ZAEBV?$basic_string@DU?$char_traits@D@std@@V?$allocator@D@2@@3@@Z 0000000180019ae8     WinSysInfo.obj
 0002:00005af1       $stateUnwindMap$??$getSystemDirImpl@P6AIPEAGI@Z@?A0x7970c2a6@SysInfo@@YA?AV?$basic_string@GU?$char_traits@G@std@@V?$allocator@G@2@@std@@P6AIPEAGI@ZAEBV?$basic_string@DU?$char_traits@D@std@@V?$allocator@D@2@@3@@Z 0000000180019af1     WinSysInfo.obj
 0002:00005b1a       $ip2state$??$getSystemDirImpl@P6AIPEAGI@Z@?A0x7970c2a6@SysInfo@@YA?AV?$basic_string@GU?$char_traits@G@std@@V?$allocator@G@2@@std@@P6AIPEAGI@ZAEBV?$basic_string@DU?$char_traits@D@std@@V?$allocator@D@2@@3@@Z 0000000180019b1a     WinSysInfo.obj
 0002:00005b34       $unwind$?getModulePath@?A0x7970c2a6@SysInfo@@YA?AV?$basic_string@GU?$char_traits@G@std@@V?$allocator@G@2@@std@@PEAUHINSTANCE__@@@Z 0000000180019b34     WinSysInfo.obj
 0002:00005b54       $cppxdata$?getModulePath@?A0x7970c2a6@SysInfo@@YA?AV?$basic_string@GU?$char_traits@G@std@@V?$allocator@G@2@@std@@PEAUHINSTANCE__@@@Z 0000000180019b54     WinSysInfo.obj
 0002:00005b5d       $stateUnwindMap$?getModulePath@?A0x7970c2a6@SysInfo@@YA?AV?$basic_string@GU?$char_traits@G@std@@V?$allocator@G@2@@std@@PEAUHINSTANCE__@@@Z 0000000180019b5d     WinSysInfo.obj
 0002:00005b71       $ip2state$?getModulePath@?A0x7970c2a6@SysInfo@@YA?AV?$basic_string@GU?$char_traits@G@std@@V?$allocator@G@2@@std@@PEAUHINSTANCE__@@@Z 0000000180019b71     WinSysInfo.obj
 0002:00005b80       $unwind$?GetLongPath@?A0x764c93a3@@YA?AV?$basic_string@GU?$char_traits@G@std@@V?$allocator@G@2@@std@@AEBV23@@Z 0000000180019b80     WindowsRegistry.obj
 0002:00005ba8       $cppxdata$?GetLongPath@?A0x764c93a3@@YA?AV?$basic_string@GU?$char_traits@G@std@@V?$allocator@G@2@@std@@AEBV23@@Z 0000000180019ba8     WindowsRegistry.obj
 0002:00005bb1       $stateUnwindMap$?GetLongPath@?A0x764c93a3@@YA?AV?$basic_string@GU?$char_traits@G@std@@V?$allocator@G@2@@std@@AEBV23@@Z 0000000180019bb1     WindowsRegistry.obj
 0002:00005bbe       $ip2state$?GetLongPath@?A0x764c93a3@@YA?AV?$basic_string@GU?$char_traits@G@std@@V?$allocator@G@2@@std@@AEBV23@@Z 0000000180019bbe     WindowsRegistry.obj
 0002:00005bcc       $unwind$Java_jdk_jpackage_internal_WindowsRegistry_readDwordValue 0000000180019bcc     WindowsRegistry.obj
 0002:00005bec       $cppxdata$Java_jdk_jpackage_internal_WindowsRegistry_readDwordValue 0000000180019bec     WindowsRegistry.obj
 0002:00005bf9       $stateUnwindMap$Java_jdk_jpackage_internal_WindowsRegistry_readDwordValue 0000000180019bf9     WindowsRegistry.obj
 0002:00005c03       $tryMap$Java_jdk_jpackage_internal_WindowsRegistry_readDwordValue 0000000180019c03     WindowsRegistry.obj
 0002:00005c0b       $handlerMap$Java_jdk_jpackage_internal_WindowsRegistry_readDwordValue 0000000180019c0b     WindowsRegistry.obj
 0002:00005c21       $ip2state$Java_jdk_jpackage_internal_WindowsRegistry_readDwordValue 0000000180019c21     WindowsRegistry.obj
 0002:00005c30       $unwind$Java_jdk_jpackage_internal_WindowsRegistry_openRegistryKey 0000000180019c30     WindowsRegistry.obj
 0002:00005c48       $cppxdata$Java_jdk_jpackage_internal_WindowsRegistry_openRegistryKey 0000000180019c48     WindowsRegistry.obj
 0002:00005c55       $tryMap$Java_jdk_jpackage_internal_WindowsRegistry_openRegistryKey 0000000180019c55     WindowsRegistry.obj
 0002:00005c5d       $handlerMap$Java_jdk_jpackage_internal_WindowsRegistry_openRegistryKey 0000000180019c5d     WindowsRegistry.obj
 0002:00005c73       $ip2state$Java_jdk_jpackage_internal_WindowsRegistry_openRegistryKey 0000000180019c73     WindowsRegistry.obj
 0002:00005c7c       $unwind$Java_jdk_jpackage_internal_WindowsRegistry_enumRegistryValue 0000000180019c7c     WindowsRegistry.obj
 0002:00005c9c       $cppxdata$Java_jdk_jpackage_internal_WindowsRegistry_enumRegistryValue 0000000180019c9c     WindowsRegistry.obj
 0002:00005ca9       $stateUnwindMap$Java_jdk_jpackage_internal_WindowsRegistry_enumRegistryValue 0000000180019ca9     WindowsRegistry.obj
 0002:00005cb2       $tryMap$Java_jdk_jpackage_internal_WindowsRegistry_enumRegistryValue 0000000180019cb2     WindowsRegistry.obj
 0002:00005cba       $handlerMap$Java_jdk_jpackage_internal_WindowsRegistry_enumRegistryValue 0000000180019cba     WindowsRegistry.obj
 0002:00005cd0       $ip2state$Java_jdk_jpackage_internal_WindowsRegistry_enumRegistryValue 0000000180019cd0     WindowsRegistry.obj
 0002:00005ce0       $unwind$Java_jdk_jpackage_internal_WindowsRegistry_enumRegistryValue$catch$4 0000000180019ce0     WindowsRegistry.obj
 0002:00005ce0       $unwind$Java_jdk_jpackage_internal_WindowsRegistry_enumRegistryValue$catch$5 0000000180019ce0     WindowsRegistry.obj
 0002:00005ce8       $unwind$Java_jdk_jpackage_internal_WindowsRegistry_comparePaths 0000000180019ce8     WindowsRegistry.obj
 0002:00005d04       $cppxdata$Java_jdk_jpackage_internal_WindowsRegistry_comparePaths 0000000180019d04     WindowsRegistry.obj
 0002:00005d11       $stateUnwindMap$Java_jdk_jpackage_internal_WindowsRegistry_comparePaths 0000000180019d11     WindowsRegistry.obj
 0002:00005d11       $stateUnwindMap$Java_jdk_jpackage_internal_ShortPathUtils_getShortPath 0000000180019d11     jpackage.obj
 0002:00005d20       $tryMap$Java_jdk_jpackage_internal_WindowsRegistry_comparePaths 0000000180019d20     WindowsRegistry.obj
 0002:00005d28       $handlerMap$Java_jdk_jpackage_internal_WindowsRegistry_comparePaths 0000000180019d28     WindowsRegistry.obj
 0002:00005d3e       $ip2state$Java_jdk_jpackage_internal_WindowsRegistry_comparePaths 0000000180019d3e     WindowsRegistry.obj
 0002:00005d4c       $unwind$?append@LastErrorLogAppender@?A0xd3578678@@UEAAXAEBULogEvent@@@Z 0000000180019d4c     app.obj
 0002:00005d60       $cppxdata$?append@LastErrorLogAppender@?A0xd3578678@@UEAAXAEBULogEvent@@@Z 0000000180019d60     app.obj
 0002:00005d69       $stateUnwindMap$?append@LastErrorLogAppender@?A0xd3578678@@UEAAXAEBULogEvent@@@Z 0000000180019d69     app.obj
 0002:00005d70       $ip2state$?append@LastErrorLogAppender@?A0xd3578678@@UEAAXAEBULogEvent@@@Z 0000000180019d70     app.obj
 0002:00005d78       $unwind$Java_jdk_jpackage_internal_ExecutableRebrander_lockResource 0000000180019d78     jpackage.obj
 0002:00005d8c       $cppxdata$Java_jdk_jpackage_internal_ExecutableRebrander_lockResource 0000000180019d8c     jpackage.obj
 0002:00005d99       $stateUnwindMap$Java_jdk_jpackage_internal_ExecutableRebrander_lockResource 0000000180019d99     jpackage.obj
 0002:00005da2       $tryMap$Java_jdk_jpackage_internal_ExecutableRebrander_lockResource 0000000180019da2     jpackage.obj
 0002:00005daa       $handlerMap$Java_jdk_jpackage_internal_ExecutableRebrander_lockResource 0000000180019daa     jpackage.obj
 0002:00005dbe       $ip2state$Java_jdk_jpackage_internal_ExecutableRebrander_lockResource 0000000180019dbe     jpackage.obj
 0002:00005dc8       $unwind$Java_jdk_jpackage_internal_ExecutableRebrander_unlockResource 0000000180019dc8     jpackage.obj
 0002:00005dd8       $cppxdata$Java_jdk_jpackage_internal_ExecutableRebrander_unlockResource 0000000180019dd8     jpackage.obj
 0002:00005de5       $tryMap$Java_jdk_jpackage_internal_ExecutableRebrander_unlockResource 0000000180019de5     jpackage.obj
 0002:00005ded       $handlerMap$Java_jdk_jpackage_internal_ExecutableRebrander_unlockResource 0000000180019ded     jpackage.obj
 0002:00005e01       $ip2state$Java_jdk_jpackage_internal_ExecutableRebrander_unlockResource 0000000180019e01     jpackage.obj
 0002:00005e04       $unwind$Java_jdk_jpackage_internal_ExecutableRebrander_iconSwap 0000000180019e04     jpackage.obj
 0002:00005e1c       $cppxdata$Java_jdk_jpackage_internal_ExecutableRebrander_iconSwap 0000000180019e1c     jpackage.obj
 0002:00005e29       $stateUnwindMap$Java_jdk_jpackage_internal_ExecutableRebrander_iconSwap 0000000180019e29     jpackage.obj
 0002:00005e38       $tryMap$Java_jdk_jpackage_internal_ExecutableRebrander_iconSwap 0000000180019e38     jpackage.obj
 0002:00005e40       $handlerMap$Java_jdk_jpackage_internal_ExecutableRebrander_iconSwap 0000000180019e40     jpackage.obj
 0002:00005e55       $ip2state$Java_jdk_jpackage_internal_ExecutableRebrander_iconSwap 0000000180019e55     jpackage.obj
 0002:00005e60       $unwind$Java_jdk_jpackage_internal_ExecutableRebrander_versionSwap 0000000180019e60     jpackage.obj
 0002:00005e80       $cppxdata$Java_jdk_jpackage_internal_ExecutableRebrander_versionSwap 0000000180019e80     jpackage.obj
 0002:00005e8d       $stateUnwindMap$Java_jdk_jpackage_internal_ExecutableRebrander_versionSwap 0000000180019e8d     jpackage.obj
 0002:00005eb0       $tryMap$Java_jdk_jpackage_internal_ExecutableRebrander_versionSwap 0000000180019eb0     jpackage.obj
 0002:00005eb8       $handlerMap$Java_jdk_jpackage_internal_ExecutableRebrander_versionSwap 0000000180019eb8     jpackage.obj
 0002:00005ece       $ip2state$Java_jdk_jpackage_internal_ExecutableRebrander_versionSwap 0000000180019ece     jpackage.obj
 0002:00005ee0       $unwind$Java_jdk_jpackage_internal_WinExeBundler_embedMSI 0000000180019ee0     jpackage.obj
 0002:00005ef8       $cppxdata$Java_jdk_jpackage_internal_WinExeBundler_embedMSI 0000000180019ef8     jpackage.obj
 0002:00005f05       $stateUnwindMap$Java_jdk_jpackage_internal_WinExeBundler_embedMSI 0000000180019f05     jpackage.obj
 0002:00005f60       $tryMap$Java_jdk_jpackage_internal_WinExeBundler_embedMSI 0000000180019f60     jpackage.obj
 0002:00005f68       $handlerMap$Java_jdk_jpackage_internal_WinExeBundler_embedMSI 0000000180019f68     jpackage.obj
 0002:00005f7e       $ip2state$Java_jdk_jpackage_internal_WinExeBundler_embedMSI 0000000180019f7e     jpackage.obj
 0002:00005fa4       $unwind$??0?$basic_istringstream@DU?$char_traits@D@std@@V?$allocator@D@2@@std@@QEAA@AEBV?$basic_string@DU?$char_traits@D@std@@V?$allocator@D@2@@1@H@Z 0000000180019fa4     jpackage.obj
 0002:00005fbc       $cppxdata$??0?$basic_istringstream@DU?$char_traits@D@std@@V?$allocator@D@2@@std@@QEAA@AEBV?$basic_string@DU?$char_traits@D@std@@V?$allocator@D@2@@1@H@Z 0000000180019fbc     jpackage.obj
 0002:00005fc5       $stateUnwindMap$??0?$basic_istringstream@DU?$char_traits@D@std@@V?$allocator@D@2@@std@@QEAA@AEBV?$basic_string@DU?$char_traits@D@std@@V?$allocator@D@2@@1@H@Z 0000000180019fc5     jpackage.obj
 0002:00005fd0       $ip2state$??0?$basic_istringstream@DU?$char_traits@D@std@@V?$allocator@D@2@@std@@QEAA@AEBV?$basic_string@DU?$char_traits@D@std@@V?$allocator@D@2@@1@H@Z 0000000180019fd0     jpackage.obj
 0002:00005fd8       $unwind$??0?$basic_stringbuf@DU?$char_traits@D@std@@V?$allocator@D@2@@std@@QEAA@AEBV?$basic_string@DU?$char_traits@D@std@@V?$allocator@D@2@@1@H@Z 0000000180019fd8     jpackage.obj
 0002:00005ff0       $cppxdata$??0?$basic_stringbuf@DU?$char_traits@D@std@@V?$allocator@D@2@@std@@QEAA@AEBV?$basic_string@DU?$char_traits@D@std@@V?$allocator@D@2@@1@H@Z 0000000180019ff0     jpackage.obj
 0002:00005ff9       $stateUnwindMap$??0?$basic_stringbuf@DU?$char_traits@D@std@@V?$allocator@D@2@@std@@QEAA@AEBV?$basic_string@DU?$char_traits@D@std@@V?$allocator@D@2@@1@H@Z 0000000180019ff9     jpackage.obj
 0002:00006000       $ip2state$??0?$basic_stringbuf@DU?$char_traits@D@std@@V?$allocator@D@2@@std@@QEAA@AEBV?$basic_string@DU?$char_traits@D@std@@V?$allocator@D@2@@1@H@Z 000000018001a000     jpackage.obj
 0002:00006008       $unwind$Java_jdk_jpackage_internal_ShortPathUtils_getShortPath 000000018001a008     jpackage.obj
 0002:0000601c       $cppxdata$Java_jdk_jpackage_internal_ShortPathUtils_getShortPath 000000018001a01c     jpackage.obj
 0002:00006029       $tryMap$Java_jdk_jpackage_internal_ShortPathUtils_getShortPath 000000018001a029     jpackage.obj
 0002:00006031       $handlerMap$Java_jdk_jpackage_internal_ShortPathUtils_getShortPath 000000018001a031     jpackage.obj
 0002:00006045       $ip2state$Java_jdk_jpackage_internal_ShortPathUtils_getShortPath 000000018001a045     jpackage.obj
 0002:00006050       $unwind$?unsafe_format@tstrings@@YA?AV?$basic_string@GU?$char_traits@G@std@@V?$allocator@G@2@@std@@PEBGZZ 000000018001a050     tstrings.obj
 0002:00006068       $cppxdata$?unsafe_format@tstrings@@YA?AV?$basic_string@GU?$char_traits@G@std@@V?$allocator@G@2@@std@@PEBGZZ 000000018001a068     tstrings.obj
 0002:00006071       $stateUnwindMap$?unsafe_format@tstrings@@YA?AV?$basic_string@GU?$char_traits@G@std@@V?$allocator@G@2@@std@@PEBGZZ 000000018001a071     tstrings.obj
 0002:00006078       $unwind$?equals@tstrings@@YA_NAEBV?$basic_string@GU?$char_traits@G@std@@V?$allocator@G@2@@std@@0W4CompareType@1@@Z 000000018001a078     tstrings.obj
 0002:00006090       $cppxdata$?equals@tstrings@@YA_NAEBV?$basic_string@GU?$char_traits@G@std@@V?$allocator@G@2@@std@@0W4CompareType@1@@Z 000000018001a090     tstrings.obj
 0002:00006099       $stateUnwindMap$?equals@tstrings@@YA_NAEBV?$basic_string@GU?$char_traits@G@std@@V?$allocator@G@2@@std@@0W4CompareType@1@@Z 000000018001a099     tstrings.obj
 0002:000060a0       $ip2state$?equals@tstrings@@YA_NAEBV?$basic_string@GU?$char_traits@G@std@@V?$allocator@G@2@@std@@0W4CompareType@1@@Z 000000018001a0a0     tstrings.obj
 0002:000060a8       $unwind$?toLower@tstrings@@YA?AV?$basic_string@GU?$char_traits@G@std@@V?$allocator@G@2@@std@@AEBV23@@Z 000000018001a0a8     tstrings.obj
 0002:000060c8       $cppxdata$?toLower@tstrings@@YA?AV?$basic_string@GU?$char_traits@G@std@@V?$allocator@G@2@@std@@AEBV23@@Z 000000018001a0c8     tstrings.obj
 0002:000060d1       $stateUnwindMap$?toLower@tstrings@@YA?AV?$basic_string@GU?$char_traits@G@std@@V?$allocator@G@2@@std@@AEBV23@@Z 000000018001a0d1     tstrings.obj
 0002:000060d7       $ip2state$?toLower@tstrings@@YA?AV?$basic_string@GU?$char_traits@G@std@@V?$allocator@G@2@@std@@AEBV23@@Z 000000018001a0d7     tstrings.obj
 0002:000060dc       $unwind$?toMultiByte@?A0xf04d92fb@tstrings@@YA?AV?$basic_string@DU?$char_traits@D@std@@V?$allocator@D@2@@std@@AEBV?$basic_string@GU?$char_traits@G@std@@V?$allocator@G@2@@4@H@Z 000000018001a0dc     tstrings.obj
 0002:000060fc       $cppxdata$?toMultiByte@?A0xf04d92fb@tstrings@@YA?AV?$basic_string@DU?$char_traits@D@std@@V?$allocator@D@2@@std@@AEBV?$basic_string@GU?$char_traits@G@std@@V?$allocator@G@2@@4@H@Z 000000018001a0fc     tstrings.obj
 0002:00006105       $stateUnwindMap$?toMultiByte@?A0xf04d92fb@tstrings@@YA?AV?$basic_string@DU?$char_traits@D@std@@V?$allocator@D@2@@std@@AEBV?$basic_string@GU?$char_traits@G@std@@V?$allocator@G@2@@4@H@Z 000000018001a105     tstrings.obj
 0002:0000610b       $ip2state$?toMultiByte@?A0xf04d92fb@tstrings@@YA?AV?$basic_string@DU?$char_traits@D@std@@V?$allocator@D@2@@std@@AEBV?$basic_string@GU?$char_traits@G@std@@V?$allocator@G@2@@4@H@Z 000000018001a10b     tstrings.obj
 0002:00006114       $unwind$?fromMultiByte@?A0xf04d92fb@tstrings@@YA?AV?$basic_string@GU?$char_traits@G@std@@V?$allocator@G@2@@std@@AEBV?$basic_string@DU?$char_traits@D@std@@V?$allocator@D@2@@4@H@Z 000000018001a114     tstrings.obj
 0002:00006134       $cppxdata$?fromMultiByte@?A0xf04d92fb@tstrings@@YA?AV?$basic_string@GU?$char_traits@G@std@@V?$allocator@G@2@@std@@AEBV?$basic_string@DU?$char_traits@D@std@@V?$allocator@D@2@@4@H@Z 000000018001a134     tstrings.obj
 0002:0000613d       $stateUnwindMap$?fromMultiByte@?A0xf04d92fb@tstrings@@YA?AV?$basic_string@GU?$char_traits@G@std@@V?$allocator@G@2@@std@@AEBV?$basic_string@DU?$char_traits@D@std@@V?$allocator@D@2@@4@H@Z 000000018001a13d     tstrings.obj
 0002:00006143       $ip2state$?fromMultiByte@?A0xf04d92fb@tstrings@@YA?AV?$basic_string@GU?$char_traits@G@std@@V?$allocator@G@2@@std@@AEBV?$basic_string@DU?$char_traits@D@std@@V?$allocator@D@2@@4@H@Z 000000018001a143     tstrings.obj
 0002:0000614c       $unwind$__GSHandlerCheckCommon 000000018001a14c     MSVCRT:gshandler.obj
 0002:00006158       $xdatasym                  000000018001a158     MSVCRT:chkstk.obj
 0002:00006160       $xdatasym                  000000018001a160     MSVCRT:amdsecgs.obj
 0002:00006164       $unwind$__report_securityfailure 000000018001a164     MSVCRT:gs_report.obj
 0002:0000616c       $unwind$__report_gsfailure 000000018001a16c     MSVCRT:gs_report.obj
 0002:00006174       $unwind$capture_current_context 000000018001a174     MSVCRT:gs_report.obj
 0002:00006180       $unwind$capture_previous_context 000000018001a180     MSVCRT:gs_report.obj
 0002:0000618c       $unwind$__scrt_is_nonwritable_in_current_image 000000018001a18c     MSVCRT:utility.obj
 0002:000061ac       $unwind$__scrt_is_nonwritable_in_current_image$filt$0 000000018001a1ac     MSVCRT:utility.obj
 0002:000061b4       $unwind$?dllmain_crt_process_attach@@YAHQEAUHINSTANCE__@@QEAX@Z 000000018001a1b4     MSVCRT:dll_dllmain.obj
 0002:000061f0       $unwind$?dllmain_crt_process_detach@@YAH_N@Z 000000018001a1f0     MSVCRT:dll_dllmain.obj
 0002:00006244       $unwind$?dllmain_dispatch@@YAHQEAUHINSTANCE__@@KQEAX@Z 000000018001a244     MSVCRT:dll_dllmain.obj
 0002:0000626c       $unwind$?filt$0@?0??dllmain_dispatch@@YAHQEAUHINSTANCE__@@KQEAX@Z@4HA 000000018001a26c     MSVCRT:dll_dllmain.obj
 0002:00006274       $unwind$__isa_available_init 000000018001a274     MSVCRT:cpu_disp.obj
 0002:00006288       $unwind$__scrt_fastfail    000000018001a288     MSVCRT:utility_desktop.obj
 0002:00006298       $unwind$__security_init_cookie 000000018001a298     MSVCRT:gs_support.obj
 0002:000062a8       $xdatasym                  000000018001a2a8     MSVCRT:guard_dispatch.obj
 0002:000062b0       $xdatasym                  000000018001a2b0     MSVCRT:guard_xfg_dispatch.obj
 0002:00006770       .edata                     000000018001a770     jpackage.exp
 0002:00006798       rgpv                       000000018001a798     jpackage.exp
 0002:000067c4       rgszName                   000000018001a7c4     jpackage.exp
 0002:000067f0       rgwOrd                     000000018001a7f0     jpackage.exp
 0002:00006806       szName                     000000018001a806     jpackage.exp
 0002:00006813       $N00001                    000000018001a813     jpackage.exp
 0002:0000684b       $N00002                    000000018001a84b     jpackage.exp
 0002:00006887       $N00003                    000000018001a887     jpackage.exp
 0002:000068c5       $N00004                    000000018001a8c5     jpackage.exp
 0002:00006900       $N00005                    000000018001a900     jpackage.exp
 0002:00006937       $N00006                    000000018001a937     jpackage.exp
 0002:00006969       $N00007                    000000018001a969     jpackage.exp
 0002:000069a5       $N00008                    000000018001a9a5     jpackage.exp
 0002:000069dd       $N00009                    000000018001a9dd     jpackage.exp
 0002:00006a1a       $N00010                    000000018001aa1a     jpackage.exp
 0002:00006a55       $N00011                    000000018001aa55     jpackage.exp
 0002:00007372       .idata$6                   000000018001b372     advapi32:ADVAPI32.dll
 0002:00007380       .idata$6                   000000018001b380     msi:msi.dll
 0002:000073aa       .idata$6                   000000018001b3aa     ole32:ole32.dll
 0002:000094fa       .idata$6                   000000018001d4fa     msvcprt:MSVCP140.dll
 0002:0000981e       .idata$6                   000000018001d81e     kernel32:KERNEL32.dll
 0002:00009908       .idata$6                   000000018001d908     vcruntime:VCRUNTIME140.dll
 0002:0000991a       .idata$6                   000000018001d91a     vcruntime:VCRUNTIME140_1.dll
 0002:00009b74       .idata$6                   000000018001db74     ucrt:api-ms-win-crt-runtime-l1-1-0.dll
 0002:00009b96       .idata$6                   000000018001db96     ucrt:api-ms-win-crt-string-l1-1-0.dll
 0002:00009bb8       .idata$6                   000000018001dbb8     ucrt:api-ms-win-crt-stdio-l1-1-0.dll
 0002:00009bd8       .idata$6                   000000018001dbd8     ucrt:api-ms-win-crt-heap-l1-1-0.dll
 0002:00009bf8       .idata$6                   000000018001dbf8     ucrt:api-ms-win-crt-filesystem-l1-1-0.dll
 0003:00000000       ?moduleName@?A0x40e1fcfd@@3PAGA 000000018001e000     PlatformLogEvent.obj
 0003:00000208       ?lastErrorLogAppender@?A0xd3578678@@3VLastErrorLogAppender@1@A 000000018001e208     app.obj
 0003:00000bd8       ??_R0?AVLastErrorLogAppender@?A0xd3578678@@@8 000000018001ebd8     app.obj
 0003:00000ca8       ?defaultLogAppenderMemory@?A0xc7174dad@@3PADA 000000018001eca8     Log.obj
 0003:00000cb8       ?defaultLoggerMemory@?A0xc7174dad@@3PADA 000000018001ecb8     Log.obj
 0003:00000cc8       ?state@?A0xc7174dad@@3W4State@1@A 000000018001ecc8     Log.obj
 0003:00000ce8       ?theLastErrorMsg@?A0xd3578678@@3PEBV?$basic_string@DU?$char_traits@D@std@@V?$allocator@D@2@@std@@EB 000000018001ece8     app.obj
 0003:00000cf0       ?nopLogAppenderMemory@?A0xd3578678@@3PADA 000000018001ecf0     app.obj
 0003:00000cf8       ?standardLogAppenderMemory@?A0xd3578678@@3PADA 000000018001ecf8     app.obj
 0003:00000d00       ?_Fac_head@std@@3PEAU_Fac_node@1@EA 000000018001ed00     msvcprt:locale0_implib.obj
 0003:00000d08       ?_Fac_tidy_reg@std@@3U_Fac_tidy_reg_t@1@B 000000018001ed08     msvcprt:locale0_implib.obj
 0003:00000d10       GS_ExceptionRecord         000000018001ed10     MSVCRT:gs_report.obj
 0003:00000db0       GS_ContextRecord           000000018001edb0     MSVCRT:gs_report.obj
 0003:00001290       ?is_initialized_as_dll@@3_NA 000000018001f290     MSVCRT:utility.obj
 0003:00001291       ?module_local_atexit_table_initialized@@3_NA 000000018001f291     MSVCRT:utility.obj
 0003:00001298       ?module_local_atexit_table@@3U_onexit_table_t@@A 000000018001f298     MSVCRT:utility.obj
 0003:000012b0       ?module_local_at_quick_exit_table@@3U_onexit_table_t@@A 000000018001f2b0     MSVCRT:utility.obj
 0003:000012c8       ?__proc_attached@@3HA      000000018001f2c8     MSVCRT:dll_dllmain.obj
 0005:00000060       $R000000                   0000000180022060     jpackage.dll.res
